 javaaccessbridge

 Timestamp is 41efdacc (reproducible build file hash)

 Preferred load address is 0000000180000000

 Start         Length     Name                   Class
 0001:00000000 00028120H .text$mn                CODE
 0001:00028120 00000060H .text$mn$00             CODE
 0001:00028180 000010e0H .text$mn$21             CODE
 0001:00029260 000005c0H .text$x                 CODE
 0002:00000000 00000328H .idata$5                DATA
 0002:00000328 00000038H .00cfg                  DATA
 0002:00000360 00000008H .CRT$XCA                DATA
 0002:00000368 00000008H .CRT$XCZ                DATA
 0002:00000370 00000008H .CRT$XIA                DATA
 0002:00000378 00000020H .CRT$XIC                DATA
 0002:00000398 00000008H .CRT$XIZ                DATA
 0002:000003a0 00000008H .CRT$XPA                DATA
 0002:000003a8 00000010H .CRT$XPX                DATA
 0002:000003b8 00000008H .CRT$XPXA               DATA
 0002:000003c0 00000008H .CRT$XPZ                DATA
 0002:000003c8 00000008H .CRT$XTA                DATA
 0002:000003d0 00000010H .CRT$XTZ                DATA
 0002:000003d8 00000000H .gehcont$y              DATA
 0002:000003d8 00000000H .gfids$y                DATA
 0002:000003e0 00017b60H .rdata                  DATA
 0002:00017f40 000001c0H .rdata$00               DATA
 0002:00018100 00000000H .rdata$CastGuardVftablesA DATA
 0002:00018100 00000000H .rdata$CastGuardVftablesC DATA
 0002:00018100 00000274H .rdata$r                DATA
 0002:00018374 000000f4H .rdata$voltmd           DATA
 0002:00018468 000003b0H .rdata$zzzdbg           DATA
 0002:00018818 00000008H .rtc$IAA                DATA
 0002:00018820 00000008H .rtc$IZZ                DATA
 0002:00018828 00000008H .rtc$TAA                DATA
 0002:00018830 00000008H .rtc$TZZ                DATA
 0002:00018838 00001680H .xdata                  DATA
 0002:00019eb8 00000158H .xdata$x                DATA
 0002:0001a010 00000a00H .edata                  DATA
 0002:0001aa10 0000003cH .idata$2                DATA
 0002:0001aa4c 00000014H .idata$3                DATA
 0002:0001aa60 00000328H .idata$4                DATA
 0002:0001ad88 0000073cH .idata$6                DATA
 0003:00000000 00000a70H .data                   DATA
 0003:00000a70 000000a8H .data$r                 DATA
 0003:00000b18 00000028H .data$rs                DATA
 0003:00000b40 00001170H .bss                    DATA
 0004:00000000 00001e24H .pdata                  DATA
 0005:00000000 00000100H .fptable                DATA
 0006:00000000 00000120H .rsrc$01                DATA
 0006:00000120 00000628H .rsrc$02                DATA

  Address         Publics by Value              Rva+Base               Lib:Object

 0000:00000000       __AbsoluteZero             0000000000000000     <absolute>
 0000:00000000       ___safe_se_handler_count   0000000000000000     <absolute>
 0000:00000000       ___safe_se_handler_table   0000000000000000     <absolute>
 0000:00000000       __arm64x_extra_rfe_table   0000000000000000     <absolute>
 0000:00000000       __arm64x_extra_rfe_table_size 0000000000000000     <absolute>
 0000:00000000       __arm64x_native_entrypoint 0000000000000000     <absolute>
 0000:00000000       __arm64x_redirection_metadata 0000000000000000     <absolute>
 0000:00000000       __arm64x_redirection_metadata_count 0000000000000000     <absolute>
 0000:00000000       __dynamic_value_reloc_table 0000000000000000     <absolute>
 0000:00000000       __enclave_config           0000000000000000     <absolute>
 0000:00000000       __guard_check_icall_a64n_fptr 0000000000000000     <absolute>
 0000:00000000       __guard_eh_cont_count      0000000000000000     <absolute>
 0000:00000000       __guard_eh_cont_table      0000000000000000     <absolute>
 0000:00000000       __guard_fids_count         0000000000000000     <absolute>
 0000:00000000       __guard_fids_table         0000000000000000     <absolute>
 0000:00000000       __guard_iat_count          0000000000000000     <absolute>
 0000:00000000       __guard_iat_table          0000000000000000     <absolute>
 0000:00000000       __guard_longjmp_count      0000000000000000     <absolute>
 0000:00000000       __guard_longjmp_table      0000000000000000     <absolute>
 0000:00000000       __hybrid_auxiliary_delayload_iat 0000000000000000     <absolute>
 0000:00000000       __hybrid_auxiliary_delayload_iat_copy 0000000000000000     <absolute>
 0000:00000000       __hybrid_auxiliary_iat     0000000000000000     <absolute>
 0000:00000000       __hybrid_auxiliary_iat_copy 0000000000000000     <absolute>
 0000:00000000       __hybrid_code_map          0000000000000000     <absolute>
 0000:00000000       __hybrid_code_map_count    0000000000000000     <absolute>
 0000:00000000       __hybrid_image_info_bitfield 0000000000000000     <absolute>
 0000:00000000       __x64_code_ranges_to_entry_points 0000000000000000     <absolute>
 0000:00000000       __x64_code_ranges_to_entry_points_count 0000000000000000     <absolute>
 0000:00000100       __guard_flags              0000000000000100     <absolute>
 0000:00000000       __ImageBase                0000000180000000     <linker-defined>
 0001:00000000       ??0AccessBridgeATInstance@@QEAA@PEAUHWND__@@0PEADPEAV0@@Z 0000000180001000 f   AccessBridgeATInstance.obj
 0001:0000003c       ??1AccessBridgeATInstance@@QEAA@XZ 000000018000103c f   AccessBridgeATInstance.obj
 0001:00000204       ?findABATInstanceFromATHWND@AccessBridgeATInstance@@QEAAPEAV1@PEAUHWND__@@@Z 0000000180001204 f   AccessBridgeATInstance.obj
 0001:00000224       ?initiateIPC@AccessBridgeATInstance@@QEAA_JXZ 0000000180001224 f   AccessBridgeATInstance.obj
 0001:0000031c       ?sendAccessibilityEventPackage@AccessBridgeATInstance@@QEAA_JPEADHJ@Z 000000018000131c f   AccessBridgeATInstance.obj
 0001:00000380       ?sendJavaEventPackage@AccessBridgeATInstance@@QEAA_JPEADHJ@Z 0000000180001380 f   AccessBridgeATInstance.obj
 0001:000003f4       PrintDebugString           00000001800013f4 f   AccessBridgeDebug.obj
 0001:00000470       __local_stdio_printf_options 0000000180001470 f i AccessBridgeDebug.obj
 0001:00000478       finalizeFileLogger         0000000180001478 f   AccessBridgeDebug.obj
 0001:0000049c       fprintf                    000000018000149c f i AccessBridgeDebug.obj
 0001:000004e0       getTimeStamp               00000001800014e0 f   AccessBridgeDebug.obj
 0001:00000518       initializeFileLogger       0000000180001518 f   AccessBridgeDebug.obj
 0001:00000624       printf                     0000000180001624 f i AccessBridgeDebug.obj
 0001:00000678       wPrintDebugString          0000000180001678 f   AccessBridgeDebug.obj
 0001:00000678       wPrintJavaDebugString      0000000180001678 f   AccessBridgeDebug.obj
 0001:000006f4       ??0AccessBridgeJavaEntryPoints@@QEAA@PEAUJNIEnv_@@PEAV_jobject@@@Z 00000001800016f4 f   AccessBridgeJavaEntryPoints.obj
 0001:0000071c       ?BuildJavaEntryPoints@AccessBridgeJavaEntryPoints@@QEAAHXZ 000000018000171c f   AccessBridgeJavaEntryPoints.obj
 0001:00002694       ?CallBooleanMethod@JNIEnv_@@QEAAEPEAV_jobject@@PEAU_jmethodID@@ZZ 0000000180003694 f i AccessBridgeJavaEntryPoints.obj
 0001:000026b8       ?CallCharMethod@JNIEnv_@@QEAAGPEAV_jobject@@PEAU_jmethodID@@ZZ 00000001800036b8 f i AccessBridgeJavaEntryPoints.obj
 0001:000026dc       ?CallFloatMethod@JNIEnv_@@QEAAMPEAV_jobject@@PEAU_jmethodID@@ZZ 00000001800036dc f i AccessBridgeJavaEntryPoints.obj
 0001:00002700       ?CallIntMethod@JNIEnv_@@QEAAHPEAV_jobject@@PEAU_jmethodID@@ZZ 0000000180003700 f i AccessBridgeJavaEntryPoints.obj
 0001:00002724       ?CallObjectMethod@JNIEnv_@@QEAAPEAV_jobject@@PEAV2@PEAU_jmethodID@@ZZ 0000000180003724 f i AccessBridgeJavaEntryPoints.obj
 0001:00002748       ?CallVoidMethod@JNIEnv_@@QEAAXPEAV_jobject@@PEAU_jmethodID@@ZZ 0000000180003748 f i AccessBridgeJavaEntryPoints.obj
 0001:0000276c       ?activateAccessibleHyperlink@AccessBridgeJavaEntryPoints@@QEAAHPEAV_jobject@@0@Z 000000018000376c f   AccessBridgeJavaEntryPoints.obj
 0001:00002818       ?addAccessibilityEventNotification@AccessBridgeJavaEntryPoints@@QEAAH_J@Z 0000000180003818 f   AccessBridgeJavaEntryPoints.obj
 0001:000028d0       ?addAccessibleSelectionFromContext@AccessBridgeJavaEntryPoints@@QEAAXPEAV_jobject@@H@Z 00000001800038d0 f   AccessBridgeJavaEntryPoints.obj
 0001:00002978       ?addJavaEventNotification@AccessBridgeJavaEntryPoints@@QEAAH_J@Z 0000000180003978 f   AccessBridgeJavaEntryPoints.obj
 0001:00002a10       ?clearAccessibleSelectionFromContext@AccessBridgeJavaEntryPoints@@QEAAXPEAV_jobject@@@Z 0000000180003a10 f   AccessBridgeJavaEntryPoints.obj
 0001:00002aa4       ?doAccessibleActions@AccessBridgeJavaEntryPoints@@QEAAHPEAV_jobject@@PEAUAccessibleActionsToDoTag@@PEAH@Z 0000000180003aa4 f   AccessBridgeJavaEntryPoints.obj
 0001:00002c28       ?getAccessibleActions@AccessBridgeJavaEntryPoints@@QEAAHPEAV_jobject@@PEAUAccessibleActionsTag@@@Z 0000000180003c28 f   AccessBridgeJavaEntryPoints.obj
 0001:00002ee4       ?getAccessibleChildFromContext@AccessBridgeJavaEntryPoints@@QEAAPEAV_jobject@@PEAV2@H@Z 0000000180003ee4 f   AccessBridgeJavaEntryPoints.obj
 0001:00002ff8       ?getAccessibleContextAt@AccessBridgeJavaEntryPoints@@QEAAPEAV_jobject@@HHPEAV2@@Z 0000000180003ff8 f   AccessBridgeJavaEntryPoints.obj
 0001:000030f0       ?getAccessibleContextFromHWND@AccessBridgeJavaEntryPoints@@QEAAPEAV_jobject@@H@Z 00000001800040f0 f   AccessBridgeJavaEntryPoints.obj
 0001:000031a8       ?getAccessibleContextInfo@AccessBridgeJavaEntryPoints@@QEAAHPEAV_jobject@@PEAUAccessibleContextInfoTag@@@Z 00000001800041a8 f   AccessBridgeJavaEntryPoints.obj
 0001:000042ac       ?getAccessibleContextWithFocus@AccessBridgeJavaEntryPoints@@QEAAPEAV_jobject@@XZ 00000001800052ac f   AccessBridgeJavaEntryPoints.obj
 0001:00004388       ?getAccessibleHyperlink@AccessBridgeJavaEntryPoints@@QEAAHQEAV_jobject@@HPEAUAccessibleHyperlinkInfoTag@@@Z 0000000180005388 f   AccessBridgeJavaEntryPoints.obj
 0001:000046a4       ?getAccessibleHyperlinkCount@AccessBridgeJavaEntryPoints@@QEAAHQEAV_jobject@@@Z 00000001800056a4 f   AccessBridgeJavaEntryPoints.obj
 0001:00004740       ?getAccessibleHypertext@AccessBridgeJavaEntryPoints@@QEAAHPEAV_jobject@@PEAUAccessibleHypertextInfoTag@@@Z 0000000180005740 f   AccessBridgeJavaEntryPoints.obj
 0001:00004ba8       ?getAccessibleHypertextExt@AccessBridgeJavaEntryPoints@@QEAAHQEAV_jobject@@HPEAUAccessibleHypertextInfoTag@@@Z 0000000180005ba8 f   AccessBridgeJavaEntryPoints.obj
 0001:00005034       ?getAccessibleHypertextLinkIndex@AccessBridgeJavaEntryPoints@@QEAAHQEAV_jobject@@H@Z 0000000180006034 f   AccessBridgeJavaEntryPoints.obj
 0001:000050e0       ?getAccessibleIcons@AccessBridgeJavaEntryPoints@@QEAAHPEAV_jobject@@PEAUAccessibleIconsTag@@@Z 00000001800060e0 f   AccessBridgeJavaEntryPoints.obj
 0001:0000545c       ?getAccessibleKeyBindings@AccessBridgeJavaEntryPoints@@QEAAHPEAV_jobject@@PEAUAccessibleKeyBindingsTag@@@Z 000000018000645c f   AccessBridgeJavaEntryPoints.obj
 0001:000055ec       ?getAccessibleParentFromContext@AccessBridgeJavaEntryPoints@@QEAAPEAV_jobject@@PEAV2@@Z 00000001800065ec f   AccessBridgeJavaEntryPoints.obj
 0001:000056f8       ?getAccessibleRelationSet@AccessBridgeJavaEntryPoints@@QEAAHPEAV_jobject@@PEAUAccessibleRelationSetInfoTag@@@Z 00000001800066f8 f   AccessBridgeJavaEntryPoints.obj
 0001:00005acc       ?getAccessibleSelectionCountFromContext@AccessBridgeJavaEntryPoints@@QEAAHPEAV_jobject@@@Z 0000000180006acc f   AccessBridgeJavaEntryPoints.obj
 0001:00005b70       ?getAccessibleSelectionFromContext@AccessBridgeJavaEntryPoints@@QEAAPEAV_jobject@@PEAV2@H@Z 0000000180006b70 f   AccessBridgeJavaEntryPoints.obj
 0001:00005c84       ?getAccessibleTableCellInfo@AccessBridgeJavaEntryPoints@@QEAAHPEAV_jobject@@HHPEAUAccessibleTableCellInfoTag@@@Z 0000000180006c84 f   AccessBridgeJavaEntryPoints.obj
 0001:00005f30       ?getAccessibleTableColumn@AccessBridgeJavaEntryPoints@@QEAAHPEAV_jobject@@H@Z 0000000180006f30 f   AccessBridgeJavaEntryPoints.obj
 0001:00005fe8       ?getAccessibleTableColumnDescription@AccessBridgeJavaEntryPoints@@QEAAPEAV_jobject@@PEAV2@H@Z 0000000180006fe8 f   AccessBridgeJavaEntryPoints.obj
 0001:000060fc       ?getAccessibleTableColumnHeader@AccessBridgeJavaEntryPoints@@QEAAHPEAV_jobject@@PEAUAccessibleTableInfoTag@@@Z 00000001800070fc f   AccessBridgeJavaEntryPoints.obj
 0001:000062b0       ?getAccessibleTableColumnSelectionCount@AccessBridgeJavaEntryPoints@@QEAAHPEAV_jobject@@@Z 00000001800072b0 f   AccessBridgeJavaEntryPoints.obj
 0001:00006354       ?getAccessibleTableColumnSelections@AccessBridgeJavaEntryPoints@@QEAAHPEAV_jobject@@HPEAH@Z 0000000180007354 f   AccessBridgeJavaEntryPoints.obj
 0001:00006440       ?getAccessibleTableIndex@AccessBridgeJavaEntryPoints@@QEAAHPEAV_jobject@@HH@Z 0000000180007440 f   AccessBridgeJavaEntryPoints.obj
 0001:0000650c       ?getAccessibleTableInfo@AccessBridgeJavaEntryPoints@@QEAAHPEAV_jobject@@PEAUAccessibleTableInfoTag@@@Z 000000018000750c f   AccessBridgeJavaEntryPoints.obj
 0001:00006778       ?getAccessibleTableRow@AccessBridgeJavaEntryPoints@@QEAAHPEAV_jobject@@H@Z 0000000180007778 f   AccessBridgeJavaEntryPoints.obj
 0001:00006830       ?getAccessibleTableRowDescription@AccessBridgeJavaEntryPoints@@QEAAPEAV_jobject@@PEAV2@H@Z 0000000180007830 f   AccessBridgeJavaEntryPoints.obj
 0001:00006944       ?getAccessibleTableRowHeader@AccessBridgeJavaEntryPoints@@QEAAHPEAV_jobject@@PEAUAccessibleTableInfoTag@@@Z 0000000180007944 f   AccessBridgeJavaEntryPoints.obj
 0001:00006af8       ?getAccessibleTableRowSelectionCount@AccessBridgeJavaEntryPoints@@QEAAHPEAV_jobject@@@Z 0000000180007af8 f   AccessBridgeJavaEntryPoints.obj
 0001:00006b9c       ?getAccessibleTableRowSelections@AccessBridgeJavaEntryPoints@@QEAAHPEAV_jobject@@HPEAH@Z 0000000180007b9c f   AccessBridgeJavaEntryPoints.obj
 0001:00006c88       ?getAccessibleTextAttributes@AccessBridgeJavaEntryPoints@@QEAAHPEAV_jobject@@HPEAUAccessibleTextAttributesInfoTag@@@Z 0000000180007c88 f   AccessBridgeJavaEntryPoints.obj
 0001:000081bc       ?getAccessibleTextInfo@AccessBridgeJavaEntryPoints@@QEAAHPEAV_jobject@@PEAUAccessibleTextInfoTag@@HH@Z 00000001800091bc f   AccessBridgeJavaEntryPoints.obj
 0001:00008368       ?getAccessibleTextItems@AccessBridgeJavaEntryPoints@@QEAAHPEAV_jobject@@PEAUAccessibleTextItemsInfoTag@@H@Z 0000000180009368 f   AccessBridgeJavaEntryPoints.obj
 0001:000088e4       ?getAccessibleTextLineBounds@AccessBridgeJavaEntryPoints@@QEAAHPEAV_jobject@@HPEAH1@Z 00000001800098e4 f   AccessBridgeJavaEntryPoints.obj
 0001:00008a18       ?getAccessibleTextRange@AccessBridgeJavaEntryPoints@@QEAAHPEAV_jobject@@HHPEAGF@Z 0000000180009a18 f   AccessBridgeJavaEntryPoints.obj
 0001:00008cd8       ?getAccessibleTextRect@AccessBridgeJavaEntryPoints@@QEAAHPEAV_jobject@@PEAUAccessibleTextRectInfoTag@@H@Z 0000000180009cd8 f   AccessBridgeJavaEntryPoints.obj
 0001:00008ec4       ?getAccessibleTextSelectionInfo@AccessBridgeJavaEntryPoints@@QEAAHPEAV_jobject@@PEAUAccessibleTextSelectionInfoTag@@@Z 0000000180009ec4 f   AccessBridgeJavaEntryPoints.obj
 0001:000091cc       ?getActiveDescendent@AccessBridgeJavaEntryPoints@@QEAAPEAV_jobject@@QEAV2@@Z 000000018000a1cc f   AccessBridgeJavaEntryPoints.obj
 0001:000092c0       ?getCaretLocation@AccessBridgeJavaEntryPoints@@QEAAHPEAV_jobject@@PEAUAccessibleTextRectInfoTag@@H@Z 000000018000a2c0 f   AccessBridgeJavaEntryPoints.obj
 0001:000094ac       ?getCurrentAccessibleValueFromContext@AccessBridgeJavaEntryPoints@@QEAAHPEAV_jobject@@PEAGF@Z 000000018000a4ac f   AccessBridgeJavaEntryPoints.obj
 0001:000096f0       ?getHWNDFromAccessibleContext@AccessBridgeJavaEntryPoints@@QEAAPEAUHWND__@@PEAV_jobject@@@Z 000000018000a6f0 f   AccessBridgeJavaEntryPoints.obj
 0001:00009794       ?getMaximumAccessibleValueFromContext@AccessBridgeJavaEntryPoints@@QEAAHPEAV_jobject@@PEAGF@Z 000000018000a794 f   AccessBridgeJavaEntryPoints.obj
 0001:000099d8       ?getMinimumAccessibleValueFromContext@AccessBridgeJavaEntryPoints@@QEAAHPEAV_jobject@@PEAGF@Z 000000018000a9d8 f   AccessBridgeJavaEntryPoints.obj
 0001:00009c1c       ?getObjectDepth@AccessBridgeJavaEntryPoints@@QEAAHQEAV_jobject@@@Z 000000018000ac1c f   AccessBridgeJavaEntryPoints.obj
 0001:00009cc4       ?getParentWithRole@AccessBridgeJavaEntryPoints@@QEAAPEAV_jobject@@QEAV2@PEBG@Z 000000018000acc4 f   AccessBridgeJavaEntryPoints.obj
 0001:00009df0       ?getParentWithRoleElseRoot@AccessBridgeJavaEntryPoints@@QEAAPEAV_jobject@@QEAV2@PEBG@Z 000000018000adf0 f   AccessBridgeJavaEntryPoints.obj
 0001:00009f1c       ?getTextAttributesInRange@AccessBridgeJavaEntryPoints@@QEAAHQEAV_jobject@@HHPEAUAccessibleTextAttributesInfoTag@@PEAF@Z 000000018000af1c f   AccessBridgeJavaEntryPoints.obj
 0001:0000a220       ?getTopLevelObject@AccessBridgeJavaEntryPoints@@QEAAPEAV_jobject@@QEAV2@@Z 000000018000b220 f   AccessBridgeJavaEntryPoints.obj
 0001:0000a314       ?getVersionInfo@AccessBridgeJavaEntryPoints@@QEAAHPEAUAccessBridgeVersionInfoTag@@@Z 000000018000b314 f   AccessBridgeJavaEntryPoints.obj
 0001:0000a564       ?getVirtualAccessibleName@AccessBridgeJavaEntryPoints@@QEAAHQEAV_jobject@@PEAGH@Z 000000018000b564 f   AccessBridgeJavaEntryPoints.obj
 0001:0000a7b4       ?getVisibleChildren@AccessBridgeJavaEntryPoints@@QEAAHQEAV_jobject@@HPEAUVisibleChildenInfoTag@@@Z 000000018000b7b4 f   AccessBridgeJavaEntryPoints.obj
 0001:0000a948       ?getVisibleChildrenCount@AccessBridgeJavaEntryPoints@@QEAAHQEAV_jobject@@@Z 000000018000b948 f   AccessBridgeJavaEntryPoints.obj
 0001:0000a9dc       ?isAccessibleChildSelectedFromContext@AccessBridgeJavaEntryPoints@@QEAAHPEAV_jobject@@H@Z 000000018000b9dc f   AccessBridgeJavaEntryPoints.obj
 0001:0000aa98       ?isAccessibleTableColumnSelected@AccessBridgeJavaEntryPoints@@QEAAHPEAV_jobject@@H@Z 000000018000ba98 f   AccessBridgeJavaEntryPoints.obj
 0001:0000ab50       ?isAccessibleTableRowSelected@AccessBridgeJavaEntryPoints@@QEAAHPEAV_jobject@@H@Z 000000018000bb50 f   AccessBridgeJavaEntryPoints.obj
 0001:0000ac08       ?isJavaWindow@AccessBridgeJavaEntryPoints@@QEAAHH@Z 000000018000bc08 f   AccessBridgeJavaEntryPoints.obj
 0001:0000ac9c       ?isSameObject@AccessBridgeJavaEntryPoints@@QEAAHPEAV_jobject@@0@Z 000000018000bc9c f   AccessBridgeJavaEntryPoints.obj
 0001:0000ad38       ?removeAccessibilityEventNotification@AccessBridgeJavaEntryPoints@@QEAAH_J@Z 000000018000bd38 f   AccessBridgeJavaEntryPoints.obj
 0001:0000add0       ?removeAccessibleSelectionFromContext@AccessBridgeJavaEntryPoints@@QEAAXPEAV_jobject@@H@Z 000000018000bdd0 f   AccessBridgeJavaEntryPoints.obj
 0001:0000ae78       ?removeJavaEventNotification@AccessBridgeJavaEntryPoints@@QEAAH_J@Z 000000018000be78 f   AccessBridgeJavaEntryPoints.obj
 0001:0000af10       ?requestFocus@AccessBridgeJavaEntryPoints@@QEAAHQEAV_jobject@@@Z 000000018000bf10 f   AccessBridgeJavaEntryPoints.obj
 0001:0000afb8       ?selectAllAccessibleSelectionFromContext@AccessBridgeJavaEntryPoints@@QEAAXPEAV_jobject@@@Z 000000018000bfb8 f   AccessBridgeJavaEntryPoints.obj
 0001:0000b04c       ?selectTextRange@AccessBridgeJavaEntryPoints@@QEAAHQEAV_jobject@@HH@Z 000000018000c04c f   AccessBridgeJavaEntryPoints.obj
 0001:0000b114       ?setCaretPosition@AccessBridgeJavaEntryPoints@@QEAAHQEAV_jobject@@H@Z 000000018000c114 f   AccessBridgeJavaEntryPoints.obj
 0001:0000b1cc       ?setTextContents@AccessBridgeJavaEntryPoints@@QEAAHQEAV_jobject@@PEBG@Z 000000018000c1cc f   AccessBridgeJavaEntryPoints.obj
 0001:0000b2b8       ?verifyAccessibleText@AccessBridgeJavaEntryPoints@@QEAAHPEAV_jobject@@@Z 000000018000c2b8 f   AccessBridgeJavaEntryPoints.obj
 0001:0000b3e0       ?initBroadcastMessageIDs@@YAHXZ 000000018000c3e0 f   AccessBridgeMessages.obj
 0001:0000b420       ??0JavaAccessBridge@@QEAA@PEAUHINSTANCE__@@@Z 000000018000c420 f   JavaAccessBridge.obj
 0001:0000b44c       ??1JavaAccessBridge@@QEAA@XZ 000000018000c44c f   JavaAccessBridge.obj
 0001:0000b51c       ?MemoryMappedFileCreated@JavaAccessBridge@@QEAA_JPEAUHWND__@@PEAD@Z 000000018000c51c f   JavaAccessBridge.obj
 0001:0000b5b8       ?WindowsATDestroyed@JavaAccessBridge@@QEAAXPEAUHWND__@@@Z 000000018000c5b8 f   JavaAccessBridge.obj
 0001:0000b66c       ?addAccessibilityEventNotification@JavaAccessBridge@@QEAAX_JPEAUHWND__@@@Z 000000018000c66c f   JavaAccessBridge.obj
 0001:0000b714       ?addJavaEventNotification@JavaAccessBridge@@QEAAX_JPEAUHWND__@@@Z 000000018000c714 f   JavaAccessBridge.obj
 0001:0000b7bc       ?fireCaretUpdate@JavaAccessBridge@@QEAAXPEAUJNIEnv_@@PEAV_jobject@@11@Z 000000018000c7bc f   JavaAccessBridge.obj
 0001:0000b8e8       ?fireFocusGained@JavaAccessBridge@@QEAAXPEAUJNIEnv_@@PEAV_jobject@@11@Z 000000018000c8e8 f   JavaAccessBridge.obj
 0001:0000ba14       ?fireFocusLost@JavaAccessBridge@@QEAAXPEAUJNIEnv_@@PEAV_jobject@@11@Z 000000018000ca14 f   JavaAccessBridge.obj
 0001:0000bb40       ?fireMenuCanceled@JavaAccessBridge@@QEAAXPEAUJNIEnv_@@PEAV_jobject@@11@Z 000000018000cb40 f   JavaAccessBridge.obj
 0001:0000bc70       ?fireMenuDeselected@JavaAccessBridge@@QEAAXPEAUJNIEnv_@@PEAV_jobject@@11@Z 000000018000cc70 f   JavaAccessBridge.obj
 0001:0000bda0       ?fireMenuSelected@JavaAccessBridge@@QEAAXPEAUJNIEnv_@@PEAV_jobject@@11@Z 000000018000cda0 f   JavaAccessBridge.obj
 0001:0000bed0       ?fireMouseClicked@JavaAccessBridge@@QEAAXPEAUJNIEnv_@@PEAV_jobject@@11@Z 000000018000ced0 f   JavaAccessBridge.obj
 0001:0000bffc       ?fireMouseEntered@JavaAccessBridge@@QEAAXPEAUJNIEnv_@@PEAV_jobject@@11@Z 000000018000cffc f   JavaAccessBridge.obj
 0001:0000c128       ?fireMouseExited@JavaAccessBridge@@QEAAXPEAUJNIEnv_@@PEAV_jobject@@11@Z 000000018000d128 f   JavaAccessBridge.obj
 0001:0000c254       ?fireMousePressed@JavaAccessBridge@@QEAAXPEAUJNIEnv_@@PEAV_jobject@@11@Z 000000018000d254 f   JavaAccessBridge.obj
 0001:0000c380       ?fireMouseReleased@JavaAccessBridge@@QEAAXPEAUJNIEnv_@@PEAV_jobject@@11@Z 000000018000d380 f   JavaAccessBridge.obj
 0001:0000c4b0       ?firePopupMenuCanceled@JavaAccessBridge@@QEAAXPEAUJNIEnv_@@PEAV_jobject@@11@Z 000000018000d4b0 f   JavaAccessBridge.obj
 0001:0000c5e0       ?firePopupMenuWillBecomeInvisible@JavaAccessBridge@@QEAAXPEAUJNIEnv_@@PEAV_jobject@@11@Z 000000018000d5e0 f   JavaAccessBridge.obj
 0001:0000c710       ?firePopupMenuWillBecomeVisible@JavaAccessBridge@@QEAAXPEAUJNIEnv_@@PEAV_jobject@@11@Z 000000018000d710 f   JavaAccessBridge.obj
 0001:0000c840       ?firePropertyActiveDescendentChange@JavaAccessBridge@@QEAAXPEAUJNIEnv_@@PEAV_jobject@@1111@Z 000000018000d840 f   JavaAccessBridge.obj
 0001:0000c998       ?firePropertyCaretChange@JavaAccessBridge@@QEAAXPEAUJNIEnv_@@PEAV_jobject@@11HH@Z 000000018000d998 f   JavaAccessBridge.obj
 0001:0000cab8       ?firePropertyChildChange@JavaAccessBridge@@QEAAXPEAUJNIEnv_@@PEAV_jobject@@1111@Z 000000018000dab8 f   JavaAccessBridge.obj
 0001:0000cc10       ?firePropertyDescriptionChange@JavaAccessBridge@@QEAAXPEAUJNIEnv_@@PEAV_jobject@@11PEAV_jstring@@2@Z 000000018000dc10 f   JavaAccessBridge.obj
 0001:0000ce38       ?firePropertyNameChange@JavaAccessBridge@@QEAAXPEAUJNIEnv_@@PEAV_jobject@@11PEAV_jstring@@2@Z 000000018000de38 f   JavaAccessBridge.obj
 0001:0000d060       ?firePropertySelectionChange@JavaAccessBridge@@QEAAXPEAUJNIEnv_@@PEAV_jobject@@11@Z 000000018000e060 f   JavaAccessBridge.obj
 0001:0000d154       ?firePropertyStateChange@JavaAccessBridge@@QEAAXPEAUJNIEnv_@@PEAV_jobject@@11PEAV_jstring@@2@Z 000000018000e154 f   JavaAccessBridge.obj
 0001:0000d37c       ?firePropertyTableModelChange@JavaAccessBridge@@QEAAXPEAUJNIEnv_@@PEAV_jobject@@11PEAV_jstring@@2@Z 000000018000e37c f   JavaAccessBridge.obj
 0001:0000d5a8       ?firePropertyTextChange@JavaAccessBridge@@QEAAXPEAUJNIEnv_@@PEAV_jobject@@11@Z 000000018000e5a8 f   JavaAccessBridge.obj
 0001:0000d69c       ?firePropertyValueChange@JavaAccessBridge@@QEAAXPEAUJNIEnv_@@PEAV_jobject@@11PEAV_jstring@@2@Z 000000018000e69c f   JavaAccessBridge.obj
 0001:0000d8c4       ?firePropertyVisibleDataChange@JavaAccessBridge@@QEAAXPEAUJNIEnv_@@PEAV_jobject@@11@Z 000000018000e8c4 f   JavaAccessBridge.obj
 0001:0000d9b8       ?initWindow@JavaAccessBridge@@QEAAHXZ 000000018000e9b8 f   JavaAccessBridge.obj
 0001:0000d9fc       ?javaRun@JavaAccessBridge@@QEAAXPEAUJNIEnv_@@PEAV_jobject@@@Z 000000018000e9fc f   JavaAccessBridge.obj
 0001:0000db9c       ?javaShutdown@JavaAccessBridge@@QEAAXPEAUJNIEnv_@@PEAV_jobject@@@Z 000000018000eb9c f   JavaAccessBridge.obj
 0001:0000dc54       ?postHelloToWindowsDLLMsg@JavaAccessBridge@@QEAAXPEAUHWND__@@@Z 000000018000ec54 f   JavaAccessBridge.obj
 0001:0000dcb0       ?processPackage@JavaAccessBridge@@QEAA_JPEADH@Z 000000018000ecb0 f   JavaAccessBridge.obj
 0001:0000ee98       ?receiveMemoryPackage@JavaAccessBridge@@QEAAHPEAUHWND__@@J@Z 000000018000fe98 f   JavaAccessBridge.obj
 0001:0000ef34       ?releaseJavaObject@JavaAccessBridge@@QEAAXPEAV_jobject@@@Z 000000018000ff34 f   JavaAccessBridge.obj
 0001:0000ef9c       ?removeAccessibilityEventNotification@JavaAccessBridge@@QEAAX_JPEAUHWND__@@@Z 000000018000ff9c f   JavaAccessBridge.obj
 0001:0000f044       ?removeJavaEventNotification@JavaAccessBridge@@QEAAX_JPEAUHWND__@@@Z 0000000180010044 f   JavaAccessBridge.obj
 0001:0000f0ec       AccessBridgeDialogProc     00000001800100ec f   JavaAccessBridge.obj
 0001:0000f20c       DllMain                    000000018001020c f   JavaAccessBridge.obj
 0001:0000f284       Java_com_sun_java_accessibility_internal_AccessBridge_caretUpdate 0000000180010284 f   JavaAccessBridge.obj
 0001:0000f2a8       Java_com_sun_java_accessibility_internal_AccessBridge_focusGained 00000001800102a8 f   JavaAccessBridge.obj
 0001:0000f2cc       Java_com_sun_java_accessibility_internal_AccessBridge_focusLost 00000001800102cc f   JavaAccessBridge.obj
 0001:0000f2f0       Java_com_sun_java_accessibility_internal_AccessBridge_javaShutdown 00000001800102f0 f   JavaAccessBridge.obj
 0001:0000f304       Java_com_sun_java_accessibility_internal_AccessBridge_jawtGetComponentFromNativeWindowHandle 0000000180010304 f   JavaAccessBridge.obj
 0001:0000f348       Java_com_sun_java_accessibility_internal_AccessBridge_jawtGetNativeWindowHandleFromComponent 0000000180010348 f   JavaAccessBridge.obj
 0001:0000f3b0       Java_com_sun_java_accessibility_internal_AccessBridge_menuCanceled 00000001800103b0 f   JavaAccessBridge.obj
 0001:0000f3d4       Java_com_sun_java_accessibility_internal_AccessBridge_menuDeselected 00000001800103d4 f   JavaAccessBridge.obj
 0001:0000f3f8       Java_com_sun_java_accessibility_internal_AccessBridge_menuSelected 00000001800103f8 f   JavaAccessBridge.obj
 0001:0000f41c       Java_com_sun_java_accessibility_internal_AccessBridge_mouseClicked 000000018001041c f   JavaAccessBridge.obj
 0001:0000f440       Java_com_sun_java_accessibility_internal_AccessBridge_mouseEntered 0000000180010440 f   JavaAccessBridge.obj
 0001:0000f464       Java_com_sun_java_accessibility_internal_AccessBridge_mouseExited 0000000180010464 f   JavaAccessBridge.obj
 0001:0000f488       Java_com_sun_java_accessibility_internal_AccessBridge_mousePressed 0000000180010488 f   JavaAccessBridge.obj
 0001:0000f4ac       Java_com_sun_java_accessibility_internal_AccessBridge_mouseReleased 00000001800104ac f   JavaAccessBridge.obj
 0001:0000f4d0       Java_com_sun_java_accessibility_internal_AccessBridge_popupMenuCanceled 00000001800104d0 f   JavaAccessBridge.obj
 0001:0000f4f4       Java_com_sun_java_accessibility_internal_AccessBridge_popupMenuWillBecomeInvisible 00000001800104f4 f   JavaAccessBridge.obj
 0001:0000f518       Java_com_sun_java_accessibility_internal_AccessBridge_popupMenuWillBecomeVisible 0000000180010518 f   JavaAccessBridge.obj
 0001:0000f53c       Java_com_sun_java_accessibility_internal_AccessBridge_propertyActiveDescendentChange 000000018001053c f   JavaAccessBridge.obj
 0001:0000f574       Java_com_sun_java_accessibility_internal_AccessBridge_propertyCaretChange 0000000180010574 f   JavaAccessBridge.obj
 0001:0000f5a8       Java_com_sun_java_accessibility_internal_AccessBridge_propertyChildChange 00000001800105a8 f   JavaAccessBridge.obj
 0001:0000f5e0       Java_com_sun_java_accessibility_internal_AccessBridge_propertyDescriptionChange 00000001800105e0 f   JavaAccessBridge.obj
 0001:0000f618       Java_com_sun_java_accessibility_internal_AccessBridge_propertyNameChange 0000000180010618 f   JavaAccessBridge.obj
 0001:0000f650       Java_com_sun_java_accessibility_internal_AccessBridge_propertySelectionChange 0000000180010650 f   JavaAccessBridge.obj
 0001:0000f674       Java_com_sun_java_accessibility_internal_AccessBridge_propertyStateChange 0000000180010674 f   JavaAccessBridge.obj
 0001:0000f6ac       Java_com_sun_java_accessibility_internal_AccessBridge_propertyTableModelChange 00000001800106ac f   JavaAccessBridge.obj
 0001:0000f6e4       Java_com_sun_java_accessibility_internal_AccessBridge_propertyTextChange 00000001800106e4 f   JavaAccessBridge.obj
 0001:0000f708       Java_com_sun_java_accessibility_internal_AccessBridge_propertyValueChange 0000000180010708 f   JavaAccessBridge.obj
 0001:0000f740       Java_com_sun_java_accessibility_internal_AccessBridge_propertyVisibleDataChange 0000000180010740 f   JavaAccessBridge.obj
 0001:0000f764       Java_com_sun_java_accessibility_internal_AccessBridge_runDLL 0000000180010764 f   JavaAccessBridge.obj
 0001:0000f79c       Java_com_sun_java_accessibility_internal_AccessBridge_sendDebugString 000000018001079c f   JavaAccessBridge.obj
 0001:0000f830       ??2@YAPEAX_K@Z             0000000180010830 f   LIBCMT:new_scalar.obj
 0001:0000f86c       ??3@YAXPEAX_K@Z            000000018001086c f   LIBCMT:delete_scalar_size.obj
 0001:0000f86c       ??_V@YAXPEAX@Z             000000018001086c f   LIBCMT:delete_array.obj
 0001:0000f874       ??_U@YAPEAX_K@Z            0000000180010874 f   LIBCMT:new_array.obj
 0001:0000f87c       __GSHandlerCheck           000000018001087c f   LIBCMT:gshandler.obj
 0001:0000f89c       __GSHandlerCheckCommon     000000018001089c f   LIBCMT:gshandler.obj
 0001:0000f910       __security_check_cookie    0000000180010910 f   LIBCMT:amdsecgs.obj
 0001:0000fc40       _DllMainCRTStartup         0000000180010c40 f   LIBCMT:dll_dllmain.obj
 0001:0000fc80       ??0bad_alloc@std@@QEAA@AEBV01@@Z 0000000180010c80 f i LIBCMT:throw_bad_alloc.obj
 0001:0000fcbc       ??0bad_alloc@std@@QEAA@XZ  0000000180010cbc f i LIBCMT:throw_bad_alloc.obj
 0001:0000fcdc       ??0bad_array_new_length@std@@QEAA@AEBV01@@Z 0000000180010cdc f i LIBCMT:throw_bad_alloc.obj
 0001:0000fd18       ??0bad_array_new_length@std@@QEAA@XZ 0000000180010d18 f i LIBCMT:throw_bad_alloc.obj
 0001:0000fd38       ??0exception@std@@QEAA@AEBV01@@Z 0000000180010d38 f i LIBCMT:throw_bad_alloc.obj
 0001:0000fd6c       ??1bad_alloc@std@@UEAA@XZ  0000000180010d6c f i LIBCMT:throw_bad_alloc.obj
 0001:0000fd6c       ??1bad_array_new_length@std@@UEAA@XZ 0000000180010d6c f i LIBCMT:throw_bad_alloc.obj
 0001:0000fd6c       ??1bad_exception@std@@UEAA@XZ 0000000180010d6c f i libvcruntime:frame.obj
 0001:0000fd80       ??_Ebad_alloc@std@@UEAAPEAXI@Z 0000000180010d80 f i LIBCMT:throw_bad_alloc.obj
 0001:0000fd80       ??_Ebad_array_new_length@std@@UEAAPEAXI@Z 0000000180010d80 f i LIBCMT:throw_bad_alloc.obj
 0001:0000fd80       ??_Ebad_exception@std@@UEAAPEAXI@Z 0000000180010d80 f i libvcruntime:frame.obj
 0001:0000fd80       ??_Eexception@std@@UEAAPEAXI@Z 0000000180010d80 f i LIBCMT:throw_bad_alloc.obj
 0001:0000fd80       ??_Gbad_alloc@std@@UEAAPEAXI@Z 0000000180010d80 f i LIBCMT:throw_bad_alloc.obj
 0001:0000fd80       ??_Gbad_array_new_length@std@@UEAAPEAXI@Z 0000000180010d80 f i LIBCMT:throw_bad_alloc.obj
 0001:0000fd80       ??_Gbad_exception@std@@UEAAPEAXI@Z 0000000180010d80 f i libvcruntime:frame.obj
 0001:0000fd80       ??_Gexception@std@@UEAAPEAXI@Z 0000000180010d80 f i LIBCMT:throw_bad_alloc.obj
 0001:0000fdc4       ?__scrt_throw_std_bad_alloc@@YAXXZ 0000000180010dc4 f   LIBCMT:throw_bad_alloc.obj
 0001:0000fde4       ?__scrt_throw_std_bad_array_new_length@@YAXXZ 0000000180010de4 f   LIBCMT:throw_bad_alloc.obj
 0001:0000fe04       ?what@exception@std@@UEBAPEBDXZ 0000000180010e04 f i LIBCMT:throw_bad_alloc.obj
 0001:0000fe18       ??3@YAXPEAX@Z              0000000180010e18 f   LIBCMT:delete_scalar.obj
 0001:0000fe20       __raise_securityfailure    0000000180010e20 f   LIBCMT:gs_report.obj
 0001:0000fe54       __report_gsfailure         0000000180010e54 f   LIBCMT:gs_report.obj
 0001:0000ff9c       __security_init_cookie     0000000180010f9c f   LIBCMT:gs_support.obj
 0001:00010048       ?__scrt_initialize_type_info@@YAXXZ 0000000180011048 f   LIBCMT:tncleanup.obj
 0001:00010058       ?__scrt_uninitialize_type_info@@YAXXZ 0000000180011058 f   LIBCMT:tncleanup.obj
 0001:00010064       __local_stdio_scanf_options 0000000180011064 f i LIBCMT:default_local_stdio_options.obj
 0001:0001006c       __scrt_initialize_default_local_stdio_options 000000018001106c f   LIBCMT:default_local_stdio_options.obj
 0001:00010088       __scrt_acquire_startup_lock 0000000180011088 f   LIBCMT:utility.obj
 0001:000100c4       __scrt_dllmain_after_initialize_c 00000001800110c4 f   LIBCMT:utility.obj
 0001:000100f8       __scrt_dllmain_before_initialize_c 00000001800110f8 f   LIBCMT:utility.obj
 0001:00010110       __scrt_dllmain_crt_thread_attach 0000000180011110 f   LIBCMT:utility.obj
 0001:00010138       __scrt_dllmain_crt_thread_detach 0000000180011138 f   LIBCMT:utility.obj
 0001:00010150       __scrt_dllmain_exception_filter 0000000180011150 f   LIBCMT:utility.obj
 0001:000101b0       __scrt_dllmain_uninitialize_c 00000001800111b0 f   LIBCMT:utility.obj
 0001:000101e0       __scrt_dllmain_uninitialize_critical 00000001800111e0 f   LIBCMT:utility.obj
 0001:000101f4       __scrt_initialize_crt      00000001800111f4 f   LIBCMT:utility.obj
 0001:00010230       __scrt_initialize_onexit_tables 0000000180011230 f   LIBCMT:utility.obj
 0001:000102bc       __scrt_is_nonwritable_in_current_image 00000001800112bc f   LIBCMT:utility.obj
 0001:00010354       __scrt_release_startup_lock 0000000180011354 f   LIBCMT:utility.obj
 0001:00010378       __scrt_uninitialize_crt    0000000180011378 f   LIBCMT:utility.obj
 0001:000103a4       __scrt_get_dyn_tls_init_callback 00000001800113a4 f   LIBCMT:dyn_tls_init.obj
 0001:000103ac       __crt_debugger_hook        00000001800113ac f   LIBCMT:utility_desktop.obj
 0001:000103b4       __scrt_fastfail            00000001800113b4 f   LIBCMT:utility_desktop.obj
 0001:000104fc       _RTC_Initialize            00000001800114fc f   LIBCMT:initsect.obj
 0001:00010538       _RTC_Terminate             0000000180011538 f   LIBCMT:initsect.obj
 0001:00010574       _guard_check_icall_nop     0000000180011574 f i LIBCMT:guard_support.obj
 0001:00010578       ??_Etype_info@@UEAAPEAXI@Z 0000000180011578 f i LIBCMT:std_type_info_static.obj
 0001:00010578       ??_Gtype_info@@UEAAPEAXI@Z 0000000180011578 f i LIBCMT:std_type_info_static.obj
 0001:000105a4       __isa_available_init       00000001800115a4 f   LIBCMT:cpu_disp.obj
 0001:00010870       _get_startup_argv_mode     0000000180011870 f   LIBCMT:argv_mode.obj
 0001:00010878       __scrt_is_ucrt_dll_in_use  0000000180011878 f   LIBCMT:ucrt_detection.obj
 0001:00010890       __C_specific_handler       0000000180011890 f   libvcruntime:riscchandler.obj
 0001:00010aa8       __std_exception_copy       0000000180011aa8 f   libvcruntime:std_exception.obj
 0001:00010b38       __std_exception_destroy    0000000180011b38 f   libvcruntime:std_exception.obj
 0001:00010b60       _CxxThrowException         0000000180011b60 f   libvcruntime:throw.obj
 0001:00010c08       __std_type_info_compare    0000000180011c08 f   libvcruntime:std_type_info.obj
 0001:00010c30       __std_type_info_destroy_list 0000000180011c30 f   libvcruntime:std_type_info.obj
 0001:00010c5c       __vcrt_initialize          0000000180011c5c f   libvcruntime:initialization.obj
 0001:00010c84       __vcrt_thread_attach       0000000180011c84 f   libvcruntime:initialization.obj
 0001:00010c98       __vcrt_thread_detach       0000000180011c98 f   libvcruntime:initialization.obj
 0001:00010ca8       __vcrt_uninitialize        0000000180011ca8 f   libvcruntime:initialization.obj
 0001:00010cc4       __vcrt_uninitialize_critical 0000000180011cc4 f   libvcruntime:initialization.obj
 0001:00010cd4       __DestructExceptionObject  0000000180011cd4 f   libvcruntime:ehhelpers.obj
 0001:00010d44       ?_CallMemberFunction0@@YAXQEAX0@Z 0000000180011d44 f i libvcruntime:ehhelpers.obj
 0001:00010d48       _IsExceptionObjectToBeDestroyed 0000000180011d48 f   libvcruntime:ehhelpers.obj
 0001:00010d78       __AdjustPointer            0000000180011d78 f   libvcruntime:ehhelpers.obj
 0001:00010d9c       __FrameUnwindFilter        0000000180011d9c f   libvcruntime:ehhelpers.obj
 0001:00010e04       __std_terminate            0000000180011e04 f   libvcruntime:ehhelpers.obj
 0001:00010e40       _NLG_Notify                0000000180011e40 f   libvcruntime:notify.obj
 0001:00010e60       __NLG_Dispatch2            0000000180011e60 f   libvcruntime:notify.obj
 0001:00010e70       __NLG_Return2              0000000180011e70 f   libvcruntime:notify.obj
 0001:00010e74       __except_validate_context_record 0000000180011e74 f   libvcruntime:jbcxrval.obj
 0001:00010eac       __vcrt_freefls             0000000180011eac f   libvcruntime:per_thread_data.obj
 0001:00010ecc       __vcrt_freeptd_for_this_thread 0000000180011ecc f   libvcruntime:per_thread_data.obj
 0001:00010f14       __vcrt_getptd              0000000180011f14 f   libvcruntime:per_thread_data.obj
 0001:00010f30       __vcrt_getptd_noexit       0000000180011f30 f   libvcruntime:per_thread_data.obj
 0001:00010ff0       __vcrt_initialize_ptd      0000000180011ff0 f   libvcruntime:per_thread_data.obj
 0001:00011038       __vcrt_uninitialize_ptd    0000000180012038 f   libvcruntime:per_thread_data.obj
 0001:0001105c       __vcrt_initialize_locks    000000018001205c f   libvcruntime:locks.obj
 0001:000110a4       __vcrt_uninitialize_locks  00000001800120a4 f   libvcruntime:locks.obj
 0001:000110dc       ??$_CallSETranslator@V__FrameHandler3@@@@YAHPEAUEHExceptionRecord@@PEA_KPEAU_CONTEXT@@PEAU_xDISPATCHER_CONTEXT@@PEBU_s_FuncInfo@@K1H@Z 00000001800120dc f i libvcruntime:risctrnsctrl.obj
 0001:00011130       ?CatchTryBlock@__FrameHandler3@@SAPEBU_s_TryBlockMapEntry@@PEBU_s_FuncInfo@@H@Z 0000000180012130 f   libvcruntime:risctrnsctrl.obj
 0001:00011194       ?ExecutionInCatch@__FrameHandler3@@SA_NPEAU_xDISPATCHER_CONTEXT@@PEBU_s_FuncInfo@@@Z 0000000180012194 f   libvcruntime:risctrnsctrl.obj
 0001:000111c0       ?FrameUnwindToEmptyState@__FrameHandler3@@SAXPEA_KPEAU_xDISPATCHER_CONTEXT@@PEBU_s_FuncInfo@@@Z 00000001800121c0 f   libvcruntime:risctrnsctrl.obj
 0001:00011224       ?GetEstablisherFrame@__FrameHandler3@@SAPEA_KPEA_KPEAU_xDISPATCHER_CONTEXT@@PEBU_s_FuncInfo@@0@Z 0000000180012224 f   libvcruntime:risctrnsctrl.obj
 0001:000112f4       ?GetRangeOfTrysToCheck@__FrameHandler3@@SA?AU?$pair@Viterator@TryBlockMap@__FrameHandler3@@V123@@std@@AEAVTryBlockMap@1@HPEAU_xDISPATCHER_CONTEXT@@PEBU_s_FuncInfo@@H@Z 00000001800122f4 f   libvcruntime:risctrnsctrl.obj
 0001:00011428       ?UnwindNestedFrames@__FrameHandler3@@SAXPEA_KPEAUEHExceptionRecord@@PEAU_CONTEXT@@0PEAXPEBU_s_FuncInfo@@HHPEBU_s_HandlerType@@PEAU_xDISPATCHER_CONTEXT@@E@Z 0000000180012428 f   libvcruntime:risctrnsctrl.obj
 0001:0001152c       _CreateFrameInfo           000000018001252c f   libvcruntime:risctrnsctrl.obj
 0001:00011568       _FindAndUnlinkFrame        0000000180012568 f   libvcruntime:risctrnsctrl.obj
 0001:000115bc       _GetImageBase              00000001800125bc f   libvcruntime:risctrnsctrl.obj
 0001:000115d0       _GetThrowImageBase         00000001800125d0 f   libvcruntime:risctrnsctrl.obj
 0001:000115e4       _SetImageBase              00000001800125e4 f   libvcruntime:risctrnsctrl.obj
 0001:000115fc       _SetThrowImageBase         00000001800125fc f   libvcruntime:risctrnsctrl.obj
 0001:00011614       __CxxFrameHandler3         0000000180012614 f   libvcruntime:risctrnsctrl.obj
 0001:000117ec       __vcrt_FlsAlloc            00000001800127ec f   libvcruntime:winapi_downlevel.obj
 0001:00011834       __vcrt_FlsFree             0000000180012834 f   libvcruntime:winapi_downlevel.obj
 0001:0001187c       __vcrt_FlsGetValue         000000018001287c f   libvcruntime:winapi_downlevel.obj
 0001:000118c4       __vcrt_FlsSetValue         00000001800128c4 f   libvcruntime:winapi_downlevel.obj
 0001:00011918       __vcrt_InitializeCriticalSectionEx 0000000180012918 f   libvcruntime:winapi_downlevel.obj
 0001:0001197c       ?GetCurrentState@__FrameHandler3@@SAHPEA_KPEAU_xDISPATCHER_CONTEXT@@PEBU_s_FuncInfo@@@Z 000000018001297c f   libvcruntime:ehstate.obj
 0001:000119a4       ?GetUnwindTryBlock@__FrameHandler3@@SAHPEA_KPEAU_xDISPATCHER_CONTEXT@@PEBU_s_FuncInfo@@@Z 00000001800129a4 f   libvcruntime:ehstate.obj
 0001:000119d0       ?SetState@__FrameHandler3@@SAXPEA_KPEBU_s_FuncInfo@@H@Z 00000001800129d0 f   libvcruntime:ehstate.obj
 0001:000119dc       ?SetUnwindTryBlock@__FrameHandler3@@SAXPEA_KPEAU_xDISPATCHER_CONTEXT@@PEBU_s_FuncInfo@@H@Z 00000001800129dc f   libvcruntime:ehstate.obj
 0001:00011a18       ?StateFromControlPc@__FrameHandler3@@SAHPEBU_s_FuncInfo@@PEAU_xDISPATCHER_CONTEXT@@@Z 0000000180012a18 f   libvcruntime:ehstate.obj
 0001:00011a20       ?StateFromIp@__FrameHandler3@@SAHPEBU_s_FuncInfo@@PEAU_xDISPATCHER_CONTEXT@@_K@Z 0000000180012a20 f   libvcruntime:ehstate.obj
 0001:0001255c       ??$TypeMatchHelper@V__FrameHandler3@@@@YAHPEBU_s_HandlerType@@PEBU_s_CatchableType@@PEBU_s_ThrowInfo@@@Z 000000018001355c f i libvcruntime:frame.obj
 0001:0001269c       ??$__InternalCxxFrameHandler@V__FrameHandler3@@@@YA?AW4_EXCEPTION_DISPOSITION@@PEAUEHExceptionRecord@@PEA_KPEAU_CONTEXT@@PEAU_xDISPATCHER_CONTEXT@@PEBU_s_FuncInfo@@H1E@Z 000000018001369c f i libvcruntime:frame.obj
 0001:000128d4       ??$__InternalCxxFrameHandlerWrapper@V__FrameHandler3@@@@YA?AW4_EXCEPTION_DISPOSITION@@PEAUEHExceptionRecord@@PEA_KPEAU_CONTEXT@@PEAU_xDISPATCHER_CONTEXT@@PEBU_s_FuncInfo@@H1E@Z 00000001800138d4 f i libvcruntime:frame.obj
 0001:000128dc       ??0bad_exception@std@@QEAA@AEBV01@@Z 00000001800138dc f i libvcruntime:frame.obj
 0001:00012918       ??0bad_exception@std@@QEAA@XZ 0000000180013918 f i libvcruntime:frame.obj
 0001:00012938       ?CxxCallCatchBlock@__FrameHandler3@@SAPEAXPEAU_EXCEPTION_RECORD@@@Z 0000000180013938 f   libvcruntime:frame.obj
 0001:00012ba8       ?FrameUnwindToState@__FrameHandler3@@SAXPEA_KPEAU_xDISPATCHER_CONTEXT@@PEBU_s_FuncInfo@@H@Z 0000000180013ba8 f   libvcruntime:frame.obj
 0001:00012d34       ?GetHandlerSearchState@__FrameHandler3@@SAHPEA_KPEAU_xDISPATCHER_CONTEXT@@PEBU_s_FuncInfo@@@Z 0000000180013d34 f i libvcruntime:frame.obj
 0001:00012f44       ?_CallMemberFunction1@@YAXQEAX00@Z 0000000180013f44 f i libvcruntime:frame.obj
 0001:00012f50       ?_CallMemberFunction2@@YAXQEAX00H@Z 0000000180013f50 f i libvcruntime:frame.obj
 0001:00012fa0       _CallSettingFrame          0000000180013fa0 f   libvcruntime:handlers.obj
 0001:00013110       _beginthreadex             0000000180014110 f   libucrt:thread.obj
 0001:000131f0       _endthreadex               00000001800141f0 f   libucrt:thread.obj
 0001:00013200       __acrt_initialize_stdio    0000000180014200 f   libucrt:_file.obj
 0001:00013320       __acrt_iob_func            0000000180014320 f   libucrt:_file.obj
 0001:00013334       __acrt_uninitialize_stdio  0000000180014334 f   libucrt:_file.obj
 0001:00013390       _lock_file                 0000000180014390 f   libucrt:_file.obj
 0001:0001339c       _unlock_file               000000018001439c f   libucrt:_file.obj
 0001:00013428       ??$ensure_buffer_is_big_enough@D@formatting_buffer@__crt_stdio_output@@QEAA_N_KAEAV__crt_cached_ptd_host@@@Z 0000000180014428 f i libucrt:output.obj
 0001:000134d0       ??$ensure_buffer_is_big_enough@_W@formatting_buffer@__crt_stdio_output@@QEAA_N_KAEAV__crt_cached_ptd_host@@@Z 00000001800144d0 f i libucrt:output.obj
 0001:0001357c       ??$is_wide_character_specifier@_W@__crt_stdio_output@@YA_N_K_WW4length_modifier@0@@Z 000000018001457c f i libucrt:output.obj
 0001:000135bc       ??$parse_integer@KV?$c_string_character_source@D@__crt_strtox@@$0A@@__crt_strtox@@YAKAEAV__crt_cached_ptd_host@@V?$c_string_character_source@D@0@H_N@Z 00000001800145bc f i libucrt:output.obj
 0001:00013870       ??$parse_integer@KV?$c_string_character_source@_W@__crt_strtox@@$0A@@__crt_strtox@@YAKAEAV__crt_cached_ptd_host@@V?$c_string_character_source@_W@0@H_N@Z 0000000180014870 f i libucrt:output.obj
 0001:00013fdc       ??$type_case_integer@$07@?$output_processor@DV?$stream_output_adapter@D@__crt_stdio_output@@V?$standard_base@DV?$stream_output_adapter@D@__crt_stdio_output@@@2@@__crt_stdio_output@@AEAA_N_N@Z 0000000180014fdc f i libucrt:output.obj
 0001:000141e0       ??$type_case_integer@$07@?$output_processor@_WV?$stream_output_adapter@_W@__crt_stdio_output@@V?$standard_base@_WV?$stream_output_adapter@_W@__crt_stdio_output@@@2@@__crt_stdio_output@@AEAA_N_N@Z 00000001800151e0 f i libucrt:output.obj
 0001:000143ec       ??$type_case_integer@$09@?$output_processor@DV?$stream_output_adapter@D@__crt_stdio_output@@V?$standard_base@DV?$stream_output_adapter@D@__crt_stdio_output@@@2@@__crt_stdio_output@@AEAA_N_N@Z 00000001800153ec f i libucrt:output.obj
 0001:000145f0       ??$type_case_integer@$09@?$output_processor@_WV?$stream_output_adapter@_W@__crt_stdio_output@@V?$standard_base@_WV?$stream_output_adapter@_W@__crt_stdio_output@@@2@@__crt_stdio_output@@AEAA_N_N@Z 00000001800155f0 f i libucrt:output.obj
 0001:000147fc       ??$type_case_integer@$0BA@@?$output_processor@DV?$stream_output_adapter@D@__crt_stdio_output@@V?$standard_base@DV?$stream_output_adapter@D@__crt_stdio_output@@@2@@__crt_stdio_output@@AEAA_N_N@Z 00000001800157fc f i libucrt:output.obj
 0001:00014a00       ??$type_case_integer@$0BA@@?$output_processor@_WV?$stream_output_adapter@_W@__crt_stdio_output@@V?$standard_base@_WV?$stream_output_adapter@_W@__crt_stdio_output@@@2@@__crt_stdio_output@@AEAA_N_N@Z 0000000180015a00 f i libucrt:output.obj
 0001:00014c0c       ??$type_case_integer_parse_into_buffer@I$07@?$output_processor@DV?$stream_output_adapter@D@__crt_stdio_output@@V?$standard_base@DV?$stream_output_adapter@D@__crt_stdio_output@@@2@@__crt_stdio_output@@AEAAXI_N@Z 0000000180015c0c f i libucrt:output.obj
 0001:00014c7c       ??$type_case_integer_parse_into_buffer@I$07@?$output_processor@_WV?$stream_output_adapter@_W@__crt_stdio_output@@V?$standard_base@_WV?$stream_output_adapter@_W@__crt_stdio_output@@@2@@__crt_stdio_output@@AEAAXI_N@Z 0000000180015c7c f i libucrt:output.obj
 0001:00014d00       ??$type_case_integer_parse_into_buffer@I$09@?$output_processor@DV?$stream_output_adapter@D@__crt_stdio_output@@V?$standard_base@DV?$stream_output_adapter@D@__crt_stdio_output@@@2@@__crt_stdio_output@@AEAAXI_N@Z 0000000180015d00 f i libucrt:output.obj
 0001:00014dac       ??$type_case_integer_parse_into_buffer@I$09@?$output_processor@_WV?$stream_output_adapter@_W@__crt_stdio_output@@V?$standard_base@_WV?$stream_output_adapter@_W@__crt_stdio_output@@@2@@__crt_stdio_output@@AEAAXI_N@Z 0000000180015dac f i libucrt:output.obj
 0001:00014e6c       ??$type_case_integer_parse_into_buffer@I$0BA@@?$output_processor@DV?$stream_output_adapter@D@__crt_stdio_output@@V?$standard_base@DV?$stream_output_adapter@D@__crt_stdio_output@@@2@@__crt_stdio_output@@AEAAXI_N@Z 0000000180015e6c f i libucrt:output.obj
 0001:00014ef0       ??$type_case_integer_parse_into_buffer@I$0BA@@?$output_processor@_WV?$stream_output_adapter@_W@__crt_stdio_output@@V?$standard_base@_WV?$stream_output_adapter@_W@__crt_stdio_output@@@2@@__crt_stdio_output@@AEAAXI_N@Z 0000000180015ef0 f i libucrt:output.obj
 0001:00014f90       ??$type_case_integer_parse_into_buffer@_K$07@?$output_processor@DV?$stream_output_adapter@D@__crt_stdio_output@@V?$standard_base@DV?$stream_output_adapter@D@__crt_stdio_output@@@2@@__crt_stdio_output@@AEAAX_K_N@Z 0000000180015f90 f i libucrt:output.obj
 0001:00015000       ??$type_case_integer_parse_into_buffer@_K$07@?$output_processor@_WV?$stream_output_adapter@_W@__crt_stdio_output@@V?$standard_base@_WV?$stream_output_adapter@_W@__crt_stdio_output@@@2@@__crt_stdio_output@@AEAAX_K_N@Z 0000000180016000 f i libucrt:output.obj
 0001:00015088       ??$type_case_integer_parse_into_buffer@_K$09@?$output_processor@DV?$stream_output_adapter@D@__crt_stdio_output@@V?$standard_base@DV?$stream_output_adapter@D@__crt_stdio_output@@@2@@__crt_stdio_output@@AEAAX_K_N@Z 0000000180016088 f i libucrt:output.obj
 0001:00015138       ??$type_case_integer_parse_into_buffer@_K$09@?$output_processor@_WV?$stream_output_adapter@_W@__crt_stdio_output@@V?$standard_base@_WV?$stream_output_adapter@_W@__crt_stdio_output@@@2@@__crt_stdio_output@@AEAAX_K_N@Z 0000000180016138 f i libucrt:output.obj
 0001:000151fc       ??$type_case_integer_parse_into_buffer@_K$0BA@@?$output_processor@DV?$stream_output_adapter@D@__crt_stdio_output@@V?$standard_base@DV?$stream_output_adapter@D@__crt_stdio_output@@@2@@__crt_stdio_output@@AEAAX_K_N@Z 00000001800161fc f i libucrt:output.obj
 0001:00015280       ??$type_case_integer_parse_into_buffer@_K$0BA@@?$output_processor@_WV?$stream_output_adapter@_W@__crt_stdio_output@@V?$standard_base@_WV?$stream_output_adapter@_W@__crt_stdio_output@@@2@@__crt_stdio_output@@AEAAX_K_N@Z 0000000180016280 f i libucrt:output.obj
 0001:00015558       ?crop_zeroes@__crt_stdio_output@@YAXPEADQEAU__crt_locale_pointers@@@Z 0000000180016558 f i libucrt:output.obj
 0001:000155d0       ?get_raw_ptd@__crt_cached_ptd_host@@QEAAPEAU__acrt_ptd@@XZ 00000001800165d0 f i libucrt:output.obj
 0001:00015638       ?parse_int_from_format_string@?$output_processor@DV?$stream_output_adapter@D@__crt_stdio_output@@V?$standard_base@DV?$stream_output_adapter@D@__crt_stdio_output@@@2@@__crt_stdio_output@@AEAA_NQEAH@Z 0000000180016638 f i libucrt:output.obj
 0001:000156c8       ?parse_int_from_format_string@?$output_processor@_WV?$stream_output_adapter@_W@__crt_stdio_output@@V?$standard_base@_WV?$stream_output_adapter@_W@__crt_stdio_output@@@2@@__crt_stdio_output@@AEAA_NQEAH@Z 00000001800166c8 f i libucrt:output.obj
 0001:00015758       ?process@?$output_processor@DV?$stream_output_adapter@D@__crt_stdio_output@@V?$standard_base@DV?$stream_output_adapter@D@__crt_stdio_output@@@2@@__crt_stdio_output@@QEAAHXZ 0000000180016758 f i libucrt:output.obj
 0001:00015adc       ?process@?$output_processor@_WV?$stream_output_adapter@_W@__crt_stdio_output@@V?$standard_base@_WV?$stream_output_adapter@_W@__crt_stdio_output@@@2@@__crt_stdio_output@@QEAAHXZ 0000000180016adc f i libucrt:output.obj
 0001:00015d9c       ?state_case_size@?$output_processor@DV?$stream_output_adapter@D@__crt_stdio_output@@V?$standard_base@DV?$stream_output_adapter@D@__crt_stdio_output@@@2@@__crt_stdio_output@@AEAA_NXZ 0000000180016d9c f i libucrt:output.obj
 0001:00015f24       ?state_case_size@?$output_processor@_WV?$stream_output_adapter@_W@__crt_stdio_output@@V?$standard_base@_WV?$stream_output_adapter@_W@__crt_stdio_output@@@2@@__crt_stdio_output@@AEAA_NXZ 0000000180016f24 f i libucrt:output.obj
 0001:000160d4       ?state_case_type@?$output_processor@DV?$stream_output_adapter@D@__crt_stdio_output@@V?$standard_base@DV?$stream_output_adapter@D@__crt_stdio_output@@@2@@__crt_stdio_output@@AEAA_NXZ 00000001800170d4 f i libucrt:output.obj
 0001:0001660c       ?state_case_type@?$output_processor@_WV?$stream_output_adapter@_W@__crt_stdio_output@@V?$standard_base@_WV?$stream_output_adapter@_W@__crt_stdio_output@@@2@@__crt_stdio_output@@AEAA_NXZ 000000018001760c f i libucrt:output.obj
 0001:00016c08       ?type_case_Z@?$output_processor@DV?$stream_output_adapter@D@__crt_stdio_output@@V?$standard_base@DV?$stream_output_adapter@D@__crt_stdio_output@@@2@@__crt_stdio_output@@AEAA_NXZ 0000000180017c08 f i libucrt:output.obj
 0001:00016c84       ?type_case_Z@?$output_processor@_WV?$stream_output_adapter@_W@__crt_stdio_output@@V?$standard_base@_WV?$stream_output_adapter@_W@__crt_stdio_output@@@2@@__crt_stdio_output@@AEAA_NXZ 0000000180017c84 f i libucrt:output.obj
 0001:00016cf8       ?type_case_a@?$output_processor@DV?$stream_output_adapter@D@__crt_stdio_output@@V?$standard_base@DV?$stream_output_adapter@D@__crt_stdio_output@@@2@@__crt_stdio_output@@AEAA_NXZ 0000000180017cf8 f i libucrt:output.obj
 0001:00016f54       ?type_case_a@?$output_processor@_WV?$stream_output_adapter@_W@__crt_stdio_output@@V?$standard_base@_WV?$stream_output_adapter@_W@__crt_stdio_output@@@2@@__crt_stdio_output@@AEAA_NXZ 0000000180017f54 f i libucrt:output.obj
 0001:000171d0       ?type_case_c_tchar@?$output_processor@DV?$stream_output_adapter@D@__crt_stdio_output@@V?$standard_base@DV?$stream_output_adapter@D@__crt_stdio_output@@@2@@__crt_stdio_output@@AEAA_ND@Z 00000001800181d0 f i libucrt:output.obj
 0001:000172a4       ?type_case_c_tchar@?$output_processor@_WV?$stream_output_adapter@_W@__crt_stdio_output@@V?$standard_base@_WV?$stream_output_adapter@_W@__crt_stdio_output@@@2@@__crt_stdio_output@@AEAA_N_W@Z 00000001800182a4 f i libucrt:output.obj
 0001:00017368       ?type_case_n@?$output_processor@DV?$stream_output_adapter@D@__crt_stdio_output@@V?$standard_base@DV?$stream_output_adapter@D@__crt_stdio_output@@@2@@__crt_stdio_output@@AEAA_NXZ 0000000180018368 f i libucrt:output.obj
 0001:00017368       ?type_case_n@?$output_processor@_WV?$stream_output_adapter@_W@__crt_stdio_output@@V?$standard_base@_WV?$stream_output_adapter@_W@__crt_stdio_output@@@2@@__crt_stdio_output@@AEAA_NXZ 0000000180018368 f i libucrt:output.obj
 0001:00017420       ?type_case_s@?$output_processor@DV?$stream_output_adapter@D@__crt_stdio_output@@V?$standard_base@DV?$stream_output_adapter@D@__crt_stdio_output@@@2@@__crt_stdio_output@@AEAA_NXZ 0000000180018420 f i libucrt:output.obj
 0001:000174bc       ?type_case_s@?$output_processor@_WV?$stream_output_adapter@_W@__crt_stdio_output@@V?$standard_base@_WV?$stream_output_adapter@_W@__crt_stdio_output@@@2@@__crt_stdio_output@@AEAA_NXZ 00000001800184bc f i libucrt:output.obj
 0001:00017558       ?type_case_s_compute_narrow_string_length@?$output_processor@_WV?$stream_output_adapter@_W@__crt_stdio_output@@V?$standard_base@_WV?$stream_output_adapter@_W@__crt_stdio_output@@@2@@__crt_stdio_output@@AEAAHH_W@Z 0000000180018558 f i libucrt:output.obj
 0001:00017620       ?update_locale_slow@__crt_cached_ptd_host@@AEAAXXZ 0000000180018620 f i libucrt:output.obj
 0001:00017698       ?validate_stream_is_ansi_if_required@?$__acrt_stdio_char_traits@D@@SA_NQEAU_iobuf@@@Z 0000000180018698 f i libucrt:output.obj
 0001:00017734       ?write_string_impl@?$output_adapter_common@DV?$stream_output_adapter@D@__crt_stdio_output@@@__crt_stdio_output@@IEBAXQEBDHQEAHAEAV__crt_cached_ptd_host@@@Z 0000000180018734 f i libucrt:output.obj
 0001:00017804       ?write_string_impl@?$output_adapter_common@_WV?$stream_output_adapter@_W@__crt_stdio_output@@@__crt_stdio_output@@IEBAXQEB_WHQEAHAEAV__crt_cached_ptd_host@@@Z 0000000180018804 f i libucrt:output.obj
 0001:000178e8       __stdio_common_vfprintf    00000001800188e8 f   libucrt:output.obj
 0001:00017a0c       __stdio_common_vfwprintf   0000000180018a0c f   libucrt:output.obj
 0001:00017c54       fclose                     0000000180018c54 f   libucrt:fclose.obj
 0001:00017da8       fopen                      0000000180018da8 f   libucrt:fopen.obj
 0001:00017ea0       getenv                     0000000180018ea0 f   libucrt:getenv.obj
 0001:00017ea8       wcscmp                     0000000180018ea8 f   libucrt:wcscmpc.obj
 0001:00017ee0       strnlen                    0000000180018ee0 f   libucrt:strnlen.obj
 0001:0001804c       wcslen                     000000018001904c f   libucrt:strnlen.obj
 0001:00018178       wcsnlen                    0000000180019178 f   libucrt:strnlen.obj
 0001:0001836c       wcsncpy                    000000018001936c f   libucrt:wcsncpy.obj
 0001:000183f0       _callnewh                  00000001800193f0 f   libucrt:new_handler.obj
 0001:00018430       __acrt_initialize_new_handler 0000000180019430 f   libucrt:new_handler.obj
 0001:00018440       _query_new_handler         0000000180019440 f   libucrt:new_handler.obj
 0001:00018480       _set_new_handler           0000000180019480 f   libucrt:new_handler.obj
 0001:000184e0       ?_set_new_handler@@YAP6AH_K@ZH@Z 00000001800194e0 f   libucrt:new_handler.obj
 0001:000184f0       malloc                     00000001800194f0 f   libucrt:malloc.obj
 0001:000184f8       _initterm                  00000001800194f8 f   libucrt:initterm.obj
 0001:00018530       _initterm_e                0000000180019530 f   libucrt:initterm.obj
 0001:00018570       free                       0000000180019570 f   libucrt:free.obj
 0001:00018578       _seh_filter_dll            0000000180019578 f   libucrt:exception_filter.obj
 0001:0001858c       _seh_filter_exe            000000018001958c f   libucrt:exception_filter.obj
 0001:00018968       __acrt_initialize_thread_local_exit_callback 0000000180019968 f   libucrt:exit.obj
 0001:00018970       _cexit                     0000000180019970 f   libucrt:exit.obj
 0001:00018980       _exit                      0000000180019980 f   libucrt:exit.obj
 0001:0001898c       _is_c_termination_complete 000000018001998c f   libucrt:exit.obj
 0001:00018b54       __acrt_allocate_buffer_for_argv 0000000180019b54 f   libucrt:argv_parsing.obj
 0001:00018bb4       _configure_narrow_argv     0000000180019bb4 f   libucrt:argv_parsing.obj
 0001:00019018       __dcrt_get_or_create_narrow_environment_nolock 000000018001a018 f   libucrt:environment_initialization.obj
 0001:00019054       __dcrt_uninitialize_environments_nolock 000000018001a054 f   libucrt:environment_initialization.obj
 0001:00019098       _initialize_narrow_environment 000000018001a098 f   libucrt:environment_initialization.obj
 0001:000191f4       _execute_onexit_table      000000018001a1f4 f   libucrt:onexit.obj
 0001:00019238       _initialize_onexit_table   000000018001a238 f   libucrt:onexit.obj
 0001:00019298       __acrt_uninitialize_command_line 000000018001a298 f   libucrt:argv_data.obj
 0001:00019390       __acrt_initialize          000000018001a390 f   libucrt:initialization.obj
 0001:000193a4       __acrt_thread_attach       000000018001a3a4 f   libucrt:initialization.obj
 0001:000193b8       __acrt_thread_detach       000000018001a3b8 f   libucrt:initialization.obj
 0001:000193c8       __acrt_uninitialize        000000018001a3c8 f   libucrt:initialization.obj
 0001:00019400       __acrt_uninitialize_critical 000000018001a400 f   libucrt:initialization.obj
 0001:00019410       terminate                  000000018001a410 f   libucrt:terminate.obj
 0001:00019430       strcpy_s                   000000018001a430 f   libucrt:strcpy_s.obj
 0001:00019490       abort                      000000018001a490 f   libucrt:abort.obj
 0001:000194f0       calloc                     000000018001a4f0 f   libucrt:calloc.obj
 0001:000194f8       wcsncmp                    000000018001a4f8 f   libucrt:wcsncmp.obj
 0001:00019524       ?get_raw_ptd_noexit@__crt_cached_ptd_host@@QEAAPEAU__acrt_ptd@@XZ 000000018001a524 f i libucrt:invalid_parameter.obj
 0001:00019590       ?value@?$dual_state_global@P6AXPEB_W00I_K@Z@__crt_state_management@@QEAAAEAP6AXPEB_W00I_K@ZAEAV__crt_cached_ptd_host@@@Z 000000018001a590 f i libucrt:invalid_parameter.obj
 0001:000195dc       __acrt_call_reportfault    000000018001a5dc f   libucrt:invalid_parameter.obj
 0001:0001974c       __acrt_initialize_invalid_parameter_handler 000000018001a74c f   libucrt:invalid_parameter.obj
 0001:00019754       _invalid_parameter         000000018001a754 f   libucrt:invalid_parameter.obj
 0001:000197f0       _invalid_parameter_internal 000000018001a7f0 f   libucrt:invalid_parameter.obj
 0001:000198a8       _invalid_parameter_noinfo  000000018001a8a8 f   libucrt:invalid_parameter.obj
 0001:000198c8       _invoke_watson             000000018001a8c8 f   libucrt:invalid_parameter.obj
 0001:00019910       __acrt_errno_from_os_error 000000018001a910 f   libucrt:errno.obj
 0001:000199e0       __acrt_errno_map_os_error  000000018001a9e0 f   libucrt:errno.obj
 0001:00019a08       __acrt_errno_map_os_error_ptd 000000018001aa08 f   libucrt:errno.obj
 0001:00019a2c       __doserrno                 000000018001aa2c f   libucrt:errno.obj
 0001:00019a50       _errno                     000000018001aa50 f   libucrt:errno.obj
 0001:00019a80       _calloc_base               000000018001aa80 f   libucrt:calloc_base.obj
 0001:00019b00       _free_base                 000000018001ab00 f   libucrt:free_base.obj
 0001:00019e68       ?internal_get_ptd_head_slow@@YAPEAU__acrt_ptd@@XZ 000000018001ae68 f   libucrt:per_thread_data.obj
 0001:00019f88       __acrt_freeptd             000000018001af88 f   libucrt:per_thread_data.obj
 0001:00019fd8       __acrt_getptd              000000018001afd8 f   libucrt:per_thread_data.obj
 0001:00019ff4       __acrt_getptd_head         000000018001aff4 f   libucrt:per_thread_data.obj
 0001:0001a038       __acrt_getptd_noexit       000000018001b038 f   libucrt:per_thread_data.obj
 0001:0001a0c8       __acrt_getptd_noexit_explicit 000000018001b0c8 f   libucrt:per_thread_data.obj
 0001:0001a124       __acrt_initialize_ptd      000000018001b124 f   libucrt:per_thread_data.obj
 0001:0001a168       __acrt_uninitialize_ptd    000000018001b168 f   libucrt:per_thread_data.obj
 0001:0001a378       __acrt_AppPolicyGetProcessTerminationMethodInternal 000000018001b378 f   libucrt:winapi_thunks.obj
 0001:0001a3d4       __acrt_AppPolicyGetThreadInitializationTypeInternal 000000018001b3d4 f   libucrt:winapi_thunks.obj
 0001:0001a430       __acrt_AreFileApisANSI     000000018001b430 f   libucrt:winapi_thunks.obj
 0001:0001a47c       __acrt_CompareStringEx     000000018001b47c f   libucrt:winapi_thunks.obj
 0001:0001a540       __acrt_FlsAlloc            000000018001b540 f   libucrt:winapi_thunks.obj
 0001:0001a548       __acrt_FlsFree             000000018001b548 f   libucrt:winapi_thunks.obj
 0001:0001a550       __acrt_FlsGetValue         000000018001b550 f   libucrt:winapi_thunks.obj
 0001:0001a558       __acrt_FlsGetValue2        000000018001b558 f   libucrt:winapi_thunks.obj
 0001:0001a564       __acrt_FlsSetValue         000000018001b564 f   libucrt:winapi_thunks.obj
 0001:0001a56c       __acrt_InitializeCriticalSectionEx 000000018001b56c f   libucrt:winapi_thunks.obj
 0001:0001a574       __acrt_LCMapStringEx       000000018001b574 f   libucrt:winapi_thunks.obj
 0001:0001a668       __acrt_LocaleNameToLCID    000000018001b668 f   libucrt:winapi_thunks.obj
 0001:0001a6cc       __acrt_RoInitialize        000000018001b6cc f   libucrt:winapi_thunks.obj
 0001:0001a71c       __acrt_RoUninitialize      000000018001b71c f   libucrt:winapi_thunks.obj
 0001:0001a760       __acrt_initialize_winapi_thunks 000000018001b760 f   libucrt:winapi_thunks.obj
 0001:0001a790       __acrt_tls2_supported      000000018001b790 f   libucrt:winapi_thunks.obj
 0001:0001a7d4       __acrt_uninitialize_winapi_thunks 000000018001b7d4 f   libucrt:winapi_thunks.obj
 0001:0001a818       __acrt_get_begin_thread_init_policy 000000018001b818 f   libucrt:win_policies.obj
 0001:0001a858       __acrt_get_process_end_policy 000000018001b858 f   libucrt:win_policies.obj
 0001:0001a890       _fcloseall                 000000018001b890 f   libucrt:closeall.obj
 0001:0001ab24       __acrt_stdio_flush_nolock  000000018001bb24 f   libucrt:fflush.obj
 0001:0001abb0       _fflush_nolock             000000018001bbb0 f   libucrt:fflush.obj
 0001:0001ac84       _flushall                  000000018001bc84 f   libucrt:fflush.obj
 0001:0001ac8c       __acrt_stdio_free_buffer_nolock 000000018001bc8c f   libucrt:_freebuf.obj
 0001:0001aed8       __acrt_initialize_lowio    000000018001bed8 f   libucrt:ioinit.obj
 0001:0001af14       __acrt_uninitialize_lowio  000000018001bf14 f   libucrt:ioinit.obj
 0001:0001af60       _malloc_base               000000018001bf60 f   libucrt:malloc_base.obj
 0001:0001afc0       __acrt_update_locale_info  000000018001bfc0 f   libucrt:locale_update.obj
 0001:0001aff4       __acrt_update_locale_info_explicit 000000018001bff4 f   libucrt:locale_update.obj
 0001:0001b02c       __acrt_update_multibyte_info 000000018001c02c f   libucrt:locale_update.obj
 0001:0001b060       __acrt_update_multibyte_info_explicit 000000018001c060 f   libucrt:locale_update.obj
 0001:0001bba8       __acrt_fp_format           000000018001cba8 f   libucrt:cvt.obj
 0001:0001be90       _wctomb_internal           000000018001ce90 f   libucrt:wctomb.obj
 0001:0001c040       _mbtowc_internal           000000018001d040 f   libucrt:mbtowc.obj
 0001:0001c1b8       ?__mblen_utf8@__crt_mbstring@@YAHPEBD@Z 000000018001d1b8 f   libucrt:mbrtoc32.obj
 0001:0001c1f0       ?__mbrtoc32_utf8@__crt_mbstring@@YA_KPEA_UPEBD_KPEAU_Mbstatet@@AEAV__crt_cached_ptd_host@@@Z 000000018001d1f0 f   libucrt:mbrtoc32.obj
 0001:0001c3b0       ?__c16rtomb_utf8@__crt_mbstring@@YA_KPEAD_SPEAU_Mbstatet@@AEAV__crt_cached_ptd_host@@@Z 000000018001d3b0 f   libucrt:c16rtomb.obj
 0001:0001c454       ?__mbrtowc_utf8@__crt_mbstring@@YA_KPEA_WPEBD_KPEAU_Mbstatet@@AEAV__crt_cached_ptd_host@@@Z 000000018001d454 f   libucrt:mbrtowc.obj
 0001:0001c49c       ?__mbsrtowcs_utf8@__crt_mbstring@@YA_KPEA_WPEAPEBD_KPEAU_Mbstatet@@AEAV__crt_cached_ptd_host@@@Z 000000018001d49c f   libucrt:mbrtowc.obj
 0001:0001c654       _fileno                    000000018001d654 f   libucrt:fileno.obj
 0001:0001c67c       _get_printf_count_output   000000018001d67c f   libucrt:printf_count_output.obj
 0001:0001c694       _fputwc_nolock_internal    000000018001d694 f   libucrt:fputwc.obj
 0001:0001c828       _fputc_nolock_internal     000000018001d828 f   libucrt:fputc.obj
 0001:0001c840       __acrt_should_use_temporary_buffer 000000018001d840 f   libucrt:_sftbuf.obj
 0001:0001c88c       __acrt_stdio_begin_temporary_buffering_nolock 000000018001d88c f   libucrt:_sftbuf.obj
 0001:0001c954       __acrt_stdio_end_temporary_buffering_nolock 000000018001d954 f   libucrt:_sftbuf.obj
 0001:0001ca04       __acrt_set_locale_changed  000000018001da04 f   libucrt:wsetlocale.obj
 0001:0001ca10       __acrt_uninitialize_locale 000000018001da10 f   libucrt:wsetlocale.obj
 0001:0001cab8       _close_internal            000000018001dab8 f   libucrt:close.obj
 0001:0001cb7c       _close_nolock              000000018001db7c f   libucrt:close.obj
 0001:0001cc14       _close_nolock_internal     000000018001dc14 f   libucrt:close.obj
 0001:0001cce4       ?__acrt_stdio_allocate_stream@@YA?AV__crt_stdio_stream@@XZ 000000018001dce4 f   libucrt:stream.obj
 0001:0001cd3c       ?__acrt_stdio_free_stream@@YAXV__crt_stdio_stream@@@Z 000000018001dd3c f   libucrt:stream.obj
 0001:0001ce44       ??$__acrt_stdio_parse_mode@D@@YA?AU__acrt_stdio_stream_mode@@QEBD@Z 000000018001de44 f i libucrt:openfile.obj
 0001:0001d108       _openfile                  000000018001e108 f   libucrt:openfile.obj
 0001:0001d1a4       ??0_LocaleUpdate@@QEAA@QEAU__crt_locale_pointers@@@Z 000000018001e1a4 f i libucrt:wcsnicol.obj
 0001:0001d240       _strnicoll                 000000018001e240 f   libucrt:strnicol.obj
 0001:0001d258       _strnicoll_l               000000018001e258 f   libucrt:strnicol.obj
 0001:0001d358       __acrt_initialize_locks    000000018001e358 f   libucrt:locks.obj
 0001:0001d3a0       __acrt_lock                000000018001e3a0 f   libucrt:locks.obj
 0001:0001d3bc       __acrt_uninitialize_locks  000000018001e3bc f   libucrt:locks.obj
 0001:0001d3f4       __acrt_unlock              000000018001e3f4 f   libucrt:locks.obj
 0001:0001d410       __acrt_app_verifier_enabled 000000018001e410 f   libucrt:peb_access.obj
 0001:0001d42c       __acrt_is_secure_process   000000018001e42c f   libucrt:peb_access.obj
 0001:0001d458       ??$__acrt_convert_wcs_mbs_cp@D_WV<lambda_7c9dea7b4ca7285d2cdb541a38da6275>@@U__crt_win32_buffer_internal_dynamic_resizing@@@@YAHQEBDAEAV?$__crt_win32_buffer@_WU__crt_win32_buffer_internal_dynamic_resizing@@@@AEBV<lambda_7c9dea7b4ca7285d2cdb541a38da6275>@@I@Z 000000018001e458 f i libucrt:argv_wildcards.obj
 0001:0001d5f8       ??$__acrt_convert_wcs_mbs_cp@_WDV<lambda_d8593a27d1aa8c02be35c86a17d324c4>@@U__crt_win32_buffer_internal_dynamic_resizing@@@@YAHQEB_WAEAV?$__crt_win32_buffer@DU__crt_win32_buffer_internal_dynamic_resizing@@@@AEBV<lambda_d8593a27d1aa8c02be35c86a17d324c4>@@I@Z 000000018001e5f8 f i libucrt:argv_wildcards.obj
 0001:0001dec4       __acrt_expand_narrow_argv_wildcards 000000018001eec4 f   libucrt:argv_wildcards.obj
 0001:0001decc       ??$__acrt_convert_wcs_mbs_cp@_WDV<lambda_f788ae46380686e8b737efdd8c720d07>@@U__crt_win32_buffer_no_resizing@@@@YAHQEB_WAEAV?$__crt_win32_buffer@DU__crt_win32_buffer_no_resizing@@@@AEBV<lambda_f788ae46380686e8b737efdd8c720d07>@@I@Z 000000018001eecc f i libucrt:getmodulefilenamea.obj
 0001:0001dfe8       __acrt_GetModuleFileNameA  000000018001efe8 f   libucrt:getmodulefilenamea.obj
 0001:0001e914       __acrt_initialize_multibyte 000000018001f914 f   libucrt:mbctype.obj
 0001:0001e974       __acrt_update_thread_multibyte_data 000000018001f974 f   libucrt:mbctype.obj
 0001:0001e990       _setmbcp_nolock            000000018001f990 f   libucrt:mbctype.obj
 0001:0001eccc       _ismbblead                 000000018001fccc f   libucrt:ismbbyte.obj
 0001:0001ece0       __acrt_initialize_command_line 000000018001fce0 f   libucrt:argv_data.obj
 0001:0001ed08       __acrt_MultiByteToWideChar 000000018001fd08 f   libucrt:multibytetowidechar.obj
 0001:0001ed98       __acrt_WideCharToMultiByte 000000018001fd98 f   libucrt:widechartomultibyte.obj
 0001:0001ee78       __dcrt_get_narrow_environment_from_os 000000018001fe78 f   libucrt:get_environment_from_os.obj
 0001:0001f3c8       __dcrt_set_variable_in_narrow_environment_nolock 00000001800203c8 f   libucrt:setenv.obj
 0001:0001f3d0       _recalloc_base             00000001800203d0 f   libucrt:recalloc.obj
 0001:0001f470       _recalloc                  0000000180020470 f   libucrt:recalloc.obj
 0001:0001f480       _get_heap_handle           0000000180020480 f   libucrt:heap_handle.obj
 0001:0001f490       __acrt_initialize_heap     0000000180020490 f   libucrt:heap_handle.obj
 0001:0001f4c0       __acrt_uninitialize_heap   00000001800204c0 f   libucrt:heap_handle.obj
 0001:0001f4e0       __acrt_getheap             00000001800204e0 f   libucrt:heap_handle.obj
 0001:0001f4e8       __acrt_execute_initializers 00000001800204e8 f   libucrt:shared_initialization.obj
 0001:0001f568       __acrt_execute_uninitializers 0000000180020568 f   libucrt:shared_initialization.obj
 0001:0001f5ec       __acrt_get_sigabrt_handler 00000001800205ec f   libucrt:signal.obj
 0001:0001f61c       __acrt_initialize_signal_handlers 000000018002061c f   libucrt:signal.obj
 0001:0001f63c       raise                      000000018002063c f   libucrt:signal.obj
 0001:0001f8a0       __acrt_has_user_matherr    00000001800208a0 f   libucrt:matherr.obj
 0001:0001f8c0       __acrt_initialize_user_matherr 00000001800208c0 f   libucrt:matherr.obj
 0001:0001f8d0       __acrt_invoke_user_matherr 00000001800208d0 f   libucrt:matherr.obj
 0001:0001f900       _query_new_mode            0000000180020900 f   libucrt:new_mode.obj
 0001:0001f910       _set_new_mode              0000000180020910 f   libucrt:new_mode.obj
 0001:0001f93c       __acrt_add_locale_ref      000000018002093c f   libucrt:locale_refcounting.obj
 0001:0001f9c8       __acrt_free_locale         00000001800209c8 f   libucrt:locale_refcounting.obj
 0001:0001fb40       __acrt_locale_add_lc_time_reference 0000000180020b40 f   libucrt:locale_refcounting.obj
 0001:0001fb68       __acrt_locale_free_lc_time_if_unreferenced 0000000180020b68 f   libucrt:locale_refcounting.obj
 0001:0001fba0       __acrt_locale_release_lc_time_reference 0000000180020ba0 f   libucrt:locale_refcounting.obj
 0001:0001fbc8       __acrt_release_locale_ref  0000000180020bc8 f   libucrt:locale_refcounting.obj
 0001:0001fc70       __acrt_update_thread_locale_data 0000000180020c70 f   libucrt:locale_refcounting.obj
 0001:0001fce0       _updatetlocinfoEx_nolock   0000000180020ce0 f   libucrt:locale_refcounting.obj
 0001:0001fd48       __acrt_DownlevelLocaleNameToLCID 0000000180020d48 f   libucrt:lcidtoname_downlevel.obj
 0001:0001fe7c       _commit                    0000000180020e7c f   libucrt:commit.obj
 0001:0002073c       _write                     000000018002173c f   libucrt:write.obj
 0001:000207d4       _write_internal            00000001800217d4 f   libucrt:write.obj
 0001:000208f4       _write_nolock              00000001800218f4 f   libucrt:write.obj
 0001:00020c24       __acrt_lowio_create_handle_array 0000000180021c24 f   libucrt:osfinfo.obj
 0001:00020ccc       __acrt_lowio_destroy_handle_array 0000000180021ccc f   libucrt:osfinfo.obj
 0001:00020d1c       __acrt_lowio_ensure_fh_exists 0000000180021d1c f   libucrt:osfinfo.obj
 0001:00020dc4       __acrt_lowio_lock_fh       0000000180021dc4 f   libucrt:osfinfo.obj
 0001:00020dec       __acrt_lowio_set_os_handle 0000000180021dec f   libucrt:osfinfo.obj
 0001:00020eac       __acrt_lowio_unlock_fh     0000000180021eac f   libucrt:osfinfo.obj
 0001:00020ed4       _alloc_osfhnd              0000000180021ed4 f   libucrt:osfinfo.obj
 0001:00021014       _free_osfhnd               0000000180022014 f   libucrt:osfinfo.obj
 0001:000210d0       _get_osfhandle             00000001800220d0 f   libucrt:osfinfo.obj
 0001:00021218       __acrt_fp_strflt_to_string 0000000180022218 f   libucrt:_fptostr.obj
 0001:00021330       ?divide@__crt_strtox@@YA_KAEAUbig_integer@1@AEBU21@@Z 0000000180022330 f i libucrt:cfout.obj
 0001:000217bc       __acrt_fltout              00000001800227bc f   libucrt:cfout.obj
 0001:00022ad0       fegetround                 0000000180023ad0 f   libucrt:fegetround.obj
 0001:00022ae4       ?__c32rtomb_utf8@__crt_mbstring@@YA_KPEAD_UPEAU_Mbstatet@@AEAV__crt_cached_ptd_host@@@Z 0000000180023ae4 f   libucrt:c32rtomb.obj
 0001:00022b88       ?reset_and_return@__crt_mbstring@@YA_K_KPEAU_Mbstatet@@@Z 0000000180023b88 f   libucrt:common_utf8.obj
 0001:00022b90       ?return_illegal_sequence@__crt_mbstring@@YA_KPEAU_Mbstatet@@AEAV__crt_cached_ptd_host@@@Z 0000000180023b90 f   libucrt:common_utf8.obj
 0001:00022e20       __acrt_stdio_flush_and_write_narrow_nolock 0000000180023e20 f   libucrt:_flsbuf.obj
 0001:00022eec       __acrt_stdio_flush_and_write_wide_nolock 0000000180023eec f   libucrt:_flsbuf.obj
 0001:00022fb8       _isatty                    0000000180023fb8 f   libucrt:isatty.obj
 0001:00023018       __acrt_locale_free_monetary 0000000180024018 f   libucrt:initmon.obj
 0001:00023124       __acrt_locale_free_numeric 0000000180024124 f   libucrt:initnum.obj
 0001:000231c4       __acrt_locale_free_time    00000001800241c4 f   libucrt:inittime.obj
 0001:000232cc       __acrt_GetStringTypeA      00000001800242cc f   libucrt:getstringtypea.obj
 0001:0002345c       __ascii_wcsnicmp           000000018002445c f   libucrt:wcsnicmp.obj
 0001:000234a8       __ascii_strnicmp           00000001800244a8 f   libucrt:strnicmp.obj
 0001:000234f4       _strnicmp                  00000001800244f4 f   libucrt:strnicmp.obj
 0001:00023544       _strnicmp_l                0000000180024544 f   libucrt:strnicmp.obj
 0001:00023c10       _sopen_nolock              0000000180024c10 f   libucrt:open.obj
 0001:00023d2c       _sopen_s                   0000000180024d2c f   libucrt:open.obj
 0001:00023d60       _wsopen_nolock             0000000180024d60 f   libucrt:open.obj
 0001:00024504       __acrt_CompareStringA      0000000180025504 f   libucrt:comparestringa.obj
 0001:00024590       qsort                      0000000180025590 f   libucrt:qsort.obj
 0001:00024928       strncpy_s                  0000000180025928 f   libucrt:strncpy_s.obj
 0001:00024a90       strpbrk                    0000000180025a90 f   libucrt:strpbrk.obj
 0001:00024e48       _mbsdec                    0000000180025e48 f   libucrt:mbsdec.obj
 0001:00024e50       _mbsdec_l                  0000000180025e50 f   libucrt:mbsdec.obj
 0001:00025218       __acrt_LCMapStringA        0000000180026218 f   libucrt:lcmapstringa.obj
 0001:000252c4       __acrt_SetEnvironmentVariableA 00000001800262c4 f   libucrt:setenvironmentvariablea.obj
 0001:00025470       _msize_base                0000000180026470 f   libucrt:msize.obj
 0001:000254b0       _msize                     00000001800264b0 f   libucrt:msize.obj
 0001:000254c0       _realloc_base              00000001800264c0 f   libucrt:realloc_base.obj
 0001:0002570c       _lseeki64                  000000018002670c f   libucrt:lseek.obj
 0001:000257a8       _lseeki64_nolock           00000001800267a8 f   libucrt:lseek.obj
 0001:00025844       _lseeki64_nolock_internal  0000000180026844 f   libucrt:lseek.obj
 0001:0002584c       _putwch_nolock             000000018002684c f   libucrt:putwch.obj
 0001:00025db8       _read_nolock               0000000180026db8 f   libucrt:read.obj
 0001:00026218       _query_app_type            0000000180027218 f   libucrt:report_runtime_error.obj
 0001:00026220       _controlfp_s               0000000180027220 f   libucrt:contrlfp.obj
 0001:00026290       fegetenv                   0000000180027290 f   libucrt:fegetenv.obj
 0001:000262b0       fesetenv                   00000001800272b0 f   libucrt:fesetenv.obj
 0001:00026320       feholdexcept               0000000180027320 f   libucrt:feholdexcept.obj
 0001:00026380       ceil                       0000000180027380 f   libucrt:ceil.obj
 0001:00026450       log10                      0000000180027450 f   libucrt:log10.obj
 0001:00026a00       __acrt_fenv_get_common_round_control 0000000180027a00 f   libucrt:_fenvutils.obj
 0001:00026a10       __acrt_fenv_get_control    0000000180027a10 f   libucrt:_fenvutils.obj
 0001:00026af0       __acrt_fenv_get_status     0000000180027af0 f   libucrt:_fenvutils.obj
 0001:00026b50       __acrt_fenv_set_control    0000000180027b50 f   libucrt:_fenvutils.obj
 0001:00026c80       __acrt_fenv_set_status     0000000180027c80 f   libucrt:_fenvutils.obj
 0001:00026cf4       __acrt_stdio_allocate_buffer_nolock 0000000180027cf4 f   libucrt:_getbuf.obj
 0001:00026d60       _get_fmode                 0000000180027d60 f   libucrt:setmode.obj
 0001:00026d90       _setmode_nolock            0000000180027d90 f   libucrt:setmode.obj
 0001:00026e74       _chsize_nolock             0000000180027e74 f   libucrt:chsize.obj
 0001:00026f0c       _chsize_nolock_internal    0000000180027f0c f   libucrt:chsize.obj
 0001:0002709c       __strncnt                  000000018002809c f   libucrt:strncnt.obj
 0001:000270b4       _guard_check_icall         00000001800280b4 f i libucrt:checkcfg.obj
 0001:000270cc       __dcrt_lowio_ensure_console_output_initialized 00000001800280cc f   libucrt:initcon.obj
 0001:00027120       __dcrt_terminate_console_output 0000000180028120 f   libucrt:initcon.obj
 0001:0002713c       __dcrt_write_console       000000018002813c f   libucrt:initcon.obj
 0001:000271fc       _clearfp                   00000001800281fc f   libucrt:ieee.obj
 0001:00027258       _control87                 0000000180028258 f   libucrt:ieee.obj
 0001:00027610       _handle_error              0000000180028610 f   libucrt:libm_error.obj
 0001:00027750       _handle_nan                0000000180028750 f   libucrt:libm_error.obj
 0001:00027770       ceil_sse41                 0000000180028770 f   libucrt:floorceil_sse41.obj
 0001:00027780       __acrt_initialize_fma3     0000000180028780 f   libucrt:fma3_available.obj
 0001:00027834       _log10_special             0000000180028834 f   libucrt:log_special.obj
 0001:000278ec       __acrt_initialize_fmode    00000001800288ec f   libucrt:txtmode.obj
 0001:00027904       _clrfp                     0000000180028904 f   libucrt:fpctrl.obj
 0001:00027924       _ctrlfp                    0000000180028924 f   libucrt:fpctrl.obj
 0001:00027998       _get_fpcsr                 0000000180028998 f   libucrt:fpctrl.obj
 0001:00027998       _get_fpsr                  0000000180028998 f   libucrt:fpctrl.obj
 0001:000279a4       _set_fpcsr                 00000001800289a4 f   libucrt:fpctrl.obj
 0001:000279a4       _set_fpsr                  00000001800289a4 f   libucrt:fpctrl.obj
 0001:000279b0       _set_statfp                00000001800289b0 f   libucrt:fpctrl.obj
 0001:000279d0       _statfp                    00000001800289d0 f   libucrt:fpctrl.obj
 0001:000279e0       _raise_exc                 00000001800289e0 f   libucrt:fpexcept.obj
 0001:00027a10       _raise_exc_ex              0000000180028a10 f   libucrt:fpexcept.obj
 0001:00027d20       _set_errno_from_matherr    0000000180028d20 f   libucrt:fpexcept.obj
 0001:00027d60       _FindPESection             0000000180028d60 f   LIBCMT:pesect.obj
 0001:00027db0       _IsNonwritableInCurrentImage 0000000180028db0 f   LIBCMT:pesect.obj
 0001:00027e00       _ValidateImageBase         0000000180028e00 f   LIBCMT:pesect.obj
 0001:00027e2c       __GSHandlerCheck_EH        0000000180028e2c f   LIBCMT:gshandlereh.obj
 0001:00027ec0       __chkstk                   0000000180028ec0 f   LIBCMT:chkstk.obj
 0001:00027ec0       _alloca_probe              0000000180028ec0 f   LIBCMT:chkstk.obj
 0001:00027f10       __C_specific_handler_noexcept 0000000180028f10 f   libvcruntime:chandler_noexcept.obj
 0001:00027f5c       strrchr                    0000000180028f5c f   libvcruntime:strrchr.obj
 0001:000280a0       strchr                     00000001800290a0 f   libvcruntime:strchr.obj
 0001:00028130       _guard_dispatch_icall_nop  0000000180029130 f   LIBCMT:guard_dispatch.obj
 0001:00028150       _guard_xfg_dispatch_icall_nop 0000000180029150 f   LIBCMT:guard_xfg_dispatch.obj
 0001:00028170       _guard_dispatch_icall      0000000180029170 f   libucrt:dispatchcfg.obj
 0001:00028170       _guard_dispatch_icall_$fo_default$ 0000000180029170     libucrt:dispatchcfg.obj
 0001:000281a0       memcpy_repmovs             00000001800291a0 f   libvcruntime:memcpy.obj
 0001:000281b0       memcpy                     00000001800291b0 f   libvcruntime:memcpy.obj
 0001:000281b0       memcpy_$fo_default$        00000001800291b0     libvcruntime:memcpy.obj
 0001:000281b0       memmove                    00000001800291b0 f   libvcruntime:memcpy.obj
 0001:00028840       memset_repstos             0000000180029840 f   libvcruntime:memset.obj
 0001:00028850       memset                     0000000180029850 f   libvcruntime:memset.obj
 0001:00028bf0       strcmp                     0000000180029bf0 f   libucrt:strcmp.obj
 0001:00028c70       strcat                     0000000180029c70 f   libucrt:strcat.obj
 0001:00028d10       strcpy                     0000000180029d10 f   libucrt:strcat.obj
 0001:00028d13       ___entry_from_strcat_in_strcpy 0000000180029d13     libucrt:strcat.obj
 0001:00028de0       strncpy                    0000000180029de0 f   libucrt:strncpy.obj
 0001:00028f60       strlen                     0000000180029f60 f   libucrt:strlen.obj
 0001:00029020       strncat                    000000018002a020 f   libucrt:strncat.obj
 0001:000291d0       strncmp                    000000018002a1d0 f   libucrt:strncmp.obj
 0002:00000000       __imp_CloseHandle          000000018002b000     kernel32:KERNEL32.dll
 0002:00000008       __imp_GetLastError         000000018002b008     kernel32:KERNEL32.dll
 0002:00000010       __imp_MapViewOfFile        000000018002b010     kernel32:KERNEL32.dll
 0002:00000018       __imp_UnmapViewOfFile      000000018002b018     kernel32:KERNEL32.dll
 0002:00000020       __imp_OpenFileMappingA     000000018002b020     kernel32:KERNEL32.dll
 0002:00000028       __imp_GetSystemTimeAsFileTime 000000018002b028     kernel32:KERNEL32.dll
 0002:00000030       __imp_InitializeCriticalSection 000000018002b030     kernel32:KERNEL32.dll
 0002:00000038       __imp_EnterCriticalSection 000000018002b038     kernel32:KERNEL32.dll
 0002:00000040       __imp_LeaveCriticalSection 000000018002b040     kernel32:KERNEL32.dll
 0002:00000048       __imp_DeleteCriticalSection 000000018002b048     kernel32:KERNEL32.dll
 0002:00000050       __imp_Sleep                000000018002b050     kernel32:KERNEL32.dll
 0002:00000058       __imp_WriteConsoleW        000000018002b058     kernel32:KERNEL32.dll
 0002:00000060       __imp_SetEndOfFile         000000018002b060     kernel32:KERNEL32.dll
 0002:00000068       __imp_ReadConsoleW         000000018002b068     kernel32:KERNEL32.dll
 0002:00000070       __imp_ReadFile             000000018002b070     kernel32:KERNEL32.dll
 0002:00000078       __imp_HeapReAlloc          000000018002b078     kernel32:KERNEL32.dll
 0002:00000080       __imp_HeapSize             000000018002b080     kernel32:KERNEL32.dll
 0002:00000088       __imp_CreateFileW          000000018002b088     kernel32:KERNEL32.dll
 0002:00000090       __imp_GetStringTypeW       000000018002b090     kernel32:KERNEL32.dll
 0002:00000098       __imp_SetFilePointerEx     000000018002b098     kernel32:KERNEL32.dll
 0002:000000a0       __imp_GetFileSizeEx        000000018002b0a0     kernel32:KERNEL32.dll
 0002:000000a8       __imp_SetStdHandle         000000018002b0a8     kernel32:KERNEL32.dll
 0002:000000b0       __imp_RtlCaptureContext    000000018002b0b0     kernel32:KERNEL32.dll
 0002:000000b8       __imp_RtlLookupFunctionEntry 000000018002b0b8     kernel32:KERNEL32.dll
 0002:000000c0       __imp_RtlVirtualUnwind     000000018002b0c0     kernel32:KERNEL32.dll
 0002:000000c8       __imp_UnhandledExceptionFilter 000000018002b0c8     kernel32:KERNEL32.dll
 0002:000000d0       __imp_SetUnhandledExceptionFilter 000000018002b0d0     kernel32:KERNEL32.dll
 0002:000000d8       __imp_GetCurrentProcess    000000018002b0d8     kernel32:KERNEL32.dll
 0002:000000e0       __imp_TerminateProcess     000000018002b0e0     kernel32:KERNEL32.dll
 0002:000000e8       __imp_IsProcessorFeaturePresent 000000018002b0e8     kernel32:KERNEL32.dll
 0002:000000f0       __imp_QueryPerformanceCounter 000000018002b0f0     kernel32:KERNEL32.dll
 0002:000000f8       __imp_GetCurrentProcessId  000000018002b0f8     kernel32:KERNEL32.dll
 0002:00000100       __imp_GetCurrentThreadId   000000018002b100     kernel32:KERNEL32.dll
 0002:00000108       __imp_InitializeSListHead  000000018002b108     kernel32:KERNEL32.dll
 0002:00000110       __imp_IsDebuggerPresent    000000018002b110     kernel32:KERNEL32.dll
 0002:00000118       __imp_GetStartupInfoW      000000018002b118     kernel32:KERNEL32.dll
 0002:00000120       __imp_GetModuleHandleW     000000018002b120     kernel32:KERNEL32.dll
 0002:00000128       __imp_RtlUnwindEx          000000018002b128     kernel32:KERNEL32.dll
 0002:00000130       __imp_RtlPcToFileHeader    000000018002b130     kernel32:KERNEL32.dll
 0002:00000138       __imp_RaiseException       000000018002b138     kernel32:KERNEL32.dll
 0002:00000140       __imp_InterlockedFlushSList 000000018002b140     kernel32:KERNEL32.dll
 0002:00000148       __imp_SetLastError         000000018002b148     kernel32:KERNEL32.dll
 0002:00000150       __imp_InitializeCriticalSectionAndSpinCount 000000018002b150     kernel32:KERNEL32.dll
 0002:00000158       __imp_TlsAlloc             000000018002b158     kernel32:KERNEL32.dll
 0002:00000160       __imp_TlsGetValue          000000018002b160     kernel32:KERNEL32.dll
 0002:00000168       __imp_TlsSetValue          000000018002b168     kernel32:KERNEL32.dll
 0002:00000170       __imp_TlsFree              000000018002b170     kernel32:KERNEL32.dll
 0002:00000178       __imp_FreeLibrary          000000018002b178     kernel32:KERNEL32.dll
 0002:00000180       __imp_GetProcAddress       000000018002b180     kernel32:KERNEL32.dll
 0002:00000188       __imp_LoadLibraryExW       000000018002b188     kernel32:KERNEL32.dll
 0002:00000190       __imp_EncodePointer        000000018002b190     kernel32:KERNEL32.dll
 0002:00000198       __imp_CreateThread         000000018002b198     kernel32:KERNEL32.dll
 0002:000001a0       __imp_ExitThread           000000018002b1a0     kernel32:KERNEL32.dll
 0002:000001a8       __imp_FreeLibraryAndExitThread 000000018002b1a8     kernel32:KERNEL32.dll
 0002:000001b0       __imp_GetModuleHandleExW   000000018002b1b0     kernel32:KERNEL32.dll
 0002:000001b8       __imp_ExitProcess          000000018002b1b8     kernel32:KERNEL32.dll
 0002:000001c0       __imp_GetModuleFileNameW   000000018002b1c0     kernel32:KERNEL32.dll
 0002:000001c8       __imp_HeapAlloc            000000018002b1c8     kernel32:KERNEL32.dll
 0002:000001d0       __imp_HeapFree             000000018002b1d0     kernel32:KERNEL32.dll
 0002:000001d8       __imp_FlsAlloc             000000018002b1d8     kernel32:KERNEL32.dll
 0002:000001e0       __imp_FlsGetValue          000000018002b1e0     kernel32:KERNEL32.dll
 0002:000001e8       __imp_FlsSetValue          000000018002b1e8     kernel32:KERNEL32.dll
 0002:000001f0       __imp_FlsFree              000000018002b1f0     kernel32:KERNEL32.dll
 0002:000001f8       __imp_InitializeCriticalSectionEx 000000018002b1f8     kernel32:KERNEL32.dll
 0002:00000200       __imp_VirtualProtect       000000018002b200     kernel32:KERNEL32.dll
 0002:00000208       __imp_CompareStringW       000000018002b208     kernel32:KERNEL32.dll
 0002:00000210       __imp_LCMapStringW         000000018002b210     kernel32:KERNEL32.dll
 0002:00000218       __imp_GetStdHandle         000000018002b218     kernel32:KERNEL32.dll
 0002:00000220       __imp_GetFileType          000000018002b220     kernel32:KERNEL32.dll
 0002:00000228       __imp_FindClose            000000018002b228     kernel32:KERNEL32.dll
 0002:00000230       __imp_FindFirstFileExW     000000018002b230     kernel32:KERNEL32.dll
 0002:00000238       __imp_FindNextFileW        000000018002b238     kernel32:KERNEL32.dll
 0002:00000240       __imp_IsValidCodePage      000000018002b240     kernel32:KERNEL32.dll
 0002:00000248       __imp_GetACP               000000018002b248     kernel32:KERNEL32.dll
 0002:00000250       __imp_GetOEMCP             000000018002b250     kernel32:KERNEL32.dll
 0002:00000258       __imp_GetCPInfo            000000018002b258     kernel32:KERNEL32.dll
 0002:00000260       __imp_GetCommandLineA      000000018002b260     kernel32:KERNEL32.dll
 0002:00000268       __imp_GetCommandLineW      000000018002b268     kernel32:KERNEL32.dll
 0002:00000270       __imp_MultiByteToWideChar  000000018002b270     kernel32:KERNEL32.dll
 0002:00000278       __imp_WideCharToMultiByte  000000018002b278     kernel32:KERNEL32.dll
 0002:00000280       __imp_GetEnvironmentStringsW 000000018002b280     kernel32:KERNEL32.dll
 0002:00000288       __imp_FreeEnvironmentStringsW 000000018002b288     kernel32:KERNEL32.dll
 0002:00000290       __imp_SetEnvironmentVariableW 000000018002b290     kernel32:KERNEL32.dll
 0002:00000298       __imp_GetProcessHeap       000000018002b298     kernel32:KERNEL32.dll
 0002:000002a0       __imp_FlushFileBuffers     000000018002b2a0     kernel32:KERNEL32.dll
 0002:000002a8       __imp_WriteFile            000000018002b2a8     kernel32:KERNEL32.dll
 0002:000002b0       __imp_GetConsoleOutputCP   000000018002b2b0     kernel32:KERNEL32.dll
 0002:000002b8       __imp_GetConsoleMode       000000018002b2b8     kernel32:KERNEL32.dll
 0002:000002c0       \177KERNEL32_NULL_THUNK_DATA 000000018002b2c0     kernel32:KERNEL32.dll
 0002:000002c8       __imp_CreateDialogParamA   000000018002b2c8     user32:USER32.dll
 0002:000002d0       __imp_PostMessageA         000000018002b2d0     user32:USER32.dll
 0002:000002d8       __imp_DispatchMessageA     000000018002b2d8     user32:USER32.dll
 0002:000002e0       __imp_TranslateMessage     000000018002b2e0     user32:USER32.dll
 0002:000002e8       __imp_RegisterWindowMessageA 000000018002b2e8     user32:USER32.dll
 0002:000002f0       __imp_GetMessageA          000000018002b2f0     user32:USER32.dll
 0002:000002f8       __imp_PostThreadMessageA   000000018002b2f8     user32:USER32.dll
 0002:00000300       __imp_SendMessageA         000000018002b300     user32:USER32.dll
 0002:00000308       __imp_PostQuitMessage      000000018002b308     user32:USER32.dll
 0002:00000310       \177USER32_NULL_THUNK_DATA 000000018002b310     user32:USER32.dll
 0002:00000318       __imp_JAWT_GetAWT          000000018002b318     jawt:jawt.dll
 0002:00000320       \177jawt_NULL_THUNK_DATA   000000018002b320     jawt:jawt.dll
 0002:00000328       __guard_check_icall_fptr   000000018002b328     LIBCMT:guard_support.obj
 0002:00000330       __guard_xfg_check_icall_fptr 000000018002b330     LIBCMT:guard_support.obj
 0002:00000338       __guard_dispatch_icall_fptr 000000018002b338     LIBCMT:guard_support.obj
 0002:00000340       __guard_xfg_dispatch_icall_fptr 000000018002b340     LIBCMT:guard_support.obj
 0002:00000348       __guard_xfg_table_dispatch_icall_fptr 000000018002b348     LIBCMT:guard_support.obj
 0002:00000350       __castguard_check_failure_os_handled_fptr 000000018002b350     LIBCMT:guard_support.obj
 0002:00000358       __guard_memcpy_fptr        000000018002b358     libvcruntime:softmemtag.obj
 0002:00000360       __xc_a                     000000018002b360     LIBCMT:initializers.obj
 0002:00000368       __xc_z                     000000018002b368     LIBCMT:initializers.obj
 0002:00000370       __xi_a                     000000018002b370     LIBCMT:initializers.obj
 0002:00000378       __acrt_stdio_initializer   000000018002b378     libucrt:stdio_initializer.obj
 0002:00000380       __acrt_multibyte_initializer 000000018002b380     libucrt:multibyte_initializer.obj
 0002:00000388       __acrt_tran_fma3_initializer 000000018002b388     libucrt:fma3_initializer.obj
 0002:00000390       __acrt_fmode_initializer   000000018002b390     libucrt:fmode_initializer.obj
 0002:00000398       __xi_z                     000000018002b398     LIBCMT:initializers.obj
 0002:000003a0       __xp_a                     000000018002b3a0     LIBCMT:initializers.obj
 0002:000003a8       __acrt_locale_terminator   000000018002b3a8     libucrt:locale_initializer.obj
 0002:000003b0       __dcrt_console_output_terminator 000000018002b3b0     libucrt:console_output_initializer.obj
 0002:000003b8       __acrt_stdio_terminator    000000018002b3b8     libucrt:stdio_initializer.obj
 0002:000003c0       __xp_z                     000000018002b3c0     LIBCMT:initializers.obj
 0002:000003c8       __xt_a                     000000018002b3c8     LIBCMT:initializers.obj
 0002:000003d0       __xt_z                     000000018002b3d0     LIBCMT:initializers.obj
 0002:000003e0       ??_C@_0DL@PNCLIPJM@?$FLINFO?$FN?3?5in?5AccessBridgeATInstan@ 000000018002b3e0     AccessBridgeATInstance.obj
 0002:00000420       ??_C@_0DA@ILNDDPNA@?$FLINFO?$FN?3?5?5?5unmapping?5memoryMappe@ 000000018002b420     AccessBridgeATInstance.obj
 0002:00000450       ??_C@_0DJ@FCAPEKK@?$FLINFO?$FN?3?5?5?5closing?5memoryMappedF@ 000000018002b450     AccessBridgeATInstance.obj
 0002:00000490       ??_C@_0DB@BBBKEEOJ@?$FLINFO?$FN?3?5In?5AccessBridgeATInstan@ 000000018002b490     AccessBridgeATInstance.obj
 0002:000004c8       ??_C@_0DJ@HCNGCGLH@?$FLERROR?$FN?3?5?5?5Failed?5to?5CreateFile@ 000000018002b4c8     AccessBridgeATInstance.obj
 0002:00000508       ??_C@_0DC@INNGAKAO@?$FLINFO?$FN?3?5?5?5CreateFileMapping?5wor@ 000000018002b508     AccessBridgeATInstance.obj
 0002:00000540       ??_C@_0DF@EKLGABNF@?$FLERROR?$FN?3?5?5?5Failed?5to?5MapViewOfF@ 000000018002b540     AccessBridgeATInstance.obj
 0002:00000578       ??_C@_0CK@LMLFEIHL@?$FLINFO?$FN?3?5?5?5MapViewOfFile?5worked?5@ 000000018002b578     AccessBridgeATInstance.obj
 0002:000005a4       ??_C@_03DJNNCAJF@OK?$DP@   000000018002b5a4     AccessBridgeATInstance.obj
 0002:000005a8       ??_C@_0DL@FPNEIEFH@?$FLERROR?$FN?3?5?5?5JavaVM?5failed?5to?5wri@ 000000018002b5a8     AccessBridgeATInstance.obj
 0002:000005e8       ??_C@_0CN@CCHCHAPN@?$FLINFO?$FN?3?5?5?5JavaVM?5successfully?5w@ 000000018002b5e8     AccessBridgeATInstance.obj
 0002:00000618       ??_C@_03ONJMBPEK@OK?$CB@   000000018002b618     AccessBridgeATInstance.obj
 0002:00000620       ??_C@_0EE@MNPDBEBN@?$FLINFO?$FN?3?5AccessBridgeATInstance?3@ 000000018002b620     AccessBridgeATInstance.obj
 0002:00000670       ??_C@_0FI@KACFLKHC@?$FLINFO?$FN?3?5AccessBridgeATInstance?3@ 000000018002b670     AccessBridgeATInstance.obj
 0002:000006d0       ??_C@_0EN@DDCKACNO@?$FLINFO?$FN?3?5AccessBridgeATInstance?3@ 000000018002b6d0     AccessBridgeATInstance.obj
 0002:00000720       ??_C@_0BJ@FKCDJFDK@JAVA_ACCESSBRIDGE_LOGDIR@ 000000018002b720     AccessBridgeDebug.obj
 0002:0000073c       ??_C@_04FPOLKAEB@?4log@    000000018002b73c     AccessBridgeDebug.obj
 0002:00000744       ??_C@_01NOFIACDB@w@        000000018002b744     AccessBridgeDebug.obj
 0002:00000748       ??_C@_04EINJHBMM@?6?$CFs?6@ 000000018002b748     AccessBridgeDebug.obj
 0002:00000750       ??_C@_0BH@PPBGFLKL@Could?5not?5open?5file?5?$CFs@ 000000018002b750     AccessBridgeDebug.obj
 0002:00000768       ??_C@_07IBOBEFLP@?$FL?$CFllu?$FN?5@ 000000018002b768     AccessBridgeDebug.obj
 0002:00000770       ??_C@_02PCIJFNDE@?$AN?6@   000000018002b770     AccessBridgeDebug.obj
 0002:00000778       ??_C@_0DD@HABIDLLD@?$FLINFO?$FN?3?5AccessBridgeJavaEntryPo@ 000000018002b778     AccessBridgeJavaEntryPoints.obj
 0002:000007b0       ??_C@_0CI@FJHGEAOO@?$FLINFO?$FN?3?5Calling?5BuildJavaEntryP@ 000000018002b7b0     AccessBridgeJavaEntryPoints.obj
 0002:000007d8       ??_C@_0DB@PHGNIPBB@com?1sun?1java?1accessibility?1inte@ 000000018002b7d8     AccessBridgeJavaEntryPoints.obj
 0002:00000810       ??_C@_0CP@OJHOIDNH@?$FLERROR?$FN?3?5?5FindClass?$CI?$CFs?$CJ?5failed?$CB@ 000000018002b810     AccessBridgeJavaEntryPoints.obj
 0002:00000840       ??_C@_0DE@FJPDGHPE@?$FLERROR?$FN?3?5FindClass?$CI?$CFs?$CJ?5failed?$CB?5@ 000000018002b840     AccessBridgeJavaEntryPoints.obj
 0002:00000878       ??_C@_0BG@JLFLBLJI@?$CILjava?1lang?1Object?$DL?$CJV@ 000000018002b878     AccessBridgeJavaEntryPoints.obj
 0002:00000890       ??_C@_0BD@PAIEAHIF@decrementReference@ 000000018002b890     AccessBridgeJavaEntryPoints.obj
 0002:000008a8       ??_C@_0DP@BBIEPKKN@?$FLERROR?$FN?3?5GetMethodID?$CI?$CFs?$CJ?5failed@ 000000018002b8a8     AccessBridgeJavaEntryPoints.obj
 0002:000008e8       ??_C@_0BF@FOHFOJOB@?$CI?$CJLjava?1lang?1String?$DL@ 000000018002b8e8     AccessBridgeJavaEntryPoints.obj
 0002:00000900       ??_C@_0BH@KKNMIJGK@getJavaVersionProperty@ 000000018002b900     AccessBridgeJavaEntryPoints.obj
 0002:00000918       ??_C@_04FJLILDCB@?$CII?$CJZ@ 000000018002b918     AccessBridgeJavaEntryPoints.obj
 0002:00000920       ??_C@_0N@MHDJENGP@isJavaWindow@ 000000018002b920     AccessBridgeJavaEntryPoints.obj
 0002:00000930       ??_C@_0CL@DDDHKJEI@?$CII?$CJLjavax?1accessibility?1Accessi@ 000000018002b930     AccessBridgeJavaEntryPoints.obj
 0002:00000960       ??_C@_0CB@JPFPCEPL@getContextFromNativeWindowHandl@ 000000018002b960     AccessBridgeJavaEntryPoints.obj
 0002:00000988       ??_C@_0CL@LNFAHLDN@?$CILjavax?1accessibility?1Accessibl@ 000000018002b988     AccessBridgeJavaEntryPoints.obj
 0002:000009b8       ??_C@_0CB@OGDNEJKI@getNativeWindowHandleFromContex@ 000000018002b9b8     AccessBridgeJavaEntryPoints.obj
 0002:000009e0       ??_C@_0FB@EAOFMHCM@?$CILjavax?1accessibility?1Accessibl@ 000000018002b9e0     AccessBridgeJavaEntryPoints.obj
 0002:00000a38       ??_C@_0BP@OKMFCEDC@getAccessibleParentFromContext@ 000000018002ba38     AccessBridgeJavaEntryPoints.obj
 0002:00000a58       ??_C@_0DN@EHCPLCMJ@?$CILjavax?1accessibility?1Accessibl@ 000000018002ba58     AccessBridgeJavaEntryPoints.obj
 0002:00000a98       ??_C@_0BA@NNDOMDNC@setTextContents@ 000000018002ba98     AccessBridgeJavaEntryPoints.obj
 0002:00000ab0       ??_C@_0GD@DBHMDOGO@?$CILjavax?1accessibility?1Accessibl@ 000000018002bab0     AccessBridgeJavaEntryPoints.obj
 0002:00000b18       ??_C@_0BC@EHMJEOIE@getParentWithRole@ 000000018002bb18     AccessBridgeJavaEntryPoints.obj
 0002:00000b30       ??_C@_0BC@CBIPDOMM@getTopLevelObject@ 000000018002bb30     AccessBridgeJavaEntryPoints.obj
 0002:00000b48       ??_C@_0BK@KAMHKCND@getParentWithRoleElseRoot@ 000000018002bb48     AccessBridgeJavaEntryPoints.obj
 0002:00000b68       ??_C@_0P@POFHEAF@getObjectDepth@ 000000018002bb68     AccessBridgeJavaEntryPoints.obj
 0002:00000b78       ??_C@_0BE@CDLLPKAM@getActiveDescendent@ 000000018002bb78     AccessBridgeJavaEntryPoints.obj
 0002:00000b90       ??_C@_0FD@CINPJKCJ@?$CIIILjavax?1accessibility?1Accessi@ 000000018002bb90     AccessBridgeJavaEntryPoints.obj
 0002:00000be8       ??_C@_0BH@BIEKBJIN@getAccessibleContextAt@ 000000018002bbe8     AccessBridgeJavaEntryPoints.obj
 0002:00000c00       ??_C@_0CK@DOBCJGDO@?$CI?$CJLjavax?1accessibility?1Accessib@ 000000018002bc00     AccessBridgeJavaEntryPoints.obj
 0002:00000c30       ??_C@_0BO@BAFCPPBG@getAccessibleContextWithFocus@ 000000018002bc30     AccessBridgeJavaEntryPoints.obj
 0002:00000c50       ??_C@_0DM@JMIIJMDP@?$CILjavax?1accessibility?1Accessibl@ 000000018002bc50     AccessBridgeJavaEntryPoints.obj
 0002:00000c90       ??_C@_0BN@DPBDCOIO@getAccessibleNameFromContext@ 000000018002bc90     AccessBridgeJavaEntryPoints.obj
 0002:00000cb0       ??_C@_0CE@IOFJICIE@getAccessibleDescriptionFromCon@ 000000018002bcb0     AccessBridgeJavaEntryPoints.obj
 0002:00000cd8       ??_C@_0CD@DDGCACMP@getAccessibleRoleStringFromCont@ 000000018002bcd8     AccessBridgeJavaEntryPoints.obj
 0002:00000d00       ??_C@_0CJ@OOFFKIOD@getAccessibleRoleStringFromCont@ 000000018002bd00     AccessBridgeJavaEntryPoints.obj
 0002:00000d30       ??_C@_0CF@JIKEBCCK@getAccessibleStatesStringFromCo@ 000000018002bd30     AccessBridgeJavaEntryPoints.obj
 0002:00000d58       ??_C@_0CL@EODHLGAL@getAccessibleStatesStringFromCo@ 000000018002bd58     AccessBridgeJavaEntryPoints.obj
 0002:00000d88       ??_C@_0CG@LAIPJCLP@getAccessibleIndexInParentFromC@ 000000018002bd88     AccessBridgeJavaEntryPoints.obj
 0002:00000db0       ??_C@_0CG@KMCKGMOL@getAccessibleChildrenCountFromC@ 000000018002bdb0     AccessBridgeJavaEntryPoints.obj
 0002:00000de0       ??_C@_0FC@MAPACPFB@?$CILjavax?1accessibility?1Accessibl@ 000000018002bde0     AccessBridgeJavaEntryPoints.obj
 0002:00000e38       ??_C@_0BO@BJCAFAFF@getAccessibleChildFromContext@ 000000018002be38     AccessBridgeJavaEntryPoints.obj
 0002:00000e58       ??_C@_0DO@DCCADJME@?$CILjavax?1accessibility?1Accessibl@ 000000018002be58     AccessBridgeJavaEntryPoints.obj
 0002:00000e98       ??_C@_0CH@EEFIDNHA@getAccessibleBoundsOnScreenFrom@ 000000018002be98     AccessBridgeJavaEntryPoints.obj
 0002:00000ec0       ??_C@_0BP@FJIKBALD@getAccessibleXcoordFromContext@ 000000018002bec0     AccessBridgeJavaEntryPoints.obj
 0002:00000ee0       ??_C@_0BP@LGNIKGFC@getAccessibleYcoordFromContext@ 000000018002bee0     AccessBridgeJavaEntryPoints.obj
 0002:00000f00       ??_C@_0BP@EMIHBOON@getAccessibleHeightFromContext@ 000000018002bf00     AccessBridgeJavaEntryPoints.obj
 0002:00000f20       ??_C@_0BO@OAEOJGNL@getAccessibleWidthFromContext@ 000000018002bf20     AccessBridgeJavaEntryPoints.obj
 0002:00000f40       ??_C@_0FD@DOBAJOLJ@?$CILjavax?1accessibility?1Accessibl@ 000000018002bf40     AccessBridgeJavaEntryPoints.obj
 0002:00000f98       ??_C@_0CC@MHPILDJI@getAccessibleComponentFromConte@ 000000018002bf98     AccessBridgeJavaEntryPoints.obj
 0002:00000fc0       ??_C@_0FA@DEIINAGF@?$CILjavax?1accessibility?1Accessibl@ 000000018002bfc0     AccessBridgeJavaEntryPoints.obj
 0002:00001010       ??_C@_0BP@PKDLLPIG@getAccessibleActionFromContext@ 000000018002c010     AccessBridgeJavaEntryPoints.obj
 0002:00001030       ??_C@_0FD@KNPEAGPM@?$CILjavax?1accessibility?1Accessibl@ 000000018002c030     AccessBridgeJavaEntryPoints.obj
 0002:00001088       ??_C@_0CC@BHJMNIGA@getAccessibleSelectionFromConte@ 000000018002c088     AccessBridgeJavaEntryPoints.obj
 0002:000010b0       ??_C@_0EO@JMGLFFGI@?$CILjavax?1accessibility?1Accessibl@ 000000018002c0b0     AccessBridgeJavaEntryPoints.obj
 0002:00001100       ??_C@_0BN@CMHLOCAB@getAccessibleTextFromContext@ 000000018002c100     AccessBridgeJavaEntryPoints.obj
 0002:00001120       ??_C@_0EP@DILHGLKF@?$CILjavax?1accessibility?1Accessibl@ 000000018002c120     AccessBridgeJavaEntryPoints.obj
 0002:00001170       ??_C@_0BO@BFBIPFI@getAccessibleValueFromContext@ 000000018002c170     AccessBridgeJavaEntryPoints.obj
 0002:00001190       ??_C@_0EP@DNAJNMPI@?$CILjavax?1accessibility?1Accessibl@ 000000018002c190     AccessBridgeJavaEntryPoints.obj
 0002:000011e0       ??_C@_0BO@PAPKMEMG@getAccessibleTableFromContext@ 000000018002c1e0     AccessBridgeJavaEntryPoints.obj
 0002:00001200       ??_C@_0EP@HGIIMPLK@?$CILjavax?1accessibility?1Accessibl@ 000000018002c200     AccessBridgeJavaEntryPoints.obj
 0002:00001250       ??_C@_0BO@PDGALDAF@getContextFromAccessibleTable@ 000000018002c250     AccessBridgeJavaEntryPoints.obj
 0002:00001270       ??_C@_0BM@FOJGHDMD@getAccessibleTableRowHeader@ 000000018002c270     AccessBridgeJavaEntryPoints.obj
 0002:00001290       ??_C@_0BP@FNCIHNLO@getAccessibleTableColumnHeader@ 000000018002c290     AccessBridgeJavaEntryPoints.obj
 0002:000012b0       ??_C@_0BL@FHMDFDAE@getAccessibleTableRowCount@ 000000018002c2b0     AccessBridgeJavaEntryPoints.obj
 0002:000012d0       ??_C@_0BO@FPCPCCIG@getAccessibleTableColumnCount@ 000000018002c2d0     AccessBridgeJavaEntryPoints.obj
 0002:000012f0       ??_C@_0FB@MHAEKEPL@?$CILjavax?1accessibility?1Accessibl@ 000000018002c2f0     AccessBridgeJavaEntryPoints.obj
 0002:00001348       ??_C@_0CI@CIBBMNLI@getAccessibleTableCellAccessibl@ 000000018002c348     AccessBridgeJavaEntryPoints.obj
 0002:00001370       ??_C@_0CL@HMHFCPKO@?$CILjavax?1accessibility?1Accessibl@ 000000018002c370     AccessBridgeJavaEntryPoints.obj
 0002:000013a0       ??_C@_0BM@BBCGJJGP@getAccessibleTableCellIndex@ 000000018002c3a0     AccessBridgeJavaEntryPoints.obj
 0002:000013c0       ??_C@_0CA@MEOFLNBC@getAccessibleTableCellRowExtent@ 000000018002c3c0     AccessBridgeJavaEntryPoints.obj
 0002:000013e0       ??_C@_0CD@GOAKABO@getAccessibleTableCellColumnExt@ 000000018002c3e0     AccessBridgeJavaEntryPoints.obj
 0002:00001408       ??_C@_0CL@BNJKGODM@?$CILjavax?1accessibility?1Accessibl@ 000000018002c408     AccessBridgeJavaEntryPoints.obj
 0002:00001438       ??_C@_0BO@KIDDCDEB@isAccessibleTableCellSelected@ 000000018002c438     AccessBridgeJavaEntryPoints.obj
 0002:00001458       ??_C@_0CE@NOEAKJPM@getAccessibleTableRowHeaderRowC@ 000000018002c458     AccessBridgeJavaEntryPoints.obj
 0002:00001480       ??_C@_0CH@NOEKFODF@getAccessibleTableColumnHeaderR@ 000000018002c480     AccessBridgeJavaEntryPoints.obj
 0002:000014a8       ??_C@_0CH@HOBKNLMK@getAccessibleTableRowHeaderColu@ 000000018002c4a8     AccessBridgeJavaEntryPoints.obj
 0002:000014d0       ??_C@_0CK@FLEMOIGB@getAccessibleTableColumnHeaderC@ 000000018002c4d0     AccessBridgeJavaEntryPoints.obj
 0002:00001500       ??_C@_0FA@NJKKHECI@?$CILjavax?1accessibility?1Accessibl@ 000000018002c500     AccessBridgeJavaEntryPoints.obj
 0002:00001550       ??_C@_0CB@KCKFJBAJ@getAccessibleTableRowDescriptio@ 000000018002c550     AccessBridgeJavaEntryPoints.obj
 0002:00001578       ??_C@_0CE@KHNFECJN@getAccessibleTableColumnDescrip@ 000000018002c578     AccessBridgeJavaEntryPoints.obj
 0002:000015a0       ??_C@_0CJ@HGNCMOOJ@?$CILjavax?1accessibility?1Accessibl@ 000000018002c5a0     AccessBridgeJavaEntryPoints.obj
 0002:000015d0       ??_C@_0CE@CDNGIBEK@getAccessibleTableRowSelectionC@ 000000018002c5d0     AccessBridgeJavaEntryPoints.obj
 0002:000015f8       ??_C@_0CK@OKAFABOP@?$CILjavax?1accessibility?1Accessibl@ 000000018002c5f8     AccessBridgeJavaEntryPoints.obj
 0002:00001628       ??_C@_0BN@PCLDBBIG@isAccessibleTableRowSelected@ 000000018002c628     AccessBridgeJavaEntryPoints.obj
 0002:00001648       ??_C@_0CK@ILOKEAHN@?$CILjavax?1accessibility?1Accessibl@ 000000018002c648     AccessBridgeJavaEntryPoints.obj
 0002:00001678       ??_C@_0CA@CNAAIKJJ@getAccessibleTableRowSelections@ 000000018002c678     AccessBridgeJavaEntryPoints.obj
 0002:00001698       ??_C@_0CH@CDNMHGID@getAccessibleTableColumnSelecti@ 000000018002c698     AccessBridgeJavaEntryPoints.obj
 0002:000016c0       ??_C@_0CA@NFOBJKJN@isAccessibleTableColumnSelected@ 000000018002c6c0     AccessBridgeJavaEntryPoints.obj
 0002:000016e0       ??_C@_0CD@FNIEANFO@getAccessibleTableColumnSelecti@ 000000018002c6e0     AccessBridgeJavaEntryPoints.obj
 0002:00001708       ??_C@_0BG@JNIAKEE@getAccessibleTableRow@ 000000018002c708     AccessBridgeJavaEntryPoints.obj
 0002:00001720       ??_C@_0BJ@DEHNOIGE@getAccessibleTableColumn@ 000000018002c720     AccessBridgeJavaEntryPoints.obj
 0002:00001740       ??_C@_0BI@MLOHLDGL@getAccessibleTableIndex@ 000000018002c740     AccessBridgeJavaEntryPoints.obj
 0002:00001758       ??_C@_0BL@NLFDIBPJ@getAccessibleRelationCount@ 000000018002c758     AccessBridgeJavaEntryPoints.obj
 0002:00001778       ??_C@_0DN@BLNOMAFI@?$CILjavax?1accessibility?1Accessibl@ 000000018002c778     AccessBridgeJavaEntryPoints.obj
 0002:000017b8       ??_C@_0BJ@DOGHLHFJ@getAccessibleRelationKey@ 000000018002c7b8     AccessBridgeJavaEntryPoints.obj
 0002:000017d8       ??_C@_0CM@KJPNEAF@?$CILjavax?1accessibility?1Accessibl@ 000000018002c7d8     AccessBridgeJavaEntryPoints.obj
 0002:00001808       ??_C@_0CB@ONJFHOJM@getAccessibleRelationTargetCoun@ 000000018002c808     AccessBridgeJavaEntryPoints.obj
 0002:00001830       ??_C@_0FD@OOMEDHDI@?$CILjavax?1accessibility?1Accessibl@ 000000018002c830     AccessBridgeJavaEntryPoints.obj
 0002:00001888       ??_C@_0BM@MFFGDMCG@getAccessibleRelationTarget@ 000000018002c888     AccessBridgeJavaEntryPoints.obj
 0002:000018b0       ??_C@_0FD@IPGDKGIL@?$CILjavax?1accessibility?1Accessibl@ 000000018002c8b0     AccessBridgeJavaEntryPoints.obj
 0002:00001908       ??_C@_0BH@IPNEFMCF@getAccessibleHypertext@ 000000018002c908     AccessBridgeJavaEntryPoints.obj
 0002:00001920       ??_C@_0FE@PMDDAMJI@?$CILjavax?1accessibility?1Accessibl@ 000000018002c920     AccessBridgeJavaEntryPoints.obj
 0002:00001978       ??_C@_0BM@JMCFFMCN@activateAccessibleHyperlink@ 000000018002c978     AccessBridgeJavaEntryPoints.obj
 0002:00001998       ??_C@_0BM@IADLHNKN@getAccessibleHyperlinkCount@ 000000018002c998     AccessBridgeJavaEntryPoints.obj
 0002:000019c0       ??_C@_0FG@JAOELFOA@?$CILjavax?1accessibility?1Accessibl@ 000000018002c9c0     AccessBridgeJavaEntryPoints.obj
 0002:00001a18       ??_C@_0BH@EAGDOOIC@getAccessibleHyperlink@ 000000018002ca18     AccessBridgeJavaEntryPoints.obj
 0002:00001a30       ??_C@_0DO@OBGKICOI@?$CILjavax?1accessibility?1Accessibl@ 000000018002ca30     AccessBridgeJavaEntryPoints.obj
 0002:00001a70       ??_C@_0BL@MPKBBMO@getAccessibleHyperlinkText@ 000000018002ca70     AccessBridgeJavaEntryPoints.obj
 0002:00001a90       ??_C@_0BK@DJNACEGJ@getAccessibleHyperlinkURL@ 000000018002ca90     AccessBridgeJavaEntryPoints.obj
 0002:00001ab0       ??_C@_0CN@CAHDBMA@?$CILjavax?1accessibility?1Accessibl@ 000000018002cab0     AccessBridgeJavaEntryPoints.obj
 0002:00001ae0       ??_C@_0CB@LKDEDAHI@getAccessibleHyperlinkStartInde@ 000000018002cae0     AccessBridgeJavaEntryPoints.obj
 0002:00001b08       ??_C@_0BP@KJGEOOIO@getAccessibleHyperlinkEndIndex@ 000000018002cb08     AccessBridgeJavaEntryPoints.obj
 0002:00001b28       ??_C@_0CO@HPBFOBHC@?$CILjavax?1accessibility?1Accessibl@ 000000018002cb28     AccessBridgeJavaEntryPoints.obj
 0002:00001b58       ??_C@_0CA@FBPINCJA@getAccessibleHypertextLinkIndex@ 000000018002cb58     AccessBridgeJavaEntryPoints.obj
 0002:00001b78       ??_C@_0BO@KGNEMCMH@getAccessibleKeyBindingsCount@ 000000018002cb78     AccessBridgeJavaEntryPoints.obj
 0002:00001b98       ??_C@_0CM@PAHADMIP@?$CILjavax?1accessibility?1Accessibl@ 000000018002cb98     AccessBridgeJavaEntryPoints.obj
 0002:00001bc8       ??_C@_0BM@HBNEDKIN@getAccessibleKeyBindingChar@ 000000018002cbc8     AccessBridgeJavaEntryPoints.obj
 0002:00001be8       ??_C@_0CB@CIMFEKNG@getAccessibleKeyBindingModifier@ 000000018002cbe8     AccessBridgeJavaEntryPoints.obj
 0002:00001c10       ??_C@_0BI@MJKKDJIF@getAccessibleIconsCount@ 000000018002cc10     AccessBridgeJavaEntryPoints.obj
 0002:00001c28       ??_C@_0BN@CJEBMOD@getAccessibleIconDescription@ 000000018002cc28     AccessBridgeJavaEntryPoints.obj
 0002:00001c48       ??_C@_0BI@MDOGDIAA@getAccessibleIconHeight@ 000000018002cc48     AccessBridgeJavaEntryPoints.obj
 0002:00001c60       ??_C@_0BH@GGKEIMGD@getAccessibleIconWidth@ 000000018002cc60     AccessBridgeJavaEntryPoints.obj
 0002:00001c78       ??_C@_0BK@PKOFGGNC@getAccessibleActionsCount@ 000000018002cc78     AccessBridgeJavaEntryPoints.obj
 0002:00001c98       ??_C@_0BI@DODALGBC@getAccessibleActionName@ 000000018002cc98     AccessBridgeJavaEntryPoints.obj
 0002:00001cb0       ??_C@_0BE@CCPKEBNJ@doAccessibleActions@ 000000018002ccb0     AccessBridgeJavaEntryPoints.obj
 0002:00001cc8       ??_C@_0CC@JCBADKJK@getAccessibleCharCountFromConte@ 000000018002ccc8     AccessBridgeJavaEntryPoints.obj
 0002:00001cf0       ??_C@_0CG@KPDPNIKI@getAccessibleCaretPositionFromC@ 000000018002ccf0     AccessBridgeJavaEntryPoints.obj
 0002:00001d18       ??_C@_0CN@CCCKKDDE@?$CILjavax?1accessibility?1Accessibl@ 000000018002cd18     AccessBridgeJavaEntryPoints.obj
 0002:00001d48       ??_C@_0CF@IPJFBKEC@getAccessibleIndexAtPointFromCo@ 000000018002cd48     AccessBridgeJavaEntryPoints.obj
 0002:00001d70       ??_C@_0CG@CGEAMPNI@getAccessibleLetterAtIndexFromC@ 000000018002cd70     AccessBridgeJavaEntryPoints.obj
 0002:00001d98       ??_C@_0CE@CLNANFEE@getAccessibleWordAtIndexFromCon@ 000000018002cd98     AccessBridgeJavaEntryPoints.obj
 0002:00001dc0       ??_C@_0CI@BJNPGKMI@getAccessibleSentenceAtIndexFro@ 000000018002cdc0     AccessBridgeJavaEntryPoints.obj
 0002:00001de8       ??_C@_0CL@HGHPNDH@getAccessibleTextSelectionStart@ 000000018002cde8     AccessBridgeJavaEntryPoints.obj
 0002:00001e18       ??_C@_0CJ@IPEBCNBB@getAccessibleTextSelectionEndFr@ 000000018002ce18     AccessBridgeJavaEntryPoints.obj
 0002:00001e48       ??_C@_0CJ@IBCLFAFA@getAccessibleTextSelectedTextFr@ 000000018002ce48     AccessBridgeJavaEntryPoints.obj
 0002:00001e78       ??_C@_0CK@JLPCFBLN@getAccessibleAttributesAtIndexF@ 000000018002ce78     AccessBridgeJavaEntryPoints.obj
 0002:00001eb0       ??_C@_0EK@JEPLCIJI@?$CILjavax?1accessibility?1Accessibl@ 000000018002ceb0     AccessBridgeJavaEntryPoints.obj
 0002:00001f00       ??_C@_0CM@LKNKHCB@getAccessibleAttributeSetAtInde@ 000000018002cf00     AccessBridgeJavaEntryPoints.obj
 0002:00001f30       ??_C@_0DP@HKEBFOCN@?$CILjavax?1accessibility?1Accessibl@ 000000018002cf30     AccessBridgeJavaEntryPoints.obj
 0002:00001f70       ??_C@_0CI@IIHCGONP@getAccessibleTextRectAtIndexFro@ 000000018002cf70     AccessBridgeJavaEntryPoints.obj
 0002:00001f98       ??_C@_0CO@OMLKOFDL@getAccessibleXcoordTextRectAtIn@ 000000018002cf98     AccessBridgeJavaEntryPoints.obj
 0002:00001fc8       ??_C@_0CO@NKEIHFMI@getAccessibleYcoordTextRectAtIn@ 000000018002cfc8     AccessBridgeJavaEntryPoints.obj
 0002:00001ff8       ??_C@_0CO@JHFMLGGO@getAccessibleHeightTextRectAtIn@ 000000018002cff8     AccessBridgeJavaEntryPoints.obj
 0002:00002028       ??_C@_0CN@COKFHFFE@getAccessibleWidthTextRectAtInd@ 000000018002d028     AccessBridgeJavaEntryPoints.obj
 0002:00002058       ??_C@_0BC@NPONPPPN@getCaretLocationX@ 000000018002d058     AccessBridgeJavaEntryPoints.obj
 0002:00002070       ??_C@_0BC@MGPGMOLM@getCaretLocationY@ 000000018002d070     AccessBridgeJavaEntryPoints.obj
 0002:00002088       ??_C@_0BH@MJJIPGPF@getCaretLocationHeight@ 000000018002d088     AccessBridgeJavaEntryPoints.obj
 0002:000020a0       ??_C@_0BG@BIMEFOON@getCaretLocationWidth@ 000000018002d0a0     AccessBridgeJavaEntryPoints.obj
 0002:000020b8       ??_C@_0CL@JPPFAPAC@getAccessibleTextLineLeftBounds@ 000000018002d0b8     AccessBridgeJavaEntryPoints.obj
 0002:000020e8       ??_C@_0CM@IBNKHADJ@getAccessibleTextLineRightBound@ 000000018002d0e8     AccessBridgeJavaEntryPoints.obj
 0002:00002118       ??_C@_0DO@MIIPGCPP@?$CILjavax?1accessibility?1Accessibl@ 000000018002d118     AccessBridgeJavaEntryPoints.obj
 0002:00002158       ??_C@_0CC@CIBLKPOK@getAccessibleTextRangeFromConte@ 000000018002d158     AccessBridgeJavaEntryPoints.obj
 0002:00002180       ??_C@_0CF@CJIJHKPD@getCurrentAccessibleValueFromCo@ 000000018002d180     AccessBridgeJavaEntryPoints.obj
 0002:000021a8       ??_C@_0CF@PMHBGBIN@getMaximumAccessibleValueFromCo@ 000000018002d1a8     AccessBridgeJavaEntryPoints.obj
 0002:000021d0       ??_C@_0CF@MEICJJIC@getMinimumAccessibleValueFromCo@ 000000018002d1d0     AccessBridgeJavaEntryPoints.obj
 0002:000021f8       ??_C@_0CM@MHMFNKJL@?$CILjavax?1accessibility?1Accessibl@ 000000018002d1f8     AccessBridgeJavaEntryPoints.obj
 0002:00002228       ??_C@_0CC@OHDKMAMO@addAccessibleSelectionFromConte@ 000000018002d228     AccessBridgeJavaEntryPoints.obj
 0002:00002250       ??_C@_0CL@HAAKHFKD@?$CILjavax?1accessibility?1Accessibl@ 000000018002d250     AccessBridgeJavaEntryPoints.obj
 0002:00002280       ??_C@_0CE@JAJNKBKJ@clearAccessibleSelectionFromCon@ 000000018002d280     AccessBridgeJavaEntryPoints.obj
 0002:000022a8       ??_C@_0CH@GOOENNPE@getAccessibleSelectionCountFrom@ 000000018002d2a8     AccessBridgeJavaEntryPoints.obj
 0002:000022d0       ??_C@_0CM@GLHAJFJH@?$CILjavax?1accessibility?1Accessibl@ 000000018002d2d0     AccessBridgeJavaEntryPoints.obj
 0002:00002300       ??_C@_0CF@PFGNJKHP@isAccessibleChildSelectedFromCo@ 000000018002d300     AccessBridgeJavaEntryPoints.obj
 0002:00002328       ??_C@_0CF@LNEMJFKL@removeAccessibleSelectionFromCo@ 000000018002d328     AccessBridgeJavaEntryPoints.obj
 0002:00002350       ??_C@_0CI@GIPFHPKO@selectAllAccessibleSelectionFro@ 000000018002d350     AccessBridgeJavaEntryPoints.obj
 0002:00002378       ??_C@_04OHLIFDMD@?$CIJ?$CJV@ 000000018002d378     AccessBridgeJavaEntryPoints.obj
 0002:00002380       ??_C@_0BJ@MPIBKFAO@addJavaEventNotification@ 000000018002d380     AccessBridgeJavaEntryPoints.obj
 0002:000023a0       ??_C@_0BM@FNBBPCEJ@removeJavaEventNotification@ 000000018002d3a0     AccessBridgeJavaEntryPoints.obj
 0002:000023c0       ??_C@_0CC@MPLKGCBM@addAccessibilityEventNotificati@ 000000018002d3c0     AccessBridgeJavaEntryPoints.obj
 0002:000023e8       ??_C@_0CF@JFMMDHHJ@removeAccessibilityEventNotific@ 000000018002d3e8     AccessBridgeJavaEntryPoints.obj
 0002:00002410       ??_C@_0CD@PFBLKFGD@?$CILjavax?1swing?1text?1AttributeSet@ 000000018002d410     AccessBridgeJavaEntryPoints.obj
 0002:00002438       ??_C@_0BI@PMOBPKB@getBoldFromAttributeSet@ 000000018002d438     AccessBridgeJavaEntryPoints.obj
 0002:00002450       ??_C@_0BK@HMLEJNMA@getItalicFromAttributeSet@ 000000018002d450     AccessBridgeJavaEntryPoints.obj
 0002:00002470       ??_C@_0BN@BGEODKID@getUnderlineFromAttributeSet@ 000000018002d470     AccessBridgeJavaEntryPoints.obj
 0002:00002490       ??_C@_0CB@BICMGOJK@getStrikethroughFromAttributeSe@ 000000018002d490     AccessBridgeJavaEntryPoints.obj
 0002:000024b8       ??_C@_0BP@BNLEAGAN@getSuperscriptFromAttributeSet@ 000000018002d4b8     AccessBridgeJavaEntryPoints.obj
 0002:000024d8       ??_C@_0BN@FENOLEGG@getSubscriptFromAttributeSet@ 000000018002d4d8     AccessBridgeJavaEntryPoints.obj
 0002:000024f8       ??_C@_0DE@PFGGMCPM@?$CILjavax?1swing?1text?1AttributeSet@ 000000018002d4f8     AccessBridgeJavaEntryPoints.obj
 0002:00002530       ??_C@_0CD@MGNACFJA@getBackgroundColorFromAttribute@ 000000018002d530     AccessBridgeJavaEntryPoints.obj
 0002:00002558       ??_C@_0CD@JFAEMBOF@getForegroundColorFromAttribute@ 000000018002d558     AccessBridgeJavaEntryPoints.obj
 0002:00002580       ??_C@_0BO@JFHBDDGD@getFontFamilyFromAttributeSet@ 000000018002d580     AccessBridgeJavaEntryPoints.obj
 0002:000025a0       ??_C@_0CD@JEPEOEPB@?$CILjavax?1swing?1text?1AttributeSet@ 000000018002d5a0     AccessBridgeJavaEntryPoints.obj
 0002:000025c8       ??_C@_0BM@OMIOBJPB@getFontSizeFromAttributeSet@ 000000018002d5c8     AccessBridgeJavaEntryPoints.obj
 0002:000025e8       ??_C@_0BN@BAFOGOJK@getAlignmentFromAttributeSet@ 000000018002d5e8     AccessBridgeJavaEntryPoints.obj
 0002:00002608       ??_C@_0BN@DEDFHCOP@getBidiLevelFromAttributeSet@ 000000018002d608     AccessBridgeJavaEntryPoints.obj
 0002:00002628       ??_C@_0CD@BDGMPIDO@?$CILjavax?1swing?1text?1AttributeSet@ 000000018002d628     AccessBridgeJavaEntryPoints.obj
 0002:00002650       ??_C@_0CD@EJOOBJDB@getFirstLineIndentFromAttribute@ 000000018002d650     AccessBridgeJavaEntryPoints.obj
 0002:00002678       ??_C@_0BO@KCBIJLNO@getLeftIndentFromAttributeSet@ 000000018002d678     AccessBridgeJavaEntryPoints.obj
 0002:00002698       ??_C@_0BP@KEIFBKEA@getRightIndentFromAttributeSet@ 000000018002d698     AccessBridgeJavaEntryPoints.obj
 0002:000026b8       ??_C@_0BP@ICDNCHPN@getLineSpacingFromAttributeSet@ 000000018002d6b8     AccessBridgeJavaEntryPoints.obj
 0002:000026d8       ??_C@_0BO@CHPMHCHE@getSpaceAboveFromAttributeSet@ 000000018002d6d8     AccessBridgeJavaEntryPoints.obj
 0002:000026f8       ??_C@_0BO@DOLMIFOK@getSpaceBelowFromAttributeSet@ 000000018002d6f8     AccessBridgeJavaEntryPoints.obj
 0002:00002718       ??_C@_0CL@NMLPDKKP@?$CILjavax?1accessibility?1Accessibl@ 000000018002d718     AccessBridgeJavaEntryPoints.obj
 0002:00002748       ??_C@_0N@CEMKNPGL@requestFocus@ 000000018002d748     AccessBridgeJavaEntryPoints.obj
 0002:00002758       ??_C@_0CN@EDMFOCKG@?$CILjavax?1accessibility?1Accessibl@ 000000018002d758     AccessBridgeJavaEntryPoints.obj
 0002:00002788       ??_C@_0BA@JKPGAJFL@selectTextRange@ 000000018002d788     AccessBridgeJavaEntryPoints.obj
 0002:00002798       ??_C@_0BI@IIOLCPFK@getVisibleChildrenCount@ 000000018002d798     AccessBridgeJavaEntryPoints.obj
 0002:000027b0       ??_C@_0BA@JIDLMKH@getVisibleChild@ 000000018002d7b0     AccessBridgeJavaEntryPoints.obj
 0002:000027c0       ??_C@_0BB@ENIAPGBO@setCaretPosition@ 000000018002d7c0     AccessBridgeJavaEntryPoints.obj
 0002:000027d8       ??_C@_0CE@MELACKPN@getVirtualAccessibleNameFromCon@ 000000018002d7d8     AccessBridgeJavaEntryPoints.obj
 0002:00002800       ??_C@_0DP@ODHDIMGL@?$FLINFO?$FN?3?5Calling?5AccessBridgeJav@ 000000018002d800     AccessBridgeJavaEntryPoints.obj
 0002:00002840       ??_C@_0DD@INJPOCHE@Getting?5isJavaWindow?5?9?5call?5to?5@ 000000018002d840     AccessBridgeJavaEntryPoints.obj
 0002:00002878       ??_C@_0DN@ENCLOLFG@?$FLERROR?$FN?3?5?$CK?$CK?$CK?5Exception?5occured?5@ 000000018002d878     AccessBridgeJavaEntryPoints.obj
 0002:000028b8       ??_C@_0DH@DHJJKMLN@?$FLERROR?$FN?3?5either?5jniEnv?5?$DN?$DN?50?5or?5@ 000000018002d8b8     AccessBridgeJavaEntryPoints.obj
 0002:000028f0       ??_C@_0DN@GKGIBPBO@?$FLINFO?$FN?3?5In?5AccessBridgeJavaEntr@ 000000018002d8f0     AccessBridgeJavaEntryPoints.obj
 0002:00002930       ??_C@_0BF@LOIOEBHF@Calling?5IsSameObject@ 000000018002d930     AccessBridgeJavaEntryPoints.obj
 0002:00002948       ??_C@_0CE@PJOLBDKG@?$FLINFO?$FN?3?5?5?5isSameObject?5returnin@ 000000018002d948     AccessBridgeJavaEntryPoints.obj
 0002:00002970       ??_C@_0EK@MPPKLDGH@?$FLINFO?$FN?3?5In?5AccessBridgeJavaEntr@ 000000018002d970     AccessBridgeJavaEntryPoints.obj
 0002:000029c0       ??_C@_0DP@INBKCEII@Getting?5AccessibleContextFromHW@ 000000018002d9c0     AccessBridgeJavaEntryPoints.obj
 0002:00002a00       ??_C@_0EI@POHJNOIF@?$FLERROR?$FN?3?5?5either?5jniEnv?5?$DN?$DN?50?5or@ 000000018002da00     AccessBridgeJavaEntryPoints.obj
 0002:00002a50       ??_C@_0EK@KGPHBKLN@?$FLINFO?$FN?3?5In?5AccessBridgeJavaEntr@ 000000018002da50     AccessBridgeJavaEntryPoints.obj
 0002:00002aa0       ??_C@_0DM@OPKABADC@Getting?5HWNDFromAccessibleConte@ 000000018002daa0     AccessBridgeJavaEntryPoints.obj
 0002:00002ae0       ??_C@_0BD@NKFEMHLM@?$FLINFO?$FN?3?5rHWND?5?$DN?5?$CFX@ 000000018002dae0     AccessBridgeJavaEntryPoints.obj
 0002:00002b00       ??_C@_0EH@MFPOIGJN@?$FLERROR?$FN?3?5either?5jniEnv?5?$DN?$DN?50?5or?5@ 000000018002db00     AccessBridgeJavaEntryPoints.obj
 0002:00002b50       ??_C@_0EC@BPPANMDJ@?$FLINFO?$FN?3?5In?5AccessBridgeJavaEntr@ 000000018002db50     AccessBridgeJavaEntryPoints.obj
 0002:00002b98       ??_C@_0BN@LGGMDMGD@?$FLERROR?$FN?3?5?5?5?5NewString?5failed@ 000000018002db98     AccessBridgeJavaEntryPoints.obj
 0002:00002bb8       ??_C@_0CO@NCDGKPGB@setTextContents?5?9?5call?5to?5CallB@ 000000018002dbb8     AccessBridgeJavaEntryPoints.obj
 0002:00002be8       ??_C@_0BI@IMHMFAIB@?$FLINFO?$FN?3?5?5?5?5?5result?5?$DN?5?$CFd@ 000000018002dbe8     AccessBridgeJavaEntryPoints.obj
 0002:00002c00       ??_C@_0DK@MGDAPF@?$FLERROR?$FN?3?5either?5jniEnv?5?$DN?$DN?50?5or?5@ 000000018002dc00     AccessBridgeJavaEntryPoints.obj
 0002:00002c40       ??_C@_0DP@LHNNHOD@?$FLINFO?$FN?3?5In?5AccessBridgeJavaEntr@ 000000018002dc40     AccessBridgeJavaEntryPoints.obj
 0002:00002c80       ??_C@_0BO@LLFKIHLA@?$FLERROR?$FN?3?5?5?5?5?5NewString?5failed@ 000000018002dc80     AccessBridgeJavaEntryPoints.obj
 0002:00002ca0       ??_C@_0DE@KBFMBJPI@Getting?5ParentWithRole?5?9?5call?5t@ 000000018002dca0     AccessBridgeJavaEntryPoints.obj
 0002:00002cd8       ??_C@_0CE@LNEDINGM@?$FLINFO?$FN?3?5?5?5?5?5rAccessibleContext?5@ 000000018002dcd8     AccessBridgeJavaEntryPoints.obj
 0002:00002d00       ??_C@_0DA@OMNPGENP@Getting?5ParentWithRole?5?9?5call?5t@ 000000018002dd00     AccessBridgeJavaEntryPoints.obj
 0002:00002d30       ??_C@_0EF@LHAMKGPK@?$FLINFO?$FN?3?5?5?5Returning?5?9?5returnedA@ 000000018002dd30     AccessBridgeJavaEntryPoints.obj
 0002:00002d78       ??_C@_0DM@OLEIFDLG@?$FLERROR?$FN?3?5either?5jniEnv?5?$DN?$DN?50?5or?5@ 000000018002dd78     AccessBridgeJavaEntryPoints.obj
 0002:00002db8       ??_C@_0DP@EPHBFJKE@?$FLINFO?$FN?3?5In?5AccessBridgeJavaEntr@ 000000018002ddb8     AccessBridgeJavaEntryPoints.obj
 0002:00002df8       ??_C@_0DE@FDIFCLEM@Getting?5TopLevelObject?5?9?5call?5t@ 000000018002ddf8     AccessBridgeJavaEntryPoints.obj
 0002:00002e30       ??_C@_0CB@GDMCCFCK@?$FLINFO?$FN?3?5?5rAccessibleContext?5?$DN?5?$CF@ 000000018002de30     AccessBridgeJavaEntryPoints.obj
 0002:00002e58       ??_C@_0DA@ELIJHKN@Getting?5TopLevelObject?5?9?5call?5t@ 000000018002de58     AccessBridgeJavaEntryPoints.obj
 0002:00002e88       ??_C@_0DM@MKIGPNDF@?$FLERROR?$FN?3?5either?5jniEnv?5?$DN?$DN?50?5or?5@ 000000018002de88     AccessBridgeJavaEntryPoints.obj
 0002:00002ed0       ??_C@_0EH@MCHGGFNF@?$FLINFO?$FN?3?5In?5AccessBridgeJavaEntr@ 000000018002ded0     AccessBridgeJavaEntryPoints.obj
 0002:00002f18       ??_C@_0DM@IKNMPPHI@Getting?5ParentWithRoleElseRoot?5@ 000000018002df18     AccessBridgeJavaEntryPoints.obj
 0002:00002f58       ??_C@_0DI@CDJCPAOF@Getting?5ParentWithRoleElseRoot?5@ 000000018002df58     AccessBridgeJavaEntryPoints.obj
 0002:00002f90       ??_C@_0EF@MODADMKL@?$FLERROR?$FN?3?5?5either?5jniEnv?5?$DN?$DN?50?5or@ 000000018002df90     AccessBridgeJavaEntryPoints.obj
 0002:00002fd8       ??_C@_0DM@EBONPKNN@?$FLINFO?$FN?3?5In?5AccessBridgeJavaEntr@ 000000018002dfd8     AccessBridgeJavaEntryPoints.obj
 0002:00003018       ??_C@_0CO@CCBFEFG@Getting?5ObjectDepth?5?9?5call?5to?5C@ 000000018002e018     AccessBridgeJavaEntryPoints.obj
 0002:00003048       ??_C@_0BJ@KJFHIGKC@?$FLINFO?$FN?3?5?5?5?5?5rResult?5?$DN?5?$CFd@ 000000018002e048     AccessBridgeJavaEntryPoints.obj
 0002:00003068       ??_C@_0DJ@NCMDONA@?$FLERROR?$FN?3?5either?5jniEnv?5?$DN?$DN?50?5or?5@ 000000018002e068     AccessBridgeJavaEntryPoints.obj
 0002:000030b0       ??_C@_0EB@OJAHMNKI@?$FLINFO?$FN?3?5In?5AccessBridgeJavaEntr@ 000000018002e0b0     AccessBridgeJavaEntryPoints.obj
 0002:000030f8       ??_C@_0DG@FKCKDOAD@Getting?5ActiveDescendent?5?9?5call@ 000000018002e0f8     AccessBridgeJavaEntryPoints.obj
 0002:00003130       ??_C@_0DC@DOJHNKHC@Getting?5ActiveDescendant?5?9?5call@ 000000018002e130     AccessBridgeJavaEntryPoints.obj
 0002:00003168       ??_C@_0DO@FBKMCPK@?$FLERROR?$FN?3?5either?5jniEnv?5?$DN?$DN?50?5or?5@ 000000018002e168     AccessBridgeJavaEntryPoints.obj
 0002:000031a8       ??_C@_0CK@IFAHAOG@?$FLINFO?$FN?3?5?5getVirtualAccessibleNa@ 000000018002e1a8     AccessBridgeJavaEntryPoints.obj
 0002:000031d8       ??_C@_0DE@GLGPLDPG@Getting?5AccessibleName?5?9?5call?5t@ 000000018002e1d8     AccessBridgeJavaEntryPoints.obj
 0002:00003210       ??_C@_0DC@LMABNHGH@Getting?5AccessibleName?5?9?5call?5t@ 000000018002e210     AccessBridgeJavaEntryPoints.obj
 0002:00003248       ??_C@_0BH@PDDJGLOG@Getting?5AccessibleName@ 000000018002e248     AccessBridgeJavaEntryPoints.obj
 0002:00003260       ??_C@_0FH@LIIILLEC@?$FLERROR?$FN?3?5?$CK?$CK?$CK?5Exception?5occured?5@ 000000018002e260     AccessBridgeJavaEntryPoints.obj
 0002:000032c0       ??_C@_0FK@LMDLLNDA@?$FLERROR?$FN?3?5?$CK?$CK?$CK?5Exception?5occured?5@ 000000018002e2c0     AccessBridgeJavaEntryPoints.obj
 0002:00003320       ??_C@_0DC@MBCPGFEL@Getting?5AccessibleName?5?9?5call?5t@ 000000018002e320     AccessBridgeJavaEntryPoints.obj
 0002:00003358       ??_C@_1DA@BACBNKJB@?$AA?5?$AA?5?$AAA?$AAc?$AAc?$AAe?$AAs?$AAs?$AAi?$AAb?$AAl?$AAe?$AA?5?$AAN?$AAa@ 000000018002e358     AccessBridgeJavaEntryPoints.obj
 0002:00003388       ??_C@_0DC@HCPEBFPJ@Getting?5AccessibleName?5?9?5call?5t@ 000000018002e388     AccessBridgeJavaEntryPoints.obj
 0002:000033c0       ??_C@_0CD@JNOMKFNM@?$FLINFO?$FN?3?5?5?5Accessible?5Name?5is?5nu@ 000000018002e3c0     AccessBridgeJavaEntryPoints.obj
 0002:000033f0       ??_C@_0EN@LBGKPBFG@?$FLINFO?$FN?3?5either?5jniEnv?5?$DN?$DN?50?5or?5g@ 000000018002e3f0     AccessBridgeJavaEntryPoints.obj
 0002:00003440       ??_C@_0DK@COLMCNJL@?$FLINFO?$FN?3?5In?5AccessBridgeJavaEntr@ 000000018002e440     AccessBridgeJavaEntryPoints.obj
 0002:00003480       ??_C@_0CL@OHFNFEAE@requestFocus?5?9?5call?5to?5CallBool@ 000000018002e480     AccessBridgeJavaEntryPoints.obj
 0002:000034b0       ??_C@_0BH@JOKEJIHH@?$FLINFO?$FN?3?5?5?5?5result?5?$DN?5?$CFd@ 000000018002e4b0     AccessBridgeJavaEntryPoints.obj
 0002:000034c8       ??_C@_0DH@OADKFKDG@?$FLERROR?$FN?3?5either?5jniEnv?5?$DN?$DN?50?5or?5@ 000000018002e4c8     AccessBridgeJavaEntryPoints.obj
 0002:00003500       ??_C@_0FB@HEEEBDKB@?$FLINFO?$FN?3?5In?5AccessBridgeJavaEntr@ 000000018002e500     AccessBridgeJavaEntryPoints.obj
 0002:00003558       ??_C@_0CO@NOPLEGNC@selectTextRange?5?9?5call?5to?5CallB@ 000000018002e558     AccessBridgeJavaEntryPoints.obj
 0002:00003588       ??_C@_0DK@EDLAMPCD@?$FLERROR?$FN?3?5either?5jniEnv?5?$DN?$DN?50?5or?5@ 000000018002e588     AccessBridgeJavaEntryPoints.obj
 0002:000035d0       ??_C@_0FK@CBBPCLFD@?$FLINFO?$FN?3?5In?5AccessBridgeJavaEntr@ 000000018002e5d0     AccessBridgeJavaEntryPoints.obj
 0002:00003630       ??_C@_0DN@CIOOGMLK@?$FLINFO?$FN?3?5?5Getting?5full?5test_attr@ 000000018002e630     AccessBridgeJavaEntryPoints.obj
 0002:00003670       ??_C@_0EB@FNOCJLAN@Getting?5AccessibleAttributesAtI@ 000000018002e670     AccessBridgeJavaEntryPoints.obj
 0002:000036b8       ??_C@_0DE@NPIJKEOK@?$FLINFO?$FN?3?5?5?5returned?5from?5CallObj@ 000000018002e6b8     AccessBridgeJavaEntryPoints.obj
 0002:000036f0       ??_C@_0DP@GAODIEPK@Getting?5AccessibleAttributesAtI@ 000000018002e6f0     AccessBridgeJavaEntryPoints.obj
 0002:00003730       ??_C@_0CE@KAHCBNHC@Getting?5AccessibleAttributesAtI@ 000000018002e730     AccessBridgeJavaEntryPoints.obj
 0002:00003758       ??_C@_0DP@BNMNDGNG@Getting?5AccessibleAttributesAtI@ 000000018002e758     AccessBridgeJavaEntryPoints.obj
 0002:000037a0       ??_C@_1FE@NAFGNNMA@?$AA?$FL?$AAI?$AAN?$AAF?$AAO?$AA?$FN?$AA?3?$AA?5?$AA?5?$AAA?$AAc?$AAc?$AAe?$AAs?$AAs@ 000000018002e7a0     AccessBridgeJavaEntryPoints.obj
 0002:000037f8       ??_C@_0DP@KOBGEGGE@Getting?5AccessibleAttributesAtI@ 000000018002e7f8     AccessBridgeJavaEntryPoints.obj
 0002:00003838       ??_C@_0CO@GBFCDBDB@?$FLWARN?$FN?3?5?5?5Accessible?5Text?5attri@ 000000018002e838     AccessBridgeJavaEntryPoints.obj
 0002:00003870       ??_C@_0FB@DKHOICMI@?$FLERROR?$FN?3?5either?5env?5?$DN?$DN?50?5or?5get@ 000000018002e870     AccessBridgeJavaEntryPoints.obj
 0002:000038d0       ??_C@_0EH@KKFBHMJC@?$FLINFO?$FN?3?5?$CD?$CD?$CD?$CD?$CD?5AccessBridgeJavaE@ 000000018002e8d0     AccessBridgeJavaEntryPoints.obj
 0002:00003918       ??_C@_0DP@MHLDKAGF@?$CD?$CD?$CD?$CD?$CD?5Getting?5visible?5children?5@ 000000018002e918     AccessBridgeJavaEntryPoints.obj
 0002:00003958       ??_C@_0CM@JAPBNGLO@?$FLINFO?$FN?3?5?5?5?$CD?$CD?$CD?$CD?$CD?5visible?5childre@ 000000018002e958     AccessBridgeJavaEntryPoints.obj
 0002:00003990       ??_C@_0FD@GLIPOPHN@?$FLINFO?$FN?3?5?$CD?$CD?$CD?$CD?$CD?5AccessBridgeJavaE@ 000000018002e990     AccessBridgeJavaEntryPoints.obj
 0002:000039e8       ??_C@_0CH@ONKDDCMN@?$FLINFO?$FN?3?5?5?5getting?5visible?5child@ 000000018002e9e8     AccessBridgeJavaEntryPoints.obj
 0002:00003a10       ??_C@_0DJ@HGPLCHEB@?$CD?$CD?$CD?$CD?$CD?5getVisibleChildMethod?5?9?5c@ 000000018002ea10     AccessBridgeJavaEntryPoints.obj
 0002:00003a50       ??_C@_0DF@JHJIJJH@?$CD?$CD?$CD?$CD?$CD?5getVisibleChildMethod?5?9?5c@ 000000018002ea50     AccessBridgeJavaEntryPoints.obj
 0002:00003a88       ??_C@_0CD@ECMHOCH@?$FLINFO?$FN?3?5?5?5?$CD?$CD?$CD?$CD?$CD?5visible?5child?5?$DN@ 000000018002ea88     AccessBridgeJavaEntryPoints.obj
 0002:00003ab0       ??_C@_0EK@GNPPBBMN@?$FLINFO?$FN?3?5?5?5?$CD?$CD?$CD?$CD?$CD?5AccessBridgeJav@ 000000018002eab0     AccessBridgeJavaEntryPoints.obj
 0002:00003b00       ??_C@_0EL@OPKFGOFA@?$FLINFO?$FN?3?5In?5AccessBridgeJavaEntr@ 000000018002eb00     AccessBridgeJavaEntryPoints.obj
 0002:00003b50       ??_C@_0CO@BDNAFHGG@setCaretPostion?5?9?5call?5to?5CallB@ 000000018002eb50     AccessBridgeJavaEntryPoints.obj
 0002:00003b80       ??_C@_0BJ@PGHBDIPI@?$FLERROR?$FN?3?5?5?5?5?5result?5?$DN?5?$CFd@ 000000018002eb80     AccessBridgeJavaEntryPoints.obj
 0002:00003ba0       ??_C@_0DL@CBEPMOL@?$FLERROR?$FN?3?5either?5jniEnv?5?$DN?$DN?50?5or?5@ 000000018002eba0     AccessBridgeJavaEntryPoints.obj
 0002:00003be0       ??_C@_0DP@DPLDEGDE@?$FLINFO?$FN?3?5Calling?5AccessBridgeJav@ 000000018002ebe0     AccessBridgeJavaEntryPoints.obj
 0002:00003c20       ??_C@_0DJ@EBEOKJAG@Getting?5JavaVersionProperty?5?9?5c@ 000000018002ec20     AccessBridgeJavaEntryPoints.obj
 0002:00003c60       ??_C@_0FC@KFJABCDE@?$FLERROR?$FN?3?5?5?$CK?$CK?$CK?5Exception?5when?5ge@ 000000018002ec60     AccessBridgeJavaEntryPoints.obj
 0002:00003cb8       ??_C@_0DL@FDAICLOI@Getting?5JavaVersionProperty?5?9?5c@ 000000018002ecb8     AccessBridgeJavaEntryPoints.obj
 0002:00003cf8       ??_C@_0DH@PEMIMKKJ@Getting?5JavaVersionProperty?5?9?5c@ 000000018002ecf8     AccessBridgeJavaEntryPoints.obj
 0002:00003d30       ??_C@_1CK@PFPDBLJ@?$AA?5?$AA?5?$AAJ?$AAa?$AAv?$AAa?$AA?5?$AAv?$AAe?$AAr?$AAs?$AAi?$AAo?$AAn?$AA?5@ 000000018002ed30     AccessBridgeJavaEntryPoints.obj
 0002:00003d60       ??_C@_0DH@EHBDLKBL@Getting?5JavaVersionProperty?5?9?5c@ 000000018002ed60     AccessBridgeJavaEntryPoints.obj
 0002:00003d98       ??_C@_0CA@KOJKOLB@?$FLWARN?$FN?3?5?5?5Java?5version?5is?5null?4@ 000000018002ed98     AccessBridgeJavaEntryPoints.obj
 0002:00003db8       ??_C@_0DP@FHBJPJDO@?$FLERROR?$FN?3?5?5either?5env?5?$DN?$DN?50?5or?5ge@ 000000018002edb8     AccessBridgeJavaEntryPoints.obj
 0002:00003e00       ??_C@_0EC@OAJCCJEK@?$FLINFO?$FN?3?5Calling?5AccessBridgeJav@ 000000018002ee00     AccessBridgeJavaEntryPoints.obj
 0002:00003e48       ??_C@_0BF@MJCCCBHB@?$FLERROR?$FN?3?5?5No?5Java?5VM@ 000000018002ee48     AccessBridgeJavaEntryPoints.obj
 0002:00003e60       ??_C@_0BH@PCLEJECO@?$FLERROR?$FN?3?5?5Null?5jobject@ 000000018002ee60     AccessBridgeJavaEntryPoints.obj
 0002:00003e78       ??_C@_0DE@FOOENAKM@Getting?5AccessibleText?5?9?5call?5t@ 000000018002ee78     AccessBridgeJavaEntryPoints.obj
 0002:00003eb0       ??_C@_0BP@NHKMDDHI@?$FLERROR?$FN?3?5?5?5AccessibleText?5?$DN?5?$CFp@ 000000018002eeb0     AccessBridgeJavaEntryPoints.obj
 0002:00003ed0       ??_C@_0DC@NHCDOGBO@Getting?5AccessibleText?5?9?5call?5t@ 000000018002eed0     AccessBridgeJavaEntryPoints.obj
 0002:00003f10       ??_C@_0EF@KPMHECBJ@?$FLERROR?$FN?3?5?5either?5env?5?$DN?$DN?50?5or?5ge@ 000000018002ef10     AccessBridgeJavaEntryPoints.obj
 0002:00003f58       ??_C@_0CL@OMBEMJIM@?$FLERROR?$FN?3?5?5jobject?5is?5not?5an?5Acc@ 000000018002ef58     AccessBridgeJavaEntryPoints.obj
 0002:00003f90       ??_C@_0FB@IMPDGAOD@?$FLINFO?$FN?3?5Calling?5AccessBridgeJav@ 000000018002ef90     AccessBridgeJavaEntryPoints.obj
 0002:00003fe8       ??_C@_0DJ@CBKJGOIB@Getting?5AccessibleContextAt?5?9?5c@ 000000018002efe8     AccessBridgeJavaEntryPoints.obj
 0002:00004028       ??_C@_0DF@PJCJKGPI@Getting?5AccessibleContextAt?5?9?5c@ 000000018002f028     AccessBridgeJavaEntryPoints.obj
 0002:00004060       ??_C@_0DP@LFOACNJN@?$FLERROR?$FN?3?5?5either?5env?5?$DN?$DN?50?5or?5ge@ 000000018002f060     AccessBridgeJavaEntryPoints.obj
 0002:000040a0       ??_C@_0EN@LHFHLFOC@?$FLINFO?$FN?3?5Calling?5AccessBridgeJav@ 000000018002f0a0     AccessBridgeJavaEntryPoints.obj
 0002:000040f0       ??_C@_0EA@NLINILPH@Getting?5AccessibleContextWithFo@ 000000018002f0f0     AccessBridgeJavaEntryPoints.obj
 0002:00004130       ??_C@_0DM@IJDJLPBO@Getting?5AccessibleContextWithFo@ 000000018002f130     AccessBridgeJavaEntryPoints.obj
 0002:00004170       ??_C@_0EJ@KBIILIHA@?$FLERROR?$FN?3?5?5either?5jniEnv?5?$DN?$DN?50?5or@ 000000018002f170     AccessBridgeJavaEntryPoints.obj
 0002:000041c0       ??_C@_0FB@NNGDGCK@?$FLINFO?$FN?3?5?$CD?$CD?$CD?$CD?$CD?5Calling?5AccessBri@ 000000018002f1c0     AccessBridgeJavaEntryPoints.obj
 0002:00004218       ??_C@_0DF@BABIDEMG@?$FLWARN?$FN?3?5?5passed?5in?5AccessibleCo@ 000000018002f218     AccessBridgeJavaEntryPoints.obj
 0002:00004250       ??_C@_1EA@IPHAHEJA@?$AA?$FL?$AAI?$AAN?$AAF?$AAO?$AA?$FN?$AA?3?$AA?5?$AA?5?$AA?5?$AAA?$AAc?$AAc?$AAe?$AAs@ 000000018002f250     AccessBridgeJavaEntryPoints.obj
 0002:00004290       ??_C@_0CD@BCDIDKCI@?$FLWARN?$FN?3?5?5?5Accessible?5Name?5is?5nu@ 000000018002f290     AccessBridgeJavaEntryPoints.obj
 0002:000042c0       ??_C@_0EF@DMNCHIBL@?$FLERROR?$FN?3?5?5either?5env?5?$DN?$DN?50?5or?5ge@ 000000018002f2c0     AccessBridgeJavaEntryPoints.obj
 0002:00004308       ??_C@_0DL@IPNAGHCP@Getting?5AccessibleDescription?5?9@ 000000018002f308     AccessBridgeJavaEntryPoints.obj
 0002:00004350       ??_C@_1EO@NBFBPIFN@?$AA?$FL?$AAI?$AAN?$AAF?$AAO?$AA?$FN?$AA?3?$AA?5?$AA?5?$AA?5?$AAA?$AAc?$AAc?$AAe?$AAs@ 000000018002f350     AccessBridgeJavaEntryPoints.obj
 0002:000043a0       ??_C@_0CK@KNEKOBNE@?$FLWARN?$FN?3?5?5?5Accessible?5Descriptio@ 000000018002f3a0     AccessBridgeJavaEntryPoints.obj
 0002:000043d0       ??_C@_0EM@LPILGNDD@?$FLERROR?$FN?3?5?5either?5env?5?$DN?$DN?50?5or?5ge@ 000000018002f3d0     AccessBridgeJavaEntryPoints.obj
 0002:00004420       ??_C@_0DE@IKDIHCF@Getting?5AccessibleRole?5?9?5call?5t@ 000000018002f420     AccessBridgeJavaEntryPoints.obj
 0002:00004458       ??_C@_0DC@FOMJEAJG@Getting?5AccessibleRole?5?9?5call?5t@ 000000018002f458     AccessBridgeJavaEntryPoints.obj
 0002:00004490       ??_C@_0BH@LHDEAMGB@Getting?5AccessibleRole@ 000000018002f490     AccessBridgeJavaEntryPoints.obj
 0002:000044a8       ??_C@_0DC@CDOHPCLK@Getting?5AccessibleRole?5?9?5call?5t@ 000000018002f4a8     AccessBridgeJavaEntryPoints.obj
 0002:000044e0       ??_C@_1EA@DFMPHGFH@?$AA?$FL?$AAI?$AAN?$AAF?$AAO?$AA?$FN?$AA?3?$AA?5?$AA?5?$AA?5?$AAA?$AAc?$AAc?$AAe?$AAs@ 000000018002f4e0     AccessBridgeJavaEntryPoints.obj
 0002:00004520       ??_C@_0DC@JADMICAI@Getting?5AccessibleRole?5?9?5call?5t@ 000000018002f520     AccessBridgeJavaEntryPoints.obj
 0002:00004558       ??_C@_0CD@DPDMNHLG@?$FLWARN?$FN?3?5?5?5Accessible?5Role?5is?5nu@ 000000018002f558     AccessBridgeJavaEntryPoints.obj
 0002:00004580       ??_C@_0EL@ENOHPPLP@?$FLERROR?$FN?3?5?5either?5env?5?$DN?$DN?50?5or?5ge@ 000000018002f580     AccessBridgeJavaEntryPoints.obj
 0002:000045d0       ??_C@_0DK@OPAANMJH@Getting?5AccessibleRole_en_US?5?9?5@ 000000018002f5d0     AccessBridgeJavaEntryPoints.obj
 0002:00004610       ??_C@_0DI@CJNJDFMD@Getting?5AccessibleRole_en_US?5?9?5@ 000000018002f610     AccessBridgeJavaEntryPoints.obj
 0002:00004648       ??_C@_0BN@HKCJIFDO@Getting?5AccessibleRole_en_US@ 000000018002f648     AccessBridgeJavaEntryPoints.obj
 0002:00004668       ??_C@_0DI@FEPHIHOP@Getting?5AccessibleRole_en_US?5?9?5@ 000000018002f668     AccessBridgeJavaEntryPoints.obj
 0002:000046a0       ??_C@_1EM@ICLLIBMO@?$AA?$FL?$AAI?$AAN?$AAF?$AAO?$AA?$FN?$AA?3?$AA?5?$AA?5?$AA?5?$AAA?$AAc?$AAc?$AAe?$AAs@ 000000018002f6a0     AccessBridgeJavaEntryPoints.obj
 0002:000046f0       ??_C@_0DI@OHCMPHFN@Getting?5AccessibleRole_en_US?5?9?5@ 000000018002f6f0     AccessBridgeJavaEntryPoints.obj
 0002:00004728       ??_C@_0CJ@JHFOCCMF@?$FLWARN?$FN?3?5?5?5Accessible?5Role?5en_US@ 000000018002f728     AccessBridgeJavaEntryPoints.obj
 0002:00004760       ??_C@_0FA@EDCBAJIO@?$FLERROR?$FN?3?5either?5env?5?$DN?$DN?50?5or?5get@ 000000018002f760     AccessBridgeJavaEntryPoints.obj
 0002:000047b0       ??_C@_0DF@HNCNCNCA@Getting?5AccessibleState?5?9?5call?5@ 000000018002f7b0     AccessBridgeJavaEntryPoints.obj
 0002:000047e8       ??_C@_0DD@FJJPIJBK@Getting?5AccessibleState?5?9?5call?5@ 000000018002f7e8     AccessBridgeJavaEntryPoints.obj
 0002:00004820       ??_C@_0BI@BBGKJOIM@Getting?5AccessibleState@ 000000018002f820     AccessBridgeJavaEntryPoints.obj
 0002:00004838       ??_C@_0DD@CELBDLDG@Getting?5AccessibleState?5?9?5call?5@ 000000018002f838     AccessBridgeJavaEntryPoints.obj
 0002:00004870       ??_C@_1EE@DCJFHGCM@?$AA?$FL?$AAI?$AAN?$AAF?$AAO?$AA?$FN?$AA?3?$AA?5?$AA?5?$AA?5?$AAA?$AAc?$AAc?$AAe?$AAs@ 000000018002f870     AccessBridgeJavaEntryPoints.obj
 0002:000048b8       ??_C@_0DD@JHGKELIE@Getting?5AccessibleState?5?9?5call?5@ 000000018002f8b8     AccessBridgeJavaEntryPoints.obj
 0002:000048f0       ??_C@_0CF@EJIKBPCF@?$FLWARN?$FN?3?5?5?5Accessible?5States?5is?5@ 000000018002f8f0     AccessBridgeJavaEntryPoints.obj
 0002:00004920       ??_C@_0EN@PLJCLDAI@?$FLERROR?$FN?3?5?5either?5env?5?$DN?$DN?50?5or?5ge@ 000000018002f920     AccessBridgeJavaEntryPoints.obj
 0002:00004970       ??_C@_0DL@NKOGKBKA@Getting?5AccessibleState_en_US?5?9@ 000000018002f970     AccessBridgeJavaEntryPoints.obj
 0002:000049b0       ??_C@_0DJ@EPIHCNDB@Getting?5AccessibleState_en_US?5?9@ 000000018002f9b0     AccessBridgeJavaEntryPoints.obj
 0002:000049f0       ??_C@_0BO@INBCKAFB@Getting?5AccessibleState_en_US@ 000000018002f9f0     AccessBridgeJavaEntryPoints.obj
 0002:00004a10       ??_C@_0DJ@DCKJJPBN@Getting?5AccessibleState_en_US?5?9@ 000000018002fa10     AccessBridgeJavaEntryPoints.obj
 0002:00004a50       ??_C@_1FA@BNDENPHM@?$AA?$FL?$AAI?$AAN?$AAF?$AAO?$AA?$FN?$AA?3?$AA?5?$AA?5?$AA?5?$AAA?$AAc?$AAc?$AAe?$AAs@ 000000018002fa50     AccessBridgeJavaEntryPoints.obj
 0002:00004aa0       ??_C@_0DJ@IBHCOPKP@Getting?5AccessibleState_en_US?5?9@ 000000018002faa0     AccessBridgeJavaEntryPoints.obj
 0002:00004ae0       ??_C@_0CL@LNKMOAJG@?$FLWARN?$FN?3?5?5?5Accessible?5States?5en_@ 000000018002fae0     AccessBridgeJavaEntryPoints.obj
 0002:00004b10       ??_C@_0FC@KNGBOCJI@?$FLERROR?$FN?3?5either?5env?5?$DN?$DN?50?5or?5get@ 000000018002fb10     AccessBridgeJavaEntryPoints.obj
 0002:00004b68       ??_C@_0DK@NAACLIEE@Getting?5AccessibleIndexInParent@ 000000018002fb68     AccessBridgeJavaEntryPoints.obj
 0002:00004ba8       ??_C@_0BP@LDKDBFNM@?$FLINFO?$FN?3?5?5?5Index?5in?5Parent?5?$DN?5?$CFd@ 000000018002fba8     AccessBridgeJavaEntryPoints.obj
 0002:00004bd0       ??_C@_0EO@FMBHNIPI@?$FLERROR?$FN?3?5?5either?5env?5?$DN?$DN?50?5or?5ge@ 000000018002fbd0     AccessBridgeJavaEntryPoints.obj
 0002:00004c20       ??_C@_0EK@BLALEJAL@?$FLINFO?$FN?3?5?$CK?$CK?$CK?5jniEnv?3?5?$CFp?$DL?5accessB@ 000000018002fc20     AccessBridgeJavaEntryPoints.obj
 0002:00004c70       ??_C@_0DK@HBEJENLO@Getting?5AccessibleChildrenCount@ 000000018002fc70     AccessBridgeJavaEntryPoints.obj
 0002:00004cb0       ??_C@_0BO@INNKBLPE@?$FLINFO?$FN?3?5?5?5Children?5count?5?$DN?5?$CFd@ 000000018002fcb0     AccessBridgeJavaEntryPoints.obj
 0002:00004cd0       ??_C@_0EO@BPNCCJLD@?$FLERROR?$FN?3?5?5either?5env?5?$DN?$DN?50?5or?5ge@ 000000018002fcd0     AccessBridgeJavaEntryPoints.obj
 0002:00004d20       ??_C@_0EK@PAPEMOFA@?$FLINFO?$FN?3?5?$CK?$CK?$CK?5jniEnv?3?5?$CFp?$DL?5accessB@ 000000018002fd20     AccessBridgeJavaEntryPoints.obj
 0002:00004d70       ??_C@_0DD@EIHALEFK@Getting?5AccessibleXcoord?5?9?5call@ 000000018002fd70     AccessBridgeJavaEntryPoints.obj
 0002:00004da8       ??_C@_0BH@EMDFCPBA@?$FLINFO?$FN?3?5?5?5X?5coord?5?$DN?5?$CFd@ 000000018002fda8     AccessBridgeJavaEntryPoints.obj
 0002:00004dc0       ??_C@_0EH@EAAFBPMN@?$FLERROR?$FN?3?5?5either?5env?5?$DN?$DN?50?5or?5ge@ 000000018002fdc0     AccessBridgeJavaEntryPoints.obj
 0002:00004e10       ??_C@_0EK@PIPPCCAB@?$FLINFO?$FN?3?5?$CK?$CK?$CK?5jniEnv?3?5?$CFX?$DL?5accessB@ 000000018002fe10     AccessBridgeJavaEntryPoints.obj
 0002:00004e60       ??_C@_0DD@HOICCEKJ@Getting?5AccessibleYcoord?5?9?5call@ 000000018002fe60     AccessBridgeJavaEntryPoints.obj
 0002:00004e98       ??_C@_0BH@JBKDPGJF@?$FLINFO?$FN?3?5?5?5Y?5coord?5?$DN?5?$CFd@ 000000018002fe98     AccessBridgeJavaEntryPoints.obj
 0002:00004eb0       ??_C@_0EH@CDACMGOJ@?$FLERROR?$FN?3?5?5either?5env?5?$DN?$DN?50?5or?5ge@ 000000018002feb0     AccessBridgeJavaEntryPoints.obj
 0002:00004ef8       ??_C@_0DC@IECDLNHB@Getting?5AccessibleWidth?5?9?5call?5@ 000000018002fef8     AccessBridgeJavaEntryPoints.obj
 0002:00004f30       ??_C@_0BF@EEAFCLIB@?$FLINFO?$FN?3?5?5?5Width?5?$DN?5?$CFd@ 000000018002ff30     AccessBridgeJavaEntryPoints.obj
 0002:00004f50       ??_C@_0EG@HOHNFBDJ@?$FLERROR?$FN?3?5?5either?5env?5?$DN?$DN?50?5or?5ge@ 000000018002ff50     AccessBridgeJavaEntryPoints.obj
 0002:00004f98       ??_C@_0DD@DDJGOHAP@Getting?5AccessibleHeight?5?9?5call@ 000000018002ff98     AccessBridgeJavaEntryPoints.obj
 0002:00004fd0       ??_C@_0BG@DJGLJFGH@?$FLINFO?$FN?3?5?5?5Height?5?$DN?5?$CFd@ 000000018002ffd0     AccessBridgeJavaEntryPoints.obj
 0002:00004ff0       ??_C@_0EH@LBBAABEE@?$FLERROR?$FN?3?5?5either?5env?5?$DN?$DN?50?5or?5ge@ 000000018002fff0     AccessBridgeJavaEntryPoints.obj
 0002:00005038       ??_C@_0DJ@LNCBBGOH@Getting?5AccessibleComponent?5?9?5c@ 0000000180030038     AccessBridgeJavaEntryPoints.obj
 0002:00005078       ??_C@_0CD@PFGFGKFI@?$FLINFO?$FN?3?5?5?5AccessibleComponent?5?$DN@ 0000000180030078     AccessBridgeJavaEntryPoints.obj
 0002:000050a0       ??_C@_0DH@KGCNAJLL@Getting?5AccessibleComponent?5?9?5c@ 00000001800300a0     AccessBridgeJavaEntryPoints.obj
 0002:000050e0       ??_C@_0EK@MOFEFKAP@?$FLERROR?$FN?3?5?5either?5env?5?$DN?$DN?50?5or?5ge@ 00000001800300e0     AccessBridgeJavaEntryPoints.obj
 0002:00005130       ??_C@_0DG@DACOODAE@Getting?5AccessibleAction?5?9?5call@ 0000000180030130     AccessBridgeJavaEntryPoints.obj
 0002:00005168       ??_C@_0CA@PJFDOLN@?$FLINFO?$FN?3?5?5?5AccessibleAction?5?$DN?5?$CFp@ 0000000180030168     AccessBridgeJavaEntryPoints.obj
 0002:00005188       ??_C@_0DE@DDPPAPLP@Getting?5AccessibleAction?5?9?5call@ 0000000180030188     AccessBridgeJavaEntryPoints.obj
 0002:000051c0       ??_C@_0EH@DKLGJNHO@?$FLERROR?$FN?3?5?5either?5env?5?$DN?$DN?50?5or?5ge@ 00000001800301c0     AccessBridgeJavaEntryPoints.obj
 0002:00005208       ??_C@_0DJ@CGHCFMLP@Getting?5AccessibleSelection?5?9?5c@ 0000000180030208     AccessBridgeJavaEntryPoints.obj
 0002:00005248       ??_C@_0CD@PJLLNPAJ@?$FLINFO?$FN?3?5?5?5AccessibleSelection?5?$DN@ 0000000180030248     AccessBridgeJavaEntryPoints.obj
 0002:00005270       ??_C@_0DH@PGPODJFA@Getting?5AccessibleSelection?5?9?5c@ 0000000180030270     AccessBridgeJavaEntryPoints.obj
 0002:000052b0       ??_C@_0EK@NDMBIFBF@?$FLERROR?$FN?3?5?5either?5env?5?$DN?$DN?50?5or?5ge@ 00000001800302b0     AccessBridgeJavaEntryPoints.obj
 0002:00005300       ??_C@_0DO@EELLKHNA@?$FLINFO?$FN?3?5?$CD?$CD?$CD?$CD?$CD?5Calling?5getAccess@ 0000000180030300     AccessBridgeJavaEntryPoints.obj
 0002:00005340       ??_C@_0EE@BBNKAGDP@?$FLINFO?$FN?3?5?$CD?$CD?$CD?$CD?$CD?5?4?4?4?5Returned?5from@ 0000000180030340     AccessBridgeJavaEntryPoints.obj
 0002:00005388       ??_C@_0DL@DIOKBKHD@?$CD?$CD?$CD?$CD?$CD?5Getting?5AccessibleTable?5?9@ 0000000180030388     AccessBridgeJavaEntryPoints.obj
 0002:000053c8       ??_C@_0CF@KFOMFGJG@?$FLINFO?$FN?3?5?5?5?$CD?$CD?$CD?$CD?$CD?5AccessibleTable@ 00000001800303c8     AccessBridgeJavaEntryPoints.obj
 0002:000053f0       ??_C@_0DJ@ELALBBFD@?$CD?$CD?$CD?$CD?$CD?5Getting?5AccessibleTable?5?9@ 00000001800303f0     AccessBridgeJavaEntryPoints.obj
 0002:00005430       ??_C@_0EF@MKDIKDJP@?$FLERROR?$FN?3?5either?5env?5?$DN?$DN?50?5or?5get@ 0000000180030430     AccessBridgeJavaEntryPoints.obj
 0002:00005478       ??_C@_0BO@PJMPGGKG@?$FLINFO?$FN?3?5?5?5AccessibleText?5?$DN?5?$CFp@ 0000000180030478     AccessBridgeJavaEntryPoints.obj
 0002:00005498       ??_C@_0DF@NJBDDCEL@Getting?5AccessibleValue?5?9?5call?5@ 0000000180030498     AccessBridgeJavaEntryPoints.obj
 0002:000054d0       ??_C@_0BP@BANALONE@?$FLINFO?$FN?3?5?5?5AccessibleValue?5?$DN?5?$CFp@ 00000001800304d0     AccessBridgeJavaEntryPoints.obj
 0002:000054f0       ??_C@_0DD@JJHMAHMH@Getting?5AccessibleValue?5?9?5call?5@ 00000001800304f0     AccessBridgeJavaEntryPoints.obj
 0002:00005530       ??_C@_0EG@HHMGAANK@?$FLERROR?$FN?3?5?5either?5env?5?$DN?$DN?50?5or?5ge@ 0000000180030530     AccessBridgeJavaEntryPoints.obj
 0002:00005578       ??_C@_0DJ@EACHBMMF@Getting?5AccessibleHypertext?5?9?5c@ 0000000180030578     AccessBridgeJavaEntryPoints.obj
 0002:000055b8       ??_C@_0CD@DNELEHHF@?$FLINFO?$FN?3?5?5?5AccessibleHypertext?5?$DN@ 00000001800305b8     AccessBridgeJavaEntryPoints.obj
 0002:000055e0       ??_C@_0DH@DONNNDKC@Getting?5AccessibleHypertext?5?9?5c@ 00000001800305e0     AccessBridgeJavaEntryPoints.obj
 0002:00005620       ??_C@_0FA@DGBOEHHP@?$FLINFO?$FN?3?5Calling?5AccessBridgeJav@ 0000000180030620     AccessBridgeJavaEntryPoints.obj
 0002:00005670       ??_C@_0DF@OGEEIIFE@Getting?5AccessibleChild?5?9?5call?5@ 0000000180030670     AccessBridgeJavaEntryPoints.obj
 0002:000056a8       ??_C@_0DB@OOCPCHE@Getting?5AccessibleChild?5?9?5call?5@ 00000001800306a8     AccessBridgeJavaEntryPoints.obj
 0002:000056e0       ??_C@_0DD@JNMELFAO@Getting?5AccessibleChild?5?9?5call?5@ 00000001800306e0     AccessBridgeJavaEntryPoints.obj
 0002:00005720       ??_C@_0EC@MDNHELGM@?$FLERROR?$FN?3?5?5either?5env?5?$DN?$DN?50?5or?5ge@ 0000000180030720     AccessBridgeJavaEntryPoints.obj
 0002:00005770       ??_C@_0FB@PNLEIBEF@?$FLINFO?$FN?3?5Calling?5AccessBridgeJav@ 0000000180030770     AccessBridgeJavaEntryPoints.obj
 0002:000057c8       ??_C@_0DG@BJCEEHCN@Getting?5AccessibleParent?5?9?5call@ 00000001800307c8     AccessBridgeJavaEntryPoints.obj
 0002:00005800       ??_C@_0DC@MKLJMCBC@Getting?5AccessibleParent?5?9?5call@ 0000000180030800     AccessBridgeJavaEntryPoints.obj
 0002:00005838       ??_C@_0DE@IILKINNI@Getting?5AccessibleParent?5?9?5call@ 0000000180030838     AccessBridgeJavaEntryPoints.obj
 0002:00005870       ??_C@_0EH@MOCAMKEC@?$FLERROR?$FN?3?5?5either?5env?5?$DN?$DN?50?5or?5ge@ 0000000180030870     AccessBridgeJavaEntryPoints.obj
 0002:000058c0       ??_C@_0EP@IDGNPODK@?$FLINFO?$FN?3?5?$CD?$CD?$CD?$CD?$CD?5Calling?5AccessBri@ 00000001800308c0     AccessBridgeJavaEntryPoints.obj
 0002:00005910       ??_C@_0EA@HDPDLION@?$CD?$CD?$CD?$CD?$CD?5Getting?5AccessibleTableRo@ 0000000180030910     AccessBridgeJavaEntryPoints.obj
 0002:00005950       ??_C@_0CF@OMEBMMOI@?$FLINFO?$FN?3?5?5?5?$CD?$CD?$CD?$CD?$CD?5table?5row?5count@ 0000000180030950     AccessBridgeJavaEntryPoints.obj
 0002:00005978       ??_C@_0DN@MNMKPHBJ@?$FLERROR?$FN?3?5either?5env?5?$DN?$DN?50?5or?5get@ 0000000180030978     AccessBridgeJavaEntryPoints.obj
 0002:000059b8       ??_C@_0DN@LHDBHOOP@Getting?5AccessibleTableColumnCo@ 00000001800309b8     AccessBridgeJavaEntryPoints.obj
 0002:000059f8       ??_C@_0CI@GJGENPPF@?$FLINFO?$FN?3?5?5?5?$CD?$CD?$CD?$CD?$CD?5table?5column?5co@ 00000001800309f8     AccessBridgeJavaEntryPoints.obj
 0002:00005a20       ??_C@_0EF@LHBDGBA@?$FLERROR?$FN?3?5either?5env?5?$DN?$DN?50?5or?5get@ 0000000180030a20     AccessBridgeJavaEntryPoints.obj
 0002:00005a68       ??_C@_0DH@GFGBCDOC@?$CD?$CD?$CD?$CD?$CD?5Getting?5AccessibleTable?5?9@ 0000000180030a68     AccessBridgeJavaEntryPoints.obj
 0002:00005aa0       ??_C@_0CF@DCCEHDEO@?$FLINFO?$FN?3?5?5?5?$CD?$CD?$CD?$CD?$CD?5accessibleTable@ 0000000180030aa0     AccessBridgeJavaEntryPoints.obj
 0002:00005ac8       ??_C@_0DP@FLHLIILD@?$FLINFO?$FN?3?5?$CD?$CD?$CD?$CD?$CD?5Calling?5getContex@ 0000000180030ac8     AccessBridgeJavaEntryPoints.obj
 0002:00005b10       ??_C@_0EF@JOJDMPNM@?$FLINFO?$FN?3?5?$CD?$CD?$CD?$CD?$CD?5?4?4?4?5Returned?5from@ 0000000180030b10     AccessBridgeJavaEntryPoints.obj
 0002:00005b58       ??_C@_0CH@GEKEKGKL@?$FLINFO?$FN?3?5?5?5?$CD?$CD?$CD?$CD?$CD?5accessibleConte@ 0000000180030b58     AccessBridgeJavaEntryPoints.obj
 0002:00005b80       ??_C@_0EG@CNEBJJDJ@?$FLERROR?$FN?3?5either?5env?5?$DN?$DN?50?5or?5get@ 0000000180030b80     AccessBridgeJavaEntryPoints.obj
 0002:00005bd0       ??_C@_0FE@GFOFNDOE@?$FLINFO?$FN?3?5?$CD?$CD?$CD?$CD?$CD?5Calling?5AccessBri@ 0000000180030bd0     AccessBridgeJavaEntryPoints.obj
 0002:00005c30       ??_C@_0GF@GDALOMIB@?$FLINFO?$FN?3?5?$CD?$CD?$CD?$CD?$CD?5Calling?5AccessBri@ 0000000180030c30     AccessBridgeJavaEntryPoints.obj
 0002:00005ca0       ??_C@_0EB@IFJOCDDE@?$CD?$CD?$CD?$CD?$CD?5Getting?5AccessibleTableCe@ 0000000180030ca0     AccessBridgeJavaEntryPoints.obj
 0002:00005ce8       ??_C@_0CG@KKOMOEPJ@?$FLINFO?$FN?3?5?5?5?$CD?$CD?$CD?$CD?$CD?5table?5cell?5inde@ 0000000180030ce8     AccessBridgeJavaEntryPoints.obj
 0002:00005d10       ??_C@_0ED@MJPDAFIJ@?$FLERROR?$FN?3?5either?5env?5?$DN?$DN?50?5or?5get@ 0000000180030d10     AccessBridgeJavaEntryPoints.obj
 0002:00005d60       ??_C@_0EK@HFAIKGKI@?$CD?$CD?$CD?$CD?$CD?5Getting?5AccessibleTableCe@ 0000000180030d60     AccessBridgeJavaEntryPoints.obj
 0002:00005db0       ??_C@_0CL@CDCOGIJD@?$FLINFO?$FN?3?5?5?5?$CD?$CD?$CD?$CD?$CD?5table?5cell?5row?5@ 0000000180030db0     AccessBridgeJavaEntryPoints.obj
 0002:00005de0       ??_C@_0EH@MFABNFMJ@?$FLERROR?$FN?3?5either?5env?5?$DN?$DN?50?5or?5get@ 0000000180030de0     AccessBridgeJavaEntryPoints.obj
 0002:00005e30       ??_C@_0EN@GIPGNDGO@?$CD?$CD?$CD?$CD?$CD?5Getting?5AccessibleTableCe@ 0000000180030e30     AccessBridgeJavaEntryPoints.obj
 0002:00005e80       ??_C@_0CN@JHPAHOLB@?$FLINFO?$FN?3?5?5?$CD?$CD?$CD?$CD?$CD?5table?5cell?5colum@ 0000000180030e80     AccessBridgeJavaEntryPoints.obj
 0002:00005eb0       ??_C@_0EK@MCJJFMIG@?$FLERROR?$FN?3?5either?5env?5?$DN?$DN?50?5or?5get@ 0000000180030eb0     AccessBridgeJavaEntryPoints.obj
 0002:00005f00       ??_C@_0EK@OAKDMNFI@?$CD?$CD?$CD?$CD?$CD?5Getting?5isAccessibleTable@ 0000000180030f00     AccessBridgeJavaEntryPoints.obj
 0002:00005f50       ??_C@_0CL@FGJJGBAG@?$FLINFO?$FN?3?5?5?5?$CD?$CD?$CD?$CD?$CD?5table?5cell?5isSe@ 0000000180030f50     AccessBridgeJavaEntryPoints.obj
 0002:00005f80       ??_C@_0EF@NDHLMIOL@?$FLERROR?$FN?3?5either?5env?5?$DN?$DN?50?5or?5isA@ 0000000180030f80     AccessBridgeJavaEntryPoints.obj
 0002:00005fd0       ??_C@_0FA@PNFLEDNO@?$CD?$CD?$CD?$CD?$CD?5Getting?5AccessibleTableCe@ 0000000180030fd0     AccessBridgeJavaEntryPoints.obj
 0002:00006020       ??_C@_0EM@CCOLAKIM@?$CD?$CD?$CD?$CD?$CD?5Getting?5AccessibleTableCe@ 0000000180031020     AccessBridgeJavaEntryPoints.obj
 0002:00006070       ??_C@_0DC@NHIEBBHC@?$FLINFO?$FN?3?5?5?5?$CD?$CD?$CD?$CD?$CD?5table?5cell?5Acce@ 0000000180031070     AccessBridgeJavaEntryPoints.obj
 0002:000060b0       ??_C@_0EP@BAKELAEL@?$FLERROR?$FN?3?5either?5env?5?$DN?$DN?50?5or?5get@ 00000001800310b0     AccessBridgeJavaEntryPoints.obj
 0002:00006100       ??_C@_0FJ@JCFFKNHH@?$FLINFO?$FN?3?5?5?$CD?$CD?$CD?$CD?$CD?5Calling?5AccessBr@ 0000000180031100     AccessBridgeJavaEntryPoints.obj
 0002:00006160       ??_C@_0FE@DGILOPPB@?$FLINFO?$FN?3?5?$CD?$CD?$CD?$CD?$CD?5Calling?5AccessBri@ 0000000180031160     AccessBridgeJavaEntryPoints.obj
 0002:000061c0       ??_C@_0EJ@OONHAJKO@?$CD?$CD?$CD?$CD?$CD?5Getting?5AccessibleTableRo@ 00000001800311c0     AccessBridgeJavaEntryPoints.obj
 0002:00006210       ??_C@_0EG@NDBCAEFO@?$FLERROR?$FN?3?5either?5env?5?$DN?$DN?50?5or?5get@ 0000000180031210     AccessBridgeJavaEntryPoints.obj
 0002:00006260       ??_C@_0EG@DALLPPNJ@Getting?5AccessibleTableRowHeade@ 0000000180031260     AccessBridgeJavaEntryPoints.obj
 0002:000062b0       ??_C@_0EO@OOHGOEEK@?$FLERROR?$FN?3?5either?5env?5?$DN?$DN?50?5or?5get@ 00000001800312b0     AccessBridgeJavaEntryPoints.obj
 0002:00006300       ??_C@_0EE@GCIECGJK@?$CD?$CD?$CD?$CD?$CD?5Getting?5AccessibleTableRo@ 0000000180031300     AccessBridgeJavaEntryPoints.obj
 0002:00006350       ??_C@_0EA@OEOKKCMN@?$CD?$CD?$CD?$CD?$CD?5Getting?5AccessibleTableRo@ 0000000180031350     AccessBridgeJavaEntryPoints.obj
 0002:00006390       ??_C@_0DA@BEAKBEEG@?$FLINFO?$FN?3?5?5?5?$CD?$CD?$CD?$CD?$CD?5row?5header?5Acce@ 0000000180031390     AccessBridgeJavaEntryPoints.obj
 0002:000063c0       ??_C@_0ED@KKINKAGC@?$FLERROR?$FN?3?5either?5env?5?$DN?$DN?50?5or?5get@ 00000001800313c0     AccessBridgeJavaEntryPoints.obj
 0002:00006410       ??_C@_0FL@PPBJDPIL@?$FLINFO?$FN?3?5?5?5?$CD?$CD?$CD?$CD?$CD?5Calling?5AccessB@ 0000000180031410     AccessBridgeJavaEntryPoints.obj
 0002:00006470       ??_C@_0FH@EJOHBEGH@?$FLINFO?$FN?3?5?$CD?$CD?$CD?$CD?$CD?5Calling?5AccessBri@ 0000000180031470     AccessBridgeJavaEntryPoints.obj
 0002:000064d0       ??_C@_0EM@ILKGOFLG@?$CD?$CD?$CD?$CD?$CD?5Getting?5AccessibleTableCo@ 00000001800314d0     AccessBridgeJavaEntryPoints.obj
 0002:00006520       ??_C@_0EK@LPGMLANE@?$FLERROR?$FN?3?5?5either?5env?5?$DN?$DN?50?5or?5ge@ 0000000180031520     AccessBridgeJavaEntryPoints.obj
 0002:00006570       ??_C@_0EJ@CKEIFDID@Getting?5AccessibleTableColumnHe@ 0000000180031570     AccessBridgeJavaEntryPoints.obj
 0002:000065c0       ??_C@_0FB@LHNIAEHP@?$FLERROR?$FN?3?5either?5env?5?$DN?$DN?50?5or?5get@ 00000001800315c0     AccessBridgeJavaEntryPoints.obj
 0002:00006620       ??_C@_0EH@JIOGAIC@?$CD?$CD?$CD?$CD?$CD?5Getting?5AccessibleTableCo@ 0000000180031620     AccessBridgeJavaEntryPoints.obj
 0002:00006670       ??_C@_0ED@DCBGPFPL@?$CD?$CD?$CD?$CD?$CD?5Getting?5AccessibleTableCo@ 0000000180031670     AccessBridgeJavaEntryPoints.obj
 0002:000066b8       ??_C@_0DD@JPNBDACB@?$FLINFO?$FN?3?5?5?5?$CD?$CD?$CD?$CD?$CD?5column?5header?5A@ 00000001800316b8     AccessBridgeJavaEntryPoints.obj
 0002:000066f0       ??_C@_0EG@EHCJNLHA@?$FLERROR?$FN?3?5either?5env?5?$DN?$DN?50?5or?5get@ 00000001800316f0     AccessBridgeJavaEntryPoints.obj
 0002:00006740       ??_C@_0FO@DKAHOFOA@?$FLINFO?$FN?3?5?5?5?$CD?$CD?$CD?$CD?$CD?5Calling?5AccessB@ 0000000180031740     AccessBridgeJavaEntryPoints.obj
 0002:000067a0       ??_C@_0FJ@IPEPPO@?$FLINFO?$FN?3?5?$CD?$CD?$CD?$CD?$CD?5Calling?5AccessBri@ 00000001800317a0     AccessBridgeJavaEntryPoints.obj
 0002:00006800       ??_C@_0ED@ECGPKBKB@Getting?5AccessibleTableRowDescr@ 0000000180031800     AccessBridgeJavaEntryPoints.obj
 0002:00006848       ??_C@_0DP@MGPIFPGE@Getting?5AccessibleTableRowDescr@ 0000000180031848     AccessBridgeJavaEntryPoints.obj
 0002:00006890       ??_C@_0EB@HPGBLABA@Getting?5AccessibleTableRowDescr@ 0000000180031890     AccessBridgeJavaEntryPoints.obj
 0002:000068e0       ??_C@_0EI@FALMFIJI@?$FLERROR?$FN?3?5either?5env?5?$DN?$DN?50?5or?5get@ 00000001800318e0     AccessBridgeJavaEntryPoints.obj
 0002:00006930       ??_C@_0FM@OGMEFLJF@?$FLINFO?$FN?3?5?$CD?$CD?$CD?$CD?$CD?5Calling?5AccessBri@ 0000000180031930     AccessBridgeJavaEntryPoints.obj
 0002:00006990       ??_C@_0EG@HNHAKGAA@Getting?5AccessibleTableColumnDe@ 0000000180031990     AccessBridgeJavaEntryPoints.obj
 0002:000069e0       ??_C@_0EC@OOIBKPKB@Getting?5AccessibleTableColumnDe@ 00000001800319e0     AccessBridgeJavaEntryPoints.obj
 0002:00006a30       ??_C@_0EE@HEFBEJHO@Getting?5AccessibleTableColumnDe@ 0000000180031a30     AccessBridgeJavaEntryPoints.obj
 0002:00006a80       ??_C@_0EL@MDADMDPK@?$FLERROR?$FN?3?5either?5env?5?$DN?$DN?50?5or?5get@ 0000000180031a80     AccessBridgeJavaEntryPoints.obj
 0002:00006ad0       ??_C@_0FD@NONCILOI@?$FLINFO?$FN?3?5?$CD?$CD?$CD?$CD?$CD?5AccessBridgeJavaE@ 0000000180031ad0     AccessBridgeJavaEntryPoints.obj
 0002:00006b30       ??_C@_0EJ@CONOFLFI@?$CD?$CD?$CD?$CD?$CD?5Getting?5AccessibleTableRo@ 0000000180031b30     AccessBridgeJavaEntryPoints.obj
 0002:00006b80       ??_C@_0CP@GJAEEGNO@?$FLINFO?$FN?3?5?5?5?$CD?$CD?$CD?$CD?$CD?5table?5row?5selec@ 0000000180031b80     AccessBridgeJavaEntryPoints.obj
 0002:00006bb0       ??_C@_0EL@JIBDDMIF@?$FLERROR?$FN?3?5either?5env?5?$DN?$DN?50?5or?5get@ 0000000180031bb0     AccessBridgeJavaEntryPoints.obj
 0002:00006c00       ??_C@_0FA@LAKDEELL@?$FLINFO?$FN?3?5?$CD?$CD?$CD?$CD?$CD?5AccessBridgeJavaE@ 0000000180031c00     AccessBridgeJavaEntryPoints.obj
 0002:00006c50       ??_C@_0EJ@PAIANDP@?$CD?$CD?$CD?$CD?$CD?5Getting?5isAccessibleTable@ 0000000180031c50     AccessBridgeJavaEntryPoints.obj
 0002:00006ca0       ??_C@_0CK@ENCKDAKJ@?$FLINFO?$FN?3?5?5?5?$CD?$CD?$CD?$CD?$CD?5table?5row?5isSel@ 0000000180031ca0     AccessBridgeJavaEntryPoints.obj
 0002:00006cd0       ??_C@_0EE@OPDECGCG@?$FLERROR?$FN?3?5either?5env?5?$DN?$DN?50?5or?5isA@ 0000000180031cd0     AccessBridgeJavaEntryPoints.obj
 0002:00006d20       ??_C@_0FG@BNGDNOAB@?$FLINFO?$FN?3?5?$CD?$CD?$CD?$CD?$CD?5AccessBridgeJavaE@ 0000000180031d20     AccessBridgeJavaEntryPoints.obj
 0002:00006d80       ??_C@_0EF@MANEDMPN@?$CD?$CD?$CD?$CD?$CD?5Getting?5AccessibleTableRo@ 0000000180031d80     AccessBridgeJavaEntryPoints.obj
 0002:00006dc8       ??_C@_0CN@EGDPALEC@?$FLINFO?$FN?3?5?5?5?$CD?$CD?$CD?$CD?$CD?5table?5row?5selec@ 0000000180031dc8     AccessBridgeJavaEntryPoints.obj
 0002:00006e00       ??_C@_0FH@IBIGBELL@?$FLINFO?$FN?3?5?5?5?$CD?$CD?$CD?$CD?$CD?5AccessBridgeJav@ 0000000180031e00     AccessBridgeJavaEntryPoints.obj
 0002:00006e60       ??_C@_0FG@LAILABJF@?$FLINFO?$FN?3?5?$CD?$CD?$CD?$CD?$CD?5AccessBridgeJavaE@ 0000000180031e60     AccessBridgeJavaEntryPoints.obj
 0002:00006ec0       ??_C@_0EM@ELKPLHEA@?$CD?$CD?$CD?$CD?$CD?5Getting?5AccessibleTableCo@ 0000000180031ec0     AccessBridgeJavaEntryPoints.obj
 0002:00006f10       ??_C@_0DC@EFKBJLFF@?$FLINFO?$FN?3?5?5?5?$CD?$CD?$CD?$CD?$CD?5table?5column?5se@ 0000000180031f10     AccessBridgeJavaEntryPoints.obj
 0002:00006f50       ??_C@_0FD@ODFPPIDD@?$FLINFO?$FN?3?5?$CD?$CD?$CD?$CD?$CD?5AccessBridgeJavaE@ 0000000180031f50     AccessBridgeJavaEntryPoints.obj
 0002:00006fb0       ??_C@_0EM@HPIPAKED@?$CD?$CD?$CD?$CD?$CD?5Getting?5isAccessibleTable@ 0000000180031fb0     AccessBridgeJavaEntryPoints.obj
 0002:00007000       ??_C@_0CN@OPIEHDOO@?$FLINFO?$FN?3?5?5?5?$CD?$CD?$CD?$CD?$CD?5table?5column?5is@ 0000000180032000     AccessBridgeJavaEntryPoints.obj
 0002:00007030       ??_C@_0EI@CBBNNOEE@?$FLERROR?$FN?3?5?5either?5env?5?$DN?$DN?50?5or?5is@ 0000000180032030     AccessBridgeJavaEntryPoints.obj
 0002:00007080       ??_C@_0FK@KHEECFFC@?$FLINFO?$FN?3?5?$CD?$CD?$CD?$CD?$CD?5AccessBridgeJavaE@ 0000000180032080     AccessBridgeJavaEntryPoints.obj
 0002:000070e0       ??_C@_0EI@NDNDKOON@?$CD?$CD?$CD?$CD?$CD?5Getting?5AccessibleTableCo@ 00000001800320e0     AccessBridgeJavaEntryPoints.obj
 0002:00007128       ??_C@_0DA@FGAFLCDN@?$FLINFO?$FN?3?5?5?5?$CD?$CD?$CD?$CD?$CD?5table?5Column?5se@ 0000000180032128     AccessBridgeJavaEntryPoints.obj
 0002:00007160       ??_C@_0FK@PECCMPIL@?$FLINFO?$FN?3?5?5?5?$CD?$CD?$CD?$CD?$CD?5AccessBridgeJav@ 0000000180032160     AccessBridgeJavaEntryPoints.obj
 0002:000071c0       ??_C@_0EP@DEKNIMFA@?$FLINFO?$FN?3?5?$CD?$CD?$CD?$CD?$CD?5AccessBridgeJavaE@ 00000001800321c0     AccessBridgeJavaEntryPoints.obj
 0002:00007210       ??_C@_0DL@DELNDLCL@?$CD?$CD?$CD?$CD?$CD?5Getting?5AccessibleTableRo@ 0000000180032210     AccessBridgeJavaEntryPoints.obj
 0002:00007250       ??_C@_0BP@MEJOIGMM@?$FLINFO?$FN?3?5?5?5?$CD?$CD?$CD?$CD?$CD?5table?5row?5?$DN?5?$CFd@ 0000000180032250     AccessBridgeJavaEntryPoints.obj
 0002:00007270       ??_C@_0DN@DIFOEGJK@?$FLERROR?$FN?3?5either?5env?5?$DN?$DN?50?5or?5get@ 0000000180032270     AccessBridgeJavaEntryPoints.obj
 0002:000072b0       ??_C@_0FC@BFBAOEGI@?$FLINFO?$FN?3?5?$CD?$CD?$CD?$CD?$CD?5AccessBridgeJavaE@ 00000001800322b0     AccessBridgeJavaEntryPoints.obj
 0002:00007308       ??_C@_0DO@MBGEOOOH@?$CD?$CD?$CD?$CD?$CD?5Getting?5AccessibleTableCo@ 0000000180032308     AccessBridgeJavaEntryPoints.obj
 0002:00007348       ??_C@_0CC@CJBEHFKG@?$FLINFO?$FN?3?5?5?5?$CD?$CD?$CD?$CD?$CD?5table?5column?5?$DN?5@ 0000000180032348     AccessBridgeJavaEntryPoints.obj
 0002:00007370       ??_C@_0EA@IFBLPNLC@?$FLERROR?$FN?3?5either?5env?5?$DN?$DN?50?5or?5get@ 0000000180032370     AccessBridgeJavaEntryPoints.obj
 0002:000073b0       ??_C@_0FH@GMMGKHHK@?$FLINFO?$FN?3?5?$CD?$CD?$CD?$CD?$CD?5AccessBridgeJavaE@ 00000001800323b0     AccessBridgeJavaEntryPoints.obj
 0002:00007410       ??_C@_0EA@IDLLLJIK@?$CD?$CD?$CD?$CD?$CD?5Getting?5getAccessibleTabl@ 0000000180032410     AccessBridgeJavaEntryPoints.obj
 0002:00007450       ??_C@_0CB@JIHDIDBK@?$FLINFO?$FN?3?5?5?5?$CD?$CD?$CD?$CD?$CD?5table?5index?5?$DN?5?$CF@ 0000000180032450     AccessBridgeJavaEntryPoints.obj
 0002:00007478       ??_C@_0DP@EPGMKJOF@?$FLERROR?$FN?3?5either?5env?5?$DN?$DN?50?5or?5get@ 0000000180032478     AccessBridgeJavaEntryPoints.obj
 0002:000074c0       ??_C@_0EM@OMNMKDMF@?$FLINFO?$FN?3?5?$CD?$CD?$CD?$CD?$CD?5AccessBridgeJavaE@ 00000001800324c0     AccessBridgeJavaEntryPoints.obj
 0002:00007510       ??_C@_0EA@LPBOBAAO@?$CD?$CD?$CD?$CD?$CD?5Getting?5AccessibleRelatio@ 0000000180032510     AccessBridgeJavaEntryPoints.obj
 0002:00007550       ??_C@_0CO@JNBGELMK@?$FLINFO?$FN?3?5?5?5?$CD?$CD?$CD?$CD?$CD?5AccessibleRelat@ 0000000180032550     AccessBridgeJavaEntryPoints.obj
 0002:00007580       ??_C@_0DL@KJPPMLJK@Getting?5AccessibleRelationKey?5?9@ 0000000180032580     AccessBridgeJavaEntryPoints.obj
 0002:000075c0       ??_C@_0DK@CJPLLCPL@Getting?5AccessibleRelation?5key?5@ 00000001800325c0     AccessBridgeJavaEntryPoints.obj
 0002:00007600       ??_C@_0BP@LFNNPMOI@Getting?5AccessibleRelation?5key@ 0000000180032600     AccessBridgeJavaEntryPoints.obj
 0002:00007620       ??_C@_0CL@LKNHIIFA@?$FLINFO?$FN?3?5?$CD?$CD?$CD?$CD?$CD?5AccessibleRelatio@ 0000000180032620     AccessBridgeJavaEntryPoints.obj
 0002:00007650       ??_C@_0DK@OHAOHAGF@Getting?5AccessibleRelation?5key?5@ 0000000180032650     AccessBridgeJavaEntryPoints.obj
 0002:00007690       ??_C@_0CK@FLLDFIHJ@?$FLWARN?$FN?3?5?5?5AccessibleRelation?5ke@ 0000000180032690     AccessBridgeJavaEntryPoints.obj
 0002:000076c0       ??_C@_0DL@FOJGEEOM@Getting?5AccessibleRelationSet?5?9@ 00000001800326c0     AccessBridgeJavaEntryPoints.obj
 0002:00007700       ??_C@_0DH@OOCHFOKL@Getting?5AccessibleRelationSet?5?9@ 0000000180032700     AccessBridgeJavaEntryPoints.obj
 0002:00007738       ??_C@_0CA@NHODALDJ@?$FLINFO?$FN?3?5?5?5relation?5set?5item?3?5?$CFp@ 0000000180032738     AccessBridgeJavaEntryPoints.obj
 0002:00007760       ??_C@_0FA@NBCFFMGI@?$FLINFO?$FN?3?5?5?5?$CD?$CD?$CD?$CD?$CD?5AccessBridgeJav@ 0000000180032760     AccessBridgeJavaEntryPoints.obj
 0002:000077b0       ??_C@_0EK@KKPLDFBH@?$FLINFO?$FN?3?5?$CD?$CD?$CD?$CD?$CD?5AccessBridgeJavaE@ 00000001800327b0     AccessBridgeJavaEntryPoints.obj
 0002:00007800       ??_C@_0DP@KAHCJAMC@?$CD?$CD?$CD?$CD?$CD?5Getting?5AccessibleHyperte@ 0000000180032800     AccessBridgeJavaEntryPoints.obj
 0002:00007840       ??_C@_0DL@BCGGEGFO@?$CD?$CD?$CD?$CD?$CD?5Getting?5AccessibleHyperte@ 0000000180032840     AccessBridgeJavaEntryPoints.obj
 0002:00007880       ??_C@_0CJ@KAIOACGL@?$FLINFO?$FN?3?5?5?5?$CD?$CD?$CD?$CD?$CD?5AccessibleHyper@ 0000000180032880     AccessBridgeJavaEntryPoints.obj
 0002:000078b0       ??_C@_0DK@IMJHJIPP@?$FLWARN?$FN?3?5?5?5?$CD?$CD?$CD?$CD?$CD?5null?5Accessible@ 00000001800328b0     AccessBridgeJavaEntryPoints.obj
 0002:000078f0       ??_C@_0DI@FEBHIMOE@?$CD?$CD?$CD?$CD?$CD?5Getting?5hyperlink?5count?5?9@ 00000001800328f0     AccessBridgeJavaEntryPoints.obj
 0002:00007928       ??_C@_0CF@OFPNIMKK@?$FLINFO?$FN?3?5?5?5?$CD?$CD?$CD?$CD?$CD?5hyperlink?5count@ 0000000180032928     AccessBridgeJavaEntryPoints.obj
 0002:00007950       ??_C@_0DP@CIGIOMPM@?$CD?$CD?$CD?$CD?$CD?5Getting?5AccessibleHyperli@ 0000000180032950     AccessBridgeJavaEntryPoints.obj
 0002:00007990       ??_C@_0DL@PDIOCHOJ@?$CD?$CD?$CD?$CD?$CD?5Getting?5AccessibleHyperli@ 0000000180032990     AccessBridgeJavaEntryPoints.obj
 0002:000079d0       ??_C@_0CJ@FJIBOEOI@?$FLINFO?$FN?3?5?5?5?$CD?$CD?$CD?$CD?$CD?5AccessibleHyper@ 00000001800329d0     AccessBridgeJavaEntryPoints.obj
 0002:00007a00       ??_C@_0DE@FAMBBMPD@Getting?5hyperlink?5text?5?9?5call?5t@ 0000000180032a00     AccessBridgeJavaEntryPoints.obj
 0002:00007a38       ??_C@_0DM@FFPIAIEA@Getting?5AccessibleHyperlink?5tex@ 0000000180032a38     AccessBridgeJavaEntryPoints.obj
 0002:00007a78       ??_C@_0CB@GINGGJOG@Getting?5AccessibleHyperlink?5tex@ 0000000180032a78     AccessBridgeJavaEntryPoints.obj
 0002:00007aa0       ??_C@_0CN@IIHGCCLN@?$FLINFO?$FN?3?5?$CD?$CD?$CD?$CD?$CD?5AccessibleHyperli@ 0000000180032aa0     AccessBridgeJavaEntryPoints.obj
 0002:00007ad0       ??_C@_0DM@JLANMKNO@Getting?5AccessibleHyperlink?5tex@ 0000000180032ad0     AccessBridgeJavaEntryPoints.obj
 0002:00007b10       ??_C@_0CM@DKPAOLF@?$FLWARN?$FN?3?5?5?5AccessibleHyperlink?5t@ 0000000180032b10     AccessBridgeJavaEntryPoints.obj
 0002:00007b40       ??_C@_0DO@DJICJOGB@?$CD?$CD?$CD?$CD?$CD?5Getting?5hyperlink?5start?5i@ 0000000180032b40     AccessBridgeJavaEntryPoints.obj
 0002:00007b80       ??_C@_0CL@GNKIIEKN@?$FLINFO?$FN?3?5?5?5?$CD?$CD?$CD?$CD?$CD?5hyperlink?5start@ 0000000180032b80     AccessBridgeJavaEntryPoints.obj
 0002:00007bb0       ??_C@_0DM@MGHLFEBK@?$CD?$CD?$CD?$CD?$CD?5Getting?5hyperlink?5end?5ind@ 0000000180032bb0     AccessBridgeJavaEntryPoints.obj
 0002:00007bf0       ??_C@_0CJ@POHPAAGA@?$FLINFO?$FN?3?5?5?5?$CD?$CD?$CD?$CD?$CD?5hyperlink?5end?5i@ 0000000180032bf0     AccessBridgeJavaEntryPoints.obj
 0002:00007c20       ??_C@_0EO@MCEJOGLJ@?$FLINFO?$FN?3?5?5?5?$CD?$CD?$CD?$CD?$CD?5AccessBridgeJav@ 0000000180032c20     AccessBridgeJavaEntryPoints.obj
 0002:00007c70       ??_C@_0FC@PJEJEFPL@?$FLINFO?$FN?3?5Calling?5AccessBridgeJav@ 0000000180032c70     AccessBridgeJavaEntryPoints.obj
 0002:00007cc8       ??_C@_0DK@IAFPEHK@activateAccessibleHyperlink?5?9?5c@ 0000000180032cc8     AccessBridgeJavaEntryPoints.obj
 0002:00007d10       ??_C@_0EG@NBDJGANF@?$FLERROR?$FN?3?5either?5jniEnv?5?$DN?$DN?50?5or?5@ 0000000180032d10     AccessBridgeJavaEntryPoints.obj
 0002:00007d60       ??_C@_0FO@LCEKGOMG@?$FLINFO?$FN?3?5?$CD?$CD?$CD?$CD?$CD?5AccessBridgeJavaE@ 0000000180032d60     AccessBridgeJavaEntryPoints.obj
 0002:00007dc0       ??_C@_0CD@FKJEEIHP@?$FLINFO?$FN?3?5?5?5getting?5hyperlink?5?$CFd?5@ 0000000180032dc0     AccessBridgeJavaEntryPoints.obj
 0002:00007df0       ??_C@_0FB@LIBMBPHJ@?$FLINFO?$FN?3?5?5?5?$CD?$CD?$CD?$CD?$CD?5AccessBridgeJav@ 0000000180032df0     AccessBridgeJavaEntryPoints.obj
 0002:00007e50       ??_C@_0EL@OJOFGNCE@?$FLINFO?$FN?3?5?$CD?$CD?$CD?$CD?$CD?5AccessBridgeJavaE@ 0000000180032e50     AccessBridgeJavaEntryPoints.obj
 0002:00007ea0       ??_C@_0FL@JFFPJPNI@?$FLINFO?$FN?3?5?$CD?$CD?$CD?$CD?$CD?5AccessBridgeJavaE@ 0000000180032ea0     AccessBridgeJavaEntryPoints.obj
 0002:00007f00       ??_C@_0DI@MNABDACM@?$CD?$CD?$CD?$CD?$CD?5Getting?5hyperlink?5index?5?9@ 0000000180032f00     AccessBridgeJavaEntryPoints.obj
 0002:00007f38       ??_C@_0CF@MJOBJPAA@?$FLINFO?$FN?3?5?5?5?$CD?$CD?$CD?$CD?$CD?5hyperlink?5index@ 0000000180032f38     AccessBridgeJavaEntryPoints.obj
 0002:00007f60       ??_C@_0FC@MDIFEEKA@?$FLINFO?$FN?3?5?$CD?$CD?$CD?$CD?$CD?5AccessBridgeJavaE@ 0000000180032f60     AccessBridgeJavaEntryPoints.obj
 0002:00007fc0       ??_C@_0EM@DFNHGKKP@?$FLINFO?$FN?3?5?$CD?$CD?$CD?$CD?$CD?5AccessBridgeJavaE@ 0000000180032fc0     AccessBridgeJavaEntryPoints.obj
 0002:00008010       ??_C@_0DL@CLKJJKNH@?$CD?$CD?$CD?$CD?$CD?5Getting?5key?5bindings?5coun@ 0000000180033010     AccessBridgeJavaEntryPoints.obj
 0002:00008050       ??_C@_0CI@OKJNHPKA@?$FLINFO?$FN?3?5?5?5?$CD?$CD?$CD?$CD?$CD?5key?5bindings?5co@ 0000000180033050     AccessBridgeJavaEntryPoints.obj
 0002:00008078       ??_C@_0DP@FMCKMBKC@?$CD?$CD?$CD?$CD?$CD?5Getting?5key?5binding?5chara@ 0000000180033078     AccessBridgeJavaEntryPoints.obj
 0002:000080c0       ??_C@_0FN@DCEDCNML@?$FLINFO?$FN?3?5?5?5?$CD?$CD?$CD?$CD?$CD?5key?5binding?5cha@ 00000001800330c0     AccessBridgeJavaEntryPoints.obj
 0002:00008120       ??_C@_0DO@HKGJEFDO@?$CD?$CD?$CD?$CD?$CD?5Getting?5key?5binding?5modif@ 0000000180033120     AccessBridgeJavaEntryPoints.obj
 0002:00008160       ??_C@_0CK@OFBJGPDI@?$FLINFO?$FN?3?5?5?$CD?$CD?$CD?$CD?$CD?5key?5binding?5modi@ 0000000180033160     AccessBridgeJavaEntryPoints.obj
 0002:00008190       ??_C@_0EG@MKCABNJD@?$FLINFO?$FN?3?5?$CD?$CD?$CD?$CD?$CD?5AccessBridgeJavaE@ 0000000180033190     AccessBridgeJavaEntryPoints.obj
 0002:000081d8       ??_C@_0CG@IDHCCFPM@?$FLWARN?$FN?3?5?5?5?$CD?$CD?$CD?$CD?$CD?5missing?5method?$CI@ 00000001800331d8     AccessBridgeJavaEntryPoints.obj
 0002:00008200       ??_C@_0DE@JDHACCPK@?$CD?$CD?$CD?$CD?$CD?5Getting?5icons?5count?5?9?5cal@ 0000000180033200     AccessBridgeJavaEntryPoints.obj
 0002:00008238       ??_C@_0CB@DPKCEABK@?$FLINFO?$FN?3?5?5?5?$CD?$CD?$CD?$CD?$CD?5icons?5count?5?$DN?5?$CF@ 0000000180033238     AccessBridgeJavaEntryPoints.obj
 0002:00008260       ??_C@_0DG@HKLCCMCD@Getting?5icon?5description?5?9?5call@ 0000000180033260     AccessBridgeJavaEntryPoints.obj
 0002:00008298       ??_C@_0DO@JICPIJF@Getting?5AccessibleIcon?5descript@ 0000000180033298     AccessBridgeJavaEntryPoints.obj
 0002:000082d8       ??_C@_0CD@GHIFDBCH@Getting?5AccessibleIcon?5descript@ 00000001800332d8     AccessBridgeJavaEntryPoints.obj
 0002:00008300       ??_C@_0CP@OGEOHJKD@?$FLINFO?$FN?3?5?$CD?$CD?$CD?$CD?$CD?5AccessibleIcon?5de@ 0000000180033300     AccessBridgeJavaEntryPoints.obj
 0002:00008330       ??_C@_0DO@MHHHDKAL@Getting?5AccessibleIcon?5descript@ 0000000180033330     AccessBridgeJavaEntryPoints.obj
 0002:00008370       ??_C@_0CO@EGEFBBBG@?$FLWARN?$FN?3?5?5?5AccessibleIcon?5descri@ 0000000180033370     AccessBridgeJavaEntryPoints.obj
 0002:000083a0       ??_C@_0DE@GOAGCEO@?$CD?$CD?$CD?$CD?$CD?5Getting?5icon?5height?5?9?5cal@ 00000001800333a0     AccessBridgeJavaEntryPoints.obj
 0002:000083d8       ??_C@_0CB@BMHPADNP@?$FLINFO?$FN?3?5?5?5?$CD?$CD?$CD?$CD?$CD?5icon?5height?5?$DN?5?$CF@ 00000001800333d8     AccessBridgeJavaEntryPoints.obj
 0002:00008400       ??_C@_0DD@EHAOAGFJ@?$CD?$CD?$CD?$CD?$CD?5Getting?5icon?5width?5?9?5call@ 0000000180033400     AccessBridgeJavaEntryPoints.obj
 0002:00008438       ??_C@_0CA@DPEBDDDD@?$FLINFO?$FN?3?5?5?5?$CD?$CD?$CD?$CD?$CD?5icon?5width?5?$DN?5?$CFd@ 0000000180033438     AccessBridgeJavaEntryPoints.obj
 0002:00008458       ??_C@_0DG@DLFAKGJK@?$CD?$CD?$CD?$CD?$CD?5Getting?5actions?5count?5?9?5c@ 0000000180033458     AccessBridgeJavaEntryPoints.obj
 0002:00008490       ??_C@_0CH@EOBAHIJB@?$FLINFO?$FN?3?5?5?5?$CD?$CD?$CD?$CD?$CD?5key?5actions?5cou@ 0000000180033490     AccessBridgeJavaEntryPoints.obj
 0002:000084b8       ??_C@_0DC@LHBGBJKA@Getting?5Action?5Name?5?5?9?5call?5to?5@ 00000001800334b8     AccessBridgeJavaEntryPoints.obj
 0002:000084f0       ??_C@_0DK@MCEEGDOO@Getting?5AccessibleAction?5Name?5?5@ 00000001800334f0     AccessBridgeJavaEntryPoints.obj
 0002:00008530       ??_C@_0BO@FCFGOMO@Getting?5AccessibleAction?5name@ 0000000180033530     AccessBridgeJavaEntryPoints.obj
 0002:00008550       ??_C@_0CL@LDPKEJLA@?$FLINFO?$FN?3?5?$CD?$CD?$CD?$CD?$CD?5AccessibleAction?5@ 0000000180033550     AccessBridgeJavaEntryPoints.obj
 0002:00008580       ??_C@_0DK@GEFGKAFF@Getting?5AccessibleAction?5name?5?5@ 0000000180033580     AccessBridgeJavaEntryPoints.obj
 0002:000085c0       ??_C@_0CK@GFGPDCKK@?$FLWARN?$FN?3?5?5?5AccessibleAction?5name@ 00000001800335c0     AccessBridgeJavaEntryPoints.obj
 0002:000085f0       ??_C@_0FG@HPHLKACM@?$FLINFO?$FN?3?5Calling?5AccessBridgeJav@ 00000001800335f0     AccessBridgeJavaEntryPoints.obj
 0002:00008648       ??_C@_0CB@NAFFMPJL@?$FLINFO?$FN?3?5?5?5?5?5doing?5?$CFd?5actions?5?4?4@ 0000000180033648     AccessBridgeJavaEntryPoints.obj
 0002:00008670       ??_C@_0CE@MIPOFJEF@?$FLINFO?$FN?3?5?5?5?5?5doing?5action?5?$CFd?3?5?$CFs@ 0000000180033670     AccessBridgeJavaEntryPoints.obj
 0002:00008698       ??_C@_0DC@PKIFPAKH@doAccessibleActions?5?9?5call?5to?5C@ 0000000180033698     AccessBridgeJavaEntryPoints.obj
 0002:000086d0       ??_C@_0BO@OONLHHCL@?$FLERROR?$FN?3?5?5?5?5?5Action?5?$CFd?5failed@ 00000001800336d0     AccessBridgeJavaEntryPoints.obj
 0002:000086f0       ??_C@_0FA@KEPHMGGF@?$FLINFO?$FN?3?5Calling?5AccessBridgeJav@ 00000001800336f0     AccessBridgeJavaEntryPoints.obj
 0002:00008740       ??_C@_0DG@GCJDNJFK@Getting?5AccessibleCharCount?5?9?5c@ 0000000180033740     AccessBridgeJavaEntryPoints.obj
 0002:00008778       ??_C@_0BK@OIDALDPI@?$FLINFO?$FN?3?5?5?5Char?5count?5?$DN?5?$CFd@ 0000000180033778     AccessBridgeJavaEntryPoints.obj
 0002:000087a0       ??_C@_0EJ@JKPJJPMH@?$FLERROR?$FN?3?5either?5env?5?$DN?$DN?50?5or?5get@ 00000001800337a0     AccessBridgeJavaEntryPoints.obj
 0002:000087f0       ??_C@_0DK@EFHALPMO@Getting?5AccessibleCaretPosition@ 00000001800337f0     AccessBridgeJavaEntryPoints.obj
 0002:00008830       ??_C@_0BO@CCCENNB@?$FLINFO?$FN?3?5?5?5Index?5at?5caret?5?$DN?5?$CFd@ 0000000180033830     AccessBridgeJavaEntryPoints.obj
 0002:00008850       ??_C@_0EN@DJGOBIMD@?$FLERROR?$FN?3?5either?5env?5?$DN?$DN?50?5or?5get@ 0000000180033850     AccessBridgeJavaEntryPoints.obj
 0002:000088a0       ??_C@_0DJ@MLOJKMJI@Getting?5AccessibleIndexAtPoint?5@ 00000001800338a0     AccessBridgeJavaEntryPoints.obj
 0002:000088e0       ??_C@_0BO@FIAABPFC@?$FLINFO?$FN?3?5?5?5Index?5at?5point?5?$DN?5?$CFd@ 00000001800338e0     AccessBridgeJavaEntryPoints.obj
 0002:00008900       ??_C@_0EM@ENNBLMPC@?$FLERROR?$FN?3?5either?5env?5?$DN?$DN?50?5or?5get@ 0000000180033900     AccessBridgeJavaEntryPoints.obj
 0002:00008950       ??_C@_0EJ@KDHBNGHD@?$FLINFO?$FN?3?5Calling?5AccessBridgeJav@ 0000000180033950     AccessBridgeJavaEntryPoints.obj
 0002:000089a0       ??_C@_0DK@CALJAPAO@Getting?5AccessibleLetterAtIndex@ 00000001800339a0     AccessBridgeJavaEntryPoints.obj
 0002:000089e0       ??_C@_0DL@JDJLEMDG@Getting?5AccessibleLetterAtIndex@ 00000001800339e0     AccessBridgeJavaEntryPoints.obj
 0002:00008a20       ??_C@_0DP@BIFOHJBB@Getting?5AccessibleLetterAtIndex@ 0000000180033a20     AccessBridgeJavaEntryPoints.obj
 0002:00008a60       ??_C@_0DL@OOLFPOBK@Getting?5AccessibleLetterAtIndex@ 0000000180033a60     AccessBridgeJavaEntryPoints.obj
 0002:00008aa0       ??_C@_0CG@BAFOKJKC@?$FLINFO?$FN?3?5?5?5Accessible?5Text?5lette@ 0000000180033aa0     AccessBridgeJavaEntryPoints.obj
 0002:00008ac8       ??_C@_0DL@FNGOIOKI@Getting?5AccessibleLetterAtIndex@ 0000000180033ac8     AccessBridgeJavaEntryPoints.obj
 0002:00008b08       ??_C@_0CK@KNLDNGDN@?$FLWARN?$FN?3?5?5?5Accessible?5Text?5lette@ 0000000180033b08     AccessBridgeJavaEntryPoints.obj
 0002:00008b40       ??_C@_0EN@GBFAECFE@?$FLERROR?$FN?3?5either?5env?5?$DN?$DN?50?5or?5get@ 0000000180033b40     AccessBridgeJavaEntryPoints.obj
 0002:00008b90       ??_C@_0DI@DFJMLOME@Getting?5AccessibleWordAtIndex?5?9@ 0000000180033b90     AccessBridgeJavaEntryPoints.obj
 0002:00008bc8       ??_C@_0DJ@OIDPECCJ@Getting?5AccessibleWordAtIndex?5?9@ 0000000180033bc8     AccessBridgeJavaEntryPoints.obj
 0002:00008c08       ??_C@_0BO@NGEDADOF@Getting?5AccessibleWordAtIndex@ 0000000180033c08     AccessBridgeJavaEntryPoints.obj
 0002:00008c28       ??_C@_0DJ@JFBBPAAF@Getting?5AccessibleWordAtIndex?5?9@ 0000000180033c28     AccessBridgeJavaEntryPoints.obj
 0002:00008c70       ??_C@_1EK@ODCBDMFL@?$AA?$FL?$AAI?$AAN?$AAF?$AAO?$AA?$FN?$AA?3?$AA?5?$AA?5?$AA?5?$AAA?$AAc?$AAc?$AAe?$AAs@ 0000000180033c70     AccessBridgeJavaEntryPoints.obj
 0002:00008cc0       ??_C@_0DJ@CGMKIALH@Getting?5AccessibleWordAtIndex?5?9@ 0000000180033cc0     AccessBridgeJavaEntryPoints.obj
 0002:00008d00       ??_C@_0CI@JLGHFNHI@?$FLWARN?$FN?3?5?5?5Accessible?5Text?5word?5@ 0000000180033d00     AccessBridgeJavaEntryPoints.obj
 0002:00008d30       ??_C@_0EL@NKGFFDIO@?$FLERROR?$FN?3?5either?5env?5?$DN?$DN?50?5or?5get@ 0000000180033d30     AccessBridgeJavaEntryPoints.obj
 0002:00008d80       ??_C@_0DP@OGFHHBKC@Getting?5AccessibleSentenceAtInd@ 0000000180033d80     AccessBridgeJavaEntryPoints.obj
 0002:00008dc0       ??_C@_0DN@MGFPCBII@Getting?5AccessibleSentenceAtInd@ 0000000180033dc0     AccessBridgeJavaEntryPoints.obj
 0002:00008e00       ??_C@_0CC@BFJMFDHP@Getting?5AccessibleSentenceAtInd@ 0000000180033e00     AccessBridgeJavaEntryPoints.obj
 0002:00008e28       ??_C@_0DN@LLHBJDKE@Getting?5AccessibleSentenceAtInd@ 0000000180033e28     AccessBridgeJavaEntryPoints.obj
 0002:00008e70       ??_C@_1FC@FOIECOHK@?$AA?$FL?$AAI?$AAN?$AAF?$AAO?$AA?$FN?$AA?3?$AA?5?$AA?5?$AA?5?$AAA?$AAc?$AAc?$AAe?$AAs@ 0000000180033e70     AccessBridgeJavaEntryPoints.obj
 0002:00008ec8       ??_C@_0DN@IKKODBG@Getting?5AccessibleSentenceAtInd@ 0000000180033ec8     AccessBridgeJavaEntryPoints.obj
 0002:00008f08       ??_C@_0CM@EBOEJDBD@?$FLWARN?$FN?3?5?5?5Accessible?5Text?5sente@ 0000000180033f08     AccessBridgeJavaEntryPoints.obj
 0002:00008f40       ??_C@_0EP@JMGAHICJ@?$FLERROR?$FN?3?5either?5env?5?$DN?$DN?50?5or?5get@ 0000000180033f40     AccessBridgeJavaEntryPoints.obj
 0002:00008f90       ??_C@_0FB@DGBDAMEN@?$FLINFO?$FN?3?5Calling?5AccessBridgeJav@ 0000000180033f90     AccessBridgeJavaEntryPoints.obj
 0002:00008fe8       ??_C@_0DP@BBIGIAAH@Getting?5AccessibleTextSelection@ 0000000180033fe8     AccessBridgeJavaEntryPoints.obj
 0002:00009028       ??_C@_0BP@MPEDAFPO@?$FLINFO?$FN?3?5?5?5Selection?5start?5?$DN?5?$CFd@ 0000000180034028     AccessBridgeJavaEntryPoints.obj
 0002:00009050       ??_C@_0FD@EDCFOMDB@?$FLERROR?$FN?3?5?5either?5env?5?$DN?$DN?50?5or?5ge@ 0000000180034050     AccessBridgeJavaEntryPoints.obj
 0002:000090a8       ??_C@_0DN@MBOJJHKP@Getting?5AccessibleTextSelection@ 00000001800340a8     AccessBridgeJavaEntryPoints.obj
 0002:000090e8       ??_C@_0BN@JAKAFPAN@?$FLINFO?$FN?3?5?5?5Selection?5end?5?$DN?5?$CFd@ 00000001800340e8     AccessBridgeJavaEntryPoints.obj
 0002:00009110       ??_C@_0FA@HPMPKGDO@?$FLERROR?$FN?3?5either?5env?5?$DN?$DN?50?5or?5get@ 0000000180034110     AccessBridgeJavaEntryPoints.obj
 0002:00009160       ??_C@_0EA@KGAPFINL@Getting?5AccessibleTextSelectedT@ 0000000180034160     AccessBridgeJavaEntryPoints.obj
 0002:000091a0       ??_C@_0DO@OMODBJBJ@Getting?5AccessibleTextSelectedT@ 00000001800341a0     AccessBridgeJavaEntryPoints.obj
 0002:000091e0       ??_C@_0CD@CMKAHLON@Getting?5AccessibleTextSelectedT@ 00000001800341e0     AccessBridgeJavaEntryPoints.obj
 0002:00009208       ??_C@_0DO@JBMNKLDF@Getting?5AccessibleTextSelectedT@ 0000000180034208     AccessBridgeJavaEntryPoints.obj
 0002:00009248       ??_C@_0CK@DDDAABEG@?$FLINFO?$FN?3?5?5?5Accessible?8s?5selected@ 0000000180034248     AccessBridgeJavaEntryPoints.obj
 0002:00009278       ??_C@_0DO@CCBGNLIH@Getting?5AccessibleTextSelectedT@ 0000000180034278     AccessBridgeJavaEntryPoints.obj
 0002:000092b8       ??_C@_0CO@GAOLMCL@?$FLWARN?$FN?3?5?5?5Accessible?8s?5selected@ 00000001800342b8     AccessBridgeJavaEntryPoints.obj
 0002:000092f0       ??_C@_0EP@FNBFNNLO@?$FLWARN?$FN?3?5either?5env?5?$DN?$DN?50?5or?5getA@ 00000001800342f0     AccessBridgeJavaEntryPoints.obj
 0002:00009340       ??_C@_0EO@HEMIPALC@?$FLINFO?$FN?3?5Calling?5AccessBridgeJav@ 0000000180034340     AccessBridgeJavaEntryPoints.obj
 0002:00009390       ??_C@_0CK@OGCGGLCF@?$FLINFO?$FN?3?5?5Getting?5AttributeSet?5a@ 0000000180034390     AccessBridgeJavaEntryPoints.obj
 0002:000093c0       ??_C@_0ED@CGONELLD@Getting?5AccessibleAttributeSetA@ 00000001800343c0     AccessBridgeJavaEntryPoints.obj
 0002:00009410       ??_C@_0FD@BNPBOBD@?$FLERROR?$FN?3?5either?5env?5?$DN?$DN?50?5or?5get@ 0000000180034410     AccessBridgeJavaEntryPoints.obj
 0002:00009470       ??_C@_0FG@OPHHFMC@?$FLWARN?$FN?3?5?5AttributeSet?5returned?5@ 0000000180034470     AccessBridgeJavaEntryPoints.obj
 0002:000094c8       ??_C@_0CL@BFGDEBIA@?$FLINFO?$FN?3?5?5Getting?5bold?5from?5Attr@ 00000001800344c8     AccessBridgeJavaEntryPoints.obj
 0002:000094f8       ??_C@_0DL@NGCGOJOD@Getting?5BoldFromAttributeSet?5?9?5@ 00000001800344f8     AccessBridgeJavaEntryPoints.obj
 0002:00009538       ??_C@_0DP@GPLAEKHL@?$FLERROR?$FN?3?5either?5env?5?$DN?$DN?50?5or?5get@ 0000000180034538     AccessBridgeJavaEntryPoints.obj
 0002:00009578       ??_C@_0DI@GHAHHMIG@Getting?5BoldFromAttributeSet?5?9?5@ 0000000180034578     AccessBridgeJavaEntryPoints.obj
 0002:000095b0       ??_C@_0DI@NENMAMDE@Getting?5BoldFromAttributeSet?5?9?5@ 00000001800345b0     AccessBridgeJavaEntryPoints.obj
 0002:000095e8       ??_C@_0CN@DLPNJKCI@?$FLINFO?$FN?3?5?5Getting?5italic?5from?5At@ 00000001800345e8     AccessBridgeJavaEntryPoints.obj
 0002:00009618       ??_C@_0DN@FALJGLGH@Getting?5ItalicFromAttributeSet?5@ 0000000180034618     AccessBridgeJavaEntryPoints.obj
 0002:00009660       ??_C@_0EC@PFKOONOF@?$FLERROR?$FN?3?5either?5env?5?$DN?$DN?50?5or?5get@ 0000000180034660     AccessBridgeJavaEntryPoints.obj
 0002:000096a8       ??_C@_0DK@CEDKJPGF@Getting?5ItalicFromAttributeSet?5@ 00000001800346a8     AccessBridgeJavaEntryPoints.obj
 0002:000096e8       ??_C@_0DK@JHOBOPNH@Getting?5ItalicFromAttributeSet?5@ 00000001800346e8     AccessBridgeJavaEntryPoints.obj
 0002:00009728       ??_C@_0DA@HJAHPBCP@?$FLINFO?$FN?3?5?5Getting?5underline?5from@ 0000000180034728     AccessBridgeJavaEntryPoints.obj
 0002:00009760       ??_C@_0EA@LFOJMIBN@Getting?5UnderlineFromAttributeS@ 0000000180034760     AccessBridgeJavaEntryPoints.obj
 0002:000097a0       ??_C@_0EF@LMCHMLNC@?$FLERROR?$FN?3?5?5either?5env?5?$DN?$DN?50?5or?5ge@ 00000001800347a0     AccessBridgeJavaEntryPoints.obj
 0002:000097e8       ??_C@_0DN@GEOGGPCN@Getting?5UnderlineFromAttributeS@ 00000001800347e8     AccessBridgeJavaEntryPoints.obj
 0002:00009828       ??_C@_0DN@NHDNBPJP@Getting?5UnderlineFromAttributeS@ 0000000180034828     AccessBridgeJavaEntryPoints.obj
 0002:00009868       ??_C@_0DE@MIAPKOHI@?$FLINFO?$FN?3?5?5Getting?5strikethrough?5@ 0000000180034868     AccessBridgeJavaEntryPoints.obj
 0002:000098a0       ??_C@_0EE@DDJIBELI@Getting?5StrikethroughFromAttrib@ 00000001800348a0     AccessBridgeJavaEntryPoints.obj
 0002:000098f0       ??_C@_0EI@HMMOGEKC@?$FLERROR?$FN?3?5either?5env?5?$DN?$DN?50?5or?5get@ 00000001800348f0     AccessBridgeJavaEntryPoints.obj
 0002:00009940       ??_C@_0EB@GCIGLCLO@Getting?5StrikethroughFromAttrib@ 0000000180034940     AccessBridgeJavaEntryPoints.obj
 0002:00009990       ??_C@_0EB@NBFNMCAM@Getting?5StrikethroughFromAttrib@ 0000000180034990     AccessBridgeJavaEntryPoints.obj
 0002:000099d8       ??_C@_0DC@ENJFOBHI@?$FLINFO?$FN?3?5?5Getting?5superscript?5fr@ 00000001800349d8     AccessBridgeJavaEntryPoints.obj
 0002:00009a10       ??_C@_0EC@BAJDPNIO@Getting?5SuperscriptFromAttribut@ 0000000180034a10     AccessBridgeJavaEntryPoints.obj
 0002:00009a60       ??_C@_0EH@EIIKEOA@?$FLERROR?$FN?3?5either?5env?5?$DN?$DN?50?5or?5get@ 0000000180034a60     AccessBridgeJavaEntryPoints.obj
 0002:00009aa8       ??_C@_0DP@LNAJFDKJ@Getting?5SuperscriptFromAttribut@ 0000000180034aa8     AccessBridgeJavaEntryPoints.obj
 0002:00009ae8       ??_C@_0DP@ONCCDBL@Getting?5SuperscriptFromAttribut@ 0000000180034ae8     AccessBridgeJavaEntryPoints.obj
 0002:00009b28       ??_C@_0DA@KLOJONPP@?$FLINFO?$FN?3?5?5Getting?5subscript?5from@ 0000000180034b28     AccessBridgeJavaEntryPoints.obj
 0002:00009b60       ??_C@_0EA@NMFFGPLI@Getting?5SubscriptFromAttributeS@ 0000000180034b60     AccessBridgeJavaEntryPoints.obj
 0002:00009ba0       ??_C@_0EE@EGHOMMOM@?$FLERROR?$FN?3?5either?5env?5?$DN?$DN?50?5or?5get@ 0000000180034ba0     AccessBridgeJavaEntryPoints.obj
 0002:00009be8       ??_C@_0DN@NJLPKKJA@Getting?5SubscriptFromAttributeS@ 0000000180034be8     AccessBridgeJavaEntryPoints.obj
 0002:00009c28       ??_C@_0DN@GKGENKCC@Getting?5SubscriptFromAttributeS@ 0000000180034c28     AccessBridgeJavaEntryPoints.obj
 0002:00009c68       ??_C@_0DG@JDMMILDN@?$FLINFO?$FN?3?5?5Getting?5backgroundColo@ 0000000180034c68     AccessBridgeJavaEntryPoints.obj
 0002:00009ca0       ??_C@_0EF@CPKEHGFF@Getting?5BackgroundColorFromAttr@ 0000000180034ca0     AccessBridgeJavaEntryPoints.obj
 0002:00009cf0       ??_C@_0ED@OOEECCFB@Getting?5BackgroundColorFromAttr@ 0000000180034cf0     AccessBridgeJavaEntryPoints.obj
 0002:00009d38       ??_C@_0CI@JBOBOECB@Getting?5BackgroundColorFromAttr@ 0000000180034d38     AccessBridgeJavaEntryPoints.obj
 0002:00009d60       ??_C@_0ED@JDGKJAHN@Getting?5BackgroundColorFromAttr@ 0000000180034d60     AccessBridgeJavaEntryPoints.obj
 0002:00009db0       ??_C@_1GA@PMLMKIMP@?$AA?$FL?$AAI?$AAN?$AAF?$AAO?$AA?$FN?$AA?3?$AA?5?$AA?5?$AA?5?$AAA?$AAt?$AAt?$AAr?$AAi@ 0000000180034db0     AccessBridgeJavaEntryPoints.obj
 0002:00009e10       ??_C@_0ED@CALBOAMP@Getting?5BackgroundColorFromAttr@ 0000000180034e10     AccessBridgeJavaEntryPoints.obj
 0002:00009e58       ??_C@_0DD@DIMBBLFG@?$FLWARN?$FN?3?5?5?5AttributeSet?8s?5backgr@ 0000000180034e58     AccessBridgeJavaEntryPoints.obj
 0002:00009e90       ??_C@_0EK@LDLFAHLP@?$FLERROR?$FN?3?5either?5env?5?$DN?$DN?50?5or?5get@ 0000000180034e90     AccessBridgeJavaEntryPoints.obj
 0002:00009ee0       ??_C@_0DG@OAPFKBJG@?$FLINFO?$FN?3?5?5Getting?5foregroundColo@ 0000000180034ee0     AccessBridgeJavaEntryPoints.obj
 0002:00009f20       ??_C@_0EF@CFMCBGOA@Getting?5ForegroundColorFromAttr@ 0000000180034f20     AccessBridgeJavaEntryPoints.obj
 0002:00009f70       ??_C@_0ED@CGONGGIL@Getting?5ForegroundColorFromAttr@ 0000000180034f70     AccessBridgeJavaEntryPoints.obj
 0002:00009fb8       ??_C@_0CI@MCDFAAFE@Getting?5ForegroundColorFromAttr@ 0000000180034fb8     AccessBridgeJavaEntryPoints.obj
 0002:00009fe0       ??_C@_0ED@FLMDNEKH@Getting?5ForegroundColorFromAttr@ 0000000180034fe0     AccessBridgeJavaEntryPoints.obj
 0002:0000a030       ??_C@_1GA@DDCOJJLA@?$AA?$FL?$AAI?$AAN?$AAF?$AAO?$AA?$FN?$AA?3?$AA?5?$AA?5?$AA?5?$AAA?$AAt?$AAt?$AAr?$AAi@ 0000000180035030     AccessBridgeJavaEntryPoints.obj
 0002:0000a090       ??_C@_0ED@OIBIKEBF@Getting?5ForegroundColorFromAttr@ 0000000180035090     AccessBridgeJavaEntryPoints.obj
 0002:0000a0d8       ??_C@_0DD@EGLIFJNP@?$FLWARN?$FN?3?5?5?5AttributeSet?8s?5foregr@ 00000001800350d8     AccessBridgeJavaEntryPoints.obj
 0002:0000a110       ??_C@_0EK@JAILLABF@?$FLERROR?$FN?3?5either?5env?5?$DN?$DN?50?5or?5get@ 0000000180035110     AccessBridgeJavaEntryPoints.obj
 0002:0000a160       ??_C@_0DB@NPCHLNMB@?$FLINFO?$FN?3?5?5Getting?5fontFamily?5fro@ 0000000180035160     AccessBridgeJavaEntryPoints.obj
 0002:0000a1a0       ??_C@_0EA@OFLFMJOA@Getting?5FontFamilyFromAttribute@ 00000001800351a0     AccessBridgeJavaEntryPoints.obj
 0002:0000a1e0       ??_C@_0DO@ECEGIKHO@Getting?5FontFamilyFromAttribute@ 00000001800351e0     AccessBridgeJavaEntryPoints.obj
 0002:0000a220       ??_C@_0CD@ELONJGOI@Getting?5FontFamilyFromAttribute@ 0000000180035220     AccessBridgeJavaEntryPoints.obj
 0002:0000a248       ??_C@_0DO@DPGIDIFC@Getting?5FontFamilyFromAttribute@ 0000000180035248     AccessBridgeJavaEntryPoints.obj
 0002:0000a290       ??_C@_1FE@LCMANMIC@?$AA?$FL?$AAI?$AAN?$AAF?$AAO?$AA?$FN?$AA?3?$AA?5?$AA?5?$AA?5?$AAA?$AAt?$AAt?$AAr?$AAi@ 0000000180035290     AccessBridgeJavaEntryPoints.obj
 0002:0000a2e8       ??_C@_0DO@IMLDEIOA@Getting?5FontFamilyFromAttribute@ 00000001800352e8     AccessBridgeJavaEntryPoints.obj
 0002:0000a328       ??_C@_0CN@DFPIBNDO@?$FLWARN?$FN?3?5?5?5AttributeSet?8s?5fontFa@ 0000000180035328     AccessBridgeJavaEntryPoints.obj
 0002:0000a360       ??_C@_0EF@MEIJBCDI@?$FLERROR?$FN?3?5either?5env?5?$DN?$DN?50?5or?5get@ 0000000180035360     AccessBridgeJavaEntryPoints.obj
 0002:0000a3a8       ??_C@_0DA@NKBCCHCB@?$FLINFO?$FN?3?5?5Getting?5font?5size?5from@ 00000001800353a8     AccessBridgeJavaEntryPoints.obj
 0002:0000a3d8       ??_C@_0DL@OGKGFGCH@Getting?5FontSizeFromAttributeSe@ 00000001800353d8     AccessBridgeJavaEntryPoints.obj
 0002:0000a418       ??_C@_0CI@MMDBDPDB@?$FLINFO?$FN?3?5?5?5AttributeSet?8s?5font?5s@ 0000000180035418     AccessBridgeJavaEntryPoints.obj
 0002:0000a440       ??_C@_0EE@EGBGOKJP@?$FLERROR?$FN?3?5either?5env?5?$DN?$DN?50?5or?5get@ 0000000180035440     AccessBridgeJavaEntryPoints.obj
 0002:0000a488       ??_C@_0DM@KMMBHJCP@Getting?5FontSizeFromAttributeSe@ 0000000180035488     AccessBridgeJavaEntryPoints.obj
 0002:0000a4c8       ??_C@_0DM@BPBKAJJN@Getting?5FontSizeFromAttributeSe@ 00000001800354c8     AccessBridgeJavaEntryPoints.obj
 0002:0000a508       ??_C@_0CI@DPJLKBCH@?5Getting?5alignment?5from?5Attribu@ 0000000180035508     AccessBridgeJavaEntryPoints.obj
 0002:0000a530       ??_C@_0DM@IEKBPPGN@Getting?5AlignmentFromAttributeS@ 0000000180035530     AccessBridgeJavaEntryPoints.obj
 0002:0000a570       ??_C@_0DN@DKKKNGAI@Getting?5AlignmentFromAttributeS@ 0000000180035570     AccessBridgeJavaEntryPoints.obj
 0002:0000a5b0       ??_C@_0DN@IJHBKGLK@Getting?5AlignmentFromAttributeS@ 00000001800355b0     AccessBridgeJavaEntryPoints.obj
 0002:0000a5f0       ??_C@_0DA@IEHDNKCA@?$FLINFO?$FN?3?5?5Getting?5bidiLevel?5from@ 00000001800355f0     AccessBridgeJavaEntryPoints.obj
 0002:0000a620       ??_C@_0DM@HHHEIBLO@Getting?5BidiLevelFromAttributeS@ 0000000180035620     AccessBridgeJavaEntryPoints.obj
 0002:0000a660       ??_C@_0EE@FHPLAGJN@?$FLERROR?$FN?3?5either?5env?5?$DN?$DN?50?5or?5get@ 0000000180035660     AccessBridgeJavaEntryPoints.obj
 0002:0000a6a8       ??_C@_0DN@CFIDIABI@Getting?5BidiLevelFromAttributeS@ 00000001800356a8     AccessBridgeJavaEntryPoints.obj
 0002:0000a6e8       ??_C@_0DN@JGFIPAKK@Getting?5BidiLevelFromAttributeS@ 00000001800356e8     AccessBridgeJavaEntryPoints.obj
 0002:0000a728       ??_C@_0DH@CAJPMJAH@?$FLERROR?$FN?3?5?5Getting?5firstLineInde@ 0000000180035728     AccessBridgeJavaEntryPoints.obj
 0002:0000a760       ??_C@_0EC@GDNCLBBP@Getting?5FirstLineIndentFromAttr@ 0000000180035760     AccessBridgeJavaEntryPoints.obj
 0002:0000a7b0       ??_C@_0EK@JNGBIMLH@?$FLERROR?$FN?3?5either?5env?5?$DN?$DN?50?5or?5get@ 00000001800357b0     AccessBridgeJavaEntryPoints.obj
 0002:0000a800       ??_C@_0ED@IEEGLFFG@Getting?5FirstLineIndentFromAttr@ 0000000180035800     AccessBridgeJavaEntryPoints.obj
 0002:0000a850       ??_C@_0ED@DHJNMFOE@Getting?5FirstLineIndentFromAttr@ 0000000180035850     AccessBridgeJavaEntryPoints.obj
 0002:0000a898       ??_C@_0DB@GIKOBABF@?$FLINFO?$FN?3?5?5Getting?5leftIndent?5fro@ 0000000180035898     AccessBridgeJavaEntryPoints.obj
 0002:0000a8d0       ??_C@_0DN@GGPJCLGF@Getting?5LeftIndentFromAttribute@ 00000001800358d0     AccessBridgeJavaEntryPoints.obj
 0002:0000a910       ??_C@_0EF@JFNBAGAC@?$FLERROR?$FN?3?5either?5env?5?$DN?$DN?50?5or?5get@ 0000000180035910     AccessBridgeJavaEntryPoints.obj
 0002:0000a958       ??_C@_0DO@DEJDAGOO@Getting?5LeftIndentFromAttribute@ 0000000180035958     AccessBridgeJavaEntryPoints.obj
 0002:0000a998       ??_C@_0DO@IHEIHGFM@Getting?5LeftIndentFromAttribute@ 0000000180035998     AccessBridgeJavaEntryPoints.obj
 0002:0000a9d8       ??_C@_0DC@OHJHAPPB@?$FLINFO?$FN?3?5?5Getting?5rightIndent?5fr@ 00000001800359d8     AccessBridgeJavaEntryPoints.obj
 0002:0000aa10       ??_C@_0DO@GPANPNCO@Getting?5RightIndentFromAttribut@ 0000000180035a10     AccessBridgeJavaEntryPoints.obj
 0002:0000aa50       ??_C@_0EG@FKGIOCMJ@?$FLERROR?$FN?3?5either?5env?5?$DN?$DN?50?5or?5get@ 0000000180035a50     AccessBridgeJavaEntryPoints.obj
 0002:0000aa98       ??_C@_0DP@NFJEGKCA@Getting?5RightIndentFromAttribut@ 0000000180035a98     AccessBridgeJavaEntryPoints.obj
 0002:0000aad8       ??_C@_0DP@GGEPBKJC@Getting?5RightIndentFromAttribut@ 0000000180035ad8     AccessBridgeJavaEntryPoints.obj
 0002:0000ab18       ??_C@_0DC@FBCMPKE@?$FLINFO?$FN?3?5?5Getting?5lineSpacing?5fr@ 0000000180035b18     AccessBridgeJavaEntryPoints.obj
 0002:0000ab50       ??_C@_0DO@OLMNNFJE@Getting?5LineSpacingFromAttribut@ 0000000180035b50     AccessBridgeJavaEntryPoints.obj
 0002:0000ab90       ??_C@_0EH@DJGGHDHL@?$FLERROR?$FN?3?5?5either?5env?5?$DN?$DN?50?5or?5ge@ 0000000180035b90     AccessBridgeJavaEntryPoints.obj
 0002:0000abd8       ??_C@_0DP@POKEPAJK@Getting?5LineSpacingFromAttribut@ 0000000180035bd8     AccessBridgeJavaEntryPoints.obj
 0002:0000ac18       ??_C@_0DP@ENHPIACI@Getting?5LineSpacingFromAttribut@ 0000000180035c18     AccessBridgeJavaEntryPoints.obj
 0002:0000ac58       ??_C@_0DB@BBFBINOC@?$FLINFO?$FN?3?5?5Getting?5spaceAbove?5fro@ 0000000180035c58     AccessBridgeJavaEntryPoints.obj
 0002:0000ac90       ??_C@_0DN@LICNMEPC@Getting?5SpaceAboveFromAttribute@ 0000000180035c90     AccessBridgeJavaEntryPoints.obj
 0002:0000acd0       ??_C@_0EG@DEAABEIJ@?$FLERROR?$FN?3?5?5either?5env?5?$DN?$DN?50?5or?5ge@ 0000000180035cd0     AccessBridgeJavaEntryPoints.obj
 0002:0000ad18       ??_C@_0DO@FKCGNEOG@Getting?5SpaceAboveFromAttribute@ 0000000180035d18     AccessBridgeJavaEntryPoints.obj
 0002:0000ad58       ??_C@_0DO@OJPNKEFE@Getting?5SpaceAboveFromAttribute@ 0000000180035d58     AccessBridgeJavaEntryPoints.obj
 0002:0000ad98       ??_C@_0DB@IPEMBOFF@?$FLINFO?$FN?3?5?5Getting?5spaceBelow?5fro@ 0000000180035d98     AccessBridgeJavaEntryPoints.obj
 0002:0000add0       ??_C@_0DN@KGEHENNL@Getting?5SpaceBelowFromAttribute@ 0000000180035dd0     AccessBridgeJavaEntryPoints.obj
 0002:0000ae10       ??_C@_0EG@PAJHHADM@?$FLERROR?$FN?3?5?5either?5env?5?$DN?$DN?50?5or?5ge@ 0000000180035e10     AccessBridgeJavaEntryPoints.obj
 0002:0000ae58       ??_C@_0DO@BIIKCGAD@Getting?5SpaceBelowFromAttribute@ 0000000180035e58     AccessBridgeJavaEntryPoints.obj
 0002:0000ae98       ??_C@_0DO@KLFBFGLB@Getting?5SpaceBelowFromAttribute@ 0000000180035e98     AccessBridgeJavaEntryPoints.obj
 0002:0000aed8       ??_C@_0DD@NEPODHGJ@?$FLINFO?$FN?3?5?5Decrementing?5reference@ 0000000180035ed8     AccessBridgeJavaEntryPoints.obj
 0002:0000af10       ??_C@_0DJ@KDCCLHCF@Releasing?5AttributeSet?5object?5?9@ 0000000180035f10     AccessBridgeJavaEntryPoints.obj
 0002:0000af50       ??_C@_0DF@KOJHMOGM@?$FLERROR?$FN?3?5?5either?5env?5?$DN?$DN?50?5or?5ac@ 0000000180035f50     AccessBridgeJavaEntryPoints.obj
 0002:0000af88       ??_C@_0DJ@BAPJMHJH@Releasing?5AttributeSet?5object?5?9@ 0000000180035f88     AccessBridgeJavaEntryPoints.obj
 0002:0000afc8       ??_C@_0DI@FAAGAOKI@?$FLINFO?$FN?3?5?5Getting?5full?5attribute@ 0000000180035fc8     AccessBridgeJavaEntryPoints.obj
 0002:0000b000       ??_C@_0DD@BPFGOEDD@?$FLINFO?$FN?3?5?5returned?5from?5CallObje@ 0000000180036000     AccessBridgeJavaEntryPoints.obj
 0002:0000b040       ??_C@_1FG@IBEGPOLG@?$AA?$FL?$AAI?$AAN?$AAF?$AAO?$AA?$FN?$AA?3?$AA?5?$AA?5?$AA?5?$AAA?$AAc?$AAc?$AAe?$AAs@ 0000000180036040     AccessBridgeJavaEntryPoints.obj
 0002:0000b0a0       ??_C@_0FC@NKKMDLMK@?$FLERROR?$FN?3?5?5either?5env?5?$DN?$DN?50?5or?5ge@ 00000001800360a0     AccessBridgeJavaEntryPoints.obj
 0002:0000b100       ??_C@_0EB@FOBGJMBG@Getting?5AccessibleAttributeSetA@ 0000000180036100     AccessBridgeJavaEntryPoints.obj
 0002:0000b150       ??_C@_0FD@ONBHOKNL@?$FLINFO?$FN?3?5Calling?5AccessBridgeJav@ 0000000180036150     AccessBridgeJavaEntryPoints.obj
 0002:0000b1a8       ??_C@_0DL@PJLLEMMJ@Getting?5AccessibleXcoordTextRec@ 00000001800361a8     AccessBridgeJavaEntryPoints.obj
 0002:0000b1e8       ??_C@_0BG@CDBEIJEJ@?$FLINFO?$FN?3?5?5X?5coord?5?$DN?5?$CFd@ 00000001800361e8     AccessBridgeJavaEntryPoints.obj
 0002:0000b200       ??_C@_0FF@CICHONC@?$FLERROR?$FN?3?5either?5env?5?$DN?$DN?50?5or?5get@ 0000000180036200     AccessBridgeJavaEntryPoints.obj
 0002:0000b258       ??_C@_0DL@BBKMNMGI@Getting?5AccessibleYcoordTextRec@ 0000000180036258     AccessBridgeJavaEntryPoints.obj
 0002:0000b2a0       ??_C@_0FF@LPGHAKKN@?$FLINFO?$FN?3?5?5either?5env?5?$DN?$DN?50?5or?5get@ 00000001800362a0     AccessBridgeJavaEntryPoints.obj
 0002:0000b2f8       ??_C@_0DK@GOMAAIJJ@Getting?5AccessibleWidthTextRect@ 00000001800362f8     AccessBridgeJavaEntryPoints.obj
 0002:0000b338       ??_C@_0BD@PFFPBFHC@?$FLINFO?$FN?3?5Width?5?$DN?5?$CFd@ 0000000180036338     AccessBridgeJavaEntryPoints.obj
 0002:0000b350       ??_C@_0FD@LFKJAPPJ@?$FLINFO?$FN?3?5either?5env?5?$DN?$DN?50?5or?5getA@ 0000000180036350     AccessBridgeJavaEntryPoints.obj
 0002:0000b3a8       ??_C@_0DL@LIFPGLAA@Getting?5AccessibleHeightTextRec@ 00000001800363a8     AccessBridgeJavaEntryPoints.obj
 0002:0000b3e8       ??_C@_0BE@BNGOGMPP@?$FLINFO?$FN?3?5Height?5?$DN?5?$CFd@ 00000001800363e8     AccessBridgeJavaEntryPoints.obj
 0002:0000b400       ??_C@_0FG@JCNMAPKJ@?$FLERROR?$FN?3?5?5either?5env?5?$DN?$DN?50?5or?5ge@ 0000000180036400     AccessBridgeJavaEntryPoints.obj
 0002:0000b460       ??_C@_0EO@GAEGCFMP@?$FLINFO?$FN?3?5Calling?5AccessBridgeJav@ 0000000180036460     AccessBridgeJavaEntryPoints.obj
 0002:0000b4b0       ??_C@_0DF@JPKJOLBB@Getting?5caret?5X?5coordinate?5?9?5ca@ 00000001800364b0     AccessBridgeJavaEntryPoints.obj
 0002:0000b4e8       ??_C@_0DK@INHGMNIG@?$FLERROR?$FN?3?5?5either?5env?5?$DN?$DN?50?5or?5ge@ 00000001800364e8     AccessBridgeJavaEntryPoints.obj
 0002:0000b528       ??_C@_0DF@NBCAOALI@Getting?5caret?5Y?5coordinate?5?9?5ca@ 0000000180036528     AccessBridgeJavaEntryPoints.obj
 0002:0000b560       ??_C@_0DK@FAOABEAD@?$FLERROR?$FN?3?5?5either?5env?5?$DN?$DN?50?5or?5ge@ 0000000180036560     AccessBridgeJavaEntryPoints.obj
 0002:0000b5a0       ??_C@_0CO@LPKJFNHN@Getting?5caret?5width?5?9?5call?5to?5C@ 00000001800365a0     AccessBridgeJavaEntryPoints.obj
 0002:0000b5d0       ??_C@_0DO@KCIKCBGA@?$FLERROR?$FN?3?5?5either?5env?5?$DN?$DN?50?5or?5ge@ 00000001800365d0     AccessBridgeJavaEntryPoints.obj
 0002:0000b610       ??_C@_0CP@DKBLCBME@Getting?5caret?5height?5?9?5call?5to?5@ 0000000180036610     AccessBridgeJavaEntryPoints.obj
 0002:0000b640       ??_C@_0DP@MHKONHOK@?$FLERROR?$FN?3?5?5either?5env?5?$DN?$DN?50?5or?5ge@ 0000000180036640     AccessBridgeJavaEntryPoints.obj
 0002:0000b680       ??_C@_0EO@OPGMODFN@?$FLINFO?$FN?3?5Calling?5AccessBridgeJav@ 0000000180036680     AccessBridgeJavaEntryPoints.obj
 0002:0000b6d0       ??_C@_0DP@HIDGMFDD@Getting?5AccessibleTextLineLeftB@ 00000001800366d0     AccessBridgeJavaEntryPoints.obj
 0002:0000b710       ??_C@_0BK@INECDNLO@?$FLINFO?$FN?3?5?5?5startIndex?5?$DN?5?$CFd@ 0000000180036710     AccessBridgeJavaEntryPoints.obj
 0002:0000b730       ??_C@_0FD@BGKHJCDH@?$FLERROR?$FN?3?5?5either?5env?5?$DN?$DN?50?5or?5ge@ 0000000180036730     AccessBridgeJavaEntryPoints.obj
 0002:0000b790       ??_C@_0EA@OJGAJNKG@Getting?5AccessibleTextLineRight@ 0000000180036790     AccessBridgeJavaEntryPoints.obj
 0002:0000b7d0       ??_C@_0BI@NAKKCMDP@?$FLINFO?$FN?3?5?5?5endIndex?5?$DN?5?$CFd@ 00000001800367d0     AccessBridgeJavaEntryPoints.obj
 0002:0000b7f0       ??_C@_0FE@HOJFBBNL@?$FLERROR?$FN?3?5?5either?5env?5?$DN?$DN?50?5or?5ge@ 00000001800367f0     AccessBridgeJavaEntryPoints.obj
 0002:0000b850       ??_C@_0FM@PBOJPFBI@?$FLINFO?$FN?3?5Calling?5AccessBridgeJav@ 0000000180036850     AccessBridgeJavaEntryPoints.obj
 0002:0000b8b0       ??_C@_0BH@GCPBFEO@?$FLERROR?$FN?3?5?5end?5?$DM?5start?$CB@ 00000001800368b0     AccessBridgeJavaEntryPoints.obj
 0002:0000b8c8       ??_C@_0DJ@OHJBLKEE@Getting?5AccessibleTextRange?5?9?5c@ 00000001800368c8     AccessBridgeJavaEntryPoints.obj
 0002:0000b908       ??_C@_0DH@MLKPAEJI@Getting?5AccessibleTextRange?5?9?5c@ 0000000180036908     AccessBridgeJavaEntryPoints.obj
 0002:0000b940       ??_C@_1HO@MOIAIALP@?$AA?$FL?$AAI?$AAN?$AAF?$AAO?$AA?$FN?$AA?3?$AA?5?$AA?5?$AA?5?$AAA?$AAc?$AAc?$AAe?$AAs@ 0000000180036940     AccessBridgeJavaEntryPoints.obj
 0002:0000b9c0       ??_C@_0DB@GEMONLMO@?$FLINFO?$FN?3?5?5Accessible?5Text?5string@ 00000001800369c0     AccessBridgeJavaEntryPoints.obj
 0002:0000ba00       ??_C@_1HM@KJDBDPH@?$AA?$FL?$AAI?$AAN?$AAF?$AAO?$AA?$FN?$AA?3?$AA?5?$AA?5?$AA?5?$AAA?$AAc?$AAc?$AAe?$AAs@ 0000000180036a00     AccessBridgeJavaEntryPoints.obj
 0002:0000ba80       ??_C@_0BM@KMPFPDHC@Getting?5AccessibleTextRange@ 0000000180036a80     AccessBridgeJavaEntryPoints.obj
 0002:0000baa0       ??_C@_0DH@LGIBLGLE@Getting?5AccessibleTextRange?5?9?5c@ 0000000180036aa0     AccessBridgeJavaEntryPoints.obj
 0002:0000bae0       ??_C@_1EM@MAOOPBBK@?$AA?$FL?$AAI?$AAN?$AAF?$AAO?$AA?$FN?$AA?3?$AA?5?$AA?5?$AA?5?$AAA?$AAc?$AAc?$AAe?$AAs@ 0000000180036ae0     AccessBridgeJavaEntryPoints.obj
 0002:0000bb30       ??_C@_0DH@FFKMGAG@Getting?5AccessibleTextRange?5?9?5c@ 0000000180036b30     AccessBridgeJavaEntryPoints.obj
 0002:0000bb68       ??_C@_0DB@ENPGLEMN@?$FLWARN?$FN?3?5?5?5current?5Accessible?5Te@ 0000000180036b68     AccessBridgeJavaEntryPoints.obj
 0002:0000bba0       ??_C@_0EJ@IGDKNKCL@?$FLERROR?$FN?3?5either?5env?5?$DN?$DN?50?5or?5get@ 0000000180036ba0     AccessBridgeJavaEntryPoints.obj
 0002:0000bbf0       ??_C@_0FH@DFGPJEBI@?$FLINFO?$FN?3?5Calling?5AccessBridgeJav@ 0000000180036bf0     AccessBridgeJavaEntryPoints.obj
 0002:0000bc48       ??_C@_0DM@FMEJNEAF@Getting?5CurrentAccessibleValue?5@ 0000000180036c48     AccessBridgeJavaEntryPoints.obj
 0002:0000bc88       ??_C@_0DK@DEBJEKPP@Getting?5CurrentAccessibleValue?5@ 0000000180036c88     AccessBridgeJavaEntryPoints.obj
 0002:0000bcc8       ??_C@_0BP@PMLFPGML@Getting?5CurrentAccessibleValue@ 0000000180036cc8     AccessBridgeJavaEntryPoints.obj
 0002:0000bce8       ??_C@_0DK@EJDHPIND@Getting?5CurrentAccessibleValue?5@ 0000000180036ce8     AccessBridgeJavaEntryPoints.obj
 0002:0000bd28       ??_C@_0CI@LHBKPIPL@?$FLINFO?$FN?3?5?5?5current?5Accessible?5Va@ 0000000180036d28     AccessBridgeJavaEntryPoints.obj
 0002:0000bd50       ??_C@_0DK@PKOMIIGB@Getting?5CurrentAccessibleValue?5@ 0000000180036d50     AccessBridgeJavaEntryPoints.obj
 0002:0000bd90       ??_C@_0CM@JBCHBMHL@?$FLWARN?$FN?3?5?5?5current?5Accessible?5Va@ 0000000180036d90     AccessBridgeJavaEntryPoints.obj
 0002:0000bdc0       ??_C@_0EN@CEFCJCHP@?$FLERROR?$FN?3?5?5either?5env?5?$DN?$DN?50?5or?5ge@ 0000000180036dc0     AccessBridgeJavaEntryPoints.obj
 0002:0000be10       ??_C@_0FH@LDANAJBK@?$FLINFO?$FN?3?5Calling?5AccessBridgeJav@ 0000000180036e10     AccessBridgeJavaEntryPoints.obj
 0002:0000be68       ??_C@_0DM@CNMGLEAD@Getting?5MaximumAccessibleValue?5@ 0000000180036e68     AccessBridgeJavaEntryPoints.obj
 0002:0000bea8       ??_C@_0DK@LPOBNFBI@Getting?5MaximumAccessibleValue?5@ 0000000180036ea8     AccessBridgeJavaEntryPoints.obj
 0002:0000bee8       ??_C@_0BP@FLCAAJND@Getting?5MaximumAccessibleValue@ 0000000180036ee8     AccessBridgeJavaEntryPoints.obj
 0002:0000bf08       ??_C@_0DK@MCMPGHDE@Getting?5MaximumAccessibleValue?5@ 0000000180036f08     AccessBridgeJavaEntryPoints.obj
 0002:0000bf48       ??_C@_0CI@MOLFAIEC@?$FLINFO?$FN?3?5?5?5maximum?5Accessible?5Va@ 0000000180036f48     AccessBridgeJavaEntryPoints.obj
 0002:0000bf70       ??_C@_0DK@HBBEBHIG@Getting?5MaximumAccessibleValue?5@ 0000000180036f70     AccessBridgeJavaEntryPoints.obj
 0002:0000bfb0       ??_C@_0CM@EENPAHAF@?$FLWARN?$FN?3?5?5?5maximum?5Accessible?5Va@ 0000000180036fb0     AccessBridgeJavaEntryPoints.obj
 0002:0000bfe0       ??_C@_0EM@DECMFMLP@?$FLERROR?$FN?3?5either?5env?5?$DN?$DN?50?5or?5get@ 0000000180036fe0     AccessBridgeJavaEntryPoints.obj
 0002:0000c030       ??_C@_0FH@NCJCNBPB@?$FLINFO?$FN?3?5Calling?5AccessBridgeJav@ 0000000180037030     AccessBridgeJavaEntryPoints.obj
 0002:0000c088       ??_C@_0DM@EKOMNNCH@Getting?5MinimumAccessibleValue?5@ 0000000180037088     AccessBridgeJavaEntryPoints.obj
 0002:0000c0c8       ??_C@_0DK@POFOBDIM@Getting?5MinimumAccessibleValue?5@ 00000001800370c8     AccessBridgeJavaEntryPoints.obj
 0002:0000c108       ??_C@_0BP@FPLKDIPJ@Getting?5MinimumAccessibleValue@ 0000000180037108     AccessBridgeJavaEntryPoints.obj
 0002:0000c128       ??_C@_0DK@IDHAKBKA@Getting?5MinimumAccessibleValue?5@ 0000000180037128     AccessBridgeJavaEntryPoints.obj
 0002:0000c168       ??_C@_0CI@HMFEBFFJ@?$FLINFO?$FN?3?5?5?5mimimum?5Accessible?5Va@ 0000000180037168     AccessBridgeJavaEntryPoints.obj
 0002:0000c190       ??_C@_0DK@DAKLNBBC@Getting?5MinimumAccessibleValue?5@ 0000000180037190     AccessBridgeJavaEntryPoints.obj
 0002:0000c1d0       ??_C@_0CM@LFDDPHLF@?$FLWARN?$FN?3?5?5?5mimimum?5Accessible?5Va@ 00000001800371d0     AccessBridgeJavaEntryPoints.obj
 0002:0000c200       ??_C@_0EM@FNBMNDID@?$FLERROR?$FN?3?5either?5env?5?$DN?$DN?50?5or?5get@ 0000000180037200     AccessBridgeJavaEntryPoints.obj
 0002:0000c250       ??_C@_0FE@GLAEHJLA@?$FLINFO?$FN?3?5Calling?5AccessBridgeJav@ 0000000180037250     AccessBridgeJavaEntryPoints.obj
 0002:0000c2a8       ??_C@_0DI@HFNIIMHH@Doing?5addAccessibleSelection?5?9?5@ 00000001800372a8     AccessBridgeJavaEntryPoints.obj
 0002:0000c2e0       ??_C@_0CP@EBNEHGHB@?$FLERROR?$FN?3?5?$CK?$CK?$CK?5Exception?5occured?5@ 00000001800372e0     AccessBridgeJavaEntryPoints.obj
 0002:0000c310       ??_C@_0CL@OKIJNCBD@?$FLINFO?$FN?3?5?5?5returned?5from?5CallObj@ 0000000180037310     AccessBridgeJavaEntryPoints.obj
 0002:0000c340       ??_C@_0EK@CMGGDKGL@?$FLERROR?$FN?3?5?5either?5env?5?$DN?$DN?50?5or?5ad@ 0000000180037340     AccessBridgeJavaEntryPoints.obj
 0002:0000c390       ??_C@_0FG@JICCBONC@?$FLINFO?$FN?3?5Calling?5AccessBridgeJav@ 0000000180037390     AccessBridgeJavaEntryPoints.obj
 0002:0000c3e8       ??_C@_0DK@GPKPKKON@Doing?5clearAccessibleSelection?5@ 00000001800373e8     AccessBridgeJavaEntryPoints.obj
 0002:0000c430       ??_C@_0EM@NKPDGGGN@?$FLERROR?$FN?3?5?5either?5env?5?$DN?$DN?50?5or?5cl@ 0000000180037430     AccessBridgeJavaEntryPoints.obj
 0002:0000c480       ??_C@_0FE@PIPHOHFI@?$FLINFO?$FN?3?5Calling?5AccessBridgeJav@ 0000000180037480     AccessBridgeJavaEntryPoints.obj
 0002:0000c4e0       ??_C@_0EA@EDHDCMHP@Getting?5AccessibleSelectionCont@ 00000001800374e0     AccessBridgeJavaEntryPoints.obj
 0002:0000c520       ??_C@_0DM@IFLFNJN@Getting?5AccessibleSelectionCont@ 0000000180037520     AccessBridgeJavaEntryPoints.obj
 0002:0000c560       ??_C@_0DO@FEBBEFGL@Getting?5AccessibleSelectionCont@ 0000000180037560     AccessBridgeJavaEntryPoints.obj
 0002:0000c5a0       ??_C@_0FA@KGJFECGD@?$FLERROR?$FN?3?5either?5env?5?$DN?$DN?50?5or?5get@ 00000001800375a0     AccessBridgeJavaEntryPoints.obj
 0002:0000c5f0       ??_C@_0FJ@KDCCHMFP@?$FLINFO?$FN?3?5Calling?5AccessBridgeJav@ 00000001800375f0     AccessBridgeJavaEntryPoints.obj
 0002:0000c650       ??_C@_0DL@JPLKCOEB@Getting?5AccessibleSelectionCoun@ 0000000180037650     AccessBridgeJavaEntryPoints.obj
 0002:0000c690       ??_C@_0EO@LLPLNNDE@?$FLERROR?$FN?3?5either?5env?5?$DN?$DN?50?5or?5get@ 0000000180037690     AccessBridgeJavaEntryPoints.obj
 0002:0000c6e0       ??_C@_0FH@BEGAHKNM@?$FLINFO?$FN?3?5Calling?5AccessBridgeJav@ 00000001800376e0     AccessBridgeJavaEntryPoints.obj
 0002:0000c738       ??_C@_0DO@DGOGEINB@Doing?5isAccessibleChildSelected@ 0000000180037738     AccessBridgeJavaEntryPoints.obj
 0002:0000c780       ??_C@_0EM@FIJEFPDC@?$FLERROR?$FN?3?5either?5env?5?$DN?$DN?50?5or?5isA@ 0000000180037780     AccessBridgeJavaEntryPoints.obj
 0002:0000c7d0       ??_C@_0FH@DBFJFKMJ@?$FLINFO?$FN?3?5Calling?5AccessBridgeJav@ 00000001800377d0     AccessBridgeJavaEntryPoints.obj
 0002:0000c828       ??_C@_0DL@BHDCMLKI@Doing?5removeAccessibleSelection@ 0000000180037828     AccessBridgeJavaEntryPoints.obj
 0002:0000c870       ??_C@_0EN@HJFMAEOO@?$FLERROR?$FN?3?5?5either?5env?5?$DN?$DN?50?5or?5re@ 0000000180037870     AccessBridgeJavaEntryPoints.obj
 0002:0000c8c0       ??_C@_0FK@MANGNIPE@?$FLINFO?$FN?3?5Calling?5AccessBridgeJav@ 00000001800378c0     AccessBridgeJavaEntryPoints.obj
 0002:0000c920       ??_C@_0DO@JHGLNKHC@Doing?5selectAllAccessibleSelect@ 0000000180037920     AccessBridgeJavaEntryPoints.obj
 0002:0000c960       ??_C@_0EP@JCKDPHMN@?$FLERROR?$FN?3?5either?5env?5?$DN?$DN?50?5or?5sel@ 0000000180037960     AccessBridgeJavaEntryPoints.obj
 0002:0000c9b0       ??_C@_0EO@IEPNANKM@?$FLINFO?$FN?3?5?5?5in?5AccessBridgeJavaEn@ 00000001800379b0     AccessBridgeJavaEntryPoints.obj
 0002:0000ca00       ??_C@_0DK@GPMPKEMH@Doing?5addJavaEventNotification?5@ 0000000180037a00     AccessBridgeJavaEntryPoints.obj
 0002:0000ca40       ??_C@_0EA@IOOHIHIM@?$FLERROR?$FN?3?5either?5env?5?$DN?$DN?50?5or?5add@ 0000000180037a40     AccessBridgeJavaEntryPoints.obj
 0002:0000ca80       ??_C@_0FA@BBNLJKAK@?$FLINFO?$FN?3?5?5in?5AccessBridgeJavaEnt@ 0000000180037a80     AccessBridgeJavaEntryPoints.obj
 0002:0000cad0       ??_C@_0DN@IBNHMLMO@Doing?5removeJavaEventNotificati@ 0000000180037ad0     AccessBridgeJavaEntryPoints.obj
 0002:0000cb10       ??_C@_0ED@LKLPMFCD@?$FLERROR?$FN?3?5either?5env?5?$DN?$DN?50?5or?5rem@ 0000000180037b10     AccessBridgeJavaEntryPoints.obj
 0002:0000cb60       ??_C@_0FH@ICFBIMPG@?$FLINFO?$FN?3?5?5?5in?5AccessBridgeJavaEn@ 0000000180037b60     AccessBridgeJavaEntryPoints.obj
 0002:0000cbc0       ??_C@_0FL@OCFIPKDP@?$FLINFO?$FN?3?5?5?5?5addAccessibilityEven@ 0000000180037bc0     AccessBridgeJavaEntryPoints.obj
 0002:0000cc20       ??_C@_0DH@DNDEHAJF@Doing?5addAccessibilityEvent?5?9?5c@ 0000000180037c20     AccessBridgeJavaEntryPoints.obj
 0002:0000cc60       ??_C@_0EJ@BAMHEIMC@?$FLERROR?$FN?3?5either?5env?5?$DN?$DN?50?5or?5add@ 0000000180037c60     AccessBridgeJavaEntryPoints.obj
 0002:0000ccb0       ??_C@_0ED@BCNEMPCF@?$FLINFO?$FN?3?5?5?5?5?5addAccessibilityEve@ 0000000180037cb0     AccessBridgeJavaEntryPoints.obj
 0002:0000cd00       ??_C@_0FJ@JPJKPKP@?$FLINFO?$FN?3?5?5in?5AccessBridgeJavaEnt@ 0000000180037d00     AccessBridgeJavaEntryPoints.obj
 0002:0000cd60       ??_C@_0DK@KGOHAMJ@Doing?5removeAccessibilityEvent?5@ 0000000180037d60     AccessBridgeJavaEntryPoints.obj
 0002:0000cda0       ??_C@_0EM@MPLDCCAE@?$FLERROR?$FN?3?5either?5env?5?$DN?$DN?50?5or?5rem@ 0000000180037da0     AccessBridgeJavaEntryPoints.obj
 0002:0000cdf0       ??_C@_0BM@BIAOFPJG@AccessBridge?9FromJava?9Hello@ 0000000180037df0     AccessBridgeMessages.obj
 0002:0000ce10       ??_C@_0BP@OELHMMDF@AccessBridge?9FromWindows?9Hello@ 0000000180037e10     AccessBridgeMessages.obj
 0002:0000ce30       ??_C@_0CN@HNEPECB@?$FLINFO?$FN?3?5JavaAccessBridge?4DLL?5ru@ 0000000180037e30     JavaAccessBridge.obj
 0002:0000ce60       ??_C@_0CN@OBDABACD@?$FLINFO?$FN?3?5In?5AccessBridgeDialog?5?9@ 0000000180037e60     JavaAccessBridge.obj
 0002:0000ce90       ??_C@_0DM@LEGKGBDC@?$FLINFO?$FN?3?5In?5AccessBridgeDialog?5?9@ 0000000180037e90     JavaAccessBridge.obj
 0002:0000ced0       ??_C@_0DP@KFGJNONL@?$FLINFO?$FN?3?5In?5AccessBridgeDialog?5?9@ 0000000180037ed0     JavaAccessBridge.obj
 0002:0000cf10       ??_C@_0DN@BOPHDCMF@?$FLINFO?$FN?3?5In?5AccessBridgeDialog?5?9@ 0000000180037f10     JavaAccessBridge.obj
 0002:0000cf50       ??_C@_0EG@LODLDNEL@?$FLINFO?$FN?3?5In?5AccessBridgeDialog?5?9@ 0000000180037f50     JavaAccessBridge.obj
 0002:0000cfa0       ??_C@_0EE@OLIPFHDH@?$FLINFO?$FN?3?5In?5AccessBridgeDialog?5?9@ 0000000180037fa0     JavaAccessBridge.obj
 0002:0000cfe8       ??_C@_0DO@KFBCLDPM@?$FLINFO?$FN?3?5In?5AccessBridgeDialog?5?9@ 0000000180037fe8     JavaAccessBridge.obj
 0002:0000d030       ??_C@_0EF@PPOLOLIM@?$FLINFO?$FN?3?5In?5AccessBridgeDialog?5?9@ 0000000180038030     JavaAccessBridge.obj
 0002:0000d078       ??_C@_0BD@BOAKDBCO@java_access_bridge@ 0000000180038078     JavaAccessBridge.obj
 0002:0000d090       ??_C@_0DB@JHKNDMME@?$FLINFO?$FN?3?5in?5JavaAccessBridge?3?3?$HOJ@ 0000000180038090     JavaAccessBridge.obj
 0002:0000d0c8       ??_C@_0CF@DJNKIAAH@?$FLINFO?$FN?3?5?5telling?5?$CFp?5we?8re?5going@ 00000001800380c8     JavaAccessBridge.obj
 0002:0000d0f0       ??_C@_0CP@BKDEGDJC@?$FLINFO?$FN?3?5?5finished?5telling?5ATs?5a@ 00000001800380f0     JavaAccessBridge.obj
 0002:0000d120       ??_C@_0CA@EIEOEDOI@?$FLINFO?$FN?3?5?5?5finished?5deleting?5ATs@ 0000000180038120     JavaAccessBridge.obj
 0002:0000d140       ??_C@_0BP@EBFMIPOK@?$FLINFO?$FN?3?5GOODBYE?5CRUEL?5WORLD?4?4?4@ 0000000180038140     JavaAccessBridge.obj
 0002:0000d160       ??_C@_0DB@BKKBMMIL@?$FLINFO?$FN?3?5JavaAccessBridge?3?3javaR@ 0000000180038160     JavaAccessBridge.obj
 0002:0000d198       ??_C@_0BJ@CDAHIMFI@?$FLINFO?$FN?3?5?5?5?9?$DO?5javaVM?5?$DN?5?$CFp@ 0000000180038198     JavaAccessBridge.obj
 0002:0000d1b8       ??_C@_0CF@HBJLLMBP@?$FLINFO?$FN?3?5?5?9?$DO?5windowsThreadJNIEnv@ 00000001800381b8     JavaAccessBridge.obj
 0002:0000d1e0       ??_C@_0DL@EDCIECNK@?$FLINFO?$FN?3?5?5?5all?5Java?5thread?5entry@ 00000001800381e0     JavaAccessBridge.obj
 0002:0000d220       ??_C@_0DO@DHHHOLPH@?$FLINFO?$FN?3?5?5?5all?5Windows?5thread?5en@ 0000000180038220     JavaAccessBridge.obj
 0002:0000d260       ??_C@_0CF@FINMKFHO@?$FLINFO?$FN?3?5?5?5Window?5created?4?5?5HWND@ 0000000180038260     JavaAccessBridge.obj
 0002:0000d288       ??_C@_0CG@KCHIBPOJ@?$FLERROR?$FN?3?5?5?5FAILED?5TO?5CREATE?5WIN@ 0000000180038288     JavaAccessBridge.obj
 0002:0000d2b0       ??_C@_0BJ@LMONFDOG@ACCESSBRIDGESTATUSWINDOW@ 00000001800382b0     JavaAccessBridge.obj
 0002:0000d2d0       ??_C@_0DG@HAJICJFK@?$FLINFO?$FN?3?5In?5JavaAccessBridge?3?3po@ 00000001800382d0     JavaAccessBridge.obj
 0002:0000d308       ??_C@_0CO@FLLNHCIG@?$FLINFO?$FN?3?5?5?5calling?5PostMessage?$CI?$CF@ 0000000180038308     JavaAccessBridge.obj
 0002:0000d338       ??_C@_0CM@DCNJAPPO@?$FLERROR?$FN?3?5ATs?5?$DN?$DN?50?$CB?5?$CIshouldn?8t?5h@ 0000000180038338     JavaAccessBridge.obj
 0002:0000d368       ??_C@_0DH@JMPJBGDF@?$FLINFO?$FN?3?5JavaAccessBridge?3?3recei@ 0000000180038368     JavaAccessBridge.obj
 0002:0000d3a0       ??_C@_0EB@GECAJJE@?$FLERROR?$FN?3?5?9?5ATs?5?$DN?$DN?50?5?$CIshouldn?8t?5@ 00000001800383a0     JavaAccessBridge.obj
 0002:0000d3e8       ??_C@_0DL@FAPEODKG@?$FLERROR?$FN?3?5receiving?5memory?5packa@ 00000001800383e8     JavaAccessBridge.obj
 0002:0000d428       ??_C@_0DM@MJCPMIJG@?$FLINFO?$FN?3?5Processing?5package?5sent@ 0000000180038428     JavaAccessBridge.obj
 0002:0000d468       ??_C@_0BL@EFABEHOK@?$FLINFO?$FN?3?5?5PackageType?5?$DN?5?$CFX?3@ 0000000180038468     JavaAccessBridge.obj
 0002:0000d488       ??_C@_0DC@HOEDKHHL@?$FLINFO?$FN?3?5?5?5type?5?$DN?$DN?5cMemoryMapped@ 0000000180038488     JavaAccessBridge.obj
 0002:0000d4c0       ??_C@_0EC@JELBKKLB@?$FLERROR?$FN?3?5?5?5?5processing?5FAILED?$CB?$CB@ 00000001800384c0     JavaAccessBridge.obj
 0002:0000d508       ??_C@_0CM@EGHIFACB@?$FLINFO?$FN?3?5?5?5type?5?$DN?$DN?5cReleaseJavaO@ 0000000180038508     JavaAccessBridge.obj
 0002:0000d540       ??_C@_0EB@PCOLNIOI@?$FLERROR?$FN?3?5?5?5processing?5FAILED?$CB?$CB?5@ 0000000180038540     JavaAccessBridge.obj
 0002:0000d588       ??_C@_0DB@HJBBLNK@?$FLINFO?$FN?3?5?5?5type?5?$DN?$DN?5cGetAccessBri@ 0000000180038588     JavaAccessBridge.obj
 0002:0000d5c0       ??_C@_0CH@OGPNINNH@?$FLINFO?$FN?3?5?5?5type?5?$DN?$DN?5cIsJavaWindow@ 00000001800385c0     JavaAccessBridge.obj
 0002:0000d5e8       ??_C@_0CF@KCGBFLNL@?$FLINFO?$FN?3?5?5?5?5?5?9?$DO?5returning?5result@ 00000001800385e8     JavaAccessBridge.obj
 0002:0000d610       ??_C@_0CH@FFMGBMGP@?$FLINFO?$FN?3?5?5?5type?5?$DN?$DN?5cIsSameObject@ 0000000180038610     JavaAccessBridge.obj
 0002:0000d638       ??_C@_0DI@FGDPIMOI@?$FLINFO?$FN?3?5?5?5?5type?5?$DN?$DN?5cGetAccessib@ 0000000180038638     JavaAccessBridge.obj
 0002:0000d670       ??_C@_0CN@KFALDIEC@?$FLINFO?$FN?3?5?5?5?5?5?5?9?$DO?5returning?5AC?5?$DN?5@ 0000000180038670     JavaAccessBridge.obj
 0002:0000d6a0       ??_C@_0DI@ICOCNDDM@?$FLINFO?$FN?3?5?5?5?5type?5?$DN?$DN?5cGetHWNDFrom@ 00000001800386a0     JavaAccessBridge.obj
 0002:0000d6d8       ??_C@_0CD@DNCFKFDK@?$FLINFO?$FN?3?5?5?5?5?5?9?$DO?5returning?5HWND?5?$DN@ 00000001800386d8     JavaAccessBridge.obj
 0002:0000d700       ??_C@_0CK@DBBKGOKJ@?$FLINFO?$FN?3?5?5?5type?5?$DN?$DN?5cSetTextConte@ 0000000180038700     JavaAccessBridge.obj
 0002:0000d730       ??_C@_0JK@BDICEONN@?$FLINFO?$FN?3?5?5?5type?5?$DN?$DN?5cGetParentWit@ 0000000180038730     JavaAccessBridge.obj
 0002:0000d7d0       ??_C@_0CM@FMGIHPCP@?$FLINFO?$FN?3?5?5?5type?5?$DN?$DN?5cGetTopLevelO@ 00000001800387d0     JavaAccessBridge.obj
 0002:0000d800       ??_C@_0DC@EMOAFCHE@?$FLINFO?$FN?3?5?5?5?5?5?5?9?$DO?5returning?5rAcce@ 0000000180038800     JavaAccessBridge.obj
 0002:0000d838       ??_C@_0DE@EHPIAHAD@?$FLINFO?$FN?3?5?5?5type?5?$DN?$DN?5cGetParentWit@ 0000000180038838     JavaAccessBridge.obj
 0002:0000d870       ??_C@_0CJ@CIIOKEJA@?$FLINFO?$FN?3?5?5?5type?5?$DN?$DN?5cGetObjectDep@ 0000000180038870     JavaAccessBridge.obj
 0002:0000d8a0       ??_C@_0CG@CCMHCDED@?$FLINFO?$FN?3?5?5?5?5?5?9?$DO?5returning?5rResul@ 00000001800388a0     JavaAccessBridge.obj
 0002:0000d8c8       ??_C@_0CO@HPDBNII@?$FLINFO?$FN?3?5?5?5type?5?$DN?$DN?5cGetActiveDes@ 00000001800388c8     JavaAccessBridge.obj
 0002:0000d8f8       ??_C@_0CO@EEGIDCBJ@?$FLINFO?$FN?3?5?5?9?$DO?5returning?5rAccessib@ 00000001800388f8     JavaAccessBridge.obj
 0002:0000d928       ??_C@_0DB@BLNOEMHA@?$FLINFO?$FN?3?5?5?5type?5?$DN?$DN?5cGetAccessibl@ 0000000180038928     JavaAccessBridge.obj
 0002:0000d960       ??_C@_0DI@BBJPLAPN@?$FLINFO?$FN?3?5?5?5type?5?$DN?$DN?5cGetAccessibl@ 0000000180038960     JavaAccessBridge.obj
 0002:0000d998       ??_C@_0DD@EKFFDOAF@?$FLINFO?$FN?3?5?5?5type?5?$DN?$DN?5cGetAccessibl@ 0000000180038998     JavaAccessBridge.obj
 0002:0000d9d0       ??_C@_0DI@HCCMIAAH@?$FLINFO?$FN?3?5?5?5type?5?$DN?$DN?5cGetAccessibl@ 00000001800389d0     JavaAccessBridge.obj
 0002:0000da08       ??_C@_0DK@EHNJMPFO@?$FLINFO?$FN?3?5?5?5?5type?5?$DN?$DN?5cGetAccessib@ 0000000180038a08     JavaAccessBridge.obj
 0002:0000da48       ??_C@_0DI@DNENMOMG@?$FLINFO?$FN?3?5?5?5?5?$CD?$CD?$CD?$CD?$CD?5type?5?$DN?$DN?5cGetAc@ 0000000180038a48     JavaAccessBridge.obj
 0002:0000da80       ??_C@_0CG@KFAMLONA@?$FLINFO?$FN?3?5?5?5?5?$CD?$CD?$CD?$CD?$CD?5processing?5suc@ 0000000180038a80     JavaAccessBridge.obj
 0002:0000dab0       ??_C@_0EI@KKCFGLCL@?$FLERROR?$FN?3?5?5?5?5?$CD?$CD?$CD?$CD?$CD?5processing?5FA@ 0000000180038ab0     JavaAccessBridge.obj
 0002:0000daf8       ??_C@_0DM@ONBKHFBE@?$FLINFO?$FN?3?5?5?5?5?$CD?$CD?$CD?$CD?$CD?5type?5?$DN?$DN?5cGetAc@ 0000000180038af8     JavaAccessBridge.obj
 0002:0000db38       ??_C@_0DN@MOEKMKGM@?$FLINFO?$FN?3?5?5?5?5?$CD?$CD?$CD?$CD?$CD?5type?5?$DN?$DN?5cGetAc@ 0000000180038b38     JavaAccessBridge.obj
 0002:0000db80       ??_C@_0EA@CAKJDHMA@?$FLINFO?$FN?3?5?5?5?5?$CD?$CD?$CD?$CD?$CD?5type?5?$DN?$DN?5cGetAc@ 0000000180038b80     JavaAccessBridge.obj
 0002:0000dbc0       ??_C@_0EC@JLIHGBEM@?$FLINFO?$FN?3?5?5?5?5?$CD?$CD?$CD?$CD?$CD?5type?5?$DN?$DN?5cGetAc@ 0000000180038bc0     JavaAccessBridge.obj
 0002:0000dc10       ??_C@_0EF@DBAFGNDK@?$FLINFO?$FN?3?5?5?5?5?$CD?$CD?$CD?$CD?$CD?5type?5?$DN?$DN?5cGetAc@ 0000000180038c10     JavaAccessBridge.obj
 0002:0000dc60       ??_C@_0EI@BCPJNOBP@?$FLINFO?$FN?3?5?5?5?5?$CD?$CD?$CD?$CD?$CD?5type?5?$DN?$DN?5cGetAc@ 0000000180038c60     JavaAccessBridge.obj
 0002:0000dcb0       ??_C@_0EF@ONIGGHFH@?$FLINFO?$FN?3?5?5?5?5?$CD?$CD?$CD?$CD?$CD?5type?5?$DN?$DN?5cGetAc@ 0000000180038cb0     JavaAccessBridge.obj
 0002:0000dcf8       ??_C@_0DO@ENBHEGBB@?$FLINFO?$FN?3?5?5?5?5?$CD?$CD?$CD?$CD?$CD?5type?5?$DN?$DN?5cIsAcc@ 0000000180038cf8     JavaAccessBridge.obj
 0002:0000dd40       ??_C@_0EB@PMALJKOF@?$FLINFO?$FN?3?5?5?5?5?$CD?$CD?$CD?$CD?$CD?5type?5?$DN?$DN?5cIsAcc@ 0000000180038d40     JavaAccessBridge.obj
 0002:0000dd90       ??_C@_0EE@NFLEEFCE@?$FLINFO?$FN?3?5?5?5?5?$CD?$CD?$CD?$CD?$CD?5type?5?$DN?$DN?5cGetAc@ 0000000180038d90     JavaAccessBridge.obj
 0002:0000dde0       ??_C@_0EH@DNDNECPC@?$FLINFO?$FN?3?5?5?5?5?5?5?$CD?$CD?$CD?$CD?$CD?5cGetAccessib@ 0000000180038de0     JavaAccessBridge.obj
 0002:0000de30       ??_C@_0EF@PFDKDHMH@?$FLINFO?$FN?3?5?5?5?5?5?5?$CD?$CD?$CD?$CD?$CD?5cGetAccessib@ 0000000180038e30     JavaAccessBridge.obj
 0002:0000de80       ??_C@_0EB@FNPEGMEK@?$FLINFO?$FN?3?5?5?5?5?$CD?$CD?$CD?$CD?$CD?5type?5?$DN?$DN?5cGetAc@ 0000000180038e80     JavaAccessBridge.obj
 0002:0000dec8       ??_C@_0DH@HGKABJI@?$FLINFO?$FN?3?5?5?5?5?$CD?$CD?$CD?$CD?$CD?5type?5?$DN?$DN?5cGetAc@ 0000000180038ec8     JavaAccessBridge.obj
 0002:0000df00       ??_C@_0DK@PHHNIBJB@?$FLINFO?$FN?3?5?5?5?5?$CD?$CD?$CD?$CD?$CD?5type?5?$DN?$DN?5cGetAc@ 0000000180038f00     JavaAccessBridge.obj
 0002:0000df40       ??_C@_0DJ@ECCDOPKO@?$FLINFO?$FN?3?5?5?5?5?$CD?$CD?$CD?$CD?$CD?5type?5?$DN?$DN?5cGetAc@ 0000000180038f40     JavaAccessBridge.obj
 0002:0000df80       ??_C@_0DK@GDIGFCLP@?$FLINFO?$FN?3?5?5?5?5?$CD?$CD?$CD?$CD?$CD?5type?5?$DN?$DN?5cGetAc@ 0000000180038f80     JavaAccessBridge.obj
 0002:0000dfc0       ??_C@_0DI@BPKDDCHO@?$FLINFO?$FN?3?5?5?5?5?$CD?$CD?$CD?$CD?$CD?5type?5?$DN?$DN?5cGetAc@ 0000000180038fc0     JavaAccessBridge.obj
 0002:0000dff8       ??_C@_0DN@OAAMPEIM@?$FLINFO?$FN?3?5?5?5?5?$CD?$CD?$CD?$CD?$CD?5type?5?$DN?$DN?5cActiv@ 0000000180038ff8     JavaAccessBridge.obj
 0002:0000e038       ??_C@_0DN@GBPFAJCJ@?$FLINFO?$FN?3?5?5?5?5?$CD?$CD?$CD?$CD?$CD?5type?5?$DN?$DN?5cGetAc@ 0000000180039038     JavaAccessBridge.obj
 0002:0000e078       ??_C@_0DM@HFKCAKHD@?$FLINFO?$FN?3?5?5?5?5?$CD?$CD?$CD?$CD?$CD?5processing?5suc@ 0000000180039078     JavaAccessBridge.obj
 0002:0000e0b8       ??_C@_0DL@BKPFGPAI@?$FLINFO?$FN?3?5?5?5?5?$CD?$CD?$CD?$CD?$CD?5type?5?$DN?$DN?5cGetAc@ 00000001800390b8     JavaAccessBridge.obj
 0002:0000e100       ??_C@_0EB@HBBMKHLL@?$FLINFO?$FN?3?5?5?5?5?$CD?$CD?$CD?$CD?$CD?5type?5?$DN?$DN?5cGetAc@ 0000000180039100     JavaAccessBridge.obj
 0002:0000e148       ??_C@_0DI@EGGEEHLE@?$FLINFO?$FN?3?5?5?5?5?$CD?$CD?$CD?$CD?$CD?5type?5?$DN?$DN?5cGetAc@ 0000000180039148     JavaAccessBridge.obj
 0002:0000e180       ??_C@_0DK@LOBFOEFG@?$FLINFO?$FN?3?5?5?5?5?$CD?$CD?$CD?$CD?$CD?5type?5?$DN?$DN?5cGetAc@ 0000000180039180     JavaAccessBridge.obj
 0002:0000e1c0       ??_C@_0DE@NCPKKLJG@?$FLINFO?$FN?3?5?5?5?5?$CD?$CD?$CD?$CD?$CD?5type?5?$DN?$DN?5cGetAc@ 00000001800391c0     JavaAccessBridge.obj
 0002:0000e200       ??_C@_0EH@OKFMNJOP@?$FLERROR?$FN?3?5?5?5?$CD?$CD?$CD?$CD?$CD?5processing?5FAI@ 0000000180039200     JavaAccessBridge.obj
 0002:0000e248       ??_C@_0DG@CDFKKFMN@?$FLINFO?$FN?3?5?5?5?5?$CD?$CD?$CD?$CD?$CD?5type?5?$DN?$DN?5cGetAc@ 0000000180039248     JavaAccessBridge.obj
 0002:0000e280       ??_C@_0DF@GOCDLFHO@?$FLINFO?$FN?3?5?5?5?5?$CD?$CD?$CD?$CD?$CD?5type?5?$DN?$DN?5cDoAcc@ 0000000180039280     JavaAccessBridge.obj
 0002:0000e2b8       ??_C@_0DJ@FOPNGHK@?$FLINFO?$FN?3?5?5?5?5?$CD?$CD?$CD?$CD?$CD?5type?5?$DN?$DN?5GetVir@ 00000001800392b8     JavaAccessBridge.obj
 0002:0000e2f8       ??_C@_0CN@KKAHFJLP@?$FLINFO?$FN?3?5?5?5?5?$CD?$CD?$CD?$CD?$CD?5type?5?$DN?$DN?5Reques@ 00000001800392f8     JavaAccessBridge.obj
 0002:0000e328       ??_C@_0DA@BDJNNLOI@?$FLINFO?$FN?3?5?5?5?5?$CD?$CD?$CD?$CD?$CD?5type?5?$DN?$DN?5Select@ 0000000180039328     JavaAccessBridge.obj
 0002:0000e358       ??_C@_0DJ@JNPDLANK@?$FLINFO?$FN?3?5?5?5?5?$CD?$CD?$CD?$CD?$CD?5type?5?$DN?$DN?5GetTex@ 0000000180039358     JavaAccessBridge.obj
 0002:0000e398       ??_C@_0DI@KCHGBBIN@?$FLINFO?$FN?3?5?5?5?5?$CD?$CD?$CD?$CD?$CD?5type?5?$DN?$DN?5GetVis@ 0000000180039398     JavaAccessBridge.obj
 0002:0000e3d0       ??_C@_0DD@HFEKHIPA@?$FLINFO?$FN?3?5?5?5?5?$CD?$CD?$CD?$CD?$CD?5type?5?$DN?$DN?5GetVis@ 00000001800393d0     JavaAccessBridge.obj
 0002:0000e408       ??_C@_0DB@HDPFDIKC@?$FLINFO?$FN?3?5?5?5?5?$CD?$CD?$CD?$CD?$CD?5type?5?$DN?$DN?5SetCar@ 0000000180039408     JavaAccessBridge.obj
 0002:0000e440       ??_C@_0DB@MBKJOFKA@?$FLINFO?$FN?3?5?5?5?5type?5?$DN?$DN?5cGetAccessib@ 0000000180039440     JavaAccessBridge.obj
 0002:0000e478       ??_C@_0DC@FACNMLJM@?$FLINFO?$FN?3?5?5?5?5type?5?$DN?$DN?5cGetAccessib@ 0000000180039478     JavaAccessBridge.obj
 0002:0000e4b0       ??_C@_0DK@BMAJHBGM@?$FLINFO?$FN?3?5?5?5?5type?5?$DN?$DN?5cGetAccessib@ 00000001800394b0     JavaAccessBridge.obj
 0002:0000e4f0       ??_C@_0DK@KLKIIEMH@?$FLINFO?$FN?3?5?5?5?5type?5?$DN?$DN?5cGetAccessib@ 00000001800394f0     JavaAccessBridge.obj
 0002:0000e530       ??_C@_0DF@LJIJJCFL@?$FLINFO?$FN?3?5?5?5?5type?5?$DN?$DN?5cGetAccessib@ 0000000180039530     JavaAccessBridge.obj
 0002:0000e568       ??_C@_0CM@DKHFKJOD@?$FLINFO?$FN?3?5?5?5?5type?5?$DN?$DN?5cGetCaretLoc@ 0000000180039568     JavaAccessBridge.obj
 0002:0000e598       ??_C@_0DH@CHPJDHJL@?$FLINFO?$FN?3?5?5?5?5type?5?$DN?$DN?5cGetAccessib@ 0000000180039598     JavaAccessBridge.obj
 0002:0000e5d0       ??_C@_0DC@HMIBGEHP@?$FLINFO?$FN?3?5?5?5?5type?5?$DN?$DN?5cGetAccessib@ 00000001800395d0     JavaAccessBridge.obj
 0002:0000e610       ??_C@_0EA@OJBBPFCG@?$FLINFO?$FN?3?5?5?5?5type?5?$DN?$DN?5cGetCurrentA@ 0000000180039610     JavaAccessBridge.obj
 0002:0000e650       ??_C@_0EA@FFJJPODP@?$FLINFO?$FN?3?5?5?5?5type?5?$DN?$DN?5cGetMaximumA@ 0000000180039650     JavaAccessBridge.obj
 0002:0000e690       ??_C@_0EA@GABLOPGB@?$FLINFO?$FN?3?5?5?5?5type?5?$DN?$DN?5cGetMinimumA@ 0000000180039690     JavaAccessBridge.obj
 0002:0000e6d0       ??_C@_0DN@NHMKNOBO@?$FLINFO?$FN?3?5?5?5?5type?5?$DN?$DN?5cAddAccessib@ 00000001800396d0     JavaAccessBridge.obj
 0002:0000e710       ??_C@_0DP@CDAIIOJL@?$FLINFO?$FN?3?5?5?5?5type?5?$DN?$DN?5cClearAccess@ 0000000180039710     JavaAccessBridge.obj
 0002:0000e750       ??_C@_0DN@FGNKIKEK@?$FLINFO?$FN?3?5?5?5?5type?5?$DN?$DN?5cGetAccessib@ 0000000180039750     JavaAccessBridge.obj
 0002:0000e790       ??_C@_0EC@JGIFJEAP@?$FLINFO?$FN?3?5?5?5?5type?5?$DN?$DN?5cGetAccessib@ 0000000180039790     JavaAccessBridge.obj
 0002:0000e7e0       ??_C@_0EA@BDFAJBM@?$FLINFO?$FN?3?5?5?5?5type?5?$DN?$DN?5cIsAccessibl@ 00000001800397e0     JavaAccessBridge.obj
 0002:0000e820       ??_C@_0EA@NOOOKPJ@?$FLINFO?$FN?3?5?5?5?5type?5?$DN?$DN?5cRemoveAcces@ 0000000180039820     JavaAccessBridge.obj
 0002:0000e860       ??_C@_0ED@CNEBOKEO@?$FLINFO?$FN?3?5?5?5?5type?5?$DN?$DN?5cSelectAllAc@ 0000000180039860     JavaAccessBridge.obj
 0002:0000e8a8       ??_C@_0DD@FDABBAIG@?$FLINFO?$FN?3?5?5?5?5type?5?$DN?5cAddJavaEvent@ 00000001800398a8     JavaAccessBridge.obj
 0002:0000e8e0       ??_C@_0DG@CJJGFHBD@?$FLINFO?$FN?3?5?5?5?5type?5?$DN?5cRemoveJavaEv@ 00000001800398e0     JavaAccessBridge.obj
 0002:0000e918       ??_C@_0DM@IHHPMOM@?$FLINFO?$FN?3?5?5?5?5type?5?$DN?5cAddAccessibi@ 0000000180039918     JavaAccessBridge.obj
 0002:0000e958       ??_C@_0DP@CLPLFGHM@?$FLINFO?$FN?3?5?5?5?5type?5?$DN?5cRemoveAccess@ 0000000180039958     JavaAccessBridge.obj
 0002:0000e9a0       ??_C@_0EG@DADDGPDA@?$FLERROR?$FN?3?5?5?5?5processing?5FAILED?$CB?$CB@ 00000001800399a0     JavaAccessBridge.obj
 0002:0000e9e8       ??_C@_0CI@PMGDCMNI@?$FLINFO?$FN?3?5?5?5?5package?5processing?5c@ 00000001800399e8     JavaAccessBridge.obj
 0002:0000ea10       ??_C@_0CO@NOIJCKLH@?$FLINFO?$FN?3?5?5?5in?5MemoryMappedFileCr@ 0000000180039a10     JavaAccessBridge.obj
 0002:0000ea40       ??_C@_0DJ@MGBOAEHL@?$FLINFO?$FN?3?5?5?5?5?5just?5created?5a?5new?5@ 0000000180039a40     JavaAccessBridge.obj
 0002:0000ea80       ??_C@_0DA@PCLBAGKL@?$FLINFO?$FN?3?5?5?5Successfully?5initiate@ 0000000180039a80     JavaAccessBridge.obj
 0002:0000eab0       ??_C@_0CL@IAFANAPB@?$FLERROR?$FN?3?5Failed?5to?5initiate?5IPC@ 0000000180039ab0     JavaAccessBridge.obj
 0002:0000eae0       ??_C@_0DE@FDNKAIDO@?$FLINFO?$FN?3?5in?5JavaAccessBridge?3?3Wi@ 0000000180039ae0     JavaAccessBridge.obj
 0002:0000eb18       ??_C@_0CO@DDCCLLBJ@?$FLERROR?$FN?3?5?9?$DO?5ATs?5?$DN?$DN?50?$CB?5?$CIshouldn?8@ 0000000180039b18     JavaAccessBridge.obj
 0002:0000eb48       ??_C@_0CP@IIHJFGGB@?$FLINFO?$FN?3?5?5?5data?5structures?5succe@ 0000000180039b48     JavaAccessBridge.obj
 0002:0000eb78       ??_C@_0DB@JABMCGEJ@?$FLERROR?$FN?3?5couldn?8t?5find?5matching@ 0000000180039b78     JavaAccessBridge.obj
 0002:0000ebb0       ??_C@_0CP@LEPCODGO@?$FLINFO?$FN?3?5In?5JavaAccessBridge?3?3re@ 0000000180039bb0     JavaAccessBridge.obj
 0002:0000ebe0       ??_C@_0BH@GNOIGMFE@?$FLINFO?$FN?3?5?5?5object?5X?3?5?$CFp@ 0000000180039be0     JavaAccessBridge.obj
 0002:0000ebf8       ??_C@_0CE@NAEKPPND@?$FLINFO?$FN?3?5?5?5global?5reference?5dele@ 0000000180039bf8     JavaAccessBridge.obj
 0002:0000ec20       ??_C@_0CC@DPMNCGAA@?$FLERROR?$FN?3?5windowsThreadJNIEnv?5?$DN?$DN@ 0000000180039c20     JavaAccessBridge.obj
 0002:0000ec48       ??_C@_0DF@HMNKBJGB@?$FLINFO?$FN?3?5?5?5adding?5Java?5event?5typ@ 0000000180039c48     JavaAccessBridge.obj
 0002:0000ec80       ??_C@_0CO@OPGCCICC@?$FLINFO?$FN?3?5?5?5found?5HWND?0?5javaEvent@ 0000000180039c80     JavaAccessBridge.obj
 0002:0000ecb0       ??_C@_0CP@MJMPLPDN@?$FLINFO?$FN?3?5?5?5union?5of?5all?5Java?5AT?5@ 0000000180039cb0     JavaAccessBridge.obj
 0002:0000ece0       ??_C@_0FO@PMMLAHPF@?$FLINFO?$FN?3?5?5?5no?5other?5AT?5wanted?5th@ 0000000180039ce0     JavaAccessBridge.obj
 0002:0000ed40       ??_C@_0DJ@DFJLLFAC@?$FLINFO?$FN?3?5?5?5removing?5Java?5event?5t@ 0000000180039d40     JavaAccessBridge.obj
 0002:0000ed80       ??_C@_0FO@LBFBGKHJ@?$FLINFO?$FN?3?5?5?5no?5other?5AT?5wanted?5th@ 0000000180039d80     JavaAccessBridge.obj
 0002:0000ede0       ??_C@_0DN@PDHOAFNL@?$FLINFO?$FN?3?5?5?5adding?5Accesibility?5e@ 0000000180039de0     JavaAccessBridge.obj
 0002:0000ee20       ??_C@_0DH@EPKDBDGJ@?$FLINFO?$FN?3?5?5?5found?5HWND?0?5accessibi@ 0000000180039e20     JavaAccessBridge.obj
 0002:0000ee58       ??_C@_0DI@IJKEHAJM@?$FLINFO?$FN?3?5?5?5union?5of?5all?5Accessib@ 0000000180039e58     JavaAccessBridge.obj
 0002:0000ee90       ??_C@_0GG@CGBBDJFJ@?$FLINFO?$FN?3?5?5?5no?5other?5AT?5wanted?5th@ 0000000180039e90     JavaAccessBridge.obj
 0002:0000ef00       ??_C@_0EB@PJLIMJAJ@?$FLINFO?$FN?3?5?5?5removing?5Accesibility@ 0000000180039f00     JavaAccessBridge.obj
 0002:0000ef50       ??_C@_0GH@FGGMCIOE@?$FLINFO?$FN?3?5?5?5no?5other?5AT?5wanted?5th@ 0000000180039f50     JavaAccessBridge.obj
 0002:0000efc0       ??_C@_0GL@DLLNHKDB@?$FLINFO?$FN?3?5Java_com_sun_java_acces@ 0000000180039fc0     JavaAccessBridge.obj
 0002:0000f030       ??_C@_0BI@GOJFHMPI@?$FLINFO?$FN?3?5?5?5sending?5to?5AT@ 000000018003a030     JavaAccessBridge.obj
 0002:0000f050       ??_C@_0EM@NDPMFJGH@?$FLINFO?$FN?3?5?5?5GlobalRef?8d?5Event?3?5?$CF0@ 000000018003a050     JavaAccessBridge.obj
 0002:0000f0a0       ??_C@_0CN@HLLEMELD@?$FLINFO?$FN?3?5?5done?5with?5propertyCare@ 000000018003a0a0     JavaAccessBridge.obj
 0002:0000f0d0       ??_C@_0HB@FIEPPBDD@?$FLINFO?$FN?3?5Java_com_sun_java_acces@ 000000018003a0d0     JavaAccessBridge.obj
 0002:0000f150       ??_C@_0ED@LNNGOPDA@?$FLINFO?$FN?3?5?5GlobalRef?8d?5Event?3?5?$CF01@ 000000018003a150     JavaAccessBridge.obj
 0002:0000f198       ??_C@_0BL@ENCPOIKC@java?1lang?1OutOfMemoryError@ 000000018003a198     JavaAccessBridge.obj
 0002:0000f1b8       ??_C@_1O@CEDCILHN@?$AA?$CI?$AAn?$AAu?$AAl?$AAl?$AA?$CJ@ 000000018003a1b8     JavaAccessBridge.obj
 0002:0000f1c8       ??_C@_0DE@IIPLELBE@?$FLINFO?$FN?3?5?5?5done?5with?5propertyDes@ 000000018003a1c8     JavaAccessBridge.obj
 0002:0000f200       ??_C@_0GK@FGEOELMA@?$FLINFO?$FN?3?5Java_com_sun_java_acces@ 000000018003a200     JavaAccessBridge.obj
 0002:0000f270       ??_C@_0EK@CCMALPPF@?$FLINFO?$FN?3?5?5GlobalRef?8d?5Event?3?5?$CF01@ 000000018003a270     JavaAccessBridge.obj
 0002:0000f2c0       ??_C@_0CM@LHIINGJI@?$FLINFO?$FN?3?5?5done?5with?5propertyName@ 000000018003a2c0     JavaAccessBridge.obj
 0002:0000f2f0       ??_C@_0GH@NDFIEILD@?$FLINFO?$FN?3?5Java_com_sun_java_acces@ 000000018003a2f0     JavaAccessBridge.obj
 0002:0000f358       ??_C@_0DC@IDEPNPKP@?$FLINFO?$FN?3?5?5?5done?5with?5propertySel@ 000000018003a358     JavaAccessBridge.obj
 0002:0000f390       ??_C@_0GL@LHHKNKCF@?$FLINFO?$FN?3?5Java_com_sun_java_acces@ 000000018003a390     JavaAccessBridge.obj
 0002:0000f400       ??_C@_0CN@HPCDPOIL@?$FLINFO?$FN?3?5?5done?5with?5propertyStat@ 000000018003a400     JavaAccessBridge.obj
 0002:0000f430       ??_C@_0GC@GKPNHBKM@?$FLINFO?$FN?3?5Java_com_sun_java_acces@ 000000018003a430     JavaAccessBridge.obj
 0002:0000f498       ??_C@_0CM@MKJMCAOF@?$FLINFO?$FN?3?5?5done?5with?5propertyText@ 000000018003a498     JavaAccessBridge.obj
 0002:0000f4d0       ??_C@_0GL@LMHLMBIC@?$FLINFO?$FN?3?5Java_com_sun_java_acces@ 000000018003a4d0     JavaAccessBridge.obj
 0002:0000f540       ??_C@_0CO@LJOPOKFE@?$FLINFO?$FN?3?5?5?5done?5with?5propertyVal@ 000000018003a540     JavaAccessBridge.obj
 0002:0000f570       ??_C@_0GJ@PEJPEKID@?$FLINFO?$FN?3?5Java_com_sun_java_acces@ 000000018003a570     JavaAccessBridge.obj
 0002:0000f5e0       ??_C@_0DD@LNFBPAKO@?$FLINFO?$FN?3?5?5done?5with?5propertyVisi@ 000000018003a5e0     JavaAccessBridge.obj
 0002:0000f620       ??_C@_0HD@JKCIIIAC@?$FLINFO?$FN?3?5Java_com_sun_java_acces@ 000000018003a620     JavaAccessBridge.obj
 0002:0000f698       ??_C@_0BH@HMENLEAO@?$FLINFO?$FN?3?5?5sending?5to?5AT@ 000000018003a698     JavaAccessBridge.obj
 0002:0000f6b0       ??_C@_0II@CFAAOCOP@?$FLINFO?$FN?3?5?5?5GlobalRef?8d?5Event?3?5?$CF0@ 000000018003a6b0     JavaAccessBridge.obj
 0002:0000f738       ??_C@_0CN@LGDOHOEO@?$FLINFO?$FN?3?5?5done?5with?5propertyChil@ 000000018003a738     JavaAccessBridge.obj
 0002:0000f770       ??_C@_0HO@MNNKGDDP@?$FLINFO?$FN?3?5Java_com_sun_java_acces@ 000000018003a770     JavaAccessBridge.obj
 0002:0000f7f0       ??_C@_0JN@BMGHKMMD@?$FLINFO?$FN?3?5?5GlobalRef?8d?5Event?3?5?$CF01@ 000000018003a7f0     JavaAccessBridge.obj
 0002:0000f890       ??_C@_0CO@GOOPPCJH@?$FLINFO?$FN?3?5?5done?5with?5propertyActi@ 000000018003a890     JavaAccessBridge.obj
 0002:0000f8c0       ??_C@_0GP@NILNKGMP@?$FLINFO?$FN?3?5Java_com_sun_java_acces@ 000000018003a8c0     JavaAccessBridge.obj
 0002:0000f930       ??_C@_0BA@KOMOFG@?5?5sending?5to?5AT@ 000000018003a930     JavaAccessBridge.obj
 0002:0000f940       ??_C@_0DC@FMNGEBKI@?$FLINFO?$FN?3?5?5done?5with?5propertyTabl@ 000000018003a940     JavaAccessBridge.obj
 0002:0000f978       ??_C@_0DA@ODJJOIDA@?$FLINFO?$FN?3?5Firing?5event?5id?5?$DN?5?$CFd?$CI?$CFp@ 000000018003a978     JavaAccessBridge.obj
 0002:0000f9a8       ??_C@_0CF@EPNHEIBO@?$FLINFO?$FN?3?5?5?5done?5with?5firing?5AWT?5@ 000000018003a9a8     JavaAccessBridge.obj
 0002:0000f9d0       ??_C@_0DI@NNGMMOBO@?$FLINFO?$FN?3?5Firing?5event?5id?5?$DN?5?$CFd?$CI?$CFp@ 000000018003a9d0     JavaAccessBridge.obj
 0002:0000fa08       ??_C@_0DJ@GLLLDFPO@?$FLINFO?$FN?3?5javaEventMask?5?$DN?5?$CFX?5even@ 000000018003aa08     JavaAccessBridge.obj
 0002:0000fa48       ??_C@_1CO@CCIONPKC@?$AAA?$AAc?$AAc?$AAe?$AAs?$AAs?$AAB?$AAr?$AAi?$AAd?$AAg?$AAe?$AA?4?$AAj?$AAa@ 000000018003aa48     JavaAccessBridge.obj
 0002:0000fa78       _pDefaultRawDllMain        000000018003aa78     LIBCMT:dll_dllmain.obj
 0002:0000fa78       _pRawDllMain               000000018003aa78     LIBCMT:dll_dllmain.obj
 0002:0000fa88       ??_7exception@std@@6B@     000000018003aa88     LIBCMT:throw_bad_alloc.obj
 0002:0000fa98       ??_C@_0BC@EOODALEL@Unknown?5exception@ 000000018003aa98     LIBCMT:throw_bad_alloc.obj
 0002:0000fab8       ??_7bad_alloc@std@@6B@     000000018003aab8     LIBCMT:throw_bad_alloc.obj
 0002:0000fac8       ??_C@_0P@GHFPNOJB@bad?5allocation@ 000000018003aac8     LIBCMT:throw_bad_alloc.obj
 0002:0000fae0       ??_7bad_array_new_length@std@@6B@ 000000018003aae0     LIBCMT:throw_bad_alloc.obj
 0002:0000faf0       ??_C@_0BF@KINCDENJ@bad?5array?5new?5length@ 000000018003aaf0     LIBCMT:throw_bad_alloc.obj
 0002:0000fb20       __xmm@ffffffffffffffffffffffffffffffff 000000018003ab20     LIBCMT:utility.obj
 0002:0000fb38       ??_7type_info@@6B@         000000018003ab38     LIBCMT:std_type_info_static.obj
 0002:0000fb40       _pDestructExceptionObject  000000018003ab40     libvcruntime:ehhelpers.obj
 0002:00010260       ??_C@_08EHJDFFNH@__based?$CI@ 000000018003b260     libvcruntime:undname.obj
 0002:00010270       ??_C@_07KOLFKCDI@__cdecl@  000000018003b270     libvcruntime:undname.obj
 0002:00010278       ??_C@_08GHMPAG@__pascal@   000000018003b278     libvcruntime:undname.obj
 0002:00010288       ??_C@_09IFJBGAPI@__stdcall@ 000000018003b288     libvcruntime:undname.obj
 0002:00010298       ??_C@_0L@NPHFGOKO@__thiscall@ 000000018003b298     libvcruntime:undname.obj
 0002:000102a8       ??_C@_0L@JMKHOMEK@__fastcall@ 000000018003b2a8     libvcruntime:undname.obj
 0002:000102b8       ??_C@_0N@BCKKPABJ@__vectorcall@ 000000018003b2b8     libvcruntime:undname.obj
 0002:000102c8       ??_C@_09HIJEGCPM@__clrcall@ 000000018003b2c8     libvcruntime:undname.obj
 0002:000102d4       ??_C@_06GHPCKEAG@__eabi@   000000018003b2d4     libvcruntime:undname.obj
 0002:000102e0       ??_C@_09IOPIDJLG@__swift_1@ 000000018003b2e0     libvcruntime:undname.obj
 0002:000102f0       ??_C@_09KFNFGKHF@__swift_2@ 000000018003b2f0     libvcruntime:undname.obj
 0002:00010300       ??_C@_09LMMOFLDE@__swift_3@ 000000018003b300     libvcruntime:undname.obj
 0002:00010310       ??_C@_07JOMMBBKO@__ptr64@  000000018003b310     libvcruntime:undname.obj
 0002:00010318       ??_C@_0L@PILCLIHE@__restrict@ 000000018003b318     libvcruntime:undname.obj
 0002:00010328       ??_C@_0M@GFIIJFMG@__unaligned@ 000000018003b328     libvcruntime:undname.obj
 0002:00010338       ??_C@_09DHDLOLLB@restrict?$CI@ 000000018003b338     libvcruntime:undname.obj
 0002:00010342       ??_C@_00CNPNBAHC@@         000000018003b342     libvcruntime:undname.obj
 0002:00010344       ??_C@_04NIHEBCM@?5new@     000000018003b344     libvcruntime:undname.obj
 0002:00010350       ??_C@_07FPCDHGMM@?5delete@ 000000018003b350     libvcruntime:undname.obj
 0002:00010358       ??_C@_01NEMOKFLO@?$DN@     000000018003b358     libvcruntime:undname.obj
 0002:0001035c       ??_C@_02GPIOPFAK@?$DO?$DO@ 000000018003b35c     libvcruntime:undname.obj
 0002:00010360       ??_C@_02FODMEDOG@?$DM?$DM@ 000000018003b360     libvcruntime:undname.obj
 0002:00010364       ??_C@_01DCLJPIOD@?$CB@     000000018003b364     libvcruntime:undname.obj
 0002:00010368       ??_C@_02EGOFBIJA@?$DN?$DN@ 000000018003b368     libvcruntime:undname.obj
 0002:0001036c       ??_C@_02FDNJECIE@?$CB?$DN@ 000000018003b36c     libvcruntime:undname.obj
 0002:00010370       ??_C@_02GPECMEKF@?$FL?$FN@ 000000018003b370     libvcruntime:undname.obj
 0002:00010378       ??_C@_08LHJFAFGD@operator@ 000000018003b378     libvcruntime:undname.obj
 0002:00010384       ??_C@_02HBOOOICD@?9?$DO@   000000018003b384     libvcruntime:undname.obj
 0002:00010388       ??_C@_01NBENCBCI@?$CK@     000000018003b388     libvcruntime:undname.obj
 0002:0001038c       ??_C@_02ECNGHCIF@?$CL?$CL@ 000000018003b38c     libvcruntime:undname.obj
 0002:00010390       ??_C@_02BAABKJLB@?9?9@     000000018003b390     libvcruntime:undname.obj
 0002:00010394       ??_C@_01JOAMLHOP@?9@       000000018003b394     libvcruntime:undname.obj
 0002:00010398       ??_C@_01MIFGBAGJ@?$CL@     000000018003b398     libvcruntime:undname.obj
 0002:0001039c       ??_C@_01HNPIGOCE@?$CG@     000000018003b39c     libvcruntime:undname.obj
 0002:000103a0       ??_C@_03MNHNFDLC@?9?$DO?$CK@ 000000018003b3a0     libvcruntime:undname.obj
 0002:000103a4       ??_C@_01KMDKNFGN@?1@       000000018003b3a4     libvcruntime:undname.obj
 0002:000103a8       ??_C@_01FGNFDNOH@?$CF@     000000018003b3a8     libvcruntime:undname.obj
 0002:000103ac       ??_C@_01MNNFJEPP@?$DM@     000000018003b3ac     libvcruntime:undname.obj
 0002:000103b0       ??_C@_02EHCHHCKH@?$DM?$DN@ 000000018003b3b0     libvcruntime:undname.obj
 0002:000103b4       ??_C@_01PPODPGHN@?$DO@     000000018003b3b4     libvcruntime:undname.obj
 0002:000103b8       ??_C@_02EEKDKGMJ@?$DO?$DN@ 000000018003b3b8     libvcruntime:undname.obj
 0002:000103bc       ??_C@_01IHBHIGKO@?0@       000000018003b3bc     libvcruntime:undname.obj
 0002:000103c0       ??_C@_02HCKGKOFO@?$CI?$CJ@ 000000018003b3c0     libvcruntime:undname.obj
 0002:000103c4       ??_C@_01PJKLJHI@?$HO@      000000018003b3c4     libvcruntime:undname.obj
 0002:000103c8       ??_C@_01JKBOJNNK@?$FO@     000000018003b3c8     libvcruntime:undname.obj
 0002:000103cc       ??_C@_01DNKMNLPK@?$HM@     000000018003b3cc     libvcruntime:undname.obj
 0002:000103d0       ??_C@_02PPKAJPJL@?$CG?$CG@ 000000018003b3d0     libvcruntime:undname.obj
 0002:000103d4       ??_C@_02NONPIBCD@?$HM?$HM@ 000000018003b3d4     libvcruntime:undname.obj
 0002:000103d8       ??_C@_02FPIMKNGF@?$CK?$DN@ 000000018003b3d8     libvcruntime:undname.obj
 0002:000103dc       ??_C@_02FOEOMHFC@?$CL?$DN@ 000000018003b3dc     libvcruntime:undname.obj
 0002:000103e0       ??_C@_02FKMDLLOA@?9?$DN@   000000018003b3e0     libvcruntime:undname.obj
 0002:000103e4       ??_C@_02FJEHGPIO@?1?$DN@   000000018003b3e4     libvcruntime:undname.obj
 0002:000103e8       ??_C@_02FENAOKFI@?$CF?$DN@ 000000018003b3e8     libvcruntime:undname.obj
 0002:000103ec       ??_C@_03IKFCCPFF@?$DO?$DO?$DN@ 000000018003b3ec     libvcruntime:undname.obj
 0002:000103f0       ??_C@_03CDNPDDLA@?$DM?$DM?$DN@ 000000018003b3f0     libvcruntime:undname.obj
 0002:000103f4       ??_C@_02FGJGFEAB@?$CG?$DN@ 000000018003b3f4     libvcruntime:undname.obj
 0002:000103f8       ??_C@_02DHLNPPGH@?$HM?$DN@ 000000018003b3f8     libvcruntime:undname.obj
 0002:000103fc       ??_C@_02MHEGNOJ@?$FO?$DN@  000000018003b3fc     libvcruntime:undname.obj
 0002:00010400       ??_C@_09IFPLHPGF@?$GAvftable?8@ 000000018003b400     libvcruntime:undname.obj
 0002:00010410       ??_C@_09BLBHBJP@?$GAvbtable?8@ 000000018003b410     libvcruntime:undname.obj
 0002:00010420       ??_C@_07FEEIOKP@?$GAvcall?8@ 000000018003b420     libvcruntime:undname.obj
 0002:00010428       ??_C@_08LLFFHHDJ@?$GAtypeof?8@ 000000018003b428     libvcruntime:undname.obj
 0002:00010438       ??_C@_0BF@KDPPACIK@?$GAlocal?5static?5guard?8@ 000000018003b438     libvcruntime:undname.obj
 0002:00010450       ??_C@_08OBABFOLI@?$GAstring?8@ 000000018003b450     libvcruntime:undname.obj
 0002:00010460       ??_C@_0BD@JDLKDPAB@?$GAvbase?5destructor?8@ 000000018003b460     libvcruntime:undname.obj
 0002:00010478       ??_C@_0BN@DEGPLNFK@?$GAvector?5deleting?5destructor?8@ 000000018003b478     libvcruntime:undname.obj
 0002:00010498       ??_C@_0BO@OBMKPJIG@?$GAdefault?5constructor?5closure?8@ 000000018003b498     libvcruntime:undname.obj
 0002:000104b8       ??_C@_0BN@IMDCHIKM@?$GAscalar?5deleting?5destructor?8@ 000000018003b4b8     libvcruntime:undname.obj
 0002:000104d8       ??_C@_0BO@PFGOCPJJ@?$GAvector?5constructor?5iterator?8@ 000000018003b4d8     libvcruntime:undname.obj
 0002:000104f8       ??_C@_0BN@LFPFMEDL@?$GAvector?5destructor?5iterator?8@ 000000018003b4f8     libvcruntime:undname.obj
 0002:00010518       ??_C@_0CE@IKBNEHA@?$GAvector?5vbase?5constructor?5itera@ 000000018003b518     libvcruntime:undname.obj
 0002:00010540       ??_C@_0BL@NILFHHPC@?$GAvirtual?5displacement?5map?8@ 000000018003b540     libvcruntime:undname.obj
 0002:00010560       ??_C@_0CB@JONCMFFK@?$GAeh?5vector?5constructor?5iterator@ 000000018003b560     libvcruntime:undname.obj
 0002:00010588       ??_C@_0CA@GCEOPDGL@?$GAeh?5vector?5destructor?5iterator?8@ 000000018003b588     libvcruntime:undname.obj
 0002:000105a8       ??_C@_0CH@OOJPLCPH@?$GAeh?5vector?5vbase?5constructor?5it@ 000000018003b5a8     libvcruntime:undname.obj
 0002:000105d0       ??_C@_0BL@LLKPOHJI@?$GAcopy?5constructor?5closure?8@ 000000018003b5d0     libvcruntime:undname.obj
 0002:000105f0       ??_C@_0BA@KBCDOMBN@?$GAudt?5returning?8@ 000000018003b5f0     libvcruntime:undname.obj
 0002:00010600       ??_C@_03KLGMFNMG@?$GAEH@   000000018003b600     libvcruntime:undname.obj
 0002:00010604       ??_C@_05KHLCHHI@?$GARTTI@  000000018003b604     libvcruntime:undname.obj
 0002:00010610       ??_C@_0BA@KKLDJDLB@?$GAlocal?5vftable?8@ 000000018003b610     libvcruntime:undname.obj
 0002:00010620       ??_C@_0CE@IIHCMGGL@?$GAlocal?5vftable?5constructor?5clos@ 000000018003b620     libvcruntime:undname.obj
 0002:00010644       ??_C@_06FHBGPFGH@?5new?$FL?$FN@ 000000018003b644     libvcruntime:undname.obj
 0002:00010650       ??_C@_09LBNFPBCA@?5delete?$FL?$FN@ 000000018003b650     libvcruntime:undname.obj
 0002:00010660       ??_C@_0P@HJKNJFNN@?$GAomni?5callsig?8@ 000000018003b660     libvcruntime:undname.obj
 0002:00010670       ??_C@_0BL@CNOONJFP@?$GAplacement?5delete?5closure?8@ 000000018003b670     libvcruntime:undname.obj
 0002:00010690       ??_C@_0BN@CKNJLHMB@?$GAplacement?5delete?$FL?$FN?5closure?8@ 000000018003b690     libvcruntime:undname.obj
 0002:000106b0       ??_C@_0CG@CFDHKGGD@?$GAmanaged?5vector?5constructor?5ite@ 000000018003b6b0     libvcruntime:undname.obj
 0002:000106d8       ??_C@_0CF@IMGKMJNO@?$GAmanaged?5vector?5destructor?5iter@ 000000018003b6d8     libvcruntime:undname.obj
 0002:00010700       ??_C@_0CG@HLDDJMAG@?$GAeh?5vector?5copy?5constructor?5ite@ 000000018003b700     libvcruntime:undname.obj
 0002:00010728       ??_C@_0CM@FCBBDIGB@?$GAeh?5vector?5vbase?5copy?5construct@ 000000018003b728     libvcruntime:undname.obj
 0002:00010758       ??_C@_0BL@CLIPGLGB@?$GAdynamic?5initializer?5for?5?8@ 000000018003b758     libvcruntime:undname.obj
 0002:00010778       ??_C@_0CB@PDBIFEP@?$GAdynamic?5atexit?5destructor?5for?5@ 000000018003b778     libvcruntime:undname.obj
 0002:000107a0       ??_C@_0CD@CGAJBKEJ@?$GAvector?5copy?5constructor?5iterat@ 000000018003b7a0     libvcruntime:undname.obj
 0002:000107c8       ??_C@_0CJ@GJELGAMM@?$GAvector?5vbase?5copy?5constructor?5@ 000000018003b7c8     libvcruntime:undname.obj
 0002:000107f8       ??_C@_0CL@FGIJHLCE@?$GAmanaged?5vector?5copy?5constructo@ 000000018003b7f8     libvcruntime:undname.obj
 0002:00010828       ??_C@_0BM@PMGGMLDN@?$GAlocal?5static?5thread?5guard?8@ 000000018003b828     libvcruntime:undname.obj
 0002:00010848       ??_C@_0N@BDNMDMOL@operator?5?$CC?$CC?5@ 000000018003b848     libvcruntime:undname.obj
 0002:00010858       ??_C@_0BC@GGEBGALA@operator?5co_await@ 000000018003b858     libvcruntime:undname.obj
 0002:00010870       ??_C@_0M@GAAIMMOH@operator?$DM?$DN?$DO@ 000000018003b870     libvcruntime:undname.obj
 0002:00010880       ??_C@_0BC@DAFEJGAK@?5Type?5Descriptor?8@ 000000018003b880     libvcruntime:undname.obj
 0002:00010898       ??_C@_0BM@LDKODKLH@?5Base?5Class?5Descriptor?5at?5?$CI@ 000000018003b898     libvcruntime:undname.obj
 0002:000108b8       ??_C@_0BD@LGICGFMM@?5Base?5Class?5Array?8@ 000000018003b8b8     libvcruntime:undname.obj
 0002:000108d0       ??_C@_0BN@MECKDCOJ@?5Class?5Hierarchy?5Descriptor?8@ 000000018003b8d0     libvcruntime:undname.obj
 0002:000108f0       ??_C@_0BK@CFCOFLF@?5Complete?5Object?5Locator?8@ 000000018003b8f0     libvcruntime:undname.obj
 0002:00010910       ??_C@_0BG@JNJLAMPM@?$GAanonymous?5namespace?8@ 000000018003b910     libvcruntime:undname.obj
 0002:000109e0       ??_C@_1DM@KHCHBNEB@?$AAa?$AAp?$AAi?$AA?9?$AAm?$AAs?$AA?9?$AAw?$AAi?$AAn?$AA?9?$AAc?$AAo?$AAr?$AAe@ 000000018003b9e0     libvcruntime:winapi_downlevel.obj
 0002:00010a20       ??_C@_1DK@LPPGFMPP@?$AAa?$AAp?$AAi?$AA?9?$AAm?$AAs?$AA?9?$AAw?$AAi?$AAn?$AA?9?$AAc?$AAo?$AAr?$AAe@ 000000018003ba20     libvcruntime:winapi_downlevel.obj
 0002:00010a60       ??_C@_1BC@GDMECMAK@?$AAk?$AAe?$AAr?$AAn?$AAe?$AAl?$AA3?$AA2@ 000000018003ba60     libvcruntime:winapi_downlevel.obj
 0002:00010a78       ??_C@_1BA@PFFKHIOG@?$AAa?$AAp?$AAi?$AA?9?$AAm?$AAs?$AA?9@ 000000018003ba78     libvcruntime:winapi_downlevel.obj
 0002:00010a90       ??_C@_08KNHFBNJ@FlsAlloc@  000000018003ba90     libvcruntime:winapi_downlevel.obj
 0002:00010aa8       ??_C@_07PEJMOBNF@FlsFree@  000000018003baa8     libvcruntime:winapi_downlevel.obj
 0002:00010ab8       ??_C@_0M@GDNOONDI@FlsGetValue@ 000000018003bab8     libvcruntime:winapi_downlevel.obj
 0002:00010ad0       ??_C@_0M@JCPCPOEF@FlsSetValue@ 000000018003bad0     libvcruntime:winapi_downlevel.obj
 0002:00010ae8       ??_C@_0BM@HCFOFFN@InitializeCriticalSectionEx@ 000000018003bae8     libvcruntime:winapi_downlevel.obj
 0002:00010b10       ??_7bad_exception@std@@6B@ 000000018003bb10     libvcruntime:frame.obj
 0002:00010b20       ??_C@_0O@DPKOEFFH@bad?5exception@ 000000018003bb20     libvcruntime:frame.obj
 0002:00010b30       ?standard_lookup_table_spectre@__crt_stdio_output@@3V?$spectre_mitigated_lookup_table@Ustate_transition_pair@__crt_stdio_output@@$0IA@@1@B 000000018003bb30     libucrt:output.obj
 0002:00010ca8       ??_C@_06OJHGLDPL@?$CInull?$CJ@ 000000018003bca8     libucrt:output.obj
 0002:00010cb0       __acrt_exception_action_table 000000018003bcb0     libucrt:exception_filter.obj
 0002:00010d70       __acrt_signal_action_table_count 000000018003bd70     libucrt:exception_filter.obj
 0002:00010d78       __acrt_signal_action_first_fpe_index 000000018003bd78     libucrt:exception_filter.obj
 0002:00010d80       __acrt_signal_action_fpe_count 000000018003bd80     libucrt:exception_filter.obj
 0002:00010dd8       ??_C@_1BI@BGOHAHKC@?$AAm?$AAs?$AAc?$AAo?$AAr?$AAe?$AAe?$AA?4?$AAd?$AAl?$AAl@ 000000018003bdd8     libucrt:exit.obj
 0002:00010df0       ??_C@_0P@MIGLKIOC@CorExitProcess@ 000000018003bdf0     libucrt:exit.obj
 0002:00011180       ??_C@_1EA@JGEFHKEI@?$AAa?$AAp?$AAi?$AA?9?$AAm?$AAs?$AA?9?$AAw?$AAi?$AAn?$AA?9?$AAc?$AAo?$AAr?$AAe@ 000000018003c180     libucrt:winapi_thunks.obj
 0002:000111c0       ??_C@_1DM@LFJCLCKP@?$AAa?$AAp?$AAi?$AA?9?$AAm?$AAs?$AA?9?$AAw?$AAi?$AAn?$AA?9?$AAc?$AAo?$AAr?$AAe@ 000000018003c1c0     libucrt:winapi_thunks.obj
 0002:00011200       ??_C@_1DI@KMEPCBPN@?$AAa?$AAp?$AAi?$AA?9?$AAm?$AAs?$AA?9?$AAw?$AAi?$AAn?$AA?9?$AAc?$AAo?$AAr?$AAe@ 000000018003c200     libucrt:winapi_thunks.obj
 0002:00011238       ??_C@_1DI@IJCEHOCB@?$AAa?$AAp?$AAi?$AA?9?$AAm?$AAs?$AA?9?$AAw?$AAi?$AAn?$AA?9?$AAc?$AAo?$AAr?$AAe@ 000000018003c238     libucrt:winapi_thunks.obj
 0002:00011270       ??_C@_1DI@FFFOPEOO@?$AAa?$AAp?$AAi?$AA?9?$AAm?$AAs?$AA?9?$AAw?$AAi?$AAn?$AA?9?$AAc?$AAo?$AAr?$AAe@ 000000018003c270     libucrt:winapi_thunks.obj
 0002:000112b0       ??_C@_1EI@MPIAOHOC@?$AAa?$AAp?$AAi?$AA?9?$AAm?$AAs?$AA?9?$AAw?$AAi?$AAn?$AA?9?$AAc?$AAo?$AAr?$AAe@ 000000018003c2b0     libucrt:winapi_thunks.obj
 0002:00011300       ??_C@_1FK@FPHCKFIE@?$AAa?$AAp?$AAi?$AA?9?$AAm?$AAs?$AA?9?$AAw?$AAi?$AAn?$AA?9?$AAc?$AAo?$AAr?$AAe@ 000000018003c300     libucrt:winapi_thunks.obj
 0002:00011360       ??_C@_1EM@DILCGIIO@?$AAa?$AAp?$AAi?$AA?9?$AAm?$AAs?$AA?9?$AAw?$AAi?$AAn?$AA?9?$AAc?$AAo?$AAr?$AAe@ 000000018003c360     libucrt:winapi_thunks.obj
 0002:000113b0       ??_C@_1DM@LNCGDDPN@?$AAa?$AAp?$AAi?$AA?9?$AAm?$AAs?$AA?9?$AAw?$AAi?$AAn?$AA?9?$AAc?$AAo?$AAr?$AAe@ 000000018003c3b0     libucrt:winapi_thunks.obj
 0002:000113f0       ??_C@_1DO@FPAPJEMD@?$AAa?$AAp?$AAi?$AA?9?$AAm?$AAs?$AA?9?$AAw?$AAi?$AAn?$AA?9?$AAc?$AAo?$AAr?$AAe@ 000000018003c3f0     libucrt:winapi_thunks.obj
 0002:00011430       ??_C@_1DK@NDHNAHIO@?$AAa?$AAp?$AAi?$AA?9?$AAm?$AAs?$AA?9?$AAw?$AAi?$AAn?$AA?9?$AAc?$AAo?$AAr?$AAe@ 000000018003c430     libucrt:winapi_thunks.obj
 0002:00011470       ??_C@_1DM@KGHDGBCM@?$AAa?$AAp?$AAi?$AA?9?$AAm?$AAs?$AA?9?$AAw?$AAi?$AAn?$AA?9?$AAc?$AAo?$AAr?$AAe@ 000000018003c470     libucrt:winapi_thunks.obj
 0002:000114b0       ??_C@_1EO@IJIOEFOH@?$AAa?$AAp?$AAi?$AA?9?$AAm?$AAs?$AA?9?$AAw?$AAi?$AAn?$AA?9?$AAr?$AAt?$AAc?$AAo@ 000000018003c4b0     libucrt:winapi_thunks.obj
 0002:00011500       ??_C@_1FG@HHGEKANL@?$AAa?$AAp?$AAi?$AA?9?$AAm?$AAs?$AA?9?$AAw?$AAi?$AAn?$AA?9?$AAs?$AAe?$AAc?$AAu@ 000000018003c500     libucrt:winapi_thunks.obj
 0002:00011560       ??_C@_1EG@DBIOJECG@?$AAe?$AAx?$AAt?$AA?9?$AAm?$AAs?$AA?9?$AAw?$AAi?$AAn?$AA?9?$AAn?$AAt?$AAu?$AAs@ 000000018003c560     libucrt:winapi_thunks.obj
 0002:000115b0       ??_C@_1EO@FIHMJCLF@?$AAe?$AAx?$AAt?$AA?9?$AAm?$AAs?$AA?9?$AAw?$AAi?$AAn?$AA?9?$AAn?$AAt?$AAu?$AAs@ 000000018003c5b0     libucrt:winapi_thunks.obj
 0002:00011600       ??_C@_1BC@DNHGCMLG@?$AAa?$AAd?$AAv?$AAa?$AAp?$AAi?$AA3?$AA2@ 000000018003c600     libucrt:winapi_thunks.obj
 0002:00011618       ??_C@_1BG@CJPGBMEF@?$AAk?$AAe?$AAr?$AAn?$AAe?$AAl?$AAb?$AAa?$AAs?$AAe@ 000000018003c618     libucrt:winapi_thunks.obj
 0002:00011630       ??_C@_1M@OAIMIKLP@?$AAn?$AAt?$AAd?$AAl?$AAl@ 000000018003c630     libucrt:winapi_thunks.obj
 0002:00011640       ??_C@_1EG@DPGNFKGC@?$AAa?$AAp?$AAi?$AA?9?$AAm?$AAs?$AA?9?$AAw?$AAi?$AAn?$AA?9?$AAa?$AAp?$AAp?$AAm@ 000000018003c640     libucrt:winapi_thunks.obj
 0002:00011688       ??_C@_1O@BCCLBEOE@?$AAu?$AAs?$AAe?$AAr?$AA3?$AA2@ 000000018003c688     libucrt:winapi_thunks.obj
 0002:00011698       ??_C@_1BA@IAIFMGEF@?$AAe?$AAx?$AAt?$AA?9?$AAm?$AAs?$AA?9@ 000000018003c698     libucrt:winapi_thunks.obj
 0002:000116b0       ??_C@_0BA@FHFNEAED@AreFileApisANSI@ 000000018003c6b0     libucrt:winapi_thunks.obj
 0002:000116c8       ??_C@_0BA@IHGNDAEB@CompareStringEx@ 000000018003c6c8     libucrt:winapi_thunks.obj
 0002:000116e0       ??_C@_0N@MFBBDCAC@FlsGetValue2@ 000000018003c6e0     libucrt:winapi_thunks.obj
 0002:000116f8       ??_C@_0O@KKBNKAPF@LCMapStringEx@ 000000018003c6f8     libucrt:winapi_thunks.obj
 0002:00011710       ??_C@_0BB@HBDEELFH@LocaleNameToLCID@ 000000018003c710     libucrt:winapi_thunks.obj
 0002:00011728       ??_C@_0N@PPOMPGGK@RoInitialize@ 000000018003c728     libucrt:winapi_thunks.obj
 0002:00011740       ??_C@_0P@LLFHBIJD@RoUninitialize@ 000000018003c740     libucrt:winapi_thunks.obj
 0002:00011758       ??_C@_0CF@OJOFEIGO@AppPolicyGetProcessTerminationM@ 000000018003c758     libucrt:winapi_thunks.obj
 0002:00011788       ??_C@_0CF@NNDFDCOC@AppPolicyGetThreadInitializatio@ 000000018003c788     libucrt:winapi_thunks.obj
 0002:00011830       ??_C@_03OEIAHPBN@INF@      000000018003c830     libucrt:cvt.obj
 0002:00011834       ??_C@_03OJHLLCGB@inf@      000000018003c834     libucrt:cvt.obj
 0002:00011838       ??_C@_03LKNCIKJB@NAN@      000000018003c838     libucrt:cvt.obj
 0002:0001183c       ??_C@_03LHCJEHON@nan@      000000018003c83c     libucrt:cvt.obj
 0002:00011840       ??_C@_09OFJJIMPC@NAN?$CISNAN?$CJ@ 000000018003c840     libucrt:cvt.obj
 0002:00011850       ??_C@_09IPFBKMDL@nan?$CIsnan?$CJ@ 000000018003c850     libucrt:cvt.obj
 0002:00011860       ??_C@_08IKHNHAJ@NAN?$CIIND?$CJ@ 000000018003c860     libucrt:cvt.obj
 0002:00011870       ??_C@_08OFCDMILK@nan?$CIind?$CJ@ 000000018003c870     libucrt:cvt.obj
 0002:0001187c       ??_C@_05KLBDPFGC@e?$CL000@ 000000018003c87c     libucrt:cvt.obj
 0002:00011890       __lc_time_c                000000018003c890     libucrt:nlsdata.obj
 0002:00011b50       ??_C@_03KOEHGMDN@Sun@      000000018003cb50     libucrt:nlsdata.obj
 0002:00011b54       ??_C@_03PDAGKDH@Mon@       000000018003cb54     libucrt:nlsdata.obj
 0002:00011b58       ??_C@_03NAGEINEP@Tue@      000000018003cb58     libucrt:nlsdata.obj
 0002:00011b5c       ??_C@_03MHOMLAJA@Wed@      000000018003cb5c     libucrt:nlsdata.obj
 0002:00011b60       ??_C@_03IOFIKPDN@Thu@      000000018003cb60     libucrt:nlsdata.obj
 0002:00011b64       ??_C@_03IDIOELNC@Fri@      000000018003cb64     libucrt:nlsdata.obj
 0002:00011b68       ??_C@_03FEFJNEK@Sat@       000000018003cb68     libucrt:nlsdata.obj
 0002:00011b6c       ??_C@_06OOPIFAJ@Sunday@    000000018003cb6c     libucrt:nlsdata.obj
 0002:00011b74       ??_C@_06JLEDEDGH@Monday@   000000018003cb74     libucrt:nlsdata.obj
 0002:00011b80       ??_C@_07BAAGCFCM@Tuesday@  000000018003cb80     libucrt:nlsdata.obj
 0002:00011b88       ??_C@_09DLIGFAKA@Wednesday@ 000000018003cb88     libucrt:nlsdata.obj
 0002:00011b98       ??_C@_08HACCIKIA@Thursday@ 000000018003cb98     libucrt:nlsdata.obj
 0002:00011ba4       ??_C@_06JECMNKMI@Friday@   000000018003cba4     libucrt:nlsdata.obj
 0002:00011bb0       ??_C@_08INBOOONO@Saturday@ 000000018003cbb0     libucrt:nlsdata.obj
 0002:00011bbc       ??_C@_03JIHJHPIE@Jan@      000000018003cbbc     libucrt:nlsdata.obj
 0002:00011bc0       ??_C@_03HJBDCHOM@Feb@      000000018003cbc0     libucrt:nlsdata.obj
 0002:00011bc4       ??_C@_03ODNJBKGA@Mar@      000000018003cbc4     libucrt:nlsdata.obj
 0002:00011bc8       ??_C@_03LEOLGMJP@Apr@      000000018003cbc8     libucrt:nlsdata.obj
 0002:00011bcc       ??_C@_03CNMDKL@May@        000000018003cbcc     libucrt:nlsdata.obj
 0002:00011bd0       ??_C@_03IDFGHECI@Jun@      000000018003cbd0     libucrt:nlsdata.obj
 0002:00011bd4       ??_C@_03LBGABGKK@Jul@      000000018003cbd4     libucrt:nlsdata.obj
 0002:00011bd8       ??_C@_03IFJFEIGA@Aug@      000000018003cbd8     libucrt:nlsdata.obj
 0002:00011bdc       ??_C@_03GGCAPAJC@Sep@      000000018003cbdc     libucrt:nlsdata.obj
 0002:00011be0       ??_C@_03BMAOKBAD@Oct@      000000018003cbe0     libucrt:nlsdata.obj
 0002:00011be4       ??_C@_03JPJOFNIA@Nov@      000000018003cbe4     libucrt:nlsdata.obj
 0002:00011be8       ??_C@_03MKABNOCG@Dec@      000000018003cbe8     libucrt:nlsdata.obj
 0002:00011bf0       ??_C@_07CGJPFGJA@January@  000000018003cbf0     libucrt:nlsdata.obj
 0002:00011bf8       ??_C@_08GNJGEPFN@February@ 000000018003cbf8     libucrt:nlsdata.obj
 0002:00011c04       ??_C@_05HPCKOFNC@March@    000000018003cc04     libucrt:nlsdata.obj
 0002:00011c0c       ??_C@_05DMJDNLEJ@April@    000000018003cc0c     libucrt:nlsdata.obj
 0002:00011c14       ??_C@_04CNLMGBGM@June@     000000018003cc14     libucrt:nlsdata.obj
 0002:00011c1c       ??_C@_04MIEPOIFP@July@     000000018003cc1c     libucrt:nlsdata.obj
 0002:00011c24       ??_C@_06LBBHFDDG@August@   000000018003cc24     libucrt:nlsdata.obj
 0002:00011c30       ??_C@_09BHHEALKD@September@ 000000018003cc30     libucrt:nlsdata.obj
 0002:00011c40       ??_C@_07JJNFCEND@October@  000000018003cc40     libucrt:nlsdata.obj
 0002:00011c48       ??_C@_08HCHEGEOA@November@ 000000018003cc48     libucrt:nlsdata.obj
 0002:00011c58       ??_C@_08EDHMEBNP@December@ 000000018003cc58     libucrt:nlsdata.obj
 0002:00011c64       ??_C@_02DEDBPAFC@AM@       000000018003cc64     libucrt:nlsdata.obj
 0002:00011c68       ??_C@_02CJNFDJBF@PM@       000000018003cc68     libucrt:nlsdata.obj
 0002:00011c70       ??_C@_08BPBNCDIB@MM?1dd?1yy@ 000000018003cc70     libucrt:nlsdata.obj
 0002:00011c80       ??_C@_0BE@CKGJFCPC@dddd?0?5MMMM?5dd?0?5yyyy@ 000000018003cc80     libucrt:nlsdata.obj
 0002:00011c98       ??_C@_08JCCMCCIL@HH?3mm?3ss@ 000000018003cc98     libucrt:nlsdata.obj
 0002:00011ca8       ??_C@_17MBGCMIPB@?$AAS?$AAu?$AAn@ 000000018003cca8     libucrt:nlsdata.obj
 0002:00011cb0       ??_C@_17KBOMKBF@?$AAM?$AAo?$AAn@ 000000018003ccb0     libucrt:nlsdata.obj
 0002:00011cb8       ??_C@_17BMKGEGOJ@?$AAT?$AAu?$AAe@ 000000018003ccb8     libucrt:nlsdata.obj
 0002:00011cc0       ??_C@_17CJEDCEPE@?$AAW?$AAe?$AAd@ 000000018003ccc0     libucrt:nlsdata.obj
 0002:00011cc8       ??_C@_17PDPHAADD@?$AAT?$AAh?$AAu@ 000000018003ccc8     libucrt:nlsdata.obj
 0002:00011cd0       ??_C@_17HFOLPPLP@?$AAF?$AAr?$AAi@ 000000018003ccd0     libucrt:nlsdata.obj
 0002:00011cd8       ??_C@_17GGIBDPIH@?$AAS?$AAa?$AAt@ 000000018003ccd8     libucrt:nlsdata.obj
 0002:00011ce0       ??_C@_1O@IHNHDHPB@?$AAS?$AAu?$AAn?$AAd?$AAa?$AAy@ 000000018003cce0     libucrt:nlsdata.obj
 0002:00011cf0       ??_C@_1O@MMNBFLIA@?$AAM?$AAo?$AAn?$AAd?$AAa?$AAy@ 000000018003ccf0     libucrt:nlsdata.obj
 0002:00011d00       ??_C@_1BA@ENFBFFEK@?$AAT?$AAu?$AAe?$AAs?$AAd?$AAa?$AAy@ 000000018003cd00     libucrt:nlsdata.obj
 0002:00011d10       ??_C@_1BE@EBOGMDOH@?$AAW?$AAe?$AAd?$AAn?$AAe?$AAs?$AAd?$AAa?$AAy@ 000000018003cd10     libucrt:nlsdata.obj
 0002:00011d28       ??_C@_1BC@HHMNLIHE@?$AAT?$AAh?$AAu?$AAr?$AAs?$AAd?$AAa?$AAy@ 000000018003cd28     libucrt:nlsdata.obj
 0002:00011d40       ??_C@_1O@PDICJHAG@?$AAF?$AAr?$AAi?$AAd?$AAa?$AAy@ 000000018003cd40     libucrt:nlsdata.obj
 0002:00011d50       ??_C@_1BC@ENMNNPAJ@?$AAS?$AAa?$AAt?$AAu?$AAr?$AAd?$AAa?$AAy@ 000000018003cd50     libucrt:nlsdata.obj
 0002:00011d68       ??_C@_17DKNBKCHM@?$AAJ?$AAa?$AAn@ 000000018003cd68     libucrt:nlsdata.obj
 0002:00011d70       ??_C@_17LMDJEKJN@?$AAF?$AAe?$AAb@ 000000018003cd70     libucrt:nlsdata.obj
 0002:00011d78       ??_C@_17CKNLEDEC@?$AAM?$AAa?$AAr@ 000000018003cd78     libucrt:nlsdata.obj
 0002:00011d80       ??_C@_17LFPOIHDD@?$AAA?$AAp?$AAr@ 000000018003cd80     libucrt:nlsdata.obj
 0002:00011d88       ??_C@_17PNNKMEED@?$AAM?$AAa?$AAy@ 000000018003cd88     libucrt:nlsdata.obj
 0002:00011d90       ??_C@_17KCJGOCPB@?$AAJ?$AAu?$AAn@ 000000018003cd90     libucrt:nlsdata.obj
 0002:00011d98       ??_C@_17IJPCKHK@?$AAJ?$AAu?$AAl@ 000000018003cd98     libucrt:nlsdata.obj
 0002:00011da0       ??_C@_17ICPELBCN@?$AAA?$AAu?$AAg@ 000000018003cda0     libucrt:nlsdata.obj
 0002:00011da8       ??_C@_17HCHCOKMG@?$AAS?$AAe?$AAp@ 000000018003cda8     libucrt:nlsdata.obj
 0002:00011db0       ??_C@_17FNLKOI@?$AAO?$AAc?$AAt@ 000000018003cdb0     libucrt:nlsdata.obj
 0002:00011db8       ??_C@_17BBDMLCIG@?$AAN?$AAo?$AAv@ 000000018003cdb8     libucrt:nlsdata.obj
 0002:00011dc0       ??_C@_17EGKACKIF@?$AAD?$AAe?$AAc@ 000000018003cdc0     libucrt:nlsdata.obj
 0002:00011dc8       ??_C@_1BA@EFMEIEBA@?$AAJ?$AAa?$AAn?$AAu?$AAa?$AAr?$AAy@ 000000018003cdc8     libucrt:nlsdata.obj
 0002:00011dd8       ??_C@_1BC@JGDDFFAM@?$AAF?$AAe?$AAb?$AAr?$AAu?$AAa?$AAr?$AAy@ 000000018003cdd8     libucrt:nlsdata.obj
 0002:00011df0       ??_C@_1M@IKEENEDF@?$AAM?$AAa?$AAr?$AAc?$AAh@ 000000018003cdf0     libucrt:nlsdata.obj
 0002:00011e00       ??_C@_1M@GJNLMHFD@?$AAA?$AAp?$AAr?$AAi?$AAl@ 000000018003ce00     libucrt:nlsdata.obj
 0002:00011e10       ??_C@_19EPFLPGAP@?$AAJ?$AAu?$AAn?$AAe@ 000000018003ce10     libucrt:nlsdata.obj
 0002:00011e20       ??_C@_19BIFMLPCD@?$AAJ?$AAu?$AAl?$AAy@ 000000018003ce20     libucrt:nlsdata.obj
 0002:00011e30       ??_C@_1O@PAHLKOAC@?$AAA?$AAu?$AAg?$AAu?$AAs?$AAt@ 000000018003ce30     libucrt:nlsdata.obj
 0002:00011e40       ??_C@_1BE@DKAAMBJL@?$AAS?$AAe?$AAp?$AAt?$AAe?$AAm?$AAb?$AAe?$AAr@ 000000018003ce40     libucrt:nlsdata.obj
 0002:00011e58       ??_C@_1BA@EPANDLNG@?$AAO?$AAc?$AAt?$AAo?$AAb?$AAe?$AAr@ 000000018003ce58     libucrt:nlsdata.obj
 0002:00011e68       ??_C@_1BC@BGLIFPF@?$AAN?$AAo?$AAv?$AAe?$AAm?$AAb?$AAe?$AAr@ 000000018003ce68     libucrt:nlsdata.obj
 0002:00011e80       ??_C@_1BC@FEMKIFH@?$AAD?$AAe?$AAc?$AAe?$AAm?$AAb?$AAe?$AAr@ 000000018003ce80     libucrt:nlsdata.obj
 0002:00011e94       ??_C@_15ODEHAHHF@?$AAA?$AAM@ 000000018003ce94     libucrt:nlsdata.obj
 0002:00011e9c       ??_C@_15CLMNNGEL@?$AAP?$AAM@ 000000018003ce9c     libucrt:nlsdata.obj
 0002:00011ea8       ??_C@_1BC@IEBCMHCM@?$AAM?$AAM?$AA?1?$AAd?$AAd?$AA?1?$AAy?$AAy@ 000000018003cea8     libucrt:nlsdata.obj
 0002:00011ec0       ??_C@_1CI@KNAKOEBC@?$AAd?$AAd?$AAd?$AAd?$AA?0?$AA?5?$AAM?$AAM?$AAM?$AAM?$AA?5?$AAd?$AAd?$AA?0?$AA?5@ 000000018003cec0     libucrt:nlsdata.obj
 0002:00011ee8       ??_C@_1BC@GDGBMEMK@?$AAH?$AAH?$AA?3?$AAm?$AAm?$AA?3?$AAs?$AAs@ 000000018003cee8     libucrt:nlsdata.obj
 0002:00011f00       ??_C@_1M@BMHNFIME@?$AAe?$AAn?$AA?9?$AAU?$AAS@ 000000018003cf00     libucrt:nlsdata.obj
 0002:00011f0c       ?ccs@?1???$__acrt_stdio_parse_mode@D@@YA?AU__acrt_stdio_stream_mode@@QEBD@Z@4QBDB 000000018003cf0c     libucrt:openfile.obj
 0002:00011f10       ?utf8_encoding@?1???$__acrt_stdio_parse_mode@D@@YA?AU__acrt_stdio_stream_mode@@QEBD@Z@4QBDB 000000018003cf10     libucrt:openfile.obj
 0002:00011f18       ?utf16_encoding@?1???$__acrt_stdio_parse_mode@D@@YA?AU__acrt_stdio_stream_mode@@QEBD@Z@4QBDB 000000018003cf18     libucrt:openfile.obj
 0002:00011f20       ?unicode_encoding@?1???$__acrt_stdio_parse_mode@D@@YA?AU__acrt_stdio_stream_mode@@QEBD@Z@4QBDB 000000018003cf20     libucrt:openfile.obj
 0002:00011f48       ??_C@_1M@HPNHIDJI@?$AAj?$AAa?$AA?9?$AAJ?$AAP@ 000000018003cf48     libucrt:mbctype.obj
 0002:00011f58       ??_C@_1M@BIBDDEMK@?$AAz?$AAh?$AA?9?$AAC?$AAN@ 000000018003cf58     libucrt:mbctype.obj
 0002:00011f68       ??_C@_1M@JLOOOEGK@?$AAk?$AAo?$AA?9?$AAK?$AAR@ 000000018003cf68     libucrt:mbctype.obj
 0002:00011f78       ??_C@_1M@CLNBBOPM@?$AAz?$AAh?$AA?9?$AAT?$AAW@ 000000018003cf78     libucrt:mbctype.obj
 0002:00011f90       __newctype                 000000018003cf90     libucrt:ctype.obj
 0002:00012290       __newclmap                 000000018003d290     libucrt:ctype.obj
 0002:00012410       __newcumap                 000000018003d410     libucrt:ctype.obj
 0002:000133d0       ??_C@_15EMKDOKLE@?$AAa?$AAr@ 000000018003e3d0     libucrt:lcidtoname_downlevel.obj
 0002:000133d8       ??_C@_15KNPADPLH@?$AAb?$AAg@ 000000018003e3d8     libucrt:lcidtoname_downlevel.obj
 0002:000133e0       ??_C@_15EDMHLDMO@?$AAc?$AAa@ 000000018003e3e0     libucrt:lcidtoname_downlevel.obj
 0002:000133e8       ??_C@_1O@BPEAJADD@?$AAz?$AAh?$AA?9?$AAC?$AAH?$AAS@ 000000018003e3e8     libucrt:lcidtoname_downlevel.obj
 0002:000133f8       ??_C@_15LJNHCMNK@?$AAc?$AAs@ 000000018003e3f8     libucrt:lcidtoname_downlevel.obj
 0002:00013400       ??_C@_15FOMCIDHG@?$AAd?$AAa@ 000000018003e400     libucrt:lcidtoname_downlevel.obj
 0002:00013408       ??_C@_15NBKABECB@?$AAd?$AAe@ 000000018003e408     libucrt:lcidtoname_downlevel.obj
 0002:00013410       ??_C@_15GHPEIIAO@?$AAe?$AAl@ 000000018003e410     libucrt:lcidtoname_downlevel.obj
 0002:00013418       ??_C@_15MNPNEAIF@?$AAe?$AAn@ 000000018003e418     libucrt:lcidtoname_downlevel.obj
 0002:00013420       ??_C@_15GPIOMPMH@?$AAe?$AAs@ 000000018003e420     libucrt:lcidtoname_downlevel.obj
 0002:00013428       ??_C@_15NGLOAKJC@?$AAf?$AAi@ 000000018003e428     libucrt:lcidtoname_downlevel.obj
 0002:00013430       ??_C@_15FBKGNKAM@?$AAf?$AAr@ 000000018003e430     libucrt:lcidtoname_downlevel.obj
 0002:00013438       ??_C@_15KGGCNEFK@?$AAh?$AAe@ 000000018003e438     libucrt:lcidtoname_downlevel.obj
 0002:00013440       ??_C@_15PGHLIDMF@?$AAh?$AAu@ 000000018003e440     libucrt:lcidtoname_downlevel.obj
 0002:00013448       ??_C@_15BIEMAPLM@?$AAi?$AAs@ 000000018003e448     libucrt:lcidtoname_downlevel.obj
 0002:00013450       ??_C@_15IFJLDHAF@?$AAi?$AAt@ 000000018003e450     libucrt:lcidtoname_downlevel.obj
 0002:00013458       ??_C@_15GEMIOCAG@?$AAj?$AAa@ 000000018003e458     libucrt:lcidtoname_downlevel.obj
 0002:00013460       ??_C@_15EPELEGJA@?$AAk?$AAo@ 000000018003e460     libucrt:lcidtoname_downlevel.obj
 0002:00013468       ??_C@_15NDDHIMN@?$AAn?$AAl@ 000000018003e468     libucrt:lcidtoname_downlevel.obj
 0002:00013470       ??_C@_15BPIGNHCD@?$AAn?$AAo@ 000000018003e470     libucrt:lcidtoname_downlevel.obj
 0002:00013478       ??_C@_15DEOPBLCG@?$AAp?$AAl@ 000000018003e478     libucrt:lcidtoname_downlevel.obj
 0002:00013480       ??_C@_15KBECGEFG@?$AAp?$AAt@ 000000018003e480     libucrt:lcidtoname_downlevel.obj
 0002:00013488       ??_C@_15GLJCBFMD@?$AAr?$AAo@ 000000018003e488     libucrt:lcidtoname_downlevel.obj
 0002:00013490       ??_C@_15FEDGKCDI@?$AAr?$AAu@ 000000018003e490     libucrt:lcidtoname_downlevel.obj
 0002:00013498       ??_C@_15GLKMLLHM@?$AAh?$AAr@ 000000018003e498     libucrt:lcidtoname_downlevel.obj
 0002:000134a0       ??_C@_15CPKMFBDB@?$AAs?$AAk@ 000000018003e4a0     libucrt:lcidtoname_downlevel.obj
 0002:000134a8       ??_C@_15BAAIOGMK@?$AAs?$AAq@ 000000018003e4a8     libucrt:lcidtoname_downlevel.obj
 0002:000134b0       ??_C@_15INNPNOHD@?$AAs?$AAv@ 000000018003e4b0     libucrt:lcidtoname_downlevel.obj
 0002:000134b8       ??_C@_15CABMMOGH@?$AAt?$AAh@ 000000018003e4b8     libucrt:lcidtoname_downlevel.obj
 0002:000134c0       ??_C@_15BPLIHJJM@?$AAt?$AAr@ 000000018003e4c0     libucrt:lcidtoname_downlevel.obj
 0002:000134c8       ??_C@_15NEOEKKDJ@?$AAu?$AAr@ 000000018003e4c8     libucrt:lcidtoname_downlevel.obj
 0002:000134d0       ??_C@_15NFICGAJK@?$AAi?$AAd@ 000000018003e4d0     libucrt:lcidtoname_downlevel.obj
 0002:000134d8       ??_C@_15PJPFLCCM@?$AAu?$AAk@ 000000018003e4d8     libucrt:lcidtoname_downlevel.obj
 0002:000134e0       ??_C@_15HPJPHDM@?$AAb?$AAe@ 000000018003e4e0     libucrt:lcidtoname_downlevel.obj
 0002:000134e8       ??_C@_15LCHLGJII@?$AAs?$AAl@ 000000018003e4e8     libucrt:lcidtoname_downlevel.obj
 0002:000134f0       ??_C@_15PCFJPHHO@?$AAe?$AAt@ 000000018003e4f0     libucrt:lcidtoname_downlevel.obj
 0002:000134f8       ??_C@_15HPFPGODN@?$AAl?$AAv@ 000000018003e4f8     libucrt:lcidtoname_downlevel.obj
 0002:00013500       ??_C@_15NFFGKGLG@?$AAl?$AAt@ 000000018003e500     libucrt:lcidtoname_downlevel.obj
 0002:00013508       ??_C@_15BDAKCCHN@?$AAf?$AAa@ 000000018003e508     libucrt:lcidtoname_downlevel.obj
 0002:00013510       ??_C@_15NFGIAIAJ@?$AAv?$AAi@ 000000018003e510     libucrt:lcidtoname_downlevel.obj
 0002:00013518       ??_C@_15LMKNDMHN@?$AAh?$AAy@ 000000018003e518     libucrt:lcidtoname_downlevel.obj
 0002:00013520       ??_C@_15IJBHMCFL@?$AAa?$AAz@ 000000018003e520     libucrt:lcidtoname_downlevel.obj
 0002:00013528       ??_C@_15EKOFJABL@?$AAe?$AAu@ 000000018003e528     libucrt:lcidtoname_downlevel.obj
 0002:00013530       ??_C@_15BGHADCNK@?$AAm?$AAk@ 000000018003e530     libucrt:lcidtoname_downlevel.obj
 0002:00013538       ??_C@_15JDNICKHM@?$AAa?$AAf@ 000000018003e538     libucrt:lcidtoname_downlevel.obj
 0002:00013540       ??_C@_15KPJEDBKD@?$AAk?$AAa@ 000000018003e540     libucrt:lcidtoname_downlevel.obj
 0002:00013548       ??_C@_15PDNFFFEO@?$AAf?$AAo@ 000000018003e548     libucrt:lcidtoname_downlevel.obj
 0002:00013550       ??_C@_15OMLEGLOC@?$AAh?$AAi@ 000000018003e550     libucrt:lcidtoname_downlevel.obj
 0002:00013558       ??_C@_15IDNNENKK@?$AAm?$AAs@ 000000018003e558     libucrt:lcidtoname_downlevel.obj
 0002:00013560       ??_C@_15MACJNBMH@?$AAk?$AAk@ 000000018003e560     libucrt:lcidtoname_downlevel.obj
 0002:00013568       ??_C@_15DKDJEOND@?$AAk?$AAy@ 000000018003e568     libucrt:lcidtoname_downlevel.obj
 0002:00013570       ??_C@_15DFGDLJBG@?$AAs?$AAw@ 000000018003e570     libucrt:lcidtoname_downlevel.obj
 0002:00013578       ??_C@_15BBFAICNG@?$AAu?$AAz@ 000000018003e578     libucrt:lcidtoname_downlevel.obj
 0002:00013580       ??_C@_15DKNDCGEA@?$AAt?$AAt@ 000000018003e580     libucrt:lcidtoname_downlevel.obj
 0002:00013588       ??_C@_15MGIFMDPL@?$AAp?$AAa@ 000000018003e588     libucrt:lcidtoname_downlevel.obj
 0002:00013590       ??_C@_15HCNDBBA@?$AAg?$AAu@ 000000018003e590     libucrt:lcidtoname_downlevel.obj
 0002:00013598       ??_C@_15FNBEIBON@?$AAt?$AAa@ 000000018003e598     libucrt:lcidtoname_downlevel.obj
 0002:000135a0       ??_C@_15NCHGBGLK@?$AAt?$AAe@ 000000018003e5a0     libucrt:lcidtoname_downlevel.obj
 0002:000135a8       ??_C@_15PHPHCBPF@?$AAk?$AAn@ 000000018003e5a8     libucrt:lcidtoname_downlevel.obj
 0002:000135b0       ??_C@_15DLGBCKMP@?$AAm?$AAr@ 000000018003e5b0     libucrt:lcidtoname_downlevel.obj
 0002:000135b8       ??_C@_15EABBLBFF@?$AAs?$AAa@ 000000018003e5b8     libucrt:lcidtoname_downlevel.obj
 0002:000135c0       ??_C@_15CBKOMCOI@?$AAm?$AAn@ 000000018003e5c0     libucrt:lcidtoname_downlevel.obj
 0002:000135c8       ??_C@_15CKDMCJAF@?$AAg?$AAl@ 000000018003e5c8     libucrt:lcidtoname_downlevel.obj
 0002:000135d0       ??_C@_17CNJFBPG@?$AAk?$AAo?$AAk@ 000000018003e5d0     libucrt:lcidtoname_downlevel.obj
 0002:000135d8       ??_C@_17FFBJICPL@?$AAs?$AAy?$AAr@ 000000018003e5d8     libucrt:lcidtoname_downlevel.obj
 0002:000135e0       ??_C@_17KPNDCPAF@?$AAd?$AAi?$AAv@ 000000018003e5e0     libucrt:lcidtoname_downlevel.obj
 0002:000135e8       ??_C@_11LOCGONAA@@         000000018003e5e8     libucrt:lcidtoname_downlevel.obj
 0002:000135f0       ??_C@_1M@OKAHONE@?$AAa?$AAr?$AA?9?$AAS?$AAA@ 000000018003e5f0     libucrt:lcidtoname_downlevel.obj
 0002:00013600       ??_C@_1M@FFFIGIGK@?$AAb?$AAg?$AA?9?$AAB?$AAG@ 000000018003e600     libucrt:lcidtoname_downlevel.obj
 0002:00013610       ??_C@_1M@BJNKEDC@?$AAc?$AAa?$AA?9?$AAE?$AAS@ 000000018003e610     libucrt:lcidtoname_downlevel.obj
 0002:00013620       ??_C@_1M@IJJHFJHA@?$AAc?$AAs?$AA?9?$AAC?$AAZ@ 000000018003e620     libucrt:lcidtoname_downlevel.obj
 0002:00013630       ??_C@_1M@CLPEOBGI@?$AAd?$AAa?$AA?9?$AAD?$AAK@ 000000018003e630     libucrt:lcidtoname_downlevel.obj
 0002:00013640       ??_C@_1M@MCMADGCB@?$AAd?$AAe?$AA?9?$AAD?$AAE@ 000000018003e640     libucrt:lcidtoname_downlevel.obj
 0002:00013650       ??_C@_1M@OOCKEMAM@?$AAe?$AAl?$AA?9?$AAG?$AAR@ 000000018003e650     libucrt:lcidtoname_downlevel.obj
 0002:00013660       ??_C@_1M@DDNJFGID@?$AAf?$AAi?$AA?9?$AAF?$AAI@ 000000018003e660     libucrt:lcidtoname_downlevel.obj
 0002:00013670       ??_C@_1M@GLIPPMAC@?$AAf?$AAr?$AA?9?$AAF?$AAR@ 000000018003e670     libucrt:lcidtoname_downlevel.obj
 0002:00013680       ??_C@_1M@GFMCHPE@?$AAh?$AAe?$AA?9?$AAI?$AAL@ 000000018003e680     libucrt:lcidtoname_downlevel.obj
 0002:00013690       ??_C@_1M@MHLPGNKM@?$AAh?$AAu?$AA?9?$AAH?$AAU@ 000000018003e690     libucrt:lcidtoname_downlevel.obj
 0002:000136a0       ??_C@_1M@LPDDNNPN@?$AAi?$AAs?$AA?9?$AAI?$AAS@ 000000018003e6a0     libucrt:lcidtoname_downlevel.obj
 0002:000136b0       ??_C@_1M@MADIPODN@?$AAi?$AAt?$AA?9?$AAI?$AAT@ 000000018003e6b0     libucrt:lcidtoname_downlevel.obj
 0002:000136c0       ??_C@_1M@IHBJJGG@?$AAn?$AAl?$AA?9?$AAN?$AAL@ 000000018003e6c0     libucrt:lcidtoname_downlevel.obj
 0002:000136d0       ??_C@_1M@EANAGDL@?$AAn?$AAb?$AA?9?$AAN?$AAO@ 000000018003e6d0     libucrt:lcidtoname_downlevel.obj
 0002:000136e0       ??_C@_1M@NEIEMEGP@?$AAp?$AAl?$AA?9?$AAP?$AAL@ 000000018003e6e0     libucrt:lcidtoname_downlevel.obj
 0002:000136f0       ??_C@_1M@BOCFIGEP@?$AAp?$AAt?$AA?9?$AAB?$AAR@ 000000018003e6f0     libucrt:lcidtoname_downlevel.obj
 0002:00013700       ??_C@_1M@IMPFOPBG@?$AAr?$AAo?$AA?9?$AAR?$AAO@ 000000018003e700     libucrt:lcidtoname_downlevel.obj
 0002:00013710       ??_C@_1M@IDNNEJMM@?$AAr?$AAu?$AA?9?$AAR?$AAU@ 000000018003e710     libucrt:lcidtoname_downlevel.obj
 0002:00013720       ??_C@_1M@LILEEOGM@?$AAh?$AAr?$AA?9?$AAH?$AAR@ 000000018003e720     libucrt:lcidtoname_downlevel.obj
 0002:00013730       ??_C@_1M@FKIFEHPB@?$AAs?$AAk?$AA?9?$AAS?$AAK@ 000000018003e730     libucrt:lcidtoname_downlevel.obj
 0002:00013740       ??_C@_1M@LJMAMNPJ@?$AAs?$AAq?$AA?9?$AAA?$AAL@ 000000018003e740     libucrt:lcidtoname_downlevel.obj
 0002:00013750       ??_C@_1M@GIAKDKJK@?$AAs?$AAv?$AA?9?$AAS?$AAE@ 000000018003e750     libucrt:lcidtoname_downlevel.obj
 0002:00013760       ??_C@_1M@MKJKIKCL@?$AAt?$AAh?$AA?9?$AAT?$AAH@ 000000018003e760     libucrt:lcidtoname_downlevel.obj
 0002:00013770       ??_C@_1M@MFLCCMPB@?$AAt?$AAr?$AA?9?$AAT?$AAR@ 000000018003e770     libucrt:lcidtoname_downlevel.obj
 0002:00013780       ??_C@_1M@OIJHDKJN@?$AAu?$AAr?$AA?9?$AAP?$AAK@ 000000018003e780     libucrt:lcidtoname_downlevel.obj
 0002:00013790       ??_C@_1M@LHIPCIEK@?$AAi?$AAd?$AA?9?$AAI?$AAD@ 000000018003e790     libucrt:lcidtoname_downlevel.obj
 0002:000137a0       ??_C@_1M@MFMOBGI@?$AAu?$AAk?$AA?9?$AAU?$AAA@ 000000018003e7a0     libucrt:lcidtoname_downlevel.obj
 0002:000137b0       ??_C@_1M@OBGLJIPL@?$AAb?$AAe?$AA?9?$AAB?$AAY@ 000000018003e7b0     libucrt:lcidtoname_downlevel.obj
 0002:000137c0       ??_C@_1M@BCFAJEAD@?$AAs?$AAl?$AA?9?$AAS?$AAI@ 000000018003e7c0     libucrt:lcidtoname_downlevel.obj
 0002:000137d0       ??_C@_1M@FKFFEDDN@?$AAe?$AAt?$AA?9?$AAE?$AAE@ 000000018003e7d0     libucrt:lcidtoname_downlevel.obj
 0002:000137e0       ??_C@_1M@KGKKAACI@?$AAl?$AAv?$AA?9?$AAL?$AAV@ 000000018003e7e0     libucrt:lcidtoname_downlevel.obj
 0002:000137f0       ??_C@_1M@IFGBIJO@?$AAl?$AAt?$AA?9?$AAL?$AAT@ 000000018003e7f0     libucrt:lcidtoname_downlevel.obj
 0002:00013800       ??_C@_1M@FGEAHEDM@?$AAf?$AAa?$AA?9?$AAI?$AAR@ 000000018003e800     libucrt:lcidtoname_downlevel.obj
 0002:00013810       ??_C@_1M@KBMAIBFN@?$AAv?$AAi?$AA?9?$AAV?$AAN@ 000000018003e810     libucrt:lcidtoname_downlevel.obj
 0002:00013820       ??_C@_1M@GPCBKDJK@?$AAh?$AAy?$AA?9?$AAA?$AAM@ 000000018003e820     libucrt:lcidtoname_downlevel.obj
 0002:00013830       ??_C@_1BG@BECMDDJB@?$AAa?$AAz?$AA?9?$AAA?$AAZ?$AA?9?$AAL?$AAa?$AAt?$AAn@ 000000018003e830     libucrt:lcidtoname_downlevel.obj
 0002:00013848       ??_C@_1M@MAOFCAEA@?$AAe?$AAu?$AA?9?$AAE?$AAS@ 000000018003e848     libucrt:lcidtoname_downlevel.obj
 0002:00013858       ??_C@_1M@IGHABKPI@?$AAm?$AAk?$AA?9?$AAM?$AAK@ 000000018003e858     libucrt:lcidtoname_downlevel.obj
 0002:00013868       ??_C@_1M@IAIGNEJG@?$AAt?$AAn?$AA?9?$AAZ?$AAA@ 000000018003e868     libucrt:lcidtoname_downlevel.obj
 0002:00013878       ??_C@_1M@IIJCOJFA@?$AAx?$AAh?$AA?9?$AAZ?$AAA@ 000000018003e878     libucrt:lcidtoname_downlevel.obj
 0002:00013888       ??_C@_1M@LGPJHNJH@?$AAz?$AAu?$AA?9?$AAZ?$AAA@ 000000018003e888     libucrt:lcidtoname_downlevel.obj
 0002:00013898       ??_C@_1M@HOKAOIO@?$AAa?$AAf?$AA?9?$AAZ?$AAA@ 000000018003e898     libucrt:lcidtoname_downlevel.obj
 0002:000138a8       ??_C@_1M@DPCLHLIE@?$AAk?$AAa?$AA?9?$AAG?$AAE@ 000000018003e8a8     libucrt:lcidtoname_downlevel.obj
 0002:000138b8       ??_C@_1M@BLKMHJBI@?$AAf?$AAo?$AA?9?$AAF?$AAO@ 000000018003e8b8     libucrt:lcidtoname_downlevel.obj
 0002:000138c8       ??_C@_1M@LGGJAPPB@?$AAh?$AAi?$AA?9?$AAI?$AAN@ 000000018003e8c8     libucrt:lcidtoname_downlevel.obj
 0002:000138d8       ??_C@_1M@FIKPIHFE@?$AAm?$AAt?$AA?9?$AAM?$AAT@ 000000018003e8d8     libucrt:lcidtoname_downlevel.obj
 0002:000138e8       ??_C@_1M@HEGGPBFA@?$AAs?$AAe?$AA?9?$AAN?$AAO@ 000000018003e8e8     libucrt:lcidtoname_downlevel.obj
 0002:000138f8       ??_C@_1M@EIBJEEPA@?$AAm?$AAs?$AA?9?$AAM?$AAY@ 000000018003e8f8     libucrt:lcidtoname_downlevel.obj
 0002:00013908       ??_C@_1M@FHLBGMPP@?$AAk?$AAk?$AA?9?$AAK?$AAZ@ 000000018003e908     libucrt:lcidtoname_downlevel.obj
 0002:00013918       ??_C@_1M@NGJJLCGI@?$AAk?$AAy?$AA?9?$AAK?$AAG@ 000000018003e918     libucrt:lcidtoname_downlevel.obj
 0002:00013928       ??_C@_1M@GIENNBFC@?$AAs?$AAw?$AA?9?$AAK?$AAE@ 000000018003e928     libucrt:lcidtoname_downlevel.obj
 0002:00013938       ??_C@_1BG@NDGMJIMJ@?$AAu?$AAz?$AA?9?$AAU?$AAZ?$AA?9?$AAL?$AAa?$AAt?$AAn@ 000000018003e938     libucrt:lcidtoname_downlevel.obj
 0002:00013950       ??_C@_1M@IDCCIHBC@?$AAt?$AAt?$AA?9?$AAR?$AAU@ 000000018003e950     libucrt:lcidtoname_downlevel.obj
 0002:00013960       ??_C@_1M@LOICPMOJ@?$AAb?$AAn?$AA?9?$AAI?$AAN@ 000000018003e960     libucrt:lcidtoname_downlevel.obj
 0002:00013970       ??_C@_1M@KPKKNEAH@?$AAp?$AAa?$AA?9?$AAI?$AAN@ 000000018003e970     libucrt:lcidtoname_downlevel.obj
 0002:00013980       ??_C@_1M@PJGPPBOG@?$AAg?$AAu?$AA?9?$AAI?$AAN@ 000000018003e980     libucrt:lcidtoname_downlevel.obj
 0002:00013990       ??_C@_1M@KMKMOPHI@?$AAt?$AAa?$AA?9?$AAI?$AAN@ 000000018003e990     libucrt:lcidtoname_downlevel.obj
 0002:000139a0       ??_C@_1M@KFEHEPAC@?$AAt?$AAe?$AA?9?$AAI?$AAN@ 000000018003e9a0     libucrt:lcidtoname_downlevel.obj
 0002:000139b0       ??_C@_1M@CDCLMGHI@?$AAk?$AAn?$AA?9?$AAI?$AAN@ 000000018003e9b0     libucrt:lcidtoname_downlevel.obj
 0002:000139c0       ??_C@_1M@MIODLDKF@?$AAm?$AAl?$AA?9?$AAI?$AAN@ 000000018003e9c0     libucrt:lcidtoname_downlevel.obj
 0002:000139d0       ??_C@_1M@PBIEACPO@?$AAm?$AAr?$AA?9?$AAI?$AAN@ 000000018003e9d0     libucrt:lcidtoname_downlevel.obj
 0002:000139e0       ??_C@_1M@NIDEAGPH@?$AAs?$AAa?$AA?9?$AAI?$AAN@ 000000018003e9e0     libucrt:lcidtoname_downlevel.obj
 0002:000139f0       ??_C@_1M@FHIHCBIO@?$AAm?$AAn?$AA?9?$AAM?$AAN@ 000000018003e9f0     libucrt:lcidtoname_downlevel.obj
 0002:00013a00       ??_C@_1M@JAIJPENP@?$AAc?$AAy?$AA?9?$AAG?$AAB@ 000000018003ea00     libucrt:lcidtoname_downlevel.obj
 0002:00013a10       ??_C@_1M@PHGFBEPN@?$AAg?$AAl?$AA?9?$AAE?$AAS@ 000000018003ea10     libucrt:lcidtoname_downlevel.obj
 0002:00013a20       ??_C@_1O@KPIPDNCP@?$AAk?$AAo?$AAk?$AA?9?$AAI?$AAN@ 000000018003ea20     libucrt:lcidtoname_downlevel.obj
 0002:00013a30       ??_C@_1O@KNHJLDJA@?$AAs?$AAy?$AAr?$AA?9?$AAS?$AAY@ 000000018003ea30     libucrt:lcidtoname_downlevel.obj
 0002:00013a40       ??_C@_1O@MKEKBLAH@?$AAd?$AAi?$AAv?$AA?9?$AAM?$AAV@ 000000018003ea40     libucrt:lcidtoname_downlevel.obj
 0002:00013a50       ??_C@_1O@OHDCKDDF@?$AAq?$AAu?$AAz?$AA?9?$AAB?$AAO@ 000000018003ea50     libucrt:lcidtoname_downlevel.obj
 0002:00013a60       ??_C@_1M@LEPJNLFD@?$AAn?$AAs?$AA?9?$AAZ?$AAA@ 000000018003ea60     libucrt:lcidtoname_downlevel.obj
 0002:00013a70       ??_C@_1M@OMLEIIJB@?$AAm?$AAi?$AA?9?$AAN?$AAZ@ 000000018003ea70     libucrt:lcidtoname_downlevel.obj
 0002:00013a80       ??_C@_1M@PMPEAILG@?$AAa?$AAr?$AA?9?$AAI?$AAQ@ 000000018003ea80     libucrt:lcidtoname_downlevel.obj
 0002:00013a90       ??_C@_1M@CNKPNOEE@?$AAd?$AAe?$AA?9?$AAC?$AAH@ 000000018003ea90     libucrt:lcidtoname_downlevel.obj
 0002:00013aa0       ??_C@_1M@LKMGMLKO@?$AAe?$AAn?$AA?9?$AAG?$AAB@ 000000018003eaa0     libucrt:lcidtoname_downlevel.obj
 0002:00013ab0       ??_C@_1M@PGKJFFGL@?$AAe?$AAs?$AA?9?$AAM?$AAX@ 000000018003eab0     libucrt:lcidtoname_downlevel.obj
 0002:00013ac0       ??_C@_1M@DNNANBDC@?$AAf?$AAr?$AA?9?$AAB?$AAE@ 000000018003eac0     libucrt:lcidtoname_downlevel.obj
 0002:00013ad0       ??_C@_1M@HLGMDFHM@?$AAi?$AAt?$AA?9?$AAC?$AAH@ 000000018003ead0     libucrt:lcidtoname_downlevel.obj
 0002:00013ae0       ??_C@_1M@CLLBGJH@?$AAn?$AAl?$AA?9?$AAB?$AAE@ 000000018003eae0     libucrt:lcidtoname_downlevel.obj
 0002:00013af0       ??_C@_1M@BODBOGLF@?$AAn?$AAn?$AA?9?$AAN?$AAO@ 000000018003eaf0     libucrt:lcidtoname_downlevel.obj
 0002:00013b00       ??_C@_1M@HFFAHKAD@?$AAp?$AAt?$AA?9?$AAP?$AAT@ 000000018003eb00     libucrt:lcidtoname_downlevel.obj
 0002:00013b10       ??_C@_1BG@LNOAKHIE@?$AAs?$AAr?$AA?9?$AAS?$AAP?$AA?9?$AAL?$AAa?$AAt?$AAn@ 000000018003eb10     libucrt:lcidtoname_downlevel.obj
 0002:00013b28       ??_C@_1M@HBMHBGAK@?$AAs?$AAv?$AA?9?$AAF?$AAI@ 000000018003eb28     libucrt:lcidtoname_downlevel.obj
 0002:00013b38       ??_C@_1BG@DGCJGJBE@?$AAa?$AAz?$AA?9?$AAA?$AAZ?$AA?9?$AAC?$AAy?$AAr?$AAl@ 000000018003eb38     libucrt:lcidtoname_downlevel.obj
 0002:00013b50       ??_C@_1M@KEJDAAHB@?$AAs?$AAe?$AA?9?$AAS?$AAE@ 000000018003eb50     libucrt:lcidtoname_downlevel.obj
 0002:00013b60       ??_C@_1M@HEIBJJAD@?$AAm?$AAs?$AA?9?$AAB?$AAN@ 000000018003eb60     libucrt:lcidtoname_downlevel.obj
 0002:00013b70       ??_C@_1BG@PBGJMCEM@?$AAu?$AAz?$AA?9?$AAU?$AAZ?$AA?9?$AAC?$AAy?$AAr?$AAl@ 000000018003eb70     libucrt:lcidtoname_downlevel.obj
 0002:00013b88       ??_C@_1O@LAOBCMDF@?$AAq?$AAu?$AAz?$AA?9?$AAE?$AAC@ 000000018003eb88     libucrt:lcidtoname_downlevel.obj
 0002:00013b98       ??_C@_1M@POEEMAIO@?$AAa?$AAr?$AA?9?$AAE?$AAG@ 000000018003eb98     libucrt:lcidtoname_downlevel.obj
 0002:00013ba8       ??_C@_1M@EFAKDEDL@?$AAz?$AAh?$AA?9?$AAH?$AAK@ 000000018003eba8     libucrt:lcidtoname_downlevel.obj
 0002:00013bb8       ??_C@_1M@HKKIJHGI@?$AAd?$AAe?$AA?9?$AAA?$AAT@ 000000018003ebb8     libucrt:lcidtoname_downlevel.obj
 0002:00013bc8       ??_C@_1M@KBFBEHJF@?$AAe?$AAn?$AA?9?$AAA?$AAU@ 000000018003ebc8     libucrt:lcidtoname_downlevel.obj
 0002:00013bd8       ??_C@_1M@MNPLFAAH@?$AAe?$AAs?$AA?9?$AAE?$AAS@ 000000018003ebd8     libucrt:lcidtoname_downlevel.obj
 0002:00013be8       ??_C@_1M@HJOOJFMA@?$AAf?$AAr?$AA?9?$AAC?$AAA@ 000000018003ebe8     libucrt:lcidtoname_downlevel.obj
 0002:00013bf8       ??_C@_1BG@JPOFPNAB@?$AAs?$AAr?$AA?9?$AAS?$AAP?$AA?9?$AAC?$AAy?$AAr?$AAl@ 000000018003ebf8     libucrt:lcidtoname_downlevel.obj
 0002:00013c10       ??_C@_1M@LNFOCMOB@?$AAs?$AAe?$AA?9?$AAF?$AAI@ 000000018003ec10     libucrt:lcidtoname_downlevel.obj
 0002:00013c20       ??_C@_1O@MGJBOAMB@?$AAq?$AAu?$AAz?$AA?9?$AAP?$AAE@ 000000018003ec20     libucrt:lcidtoname_downlevel.obj
 0002:00013c30       ??_C@_1M@GJINLBOK@?$AAa?$AAr?$AA?9?$AAL?$AAY@ 000000018003ec30     libucrt:lcidtoname_downlevel.obj
 0002:00013c40       ??_C@_1M@GGMNHJNL@?$AAz?$AAh?$AA?9?$AAS?$AAG@ 000000018003ec40     libucrt:lcidtoname_downlevel.obj
 0002:00013c50       ??_C@_1M@HOIKODND@?$AAd?$AAe?$AA?9?$AAL?$AAU@ 000000018003ec50     libucrt:lcidtoname_downlevel.obj
 0002:00013c60       ??_C@_1M@DDOCCGFG@?$AAe?$AAn?$AA?9?$AAC?$AAA@ 000000018003ec60     libucrt:lcidtoname_downlevel.obj
 0002:00013c70       ??_C@_1M@BNOEMJLF@?$AAe?$AAs?$AA?9?$AAG?$AAT@ 000000018003ec70     libucrt:lcidtoname_downlevel.obj
 0002:00013c80       ??_C@_1M@EOGNKEK@?$AAf?$AAr?$AA?9?$AAC?$AAH@ 000000018003ec80     libucrt:lcidtoname_downlevel.obj
 0002:00013c90       ??_C@_1M@FLIDJFHL@?$AAh?$AAr?$AA?9?$AAB?$AAA@ 000000018003ec90     libucrt:lcidtoname_downlevel.obj
 0002:00013ca0       ??_C@_1O@FMCELNAJ@?$AAs?$AAm?$AAj?$AA?9?$AAN?$AAO@ 000000018003eca0     libucrt:lcidtoname_downlevel.obj
 0002:00013cb0       ??_C@_1M@JHGLJMGJ@?$AAa?$AAr?$AA?9?$AAD?$AAZ@ 000000018003ecb0     libucrt:lcidtoname_downlevel.obj
 0002:00013cc0       ??_C@_1M@JKKFDCNP@?$AAz?$AAh?$AA?9?$AAM?$AAO@ 000000018003ecc0     libucrt:lcidtoname_downlevel.obj
 0002:00013cd0       ??_C@_1M@GEEFALPE@?$AAd?$AAe?$AA?9?$AAL?$AAI@ 000000018003ecd0     libucrt:lcidtoname_downlevel.obj
 0002:00013ce0       ??_C@_1M@IGEOFBG@?$AAe?$AAn?$AA?9?$AAN?$AAZ@ 000000018003ece0     libucrt:lcidtoname_downlevel.obj
 0002:00013cf0       ??_C@_1M@KDBONEHP@?$AAe?$AAs?$AA?9?$AAC?$AAR@ 000000018003ecf0     libucrt:lcidtoname_downlevel.obj
 0002:00013d00       ??_C@_1M@FHMDOHNN@?$AAf?$AAr?$AA?9?$AAL?$AAU@ 000000018003ed00     libucrt:lcidtoname_downlevel.obj
 0002:00013d10       ??_C@_1BG@NFKKMAFG@?$AAb?$AAs?$AA?9?$AAB?$AAA?$AA?9?$AAL?$AAa?$AAt?$AAn@ 000000018003ed10     libucrt:lcidtoname_downlevel.obj
 0002:00013d28       ??_C@_1O@IMNBEMCI@?$AAs?$AAm?$AAj?$AA?9?$AAS?$AAE@ 000000018003ed28     libucrt:lcidtoname_downlevel.obj
 0002:00013d38       ??_C@_1M@DHHMBNDP@?$AAa?$AAr?$AA?9?$AAM?$AAA@ 000000018003ed38     libucrt:lcidtoname_downlevel.obj
 0002:00013d48       ??_C@_1M@BNBLJCGH@?$AAe?$AAn?$AA?9?$AAI?$AAE@ 000000018003ed48     libucrt:lcidtoname_downlevel.obj
 0002:00013d58       ??_C@_1M@GEPAFMDL@?$AAe?$AAs?$AA?9?$AAP?$AAA@ 000000018003ed58     libucrt:lcidtoname_downlevel.obj
 0002:00013d68       ??_C@_1M@OJONDMDL@?$AAf?$AAr?$AA?9?$AAM?$AAC@ 000000018003ed68     libucrt:lcidtoname_downlevel.obj
 0002:00013d78       ??_C@_1BG@OBCNFJB@?$AAs?$AAr?$AA?9?$AAB?$AAA?$AA?9?$AAL?$AAa?$AAt?$AAn@ 000000018003ed78     libucrt:lcidtoname_downlevel.obj
 0002:00013d90       ??_C@_1O@KEMEEGPO@?$AAs?$AAm?$AAa?$AA?9?$AAN?$AAO@ 000000018003ed90     libucrt:lcidtoname_downlevel.obj
 0002:00013da0       ??_C@_1M@ELMGFODK@?$AAa?$AAr?$AA?9?$AAT?$AAN@ 000000018003eda0     libucrt:lcidtoname_downlevel.obj
 0002:00013db0       ??_C@_1M@BHDLHFAF@?$AAe?$AAn?$AA?9?$AAZ?$AAA@ 000000018003edb0     libucrt:lcidtoname_downlevel.obj
 0002:00013dc0       ??_C@_1M@BMGIGLIF@?$AAe?$AAs?$AA?9?$AAD?$AAO@ 000000018003edc0     libucrt:lcidtoname_downlevel.obj
 0002:00013dd0       ??_C@_1BG@CMBHIPBE@?$AAs?$AAr?$AA?9?$AAB?$AAA?$AA?9?$AAC?$AAy?$AAr?$AAl@ 000000018003edd0     libucrt:lcidtoname_downlevel.obj
 0002:00013de8       ??_C@_1O@HEDBLHNP@?$AAs?$AAm?$AAa?$AA?9?$AAS?$AAE@ 000000018003ede8     libucrt:lcidtoname_downlevel.obj
 0002:00013df8       ??_C@_1M@DAGCADIM@?$AAa?$AAr?$AA?9?$AAO?$AAM@ 000000018003edf8     libucrt:lcidtoname_downlevel.obj
 0002:00013e08       ??_C@_1M@FODLMICG@?$AAe?$AAn?$AA?9?$AAJ?$AAM@ 000000018003ee08     libucrt:lcidtoname_downlevel.obj
 0002:00013e18       ??_C@_1M@DNMLCIHB@?$AAe?$AAs?$AA?9?$AAV?$AAE@ 000000018003ee18     libucrt:lcidtoname_downlevel.obj
 0002:00013e28       ??_C@_1O@EOKHMKJK@?$AAs?$AAm?$AAs?$AA?9?$AAF?$AAI@ 000000018003ee28     libucrt:lcidtoname_downlevel.obj
 0002:00013e38       ??_C@_1M@CAFJMKOF@?$AAa?$AAr?$AA?9?$AAY?$AAE@ 000000018003ee38     libucrt:lcidtoname_downlevel.obj
 0002:00013e48       ??_C@_1M@CBFHIJLI@?$AAe?$AAn?$AA?9?$AAC?$AAB@ 000000018003ee48     libucrt:lcidtoname_downlevel.obj
 0002:00013e58       ??_C@_1M@BGNFLDN@?$AAe?$AAs?$AA?9?$AAC?$AAO@ 000000018003ee58     libucrt:lcidtoname_downlevel.obj
 0002:00013e68       ??_C@_1O@JMPHMAMC@?$AAs?$AAm?$AAn?$AA?9?$AAF?$AAI@ 000000018003ee68     libucrt:lcidtoname_downlevel.obj
 0002:00013e78       ??_C@_1M@JLANABKE@?$AAa?$AAr?$AA?9?$AAS?$AAY@ 000000018003ee78     libucrt:lcidtoname_downlevel.obj
 0002:00013e88       ??_C@_1M@HPKGCFGN@?$AAe?$AAn?$AA?9?$AAB?$AAZ@ 000000018003ee88     libucrt:lcidtoname_downlevel.obj
 0002:00013e98       ??_C@_1M@OLJCMLGM@?$AAe?$AAs?$AA?9?$AAP?$AAE@ 000000018003ee98     libucrt:lcidtoname_downlevel.obj
 0002:00013ea8       ??_C@_1M@MKKGFKLE@?$AAa?$AAr?$AA?9?$AAJ?$AAO@ 000000018003eea8     libucrt:lcidtoname_downlevel.obj
 0002:00013eb8       ??_C@_1M@EKPGLDNI@?$AAe?$AAn?$AA?9?$AAT?$AAT@ 000000018003eeb8     libucrt:lcidtoname_downlevel.obj
 0002:00013ec8       ??_C@_1M@OONGHFHE@?$AAe?$AAs?$AA?9?$AAA?$AAR@ 000000018003eec8     libucrt:lcidtoname_downlevel.obj
 0002:00013ed8       ??_C@_1M@OOJFGBHE@?$AAa?$AAr?$AA?9?$AAL?$AAB@ 000000018003eed8     libucrt:lcidtoname_downlevel.obj
 0002:00013ee8       ??_C@_1M@GCEJHNEG@?$AAe?$AAn?$AA?9?$AAZ?$AAW@ 000000018003eee8     libucrt:lcidtoname_downlevel.obj
 0002:00013ef8       ??_C@_1M@JNOCAHJI@?$AAe?$AAs?$AA?9?$AAE?$AAC@ 000000018003eef8     libucrt:lcidtoname_downlevel.obj
 0002:00013f08       ??_C@_1M@JEFHPGGB@?$AAa?$AAr?$AA?9?$AAK?$AAW@ 000000018003ef08     libucrt:lcidtoname_downlevel.obj
 0002:00013f18       ??_C@_1M@MLKIBJOJ@?$AAe?$AAn?$AA?9?$AAP?$AAH@ 000000018003ef18     libucrt:lcidtoname_downlevel.obj
 0002:00013f28       ??_C@_1M@BDNIPEND@?$AAe?$AAs?$AA?9?$AAC?$AAL@ 000000018003ef28     libucrt:lcidtoname_downlevel.obj
 0002:00013f38       ??_C@_1M@MPNMEKBD@?$AAa?$AAr?$AA?9?$AAA?$AAE@ 000000018003ef38     libucrt:lcidtoname_downlevel.obj
 0002:00013f48       ??_C@_1M@KBJALCPI@?$AAe?$AAs?$AA?9?$AAU?$AAY@ 000000018003ef48     libucrt:lcidtoname_downlevel.obj
 0002:00013f58       ??_C@_1M@LLCCOAGA@?$AAa?$AAr?$AA?9?$AAB?$AAH@ 000000018003ef58     libucrt:lcidtoname_downlevel.obj
 0002:00013f68       ??_C@_1M@PBFNCDEL@?$AAe?$AAs?$AA?9?$AAP?$AAY@ 000000018003ef68     libucrt:lcidtoname_downlevel.obj
 0002:00013f78       ??_C@_1M@EDGINPNP@?$AAa?$AAr?$AA?9?$AAQ?$AAA@ 000000018003ef78     libucrt:lcidtoname_downlevel.obj
 0002:00013f88       ??_C@_1M@MKDBIIJI@?$AAe?$AAs?$AA?9?$AAB?$AAO@ 000000018003ef88     libucrt:lcidtoname_downlevel.obj
 0002:00013f98       ??_C@_1M@CPKKEBLD@?$AAe?$AAs?$AA?9?$AAS?$AAV@ 000000018003ef98     libucrt:lcidtoname_downlevel.obj
 0002:00013fa8       ??_C@_1M@NDBGMMJL@?$AAe?$AAs?$AA?9?$AAH?$AAN@ 000000018003efa8     libucrt:lcidtoname_downlevel.obj
 0002:00013fb8       ??_C@_1M@JIJIBHDP@?$AAe?$AAs?$AA?9?$AAN?$AAI@ 000000018003efb8     libucrt:lcidtoname_downlevel.obj
 0002:00013fc8       ??_C@_1M@CGFMKEEK@?$AAe?$AAs?$AA?9?$AAP?$AAR@ 000000018003efc8     libucrt:lcidtoname_downlevel.obj
 0002:00013fd8       ??_C@_1O@ICJHKIIK@?$AAz?$AAh?$AA?9?$AAC?$AAH?$AAT@ 000000018003efd8     libucrt:lcidtoname_downlevel.obj
 0002:00013fe8       ??_C@_15CLNEJCE@?$AAs?$AAr@ 000000018003efe8     libucrt:lcidtoname_downlevel.obj
 0002:00014e30       ??_C@_1M@KAHEKEIG@?$AAa?$AAf?$AA?9?$AAz?$AAa@ 000000018003fe30     libucrt:lcidtoname_downlevel.obj
 0002:00014e40       ??_C@_1M@GIECOABL@?$AAa?$AAr?$AA?9?$AAa?$AAe@ 000000018003fe40     libucrt:lcidtoname_downlevel.obj
 0002:00014e50       ??_C@_1M@BMLMEKGI@?$AAa?$AAr?$AA?9?$AAb?$AAh@ 000000018003fe50     libucrt:lcidtoname_downlevel.obj
 0002:00014e60       ??_C@_1M@DAPFDGGB@?$AAa?$AAr?$AA?9?$AAd?$AAz@ 000000018003fe60     libucrt:lcidtoname_downlevel.obj
 0002:00014e70       ??_C@_1M@FJNKGKIG@?$AAa?$AAr?$AA?9?$AAe?$AAg@ 000000018003fe70     libucrt:lcidtoname_downlevel.obj
 0002:00014e80       ??_C@_1M@FLGKKCLO@?$AAa?$AAr?$AA?9?$AAi?$AAq@ 000000018003fe80     libucrt:lcidtoname_downlevel.obj
 0002:00014e90       ??_C@_1M@GNDIPALM@?$AAa?$AAr?$AA?9?$AAj?$AAo@ 000000018003fe90     libucrt:lcidtoname_downlevel.obj
 0002:00014ea0       ??_C@_1M@DDMJFMGJ@?$AAa?$AAr?$AA?9?$AAk?$AAw@ 000000018003fea0     libucrt:lcidtoname_downlevel.obj
 0002:00014eb0       ??_C@_1M@EJALMLHM@?$AAa?$AAr?$AA?9?$AAl?$AAb@ 000000018003feb0     libucrt:lcidtoname_downlevel.obj
 0002:00014ec0       ??_C@_1M@MOBDBLOC@?$AAa?$AAr?$AA?9?$AAl?$AAy@ 000000018003fec0     libucrt:lcidtoname_downlevel.obj
 0002:00014ed0       ??_C@_1M@JAOCLHDH@?$AAa?$AAr?$AA?9?$AAm?$AAa@ 000000018003fed0     libucrt:lcidtoname_downlevel.obj
 0002:00014ee0       ??_C@_1M@JHPMKJIE@?$AAa?$AAr?$AA?9?$AAo?$AAm@ 000000018003fee0     libucrt:lcidtoname_downlevel.obj
 0002:00014ef0       ??_C@_1M@OEPGHFNH@?$AAa?$AAr?$AA?9?$AAq?$AAa@ 000000018003fef0     libucrt:lcidtoname_downlevel.obj
 0002:00014f00       ??_C@_1M@KJDONENM@?$AAa?$AAr?$AA?9?$AAs?$AAa@ 000000018003ff00     libucrt:lcidtoname_downlevel.obj
 0002:00014f10       ??_C@_1M@DMJDKLKM@?$AAa?$AAr?$AA?9?$AAs?$AAy@ 000000018003ff10     libucrt:lcidtoname_downlevel.obj
 0002:00014f20       ??_C@_1M@OMFIPEDC@?$AAa?$AAr?$AA?9?$AAt?$AAn@ 000000018003ff20     libucrt:lcidtoname_downlevel.obj
 0002:00014f30       ??_C@_1M@IHMHGAON@?$AAa?$AAr?$AA?9?$AAy?$AAe@ 000000018003ff30     libucrt:lcidtoname_downlevel.obj
 0002:00014f40       ??_C@_1BG@KDCPGJGB@?$AAa?$AAz?$AA?9?$AAa?$AAz?$AA?9?$AAc?$AAy?$AAr?$AAl@ 000000018003ff40     libucrt:lcidtoname_downlevel.obj
 0002:00014f58       ??_C@_1BG@IBCKDDOE@?$AAa?$AAz?$AA?9?$AAa?$AAz?$AA?9?$AAl?$AAa?$AAt?$AAn@ 000000018003ff58     libucrt:lcidtoname_downlevel.obj
 0002:00014f70       ??_C@_1M@EGPFDCPD@?$AAb?$AAe?$AA?9?$AAb?$AAy@ 000000018003ff70     libucrt:lcidtoname_downlevel.obj
 0002:00014f80       ??_C@_1M@PCMGMCGC@?$AAb?$AAg?$AA?9?$AAb?$AAg@ 000000018003ff80     libucrt:lcidtoname_downlevel.obj
 0002:00014f90       ??_C@_1M@BJBMFGOB@?$AAb?$AAn?$AA?9?$AAi?$AAn@ 000000018003ff90     libucrt:lcidtoname_downlevel.obj
 0002:00014fa0       ??_C@_1BG@EAKMMACD@?$AAb?$AAs?$AA?9?$AAb?$AAa?$AA?9?$AAl?$AAa?$AAt?$AAn@ 000000018003ffa0     libucrt:lcidtoname_downlevel.obj
 0002:00014fb8       ??_C@_1M@KGADAODK@?$AAc?$AAa?$AA?9?$AAe?$AAs@ 000000018003ffb8     libucrt:lcidtoname_downlevel.obj
 0002:00014fc8       ??_C@_1M@COAJPDHI@?$AAc?$AAs?$AA?9?$AAc?$AAz@ 000000018003ffc8     libucrt:lcidtoname_downlevel.obj
 0002:00014fd8       ??_C@_1M@DHBHFONH@?$AAc?$AAy?$AA?9?$AAg?$AAb@ 000000018003ffd8     libucrt:lcidtoname_downlevel.obj
 0002:00014fe8       ??_C@_1M@IMGKELGA@?$AAd?$AAa?$AA?9?$AAd?$AAk@ 000000018003ffe8     libucrt:lcidtoname_downlevel.obj
 0002:00014ff8       ??_C@_1M@NNDGDNGA@?$AAd?$AAe?$AA?9?$AAa?$AAt@ 000000018003fff8     libucrt:lcidtoname_downlevel.obj
 0002:00015008       ??_C@_1M@IKDBHEEM@?$AAd?$AAe?$AA?9?$AAc?$AAh@ 0000000180040008     libucrt:lcidtoname_downlevel.obj
 0002:00015018       ??_C@_1M@GFFOJMCJ@?$AAd?$AAe?$AA?9?$AAd?$AAe@ 0000000180040018     libucrt:lcidtoname_downlevel.obj
 0002:00015028       ??_C@_1M@MDNLKBPM@?$AAd?$AAe?$AA?9?$AAl?$AAi@ 0000000180040028     libucrt:lcidtoname_downlevel.obj
 0002:00015038       ??_C@_1M@NJBEEJNL@?$AAd?$AAe?$AA?9?$AAl?$AAu@ 0000000180040038     libucrt:lcidtoname_downlevel.obj
 0002:00015048       ??_C@_1O@GNNELBAP@?$AAd?$AAi?$AAv?$AA?9?$AAm?$AAv@ 0000000180040048     libucrt:lcidtoname_downlevel.obj
 0002:00015058       ??_C@_1M@EJLEOGAE@?$AAe?$AAl?$AA?9?$AAg?$AAr@ 0000000180040058     libucrt:lcidtoname_downlevel.obj
 0002:00015068       ??_C@_1M@GMPONJN@?$AAe?$AAn?$AA?9?$AAa?$AAu@ 0000000180040068     libucrt:lcidtoname_downlevel.obj
 0002:00015078       ??_C@_1M@NIDIIPGF@?$AAe?$AAn?$AA?9?$AAb?$AAz@ 0000000180040078     libucrt:lcidtoname_downlevel.obj
 0002:00015088       ??_C@_1M@JEHMIMFO@?$AAe?$AAn?$AA?9?$AAc?$AAa@ 0000000180040088     libucrt:lcidtoname_downlevel.obj
 0002:00015098       ??_C@_1M@IGMJCDLA@?$AAe?$AAn?$AA?9?$AAc?$AAb@ 0000000180040098     libucrt:lcidtoname_downlevel.obj
 0002:000150a8       ??_C@_1M@BNFIGBKG@?$AAe?$AAn?$AA?9?$AAg?$AAb@ 00000001800400a8     libucrt:lcidtoname_downlevel.obj
 0002:000150b8       ??_C@_1M@LKIFDIGP@?$AAe?$AAn?$AA?9?$AAi?$AAe@ 00000001800400b8     libucrt:lcidtoname_downlevel.obj
 0002:000150c8       ??_C@_1M@PJKFGCCO@?$AAe?$AAn?$AA?9?$AAj?$AAm@ 00000001800400c8     libucrt:lcidtoname_downlevel.obj
 0002:000150d8       ??_C@_1M@KPPKEPBO@?$AAe?$AAn?$AA?9?$AAn?$AAz@ 00000001800400d8     libucrt:lcidtoname_downlevel.obj
 0002:000150e8       ??_C@_1M@GMDGLDOB@?$AAe?$AAn?$AA?9?$AAp?$AAh@ 00000001800400e8     libucrt:lcidtoname_downlevel.obj
 0002:000150f8       ??_C@_1M@ONGIBJNA@?$AAe?$AAn?$AA?9?$AAt?$AAt@ 00000001800400f8     libucrt:lcidtoname_downlevel.obj
 0002:00015108       ??_C@_1M@LLODPCMM@?$AAe?$AAn?$AA?9?$AAu?$AAs@ 0000000180040108     libucrt:lcidtoname_downlevel.obj
 0002:00015118       ??_C@_1M@LAKFNPAN@?$AAe?$AAn?$AA?9?$AAz?$AAa@ 0000000180040118     libucrt:lcidtoname_downlevel.obj
 0002:00015128       ??_C@_1M@MFNHNHEO@?$AAe?$AAn?$AA?9?$AAz?$AAw@ 0000000180040128     libucrt:lcidtoname_downlevel.obj
 0002:00015138       ??_C@_1M@EJEINPHM@?$AAe?$AAs?$AA?9?$AAa?$AAr@ 0000000180040138     libucrt:lcidtoname_downlevel.obj
 0002:00015148       ??_C@_1M@GNKPCCJA@?$AAe?$AAs?$AA?9?$AAb?$AAo@ 0000000180040148     libucrt:lcidtoname_downlevel.obj
 0002:00015158       ??_C@_1M@LEEGFONL@?$AAe?$AAs?$AA?9?$AAc?$AAl@ 0000000180040158     libucrt:lcidtoname_downlevel.obj
 0002:00015168       ??_C@_1M@KGPDPBDF@?$AAe?$AAs?$AA?9?$AAc?$AAo@ 0000000180040168     libucrt:lcidtoname_downlevel.obj
 0002:00015178       ??_C@_1M@EIAHOHH@?$AAe?$AAs?$AA?9?$AAc?$AAr@ 0000000180040178     libucrt:lcidtoname_downlevel.obj
 0002:00015188       ??_C@_1M@LLPGMBIN@?$AAe?$AAs?$AA?9?$AAd?$AAo@ 0000000180040188     libucrt:lcidtoname_downlevel.obj
 0002:00015198       ??_C@_1M@DKHMKNJA@?$AAe?$AAs?$AA?9?$AAe?$AAc@ 0000000180040198     libucrt:lcidtoname_downlevel.obj
 0002:000151a8       ??_C@_1M@GKGFPKAP@?$AAe?$AAs?$AA?9?$AAe?$AAs@ 00000001800401a8     libucrt:lcidtoname_downlevel.obj
 0002:000151b8       ??_C@_1M@LKHKGDLN@?$AAe?$AAs?$AA?9?$AAg?$AAt@ 00000001800401b8     libucrt:lcidtoname_downlevel.obj
 0002:000151c8       ??_C@_1M@HEIIGGJD@?$AAe?$AAs?$AA?9?$AAh?$AAn@ 00000001800401c8     libucrt:lcidtoname_downlevel.obj
 0002:000151d8       ??_C@_1M@FBDHPPGD@?$AAe?$AAs?$AA?9?$AAm?$AAx@ 00000001800401d8     libucrt:lcidtoname_downlevel.obj
 0002:000151e8       ??_C@_1M@DPAGLNDH@?$AAe?$AAs?$AA?9?$AAn?$AAi@ 00000001800401e8     libucrt:lcidtoname_downlevel.obj
 0002:000151f8       ??_C@_1M@MDGOPGDD@?$AAe?$AAs?$AA?9?$AAp?$AAa@ 00000001800401f8     libucrt:lcidtoname_downlevel.obj
 0002:00015208       ??_C@_1M@EMAMGBGE@?$AAe?$AAs?$AA?9?$AAp?$AAe@ 0000000180040208     libucrt:lcidtoname_downlevel.obj
 0002:00015218       ??_C@_1M@IBMCAOEC@?$AAe?$AAs?$AA?9?$AAp?$AAr@ 0000000180040218     libucrt:lcidtoname_downlevel.obj
 0002:00015228       ??_C@_1M@FGMDIJED@?$AAe?$AAs?$AA?9?$AAp?$AAy@ 0000000180040228     libucrt:lcidtoname_downlevel.obj
 0002:00015238       ??_C@_1M@IIDEOLLL@?$AAe?$AAs?$AA?9?$AAs?$AAv@ 0000000180040238     libucrt:lcidtoname_downlevel.obj
 0002:00015248       ??_C@_1M@GAOBIPA@?$AAe?$AAs?$AA?9?$AAu?$AAy@ 0000000180040248     libucrt:lcidtoname_downlevel.obj
 0002:00015258       ??_C@_1M@JKFFICHJ@?$AAe?$AAs?$AA?9?$AAv?$AAe@ 0000000180040258     libucrt:lcidtoname_downlevel.obj
 0002:00015268       ??_C@_1M@PNMLOJDF@?$AAe?$AAt?$AA?9?$AAe?$AAe@ 0000000180040268     libucrt:lcidtoname_downlevel.obj
 0002:00015278       ??_C@_1M@GHHLIKEI@?$AAe?$AAu?$AA?9?$AAe?$AAs@ 0000000180040278     libucrt:lcidtoname_downlevel.obj
 0002:00015288       ??_C@_1M@PBNONODE@?$AAf?$AAa?$AA?9?$AAi?$AAr@ 0000000180040288     libucrt:lcidtoname_downlevel.obj
 0002:00015298       ??_C@_1M@JEEHPMIL@?$AAf?$AAi?$AA?9?$AAf?$AAi@ 0000000180040298     libucrt:lcidtoname_downlevel.obj
 0002:000152a8       ??_C@_1M@LMDCNDBA@?$AAf?$AAo?$AA?9?$AAf?$AAo@ 00000001800402a8     libucrt:lcidtoname_downlevel.obj
 0002:000152b8       ??_C@_1M@JKEOHLDK@?$AAf?$AAr?$AA?9?$AAb?$AAe@ 00000001800402b8     libucrt:lcidtoname_downlevel.obj
 0002:000152c8       ??_C@_1M@NOHADPMI@?$AAf?$AAr?$AA?9?$AAc?$AAa@ 00000001800402c8     libucrt:lcidtoname_downlevel.obj
 0002:000152d8       ??_C@_1M@KDHIHAEC@?$AAf?$AAr?$AA?9?$AAc?$AAh@ 00000001800402d8     libucrt:lcidtoname_downlevel.obj
 0002:000152e8       ??_C@_1M@MMBBFGAK@?$AAf?$AAr?$AA?9?$AAf?$AAr@ 00000001800402e8     libucrt:lcidtoname_downlevel.obj
 0002:000152f8       ??_C@_1M@PAFNENNF@?$AAf?$AAr?$AA?9?$AAl?$AAu@ 00000001800402f8     libucrt:lcidtoname_downlevel.obj
 0002:00015308       ??_C@_1M@EOHDJGDD@?$AAf?$AAr?$AA?9?$AAm?$AAc@ 0000000180040308     libucrt:lcidtoname_downlevel.obj
 0002:00015318       ??_C@_1M@FAPLLOPF@?$AAg?$AAl?$AA?9?$AAe?$AAs@ 0000000180040318     libucrt:lcidtoname_downlevel.obj
 0002:00015328       ??_C@_1M@FOPBFLOO@?$AAg?$AAu?$AA?9?$AAi?$AAn@ 0000000180040328     libucrt:lcidtoname_downlevel.obj
 0002:00015338       ??_C@_1M@KBMCINPM@?$AAh?$AAe?$AA?9?$AAi?$AAl@ 0000000180040338     libucrt:lcidtoname_downlevel.obj
 0002:00015348       ??_C@_1M@BBPHKFPJ@?$AAh?$AAi?$AA?9?$AAi?$AAn@ 0000000180040348     libucrt:lcidtoname_downlevel.obj
 0002:00015358       ??_C@_1M@PMBNDPHD@?$AAh?$AAr?$AA?9?$AAb?$AAa@ 0000000180040358     libucrt:lcidtoname_downlevel.obj
 0002:00015368       ??_C@_1M@BPCKOEGE@?$AAh?$AAr?$AA?9?$AAh?$AAr@ 0000000180040368     libucrt:lcidtoname_downlevel.obj
 0002:00015378       ??_C@_1M@GACBMHKE@?$AAh?$AAu?$AA?9?$AAh?$AAu@ 0000000180040378     libucrt:lcidtoname_downlevel.obj
 0002:00015388       ??_C@_1M@MILPAJJC@?$AAh?$AAy?$AA?9?$AAa?$AAm@ 0000000180040388     libucrt:lcidtoname_downlevel.obj
 0002:00015398       ??_C@_1M@BABBICEC@?$AAi?$AAd?$AA?9?$AAi?$AAd@ 0000000180040398     libucrt:lcidtoname_downlevel.obj
 0002:000153a8       ??_C@_1M@BIKNHHPF@?$AAi?$AAs?$AA?9?$AAi?$AAs@ 00000001800403a8     libucrt:lcidtoname_downlevel.obj
 0002:000153b8       ??_C@_1M@NMPCJPHE@?$AAi?$AAt?$AA?9?$AAc?$AAh@ 00000001800403b8     libucrt:lcidtoname_downlevel.obj
 0002:000153c8       ??_C@_1M@GHKGFEDF@?$AAi?$AAt?$AA?9?$AAi?$AAt@ 00000001800403c8     libucrt:lcidtoname_downlevel.obj
 0002:000153d8       ??_C@_1M@NIEJCJJA@?$AAj?$AAa?$AA?9?$AAj?$AAp@ 00000001800403d8     libucrt:lcidtoname_downlevel.obj
 0002:000153e8       ??_C@_1M@JILFNBIM@?$AAk?$AAa?$AA?9?$AAg?$AAe@ 00000001800403e8     libucrt:lcidtoname_downlevel.obj
 0002:000153f8       ??_C@_1M@PACPMGPH@?$AAk?$AAk?$AA?9?$AAk?$AAz@ 00000001800403f8     libucrt:lcidtoname_downlevel.obj
 0002:00015408       ??_C@_1M@IELFGMHA@?$AAk?$AAn?$AA?9?$AAi?$AAn@ 0000000180040408     libucrt:lcidtoname_downlevel.obj
 0002:00015418       ??_C@_1O@IBBJHCH@?$AAk?$AAo?$AAk?$AA?9?$AAi?$AAn@ 0000000180040418     libucrt:lcidtoname_downlevel.obj
 0002:00015428       ??_C@_1M@DMHAEOGC@?$AAk?$AAo?$AA?9?$AAk?$AAr@ 0000000180040428     libucrt:lcidtoname_downlevel.obj
 0002:00015438       ??_C@_1M@HBAHBIGA@?$AAk?$AAy?$AA?9?$AAk?$AAg@ 0000000180040438     libucrt:lcidtoname_downlevel.obj
 0002:00015448       ??_C@_1M@KPMILCJG@?$AAl?$AAt?$AA?9?$AAl?$AAt@ 0000000180040448     libucrt:lcidtoname_downlevel.obj
 0002:00015458       ??_C@_1M@BDEKKCA@?$AAl?$AAv?$AA?9?$AAl?$AAv@ 0000000180040458     libucrt:lcidtoname_downlevel.obj
 0002:00015468       ??_C@_1M@ELCKCCJJ@?$AAm?$AAi?$AA?9?$AAn?$AAz@ 0000000180040468     libucrt:lcidtoname_downlevel.obj
 0002:00015478       ??_C@_1M@CBOOLAPA@?$AAm?$AAk?$AA?9?$AAm?$AAk@ 0000000180040478     libucrt:lcidtoname_downlevel.obj
 0002:00015488       ??_C@_1M@GPHNBJKN@?$AAm?$AAl?$AA?9?$AAi?$AAn@ 0000000180040488     libucrt:lcidtoname_downlevel.obj
 0002:00015498       ??_C@_1M@PABJILIG@?$AAm?$AAn?$AA?9?$AAm?$AAn@ 0000000180040498     libucrt:lcidtoname_downlevel.obj
 0002:000154a8       ??_C@_1M@FGBKKIPG@?$AAm?$AAr?$AA?9?$AAi?$AAn@ 00000001800404a8     libucrt:lcidtoname_downlevel.obj
 0002:000154b8       ??_C@_1M@NDBPDDAL@?$AAm?$AAs?$AA?9?$AAb?$AAn@ 00000001800404b8     libucrt:lcidtoname_downlevel.obj
 0002:000154c8       ??_C@_1M@OPIHOOPI@?$AAm?$AAs?$AA?9?$AAm?$AAy@ 00000001800404c8     libucrt:lcidtoname_downlevel.obj
 0002:000154d8       ??_C@_1M@PPDBCNFM@?$AAm?$AAt?$AA?9?$AAm?$AAt@ 00000001800404d8     libucrt:lcidtoname_downlevel.obj
 0002:000154e8       ??_C@_1M@KDJDKMDD@?$AAn?$AAb?$AA?9?$AAn?$AAo@ 00000001800404e8     libucrt:lcidtoname_downlevel.obj
 0002:000154f8       ??_C@_1M@KFCFLMJP@?$AAn?$AAl?$AA?9?$AAb?$AAe@ 00000001800404f8     libucrt:lcidtoname_downlevel.obj
 0002:00015508       ??_C@_1M@KPOPDDGO@?$AAn?$AAl?$AA?9?$AAn?$AAl@ 0000000180040508     libucrt:lcidtoname_downlevel.obj
 0002:00015518       ??_C@_1M@LJKPEMLN@?$AAn?$AAn?$AA?9?$AAn?$AAo@ 0000000180040518     libucrt:lcidtoname_downlevel.obj
 0002:00015528       ??_C@_1M@BDGHHBFL@?$AAn?$AAs?$AA?9?$AAz?$AAa@ 0000000180040528     libucrt:lcidtoname_downlevel.obj
 0002:00015538       ??_C@_1M@IDEHOAP@?$AAp?$AAa?$AA?9?$AAi?$AAn@ 0000000180040538     libucrt:lcidtoname_downlevel.obj
 0002:00015548       ??_C@_1M@HDBKGOGH@?$AAp?$AAl?$AA?9?$AAp?$AAl@ 0000000180040548     libucrt:lcidtoname_downlevel.obj
 0002:00015558       ??_C@_1M@LJLLCMEH@?$AAp?$AAt?$AA?9?$AAb?$AAr@ 0000000180040558     libucrt:lcidtoname_downlevel.obj
 0002:00015568       ??_C@_1M@NCMONAAL@?$AAp?$AAt?$AA?9?$AAp?$AAt@ 0000000180040568     libucrt:lcidtoname_downlevel.obj
 0002:00015578       ??_C@_1O@EAKMAJDN@?$AAq?$AAu?$AAz?$AA?9?$AAb?$AAo@ 0000000180040578     libucrt:lcidtoname_downlevel.obj
 0002:00015588       ??_C@_1O@BHHPIGDN@?$AAq?$AAu?$AAz?$AA?9?$AAe?$AAc@ 0000000180040588     libucrt:lcidtoname_downlevel.obj
 0002:00015598       ??_C@_1O@GBAPEKMJ@?$AAq?$AAu?$AAz?$AA?9?$AAp?$AAe@ 0000000180040598     libucrt:lcidtoname_downlevel.obj
 0002:000155a8       ??_C@_1M@CLGLEFBO@?$AAr?$AAo?$AA?9?$AAr?$AAo@ 00000001800405a8     libucrt:lcidtoname_downlevel.obj
 0002:000155b8       ??_C@_1M@CEEDODME@?$AAr?$AAu?$AA?9?$AAr?$AAu@ 00000001800405b8     libucrt:lcidtoname_downlevel.obj
 0002:000155c8       ??_C@_1M@HPKKKMPP@?$AAs?$AAa?$AA?9?$AAi?$AAn@ 00000001800405c8     libucrt:lcidtoname_downlevel.obj
 0002:000155d8       ??_C@_1M@BKMAIGOJ@?$AAs?$AAe?$AA?9?$AAf?$AAi@ 00000001800405d8     libucrt:lcidtoname_downlevel.obj
 0002:000155e8       ??_C@_1M@NDPIFLFI@?$AAs?$AAe?$AA?9?$AAn?$AAo@ 00000001800405e8     libucrt:lcidtoname_downlevel.obj
 0002:000155f8       ??_C@_1M@DANKKHJ@?$AAs?$AAe?$AA?9?$AAs?$AAe@ 00000001800405f8     libucrt:lcidtoname_downlevel.obj
 0002:00015608       ??_C@_1M@PNBLONPJ@?$AAs?$AAk?$AA?9?$AAs?$AAk@ 0000000180040608     libucrt:lcidtoname_downlevel.obj
 0002:00015618       ??_C@_1M@LFMODOAL@?$AAs?$AAl?$AA?9?$AAs?$AAi@ 0000000180040618     libucrt:lcidtoname_downlevel.obj
 0002:00015628       ??_C@_1O@DFKOMPG@?$AAs?$AAm?$AAa?$AA?9?$AAn?$AAo@ 0000000180040628     libucrt:lcidtoname_downlevel.obj
 0002:00015638       ??_C@_1O@NDKPBNNH@?$AAs?$AAm?$AAa?$AA?9?$AAs?$AAe@ 0000000180040638     libucrt:lcidtoname_downlevel.obj
 0002:00015648       ??_C@_1O@PLLKBHAB@?$AAs?$AAm?$AAj?$AA?9?$AAn?$AAo@ 0000000180040648     libucrt:lcidtoname_downlevel.obj
 0002:00015658       ??_C@_1O@CLEPOGCA@?$AAs?$AAm?$AAj?$AA?9?$AAs?$AAe@ 0000000180040658     libucrt:lcidtoname_downlevel.obj
 0002:00015668       ??_C@_1O@DLGJGKMK@?$AAs?$AAm?$AAn?$AA?9?$AAf?$AAi@ 0000000180040668     libucrt:lcidtoname_downlevel.obj
 0002:00015678       ??_C@_1O@OJDJGAJC@?$AAs?$AAm?$AAs?$AA?9?$AAf?$AAi@ 0000000180040678     libucrt:lcidtoname_downlevel.obj
 0002:00015688       ??_C@_1M@BOFOGHPB@?$AAs?$AAq?$AA?9?$AAa?$AAl@ 0000000180040688     libucrt:lcidtoname_downlevel.obj
 0002:00015698       ??_C@_1BG@LJBBIPGB@?$AAs?$AAr?$AA?9?$AAb?$AAa?$AA?9?$AAc?$AAy?$AAr?$AAl@ 0000000180040698     libucrt:lcidtoname_downlevel.obj
 0002:000156b0       ??_C@_1BG@JLBENFOE@?$AAs?$AAr?$AA?9?$AAb?$AAa?$AA?9?$AAl?$AAa?$AAt?$AAn@ 00000001800406b0     libucrt:lcidtoname_downlevel.obj
 0002:000156c8       ??_C@_1BG@KODPNHE@?$AAs?$AAr?$AA?9?$AAs?$AAp?$AA?9?$AAc?$AAy?$AAr?$AAl@ 00000001800406c8     libucrt:lcidtoname_downlevel.obj
 0002:000156e0       ??_C@_1BG@CIOGKHPB@?$AAs?$AAr?$AA?9?$AAs?$AAp?$AA?9?$AAl?$AAa?$AAt?$AAn@ 00000001800406e0     libucrt:lcidtoname_downlevel.obj
 0002:000156f8       ??_C@_1M@NGFJLMAC@?$AAs?$AAv?$AA?9?$AAf?$AAi@ 00000001800406f8     libucrt:lcidtoname_downlevel.obj
 0002:00015708       ??_C@_1M@MPJEJAJC@?$AAs?$AAv?$AA?9?$AAs?$AAe@ 0000000180040708     libucrt:lcidtoname_downlevel.obj
 0002:00015718       ??_C@_1M@MPNDHLFK@?$AAs?$AAw?$AA?9?$AAk?$AAe@ 0000000180040718     libucrt:lcidtoname_downlevel.obj
 0002:00015728       ??_C@_1O@KOHBJJI@?$AAs?$AAy?$AAr?$AA?9?$AAs?$AAy@ 0000000180040728     libucrt:lcidtoname_downlevel.obj
 0002:00015738       ??_C@_1M@LDCEFHA@?$AAt?$AAa?$AA?9?$AAi?$AAn@ 0000000180040738     libucrt:lcidtoname_downlevel.obj
 0002:00015748       ??_C@_1M@CNJOFAK@?$AAt?$AAe?$AA?9?$AAi?$AAn@ 0000000180040748     libucrt:lcidtoname_downlevel.obj
 0002:00015758       ??_C@_1M@GNAECACD@?$AAt?$AAh?$AA?9?$AAt?$AAh@ 0000000180040758     libucrt:lcidtoname_downlevel.obj
 0002:00015768       ??_C@_1M@CHBIHOJO@?$AAt?$AAn?$AA?9?$AAz?$AAa@ 0000000180040768     libucrt:lcidtoname_downlevel.obj
 0002:00015778       ??_C@_1M@GCCMIGPJ@?$AAt?$AAr?$AA?9?$AAt?$AAr@ 0000000180040778     libucrt:lcidtoname_downlevel.obj
 0002:00015788       ??_C@_1M@CELMCNBK@?$AAt?$AAt?$AA?9?$AAr?$AAu@ 0000000180040788     libucrt:lcidtoname_downlevel.obj
 0002:00015798       ??_C@_1M@KLMCELGA@?$AAu?$AAk?$AA?9?$AAu?$AAa@ 0000000180040798     libucrt:lcidtoname_downlevel.obj
 0002:000157a8       ??_C@_1M@EPAJJAJF@?$AAu?$AAr?$AA?9?$AAp?$AAk@ 00000001800407a8     libucrt:lcidtoname_downlevel.obj
 0002:000157b8       ??_C@_1BG@GEGPMCDJ@?$AAu?$AAz?$AA?9?$AAu?$AAz?$AA?9?$AAc?$AAy?$AAr?$AAl@ 00000001800407b8     libucrt:lcidtoname_downlevel.obj
 0002:000157d0       ??_C@_1BG@EGGKJILM@?$AAu?$AAz?$AA?9?$AAu?$AAz?$AA?9?$AAl?$AAa?$AAt?$AAn@ 00000001800407d0     libucrt:lcidtoname_downlevel.obj
 0002:000157e8       ??_C@_1M@GFOCLFF@?$AAv?$AAi?$AA?9?$AAv?$AAn@ 00000001800407e8     libucrt:lcidtoname_downlevel.obj
 0002:000157f8       ??_C@_1M@CPAMEDFI@?$AAx?$AAh?$AA?9?$AAz?$AAa@ 00000001800407f8     libucrt:lcidtoname_downlevel.obj
 0002:00015808       ??_C@_1O@EBKIFIGN@?$AAz?$AAh?$AA?9?$AAc?$AAh?$AAs@ 0000000180040808     libucrt:lcidtoname_downlevel.obj
 0002:00015818       ??_C@_1O@NMHPGANE@?$AAz?$AAh?$AA?9?$AAc?$AAh?$AAt@ 0000000180040818     libucrt:lcidtoname_downlevel.obj
 0002:00015828       ??_C@_1M@LPINJOMC@?$AAz?$AAh?$AA?9?$AAc?$AAn@ 0000000180040828     libucrt:lcidtoname_downlevel.obj
 0002:00015838       ??_C@_1M@OCJEJODD@?$AAz?$AAh?$AA?9?$AAh?$AAk@ 0000000180040838     libucrt:lcidtoname_downlevel.obj
 0002:00015848       ??_C@_1M@DNDLJINH@?$AAz?$AAh?$AA?9?$AAm?$AAo@ 0000000180040848     libucrt:lcidtoname_downlevel.obj
 0002:00015858       ??_C@_1M@MBFDNDND@?$AAz?$AAh?$AA?9?$AAs?$AAg@ 0000000180040858     libucrt:lcidtoname_downlevel.obj
 0002:00015868       ??_C@_1M@IMEPLEPE@?$AAz?$AAh?$AA?9?$AAt?$AAw@ 0000000180040868     libucrt:lcidtoname_downlevel.obj
 0002:00015878       ??_C@_1M@BBGHNHJP@?$AAz?$AAu?$AA?9?$AAz?$AAa@ 0000000180040878     libucrt:lcidtoname_downlevel.obj
 0002:000158b0       ?large_power_data@?1??multiply_by_power_of_ten@__crt_strtox@@YA_NAEAUbig_integer@2@I@Z@4QBIB 00000001800408b0     libucrt:cfout.obj
 0002:000161c0       ?large_power_indices@?1??multiply_by_power_of_ten@__crt_strtox@@YA_NAEAUbig_integer@2@I@Z@4QBUunpack_index@?1??12@YA_N0I@Z@B 00000001800411c0     libucrt:cfout.obj
 0002:00016258       ?small_powers_of_ten@?1??multiply_by_power_of_ten@__crt_strtox@@YA_NAEAUbig_integer@2@I@Z@4QBIB 0000000180041258     libucrt:cfout.obj
 0002:0001627c       ??_C@_01GBGANLPD@0@        000000018004127c     libucrt:cfout.obj
 0002:00016280       ??_C@_05DNEBIAHO@1?$CDINF@ 0000000180041280     libucrt:cfout.obj
 0002:00016288       ??_C@_06IMKFLFPG@1?$CDQNAN@ 0000000180041288     libucrt:cfout.obj
 0002:00016290       ??_C@_06PGGFOGJG@1?$CDSNAN@ 0000000180041290     libucrt:cfout.obj
 0002:00016298       ??_C@_05PHHOCPM@1?$CDIND@  0000000180041298     libucrt:cfout.obj
 0002:000162a0       __real@3ff0000000000000    00000001800412a0     libucrt:ceil.obj
 0002:00016500       ??_C@_1BA@BALFACEM@?$AAC?$AAO?$AAN?$AAO?$AAU?$AAT?$AA$@ 0000000180041500     libucrt:initcon.obj
 0002:00016550       __log10_256_lead           0000000180041550     libucrt:log10_256_lead_tail_table.obj
 0002:00016d60       __log10_256_tail           0000000180041d60     libucrt:log10_256_lead_tail_table.obj
 0002:00017570       __log_F_inv_qword          0000000180042570     libucrt:log_f_inv_qword_table.obj
 0002:00017d80       ??_C@_05HGHHAHAP@log10@    0000000180042d80     libucrt:log_special.obj
 0002:00017d90       _load_config_used          0000000180042d90     LIBCMT:loadcfg.obj
 0002:00018100       ??_R4exception@std@@6B@    0000000180043100     LIBCMT:throw_bad_alloc.obj
 0002:00018128       ??_R3exception@std@@8      0000000180043128     LIBCMT:throw_bad_alloc.obj
 0002:00018140       ??_R2exception@std@@8      0000000180043140     LIBCMT:throw_bad_alloc.obj
 0002:00018150       ??_R1A@?0A@EA@exception@std@@8 0000000180043150     LIBCMT:throw_bad_alloc.obj
 0002:00018178       ??_R4bad_array_new_length@std@@6B@ 0000000180043178     LIBCMT:throw_bad_alloc.obj
 0002:000181a0       ??_R3bad_array_new_length@std@@8 00000001800431a0     LIBCMT:throw_bad_alloc.obj
 0002:000181b8       ??_R2bad_array_new_length@std@@8 00000001800431b8     LIBCMT:throw_bad_alloc.obj
 0002:000181d8       ??_R1A@?0A@EA@bad_array_new_length@std@@8 00000001800431d8     LIBCMT:throw_bad_alloc.obj
 0002:00018200       ??_R1A@?0A@EA@bad_alloc@std@@8 0000000180043200     LIBCMT:throw_bad_alloc.obj
 0002:00018228       ??_R3bad_alloc@std@@8      0000000180043228     LIBCMT:throw_bad_alloc.obj
 0002:00018240       ??_R2bad_alloc@std@@8      0000000180043240     LIBCMT:throw_bad_alloc.obj
 0002:00018258       ??_R4bad_alloc@std@@6B@    0000000180043258     LIBCMT:throw_bad_alloc.obj
 0002:00018280       ??_R4type_info@@6B@        0000000180043280     LIBCMT:std_type_info_static.obj
 0002:000182a8       ??_R3type_info@@8          00000001800432a8     LIBCMT:std_type_info_static.obj
 0002:000182c0       ??_R2type_info@@8          00000001800432c0     LIBCMT:std_type_info_static.obj
 0002:000182d0       ??_R1A@?0A@EA@type_info@@8 00000001800432d0     LIBCMT:std_type_info_static.obj
 0002:000182f8       ??_R4bad_exception@std@@6B@ 00000001800432f8     libvcruntime:frame.obj
 0002:00018320       ??_R3bad_exception@std@@8  0000000180043320     libvcruntime:frame.obj
 0002:00018338       ??_R2bad_exception@std@@8  0000000180043338     libvcruntime:frame.obj
 0002:00018350       ??_R1A@?0A@EA@bad_exception@std@@8 0000000180043350     libvcruntime:frame.obj
 0002:00018374       __volatile_metadata        0000000180043374     <linker-defined>
 0002:00018818       __rtc_iaa                  0000000180043818     LIBCMT:initsect.obj
 0002:00018820       __rtc_izz                  0000000180043820     LIBCMT:initsect.obj
 0002:00018828       __rtc_taa                  0000000180043828     LIBCMT:initsect.obj
 0002:00018830       __rtc_tzz                  0000000180043830     LIBCMT:initsect.obj
 0002:00019eb8       _TI2?AVbad_alloc@std@@     0000000180044eb8     LIBCMT:throw_bad_alloc.obj
 0002:00019ed8       _CTA2?AVbad_alloc@std@@    0000000180044ed8     LIBCMT:throw_bad_alloc.obj
 0002:00019ef0       _CT??_R0?AVbad_alloc@std@@@8??0bad_alloc@std@@QEAA@AEBV01@@Z24 0000000180044ef0     LIBCMT:throw_bad_alloc.obj
 0002:00019f18       _CT??_R0?AVexception@std@@@8??0exception@std@@QEAA@AEBV01@@Z24 0000000180044f18     LIBCMT:throw_bad_alloc.obj
 0002:00019f40       _TI3?AVbad_array_new_length@std@@ 0000000180044f40     LIBCMT:throw_bad_alloc.obj
 0002:00019f60       _CTA3?AVbad_array_new_length@std@@ 0000000180044f60     LIBCMT:throw_bad_alloc.obj
 0002:00019f80       _CT??_R0?AVbad_array_new_length@std@@@8??0bad_array_new_length@std@@QEAA@AEBV01@@Z24 0000000180044f80     LIBCMT:throw_bad_alloc.obj
 0002:00019fa8       _TI2?AVbad_exception@std@@ 0000000180044fa8     libvcruntime:frame.obj
 0002:00019fc8       _CTA2?AVbad_exception@std@@ 0000000180044fc8     libvcruntime:frame.obj
 0002:00019fe0       _CT??_R0?AVbad_exception@std@@@8??0bad_exception@std@@QEAA@AEBV01@@Z24 0000000180044fe0     libvcruntime:frame.obj
 0002:0001aa10       __IMPORT_DESCRIPTOR_jawt   0000000180045a10     jawt:jawt.dll
 0002:0001aa24       __IMPORT_DESCRIPTOR_KERNEL32 0000000180045a24     kernel32:KERNEL32.dll
 0002:0001aa38       __IMPORT_DESCRIPTOR_USER32 0000000180045a38     user32:USER32.dll
 0002:0001aa4c       __NULL_IMPORT_DESCRIPTOR   0000000180045a4c     jawt:jawt.dll
 0003:00000000       __security_cookie          0000000180047000     LIBCMT:gs_cookie.obj
 0003:00000040       __security_cookie_complement 0000000180047040     LIBCMT:gs_cookie.obj
 0003:00000048       _fltused                   0000000180047048     LIBCMT:fltused.obj
 0003:0000004c       __scrt_native_dllmain_reason 000000018004704c     LIBCMT:utility.obj
 0003:00000050       __isa_inverted             0000000180047050     LIBCMT:cpu_disp.obj
 0003:00000058       __isa_available            0000000180047058     LIBCMT:cpu_disp.obj
 0003:0000005c       __isa_enabled              000000018004705c     LIBCMT:cpu_disp.obj
 0003:00000060       __memset_fast_string_threshold 0000000180047060     LIBCMT:cpu_disp.obj
 0003:00000068       __memset_nt_threshold      0000000180047068     LIBCMT:cpu_disp.obj
 0003:00000080       _iob                       0000000180047080     libucrt:_file.obj
 0003:00000188       __abort_behavior           0000000180047188     libucrt:abort.obj
 0003:000001a0       __badioinfo                00000001800471a0     libucrt:ioinit.obj
 0003:000001f0       __acrt_initial_locale_data 00000001800471f0     libucrt:nlsdata.obj
 0003:00000348       __acrt_initial_locale_pointers 0000000180047348     libucrt:nlsdata.obj
 0003:00000358       __acrt_wide_c_locale_string 0000000180047358     libucrt:nlsdata.obj
 0003:00000360       __acrt_initial_multibyte_data 0000000180047360     libucrt:mbctype.obj
 0003:000008a0       __globallocalestatus       00000001800478a0     libucrt:glstatus.obj
 0003:000008b0       __acrt_lconv_c             00000001800478b0     libucrt:localeconv.obj
 0003:00000948       __acrt_lconv_static_decimal 0000000180047948     libucrt:localeconv.obj
 0003:0000094c       __acrt_lconv_static_W_decimal 000000018004794c     libucrt:localeconv.obj
 0003:00000950       _lookuptrailbytes          0000000180047950     libucrt:read.obj
 0003:00000a50       _guard_check_icall_$fo_default$ 0000000180047a50     libucrt:checkcfg.obj
 0003:00000a70       ??_R0?AVbad_alloc@std@@@8  0000000180047a70     LIBCMT:throw_bad_alloc.obj
 0003:00000a98       ??_R0?AVexception@std@@@8  0000000180047a98     LIBCMT:throw_bad_alloc.obj
 0003:00000ac0       ??_R0?AVbad_array_new_length@std@@@8 0000000180047ac0     LIBCMT:throw_bad_alloc.obj
 0003:00000af0       ??_R0?AVbad_exception@std@@@8 0000000180047af0     libvcruntime:frame.obj
 0003:00000b18       ??_R0?AVtype_info@@@8      0000000180047b18     LIBCMT:std_type_info_static.obj
 0003:00000b40       ?JavaBridgeThreadId@@3KA   0000000180047b40     AccessBridgeATInstance.obj
 0003:00000b48       ?_OptionsStorage@?1??__local_stdio_printf_options@@9@4_KA 0000000180047b48     AccessBridgeDebug.obj
 0003:00000b58       ?theFromJavaHelloMsgID@@3IA 0000000180047b58     AccessBridgeMessages.obj
 0003:00000b5c       ?theFromWindowsHelloMsgID@@3IA 0000000180047b5c     AccessBridgeMessages.obj
 0003:00000b60       ?theJavaAccessBridge@@3PEAVJavaAccessBridge@@EA 0000000180047b60     JavaAccessBridge.obj
 0003:00000b68       ?theDialogWindow@@3PEAUHWND__@@EA 0000000180047b68     JavaAccessBridge.obj
 0003:00000b70       ?receiveMemoryIPCLock@@3U_RTL_CRITICAL_SECTION@@A 0000000180047b70     JavaAccessBridge.obj
 0003:00001110       ?__type_info_root_node@@3U__type_info_node@@A 0000000180048110     LIBCMT:tncleanup.obj
 0003:00001120       ?_OptionsStorage@?1??__local_stdio_scanf_options@@9@4_KA 0000000180048120     LIBCMT:default_local_stdio_options.obj
 0003:00001128       __scrt_current_native_startup_state 0000000180048128     LIBCMT:utility.obj
 0003:00001130       __scrt_native_startup_lock 0000000180048130     LIBCMT:utility.obj
 0003:00001170       __scrt_debugger_hook_flag  0000000180048170     LIBCMT:utility_desktop.obj
 0003:00001174       __avx10_version            0000000180048174     LIBCMT:cpu_disp.obj
 0003:00001178       __favor                    0000000180048178     LIBCMT:cpu_disp.obj
 0003:00001180       ?__WinRTOutOfMemoryExceptionCallback@@3P6APEAXXZEA 0000000180048180     libvcruntime:ehhelpers.obj
 0003:00001188       ?pArgList@UnDecorator@@0PEAVReplicator@@EA 0000000180048188     libvcruntime:undname.obj
 0003:00001190       ?pZNameList@UnDecorator@@0PEAVReplicator@@EA 0000000180048190     libvcruntime:undname.obj
 0003:00001198       ?pTemplateArgList@UnDecorator@@0PEAVReplicator@@EA 0000000180048198     libvcruntime:undname.obj
 0003:000011a0       ?gName@UnDecorator@@0PEBDEB 00000001800481a0     libvcruntime:undname.obj
 0003:000011a8       ?name@UnDecorator@@0PEBDEB 00000001800481a8     libvcruntime:undname.obj
 0003:000011b0       ?disableFlags@UnDecorator@@0KA 00000001800481b0     libvcruntime:undname.obj
 0003:000011b4       ?fExplicitTemplateParams@UnDecorator@@0_NA 00000001800481b4     libvcruntime:undname.obj
 0003:000011b5       ?fGetTemplateArgumentList@UnDecorator@@0_NA 00000001800481b5     libvcruntime:undname.obj
 0003:000011b8       ?m_pGetParameter@UnDecorator@@0P6APEADJ@ZEA 00000001800481b8     libvcruntime:undname.obj
 0003:000011c0       ?m_CHPENameOffset@UnDecorator@@0KA 00000001800481c0     libvcruntime:undname.obj
 0003:000011c4       ?m_recursionLevel@UnDecorator@@0KA 00000001800481c4     libvcruntime:undname.obj
 0003:000012e0       __pPurecall                00000001800482e0     libvcruntime:purevirt_data.obj
 0003:000012e8       _nstream                   00000001800482e8     libucrt:_file.obj
 0003:000012f0       __piob                     00000001800482f0     libucrt:_file.obj
 0003:000012f8       _cflush                    00000001800482f8     libucrt:_file.obj
 0003:00001428       _environ_table             0000000180048428     libucrt:environment_initialization.obj
 0003:00001430       _wenviron_table            0000000180048430     libucrt:environment_initialization.obj
 0003:00001438       __dcrt_initial_wide_environment 0000000180048438     libucrt:environment_initialization.obj
 0003:00001440       __dcrt_initial_narrow_environment 0000000180048440     libucrt:environment_initialization.obj
 0003:00001448       __acrt_atexit_table        0000000180048448     libucrt:onexit.obj
 0003:00001460       __acrt_at_quick_exit_table 0000000180048460     libucrt:onexit.obj
 0003:00001480       ?__acrt_use_tls2_apis@@3_NA 0000000180048480     libucrt:per_thread_data.obj
 0003:00001550       __pioinfo                  0000000180048550     libucrt:ioinit.obj
 0003:00001950       _nhandle                   0000000180048950     libucrt:ioinit.obj
 0003:00001978       __acrt_stdout_buffer       0000000180048978     libucrt:_sftbuf.obj
 0003:00001980       __acrt_stderr_buffer       0000000180048980     libucrt:_sftbuf.obj
 0003:00001988       __acrt_locale_changed_data 0000000180048988     libucrt:wsetlocale.obj
 0003:00001990       __acrt_current_locale_data 0000000180048990     libucrt:nlsdata.obj
 0003:00001c00       _mbctype                   0000000180048c00     libucrt:mbctype.obj
 0003:00001c08       _mbcasemap                 0000000180048c08     libucrt:mbctype.obj
 0003:00001c10       __acrt_current_multibyte_data 0000000180048c10     libucrt:mbctype.obj
 0003:00001c20       _pgmptr                    0000000180048c20     libucrt:argv_data.obj
 0003:00001c28       __argc                     0000000180048c28     libucrt:argv_data.obj
 0003:00001c30       __argv                     0000000180048c30     libucrt:argv_data.obj
 0003:00001c38       __wargv                    0000000180048c38     libucrt:argv_data.obj
 0003:00001c40       _acmdln                    0000000180048c40     libucrt:argv_data.obj
 0003:00001c48       _wcmdln                    0000000180048c48     libucrt:argv_data.obj
 0003:00001c50       __acrt_heap                0000000180048c50     libucrt:heap_handle.obj
 0003:00001c84       __acrt_lconv_static_null   0000000180048c84     libucrt:localeconv.obj
 0003:00001c88       __acrt_lconv_static_W_null 0000000180048c88     libucrt:localeconv.obj
 0003:00001c8c       _commode                   0000000180048c8c     libucrt:ncommode.obj
 0003:00001c94       _umaskval                  0000000180048c94     libucrt:umask.obj
 0003:00001c98       __use_fma3_lib             0000000180048c98     libucrt:fma3_available.obj
 0003:00001c9c       __fma3_is_available        0000000180048c9c     libucrt:fma3_available.obj
 0003:00001ca0       _fmode                     0000000180048ca0     libucrt:txtmode.obj
 0003:00001ca4       __scrt_ucrt_dll_is_in_use  0000000180048ca4     <common>
 0003:00001ca8       __dyn_tls_init_callback    0000000180048ca8     <common>

 entry point at        0001:0000fc40

 Static symbols

 0000:fffb2000       .debug$S                   0000000180000000     javaaccessbridge.exp
 0000:fffb2000       .debug$S                   0000000180000000     kernel32:KERNEL32.dll
 0000:fffb2000       .debug$S                   0000000180000000     kernel32:KERNEL32.dll
 0000:fffb2000       .debug$S                   0000000180000000     kernel32:KERNEL32.dll
 0000:fffb2000       .debug$S                   0000000180000000     kernel32:KERNEL32.dll
 0000:fffb2000       .debug$S                   0000000180000000     kernel32:KERNEL32.dll
 0000:fffb2000       .debug$S                   0000000180000000     kernel32:KERNEL32.dll
 0000:fffb2000       .debug$S                   0000000180000000     kernel32:KERNEL32.dll
 0000:fffb2000       .debug$S                   0000000180000000     kernel32:KERNEL32.dll
 0000:fffb2000       .debug$S                   0000000180000000     kernel32:KERNEL32.dll
 0000:fffb2000       .debug$S                   0000000180000000     kernel32:KERNEL32.dll
 0000:fffb2000       .debug$S                   0000000180000000     kernel32:KERNEL32.dll
 0000:fffb2000       .debug$S                   0000000180000000     kernel32:KERNEL32.dll
 0000:fffb2000       .debug$S                   0000000180000000     kernel32:KERNEL32.dll
 0000:fffb2000       .debug$S                   0000000180000000     kernel32:KERNEL32.dll
 0000:fffb2000       .debug$S                   0000000180000000     kernel32:KERNEL32.dll
 0000:fffb2000       .debug$S                   0000000180000000     kernel32:KERNEL32.dll
 0000:fffb2000       .debug$S                   0000000180000000     kernel32:KERNEL32.dll
 0000:fffb2000       .debug$S                   0000000180000000     kernel32:KERNEL32.dll
 0000:fffb2000       .debug$S                   0000000180000000     kernel32:KERNEL32.dll
 0000:fffb2000       .debug$S                   0000000180000000     kernel32:KERNEL32.dll
 0000:fffb2000       .debug$S                   0000000180000000     kernel32:KERNEL32.dll
 0000:fffb2000       .debug$S                   0000000180000000     kernel32:KERNEL32.dll
 0000:fffb2000       .debug$S                   0000000180000000     kernel32:KERNEL32.dll
 0000:fffb2000       .debug$S                   0000000180000000     kernel32:KERNEL32.dll
 0000:fffb2000       .debug$S                   0000000180000000     kernel32:KERNEL32.dll
 0000:fffb2000       .debug$S                   0000000180000000     kernel32:KERNEL32.dll
 0000:fffb2000       .debug$S                   0000000180000000     kernel32:KERNEL32.dll
 0000:fffb2000       .debug$S                   0000000180000000     kernel32:KERNEL32.dll
 0000:fffb2000       .debug$S                   0000000180000000     kernel32:KERNEL32.dll
 0000:fffb2000       .debug$S                   0000000180000000     kernel32:KERNEL32.dll
 0000:fffb2000       .debug$S                   0000000180000000     kernel32:KERNEL32.dll
 0000:fffb2000       .debug$S                   0000000180000000     kernel32:KERNEL32.dll
 0000:fffb2000       .debug$S                   0000000180000000     kernel32:KERNEL32.dll
 0000:fffb2000       .debug$S                   0000000180000000     kernel32:KERNEL32.dll
 0000:fffb2000       .debug$S                   0000000180000000     kernel32:KERNEL32.dll
 0000:fffb2000       .debug$S                   0000000180000000     kernel32:KERNEL32.dll
 0000:fffb2000       .debug$S                   0000000180000000     kernel32:KERNEL32.dll
 0000:fffb2000       .debug$S                   0000000180000000     kernel32:KERNEL32.dll
 0000:fffb2000       .debug$S                   0000000180000000     kernel32:KERNEL32.dll
 0000:fffb2000       .debug$S                   0000000180000000     kernel32:KERNEL32.dll
 0000:fffb2000       .debug$S                   0000000180000000     kernel32:KERNEL32.dll
 0000:fffb2000       .debug$S                   0000000180000000     kernel32:KERNEL32.dll
 0000:fffb2000       .debug$S                   0000000180000000     kernel32:KERNEL32.dll
 0000:fffb2000       .debug$S                   0000000180000000     kernel32:KERNEL32.dll
 0000:fffb2000       .debug$S                   0000000180000000     kernel32:KERNEL32.dll
 0000:fffb2000       .debug$S                   0000000180000000     kernel32:KERNEL32.dll
 0000:fffb2000       .debug$S                   0000000180000000     kernel32:KERNEL32.dll
 0000:fffb2000       .debug$S                   0000000180000000     kernel32:KERNEL32.dll
 0000:fffb2000       .debug$S                   0000000180000000     kernel32:KERNEL32.dll
 0000:fffb2000       .debug$S                   0000000180000000     kernel32:KERNEL32.dll
 0000:fffb2000       .debug$S                   0000000180000000     kernel32:KERNEL32.dll
 0000:fffb2000       .debug$S                   0000000180000000     kernel32:KERNEL32.dll
 0000:fffb2000       .debug$S                   0000000180000000     kernel32:KERNEL32.dll
 0000:fffb2000       .debug$S                   0000000180000000     kernel32:KERNEL32.dll
 0000:fffb2000       .debug$S                   0000000180000000     kernel32:KERNEL32.dll
 0000:fffb2000       .debug$S                   0000000180000000     kernel32:KERNEL32.dll
 0000:fffb2000       .debug$S                   0000000180000000     kernel32:KERNEL32.dll
 0000:fffb2000       .debug$S                   0000000180000000     kernel32:KERNEL32.dll
 0000:fffb2000       .debug$S                   0000000180000000     kernel32:KERNEL32.dll
 0000:fffb2000       .debug$S                   0000000180000000     kernel32:KERNEL32.dll
 0000:fffb2000       .debug$S                   0000000180000000     kernel32:KERNEL32.dll
 0000:fffb2000       .debug$S                   0000000180000000     kernel32:KERNEL32.dll
 0000:fffb2000       .debug$S                   0000000180000000     kernel32:KERNEL32.dll
 0000:fffb2000       .debug$S                   0000000180000000     kernel32:KERNEL32.dll
 0000:fffb2000       .debug$S                   0000000180000000     kernel32:KERNEL32.dll
 0000:fffb2000       .debug$S                   0000000180000000     kernel32:KERNEL32.dll
 0000:fffb2000       .debug$S                   0000000180000000     kernel32:KERNEL32.dll
 0000:fffb2000       .debug$S                   0000000180000000     kernel32:KERNEL32.dll
 0000:fffb2000       .debug$S                   0000000180000000     kernel32:KERNEL32.dll
 0000:fffb2000       .debug$S                   0000000180000000     kernel32:KERNEL32.dll
 0000:fffb2000       .debug$S                   0000000180000000     kernel32:KERNEL32.dll
 0000:fffb2000       .debug$S                   0000000180000000     kernel32:KERNEL32.dll
 0000:fffb2000       .debug$S                   0000000180000000     kernel32:KERNEL32.dll
 0000:fffb2000       .debug$S                   0000000180000000     kernel32:KERNEL32.dll
 0000:fffb2000       .debug$S                   0000000180000000     kernel32:KERNEL32.dll
 0000:fffb2000       .debug$S                   0000000180000000     kernel32:KERNEL32.dll
 0000:fffb2000       .debug$S                   0000000180000000     kernel32:KERNEL32.dll
 0000:fffb2000       .debug$S                   0000000180000000     kernel32:KERNEL32.dll
 0000:fffb2000       .debug$S                   0000000180000000     kernel32:KERNEL32.dll
 0000:fffb2000       .debug$S                   0000000180000000     kernel32:KERNEL32.dll
 0000:fffb2000       .debug$S                   0000000180000000     kernel32:KERNEL32.dll
 0000:fffb2000       .debug$S                   0000000180000000     kernel32:KERNEL32.dll
 0000:fffb2000       .debug$S                   0000000180000000     kernel32:KERNEL32.dll
 0000:fffb2000       .debug$S                   0000000180000000     kernel32:KERNEL32.dll
 0000:fffb2000       .debug$S                   0000000180000000     kernel32:KERNEL32.dll
 0000:fffb2000       .debug$S                   0000000180000000     kernel32:KERNEL32.dll
 0000:fffb2000       .debug$S                   0000000180000000     kernel32:KERNEL32.dll
 0000:fffb2000       .debug$S                   0000000180000000     kernel32:KERNEL32.dll
 0000:fffb2000       .debug$S                   0000000180000000     kernel32:KERNEL32.dll
 0000:fffb2000       .debug$S                   0000000180000000     kernel32:KERNEL32.dll
 0000:fffb2000       .debug$S                   0000000180000000     kernel32:KERNEL32.dll
 0000:fffb2000       .debug$S                   0000000180000000     kernel32:KERNEL32.dll
 0000:fffb2000       .debug$S                   0000000180000000     kernel32:KERNEL32.dll
 0000:fffb2000       .debug$S                   0000000180000000     kernel32:KERNEL32.dll
 0000:fffb2000       .debug$S                   0000000180000000     kernel32:KERNEL32.dll
 0000:fffb2000       .debug$S                   0000000180000000     kernel32:KERNEL32.dll
 0000:fffb2000       .debug$S                   0000000180000000     kernel32:KERNEL32.dll
 0000:fffb2000       .debug$S                   0000000180000000     kernel32:KERNEL32.dll
 0000:fffb2000       .debug$S                   0000000180000000     kernel32:KERNEL32.dll
 0000:fffb2000       .debug$S                   0000000180000000     kernel32:KERNEL32.dll
 0000:fffb2000       .debug$S                   0000000180000000     kernel32:KERNEL32.dll
 0000:fffb2000       .debug$S                   0000000180000000     kernel32:KERNEL32.dll
 0000:fffb2000       .debug$S                   0000000180000000     kernel32:KERNEL32.dll
 0000:fffb2000       .debug$S                   0000000180000000     kernel32:KERNEL32.dll
 0000:fffb2000       .debug$S                   0000000180000000     user32:USER32.dll
 0000:fffb2000       .debug$S                   0000000180000000     user32:USER32.dll
 0000:fffb2000       .debug$S                   0000000180000000     user32:USER32.dll
 0000:fffb2000       .debug$S                   0000000180000000     user32:USER32.dll
 0000:fffb2000       .debug$S                   0000000180000000     user32:USER32.dll
 0000:fffb2000       .debug$S                   0000000180000000     user32:USER32.dll
 0000:fffb2000       .debug$S                   0000000180000000     user32:USER32.dll
 0000:fffb2000       .debug$S                   0000000180000000     user32:USER32.dll
 0000:fffb2000       .debug$S                   0000000180000000     user32:USER32.dll
 0000:fffb2000       .debug$S                   0000000180000000     jawt:jawt.dll
 0001:000000a0       ?JavaBridgeThread@@YAIPEAX@Z 00000001800010a0 f   AccessBridgeATInstance.obj
 0001:0000013c       ?do_event@@YAXPEADHPEAUHWND__@@1@Z 000000018000113c f   AccessBridgeATInstance.obj
 0001:0000f900       $$000000                   0000000180010900     LIBCMT:amdsecgs.obj
 0001:0000f930       ?dllmain_crt_dispatch@@YAHQEAUHINSTANCE__@@KQEAX@Z 0000000180010930 f   LIBCMT:dll_dllmain.obj
 0001:0000f980       ?dllmain_crt_process_attach@@YAHQEAUHINSTANCE__@@QEAX@Z 0000000180010980 f   LIBCMT:dll_dllmain.obj
 0001:0000fa98       ?dllmain_crt_process_detach@@YAH_N@Z 0000000180010a98 f   LIBCMT:dll_dllmain.obj
 0001:0000fb18       ?dllmain_dispatch@@YAHQEAUHINSTANCE__@@KQEAX@Z 0000000180010b18 f   LIBCMT:dll_dllmain.obj
 0001:0000ff28       capture_previous_context   0000000180010f28 f   LIBCMT:gs_report.obj
 0001:00010e40       $$000000                   0000000180011e40     libvcruntime:notify.obj
 0001:00010e60       $$000000                   0000000180011e60     libvcruntime:notify.obj
 0001:00010e70       $$000000                   0000000180011e70     libvcruntime:notify.obj
 0001:0001169c       ?try_get_function@@YAPEAXW4function_id@?A0x14174aea@@QEBDQEBW4module_id@2@2@Z 000000018001269c f   libvcruntime:winapi_downlevel.obj
 0001:00011a88       ??$BuildCatchObjectHelperInternal@V__FrameHandler3@@@@YAHPEAUEHExceptionRecord@@PEAXPEBU_s_HandlerType@@PEBU_s_CatchableType@@@Z 0000000180012a88 f   libvcruntime:frame.obj
 0001:00011c88       ??$BuildCatchObjectInternal@V__FrameHandler3@@@@YAXPEAUEHExceptionRecord@@PEAXPEBU_s_HandlerType@@PEBU_s_CatchableType@@@Z 0000000180012c88 f   libvcruntime:frame.obj
 0001:00011d48       ??$CatchIt@V__FrameHandler3@@@@YAXPEAUEHExceptionRecord@@PEA_KPEAU_CONTEXT@@PEAU_xDISPATCHER_CONTEXT@@PEBU_s_FuncInfo@@PEBU_s_HandlerType@@PEBU_s_CatchableType@@PEBU_s_TryBlockMapEntry@@H1EE@Z 0000000180012d48 f   libvcruntime:frame.obj
 0001:00011e1c       ??$FindHandler@V__FrameHandler3@@@@YAXPEAUEHExceptionRecord@@PEA_KPEAU_CONTEXT@@PEAU_xDISPATCHER_CONTEXT@@PEBU_s_FuncInfo@@EH1@Z 0000000180012e1c f   libvcruntime:frame.obj
 0001:000122ec       ??$FindHandlerForForeignException@V__FrameHandler3@@@@YAXPEAUEHExceptionRecord@@PEA_KPEAU_CONTEXT@@PEAU_xDISPATCHER_CONTEXT@@PEBU_s_FuncInfo@@HH1@Z 00000001800132ec f   libvcruntime:frame.obj
 0001:00012b24       ?ExFilterRethrow@@YAHPEAU_EXCEPTION_POINTERS@@PEAUEHExceptionRecord@@PEAH@Z 0000000180013b24 f   libvcruntime:frame.obj
 0001:00012dcc       ?IsInExceptionSpec@@YAEPEAUEHExceptionRecord@@PEBU_s_ESTypeList@@@Z 0000000180013dcc f   libvcruntime:frame.obj
 0001:00012ebc       ?Is_bad_exception_allowed@@YAEPEBU_s_ESTypeList@@@Z 0000000180013ebc f   libvcruntime:frame.obj
 0001:00012fa0       $$000000                   0000000180013fa0     libvcruntime:handlers.obj
 0001:00012fe0       ??$thread_start@P6AIPEAX@Z$00@@YAKQEAX@Z 0000000180013fe0 f   libucrt:thread.obj
 0001:00013048       ?common_end_thread@@YAXI@Z 0000000180014048 f   libucrt:thread.obj
 0001:000130ac       ?create_thread_parameter@@YAPEAU__acrt_thread_parameter@@QEAX0@Z 00000001800140ac f   libucrt:thread.obj
 0001:000133a8       ??$?RV<lambda_613eff765f5c257adf68e381dfe80f05>@@AEAV<lambda_ebf663be9fcd9e0b17ed57bdb95b0759>@@V<lambda_872abebd861b7db59b42e49ea65623b0>@@@?$__crt_seh_guarded_call@H@@QEAAH$$QEAV<lambda_613eff765f5c257adf68e381dfe80f05>@@AEAV<lambda_ebf663be9fcd9e0b17ed57bdb95b0759>@@$$QEAV<lambda_872abebd861b7db59b42e49ea65623b0>@@@Z 00000001800143a8 f   libucrt:output.obj
 0001:000133e8       ??$?RV<lambda_d854c62834386a3b23916ad6dae2782d>@@AEAV<lambda_303760bc4008a2b3ec4768a30b06a80c>@@V<lambda_4780a7ea4f8cbd2590aec34bd14e2bbf>@@@?$__crt_seh_guarded_call@H@@QEAAH$$QEAV<lambda_d854c62834386a3b23916ad6dae2782d>@@AEAV<lambda_303760bc4008a2b3ec4768a30b06a80c>@@$$QEAV<lambda_4780a7ea4f8cbd2590aec34bd14e2bbf>@@@Z 00000001800143e8 f   libucrt:output.obj
 0001:00015320       ??R<lambda_303760bc4008a2b3ec4768a30b06a80c>@@QEBAHXZ 0000000180016320 f   libucrt:output.obj
 0001:0001543c       ??R<lambda_ebf663be9fcd9e0b17ed57bdb95b0759>@@QEBAHXZ 000000018001643c f   libucrt:output.obj
 0001:00017b30       ?_fclose_internal@@YAHQEAU_iobuf@@AEAV__crt_cached_ptd_host@@@Z 0000000180018b30 f   libucrt:fclose.obj
 0001:00017bac       ?_fclose_nolock_internal@@YAHQEAU_iobuf@@AEAV__crt_cached_ptd_host@@@Z 0000000180018bac f   libucrt:fclose.obj
 0001:00017cec       ??$common_fsopen@D@@YAPEAU_iobuf@@QEBD0H@Z 0000000180018cec f   libucrt:fopen.obj
 0001:00017db4       ??$common_getenv@D@@YAPEADQEBD@Z 0000000180018db4 f   libucrt:getenv.obj
 0001:00017e14       ??$common_getenv_nolock@D@@YAPEADQEBD@Z 0000000180018e14 f   libucrt:getenv.obj
 0001:000186f8       ??$?RV<lambda_d80eeec6fff315bfe5c115232f3240e3>@@AEAV<lambda_6e4b09c48022b2350581041d5f6b0c4c>@@V<lambda_2358e3775559c9db80273638284d5e45>@@@?$__crt_seh_guarded_call@X@@QEAAX$$QEAV<lambda_d80eeec6fff315bfe5c115232f3240e3>@@AEAV<lambda_6e4b09c48022b2350581041d5f6b0c4c>@@$$QEAV<lambda_2358e3775559c9db80273638284d5e45>@@@Z 00000001800196f8 f   libucrt:exit.obj
 0001:00018730       ??R<lambda_6e4b09c48022b2350581041d5f6b0c4c>@@QEBA@XZ 0000000180019730 f   libucrt:exit.obj
 0001:000187f0       ?common_exit@@YAXHW4_crt_exit_cleanup_mode@@W4_crt_exit_return_mode@@@Z 00000001800197f0 f   libucrt:exit.obj
 0001:000188d4       ?exit_or_terminate_process@@YAXI_N@Z 00000001800198d4 f   libucrt:exit.obj
 0001:00018904       ?try_cor_exit_process@@YAXI@Z 0000000180019904 f   libucrt:exit.obj
 0001:00018994       ??$parse_command_line@D@@YAXPEADPEAPEAD0PEA_K2@Z 0000000180019994 f   libucrt:argv_parsing.obj
 0001:00018d34       ??$common_initialize_environment_nolock@D@@YAHXZ 0000000180019d34 f   libucrt:environment_initialization.obj
 0001:00018da8       ??$create_environment@D@@YAQEAPEADQEAD@Z 0000000180019da8 f   libucrt:environment_initialization.obj
 0001:00018ebc       ??$free_environment@D@@YAXQEAPEAD@Z 0000000180019ebc f   libucrt:environment_initialization.obj
 0001:00018ebc       ??$free_environment@_W@@YAXQEAPEA_W@Z 0000000180019ebc f   libucrt:environment_initialization.obj
 0001:00018f00       ??$initialize_environment_by_cloning_nolock@D@@YAHXZ 0000000180019f00 f   libucrt:environment_initialization.obj
 0001:00018fe0       ??$uninitialize_environment_internal@D@@YAXAEAPEAPEAD@Z 0000000180019fe0 f   libucrt:environment_initialization.obj
 0001:00018ffc       ??$uninitialize_environment_internal@_W@@YAXAEAPEAPEA_W@Z 0000000180019ffc f   libucrt:environment_initialization.obj
 0001:000190a0       ??$?RV<lambda_7777bce6b2f8c936911f934f8298dc43>@@AEAV<lambda_f03950bc5685219e0bcd2087efbe011e>@@V<lambda_3883c3dff614d5e0c5f61bb1ac94921c>@@@?$__crt_seh_guarded_call@H@@QEAAH$$QEAV<lambda_7777bce6b2f8c936911f934f8298dc43>@@AEAV<lambda_f03950bc5685219e0bcd2087efbe011e>@@$$QEAV<lambda_3883c3dff614d5e0c5f61bb1ac94921c>@@@Z 000000018001a0a0 f   libucrt:onexit.obj
 0001:000190dc       ??R<lambda_f03950bc5685219e0bcd2087efbe011e>@@QEBA@XZ 000000018001a0dc f   libucrt:onexit.obj
 0001:00019260       initialize_global_variables 000000018001a260 f   libucrt:initialization.obj
 0001:00019274       initialize_c               000000018001a274 f   libucrt:initialization.obj
 0001:00019298       initialize_environment     000000018001a298 f   libucrt:initialization.obj
 0001:00019298       initialize_global_state_isolation 000000018001a298 f   libucrt:initialization.obj
 0001:00019298       report_memory_leaks        000000018001a298 f   libucrt:initialization.obj
 0001:00019298       uninitialize_c             000000018001a298 f   libucrt:initialization.obj
 0001:00019298       uninitialize_global_state_isolation 000000018001a298 f   libucrt:initialization.obj
 0001:0001929c       uninitialize_environment   000000018001a29c f   libucrt:initialization.obj
 0001:000192ac       initialize_pointers        000000018001a2ac f   libucrt:initialization.obj
 0001:000192ec       uninitialize_vcruntime     000000018001a2ec f   libucrt:initialization.obj
 0001:000192f4       uninitialize_allocated_memory 000000018001a2f4 f   libucrt:initialization.obj
 0001:00019334       uninitialize_allocated_io_buffers 000000018001a334 f   libucrt:initialization.obj
 0001:00019b50       ?select_heap@@YAPEAXQEAX@Z 000000018001ab50 f   libucrt:free_base.obj
 0001:00019b58       ??$?RV<lambda_0ae27a3a962d80f24befdcbee591983d>@@AEAV<lambda_8d0ee55de4b1038c4002e0adecdf1839>@@V<lambda_dc504788e8f1664fe9b84e20bfb512f2>@@@?$__crt_seh_guarded_call@X@@QEAAX$$QEAV<lambda_0ae27a3a962d80f24befdcbee591983d>@@AEAV<lambda_8d0ee55de4b1038c4002e0adecdf1839>@@$$QEAV<lambda_dc504788e8f1664fe9b84e20bfb512f2>@@@Z 000000018001ab58 f   libucrt:per_thread_data.obj
 0001:00019b98       ??$?RV<lambda_2d41944a1d46af3157314b8a01080d33>@@AEAV<lambda_8f455de75cd7d7f24b4096f044d8b9e6>@@V<lambda_aa500f224e6afead328df44964fe2772>@@@?$__crt_seh_guarded_call@X@@QEAAX$$QEAV<lambda_2d41944a1d46af3157314b8a01080d33>@@AEAV<lambda_8f455de75cd7d7f24b4096f044d8b9e6>@@$$QEAV<lambda_aa500f224e6afead328df44964fe2772>@@@Z 000000018001ab98 f   libucrt:per_thread_data.obj
 0001:00019bd8       ??$?RV<lambda_aa87e3671a710a21b5dc78c0bdf72e11>@@AEAV<lambda_92619d2358a28f41a33ba319515a20b9>@@V<lambda_6992ecaafeb10aed2b74cb1fae11a551>@@@?$__crt_seh_guarded_call@X@@QEAAX$$QEAV<lambda_aa87e3671a710a21b5dc78c0bdf72e11>@@AEAV<lambda_92619d2358a28f41a33ba319515a20b9>@@$$QEAV<lambda_6992ecaafeb10aed2b74cb1fae11a551>@@@Z 000000018001abd8 f   libucrt:per_thread_data.obj
 0001:00019c20       ??$?RV<lambda_f2e299630e499de9f9a165e60fcd3db5>@@AEAV<lambda_2ae9d31cdba2644fcbeaf08da7c24588>@@V<lambda_40d01ff24d0e7b3814fdbdcee8eab3c7>@@@?$__crt_seh_guarded_call@X@@QEAAX$$QEAV<lambda_f2e299630e499de9f9a165e60fcd3db5>@@AEAV<lambda_2ae9d31cdba2644fcbeaf08da7c24588>@@$$QEAV<lambda_40d01ff24d0e7b3814fdbdcee8eab3c7>@@@Z 000000018001ac20 f   libucrt:per_thread_data.obj
 0001:00019c80       ?construct_ptd_array@@YAXQEAU__acrt_ptd@@@Z 000000018001ac80 f   libucrt:per_thread_data.obj
 0001:00019d50       ?destroy_fls@@YAXPEAX@Z    000000018001ad50 f   libucrt:per_thread_data.obj
 0001:00019d70       ?destroy_ptd_array@@YAXQEAU__acrt_ptd@@@Z 000000018001ad70 f   libucrt:per_thread_data.obj
 0001:00019f20       ?replace_current_thread_locale_nolock@@YAXQEAU__acrt_ptd@@QEAU__crt_locale_data@@@Z 000000018001af20 f   libucrt:per_thread_data.obj
 0001:0001a18c       ?try_get_CompareStringEx@@YAP6AHPEB_WK0H0HPEAU_nlsversioninfo@@PEAX_J@ZXZ 000000018001b18c f   libucrt:winapi_thunks.obj
 0001:0001a1c4       ?try_get_function_slow@@YAPEAXW4function_id@?A0x391cf84c@@QEBDQEBW4module_id@2@2@Z 000000018001b1c4 f   libucrt:winapi_thunks.obj
 0001:0001a944       ??$?RV<lambda_842d9ff0dc9ef11c61343bbaebe7f885>@@AEAV<lambda_c5860995281e5c4ce005b3de8f5874ee>@@V<lambda_d90129c13df834fdcbf8d2b88dafcf2d>@@@?$__crt_seh_guarded_call@X@@QEAAX$$QEAV<lambda_842d9ff0dc9ef11c61343bbaebe7f885>@@AEAV<lambda_c5860995281e5c4ce005b3de8f5874ee>@@$$QEAV<lambda_d90129c13df834fdcbf8d2b88dafcf2d>@@@Z 000000018001b944 f   libucrt:fflush.obj
 0001:0001a9e0       ??$?RV<lambda_886d6c58226a84441f68b9f2b8217b83>@@AEAV<lambda_ab61a845afdef5b7c387490eaf3616ee>@@V<lambda_f7f22ab5edc0698d5f6905b0d3f44752>@@@?$__crt_seh_guarded_call@X@@QEAAX$$QEAV<lambda_886d6c58226a84441f68b9f2b8217b83>@@AEAV<lambda_ab61a845afdef5b7c387490eaf3616ee>@@$$QEAV<lambda_f7f22ab5edc0698d5f6905b0d3f44752>@@@Z 000000018001b9e0 f   libucrt:fflush.obj
 0001:0001aac4       ?common_flush_all@@YAH_N@Z 000000018001bac4 f   libucrt:fflush.obj
 0001:0001acd0       ?initialize_inherited_file_handles_nolock@@YAXXZ 000000018001bcd0 f   libucrt:ioinit.obj
 0001:0001add0       ?initialize_stdio_handles_nolock@@YAXXZ 000000018001bdd0 f   libucrt:ioinit.obj
 0001:0001b098       ?fp_format_a@@YAHQEBNPEAD_KQEAD2H_NIW4__acrt_rounding_mode@@AEAV__crt_cached_ptd_host@@@Z 000000018001c098 f   libucrt:cvt.obj
 0001:0001b42c       ?fp_format_e@@YAHQEBNQEAD_K12H_NIW4__acrt_rounding_mode@@AEAV__crt_cached_ptd_host@@@Z 000000018001c42c f   libucrt:cvt.obj
 0001:0001b530       ?fp_format_e_internal@@YAHQEAD_KH_NIQEAU_strflt@@2AEAV__crt_cached_ptd_host@@@Z 000000018001c530 f   libucrt:cvt.obj
 0001:0001b714       ?fp_format_f@@YAHQEBNQEAD_K12HW4__acrt_rounding_mode@@AEAV__crt_cached_ptd_host@@@Z 000000018001c714 f   libucrt:cvt.obj
 0001:0001b7ec       ?fp_format_f_internal@@YAHQEAD_KHQEAU_strflt@@_NAEAV__crt_cached_ptd_host@@@Z 000000018001c7ec f   libucrt:cvt.obj
 0001:0001b93c       ?fp_format_g@@YAHQEBNQEAD_K12H_NIW4__acrt_rounding_mode@@AEAV__crt_cached_ptd_host@@@Z 000000018001c93c f   libucrt:cvt.obj
 0001:0001ba90       ?should_round_up@@YA_NQEBN_KFW4__acrt_rounding_mode@@@Z 000000018001ca90 f   libucrt:cvt.obj
 0001:0001c994       ??$?RV<lambda_410d79af7f07d98d83a3f525b3859a53>@@AEAV<lambda_3e16ef9562a7dcce91392c22ab16ea36>@@V<lambda_38119f0e861e05405d8a144b9b982f0a>@@@?$__crt_seh_guarded_call@X@@QEAAX$$QEAV<lambda_410d79af7f07d98d83a3f525b3859a53>@@AEAV<lambda_3e16ef9562a7dcce91392c22ab16ea36>@@$$QEAV<lambda_38119f0e861e05405d8a144b9b982f0a>@@@Z 000000018001d994 f   libucrt:wsetlocale.obj
 0001:0001ca40       ??$?RV<lambda_ad8af0d99a0adf03d037d7dffe354bb5>@@AEAV<lambda_c9ba49e555ba839a7b07aa3fbecb7617>@@V<lambda_2f1ebd5d68526518146ae959c9e734c8>@@@?$__crt_seh_guarded_call@H@@QEAAH$$QEAV<lambda_ad8af0d99a0adf03d037d7dffe354bb5>@@AEAV<lambda_c9ba49e555ba839a7b07aa3fbecb7617>@@$$QEAV<lambda_2f1ebd5d68526518146ae959c9e734c8>@@@Z 000000018001da40 f   libucrt:close.obj
 0001:0001cd58       ?find_or_allocate_unused_stream_nolock@@YA?AV__crt_stdio_stream@@XZ 000000018001dd58 f   libucrt:stream.obj
 0001:0001d444       ?<lambda_invoker_cdecl>@<lambda_a1ce4c8ae42411fd470c77163914f50e>@@CAHPEBX0@Z 000000018001e444 f   libucrt:argv_wildcards.obj
 0001:0001d7a4       ??$common_expand_argv_wildcards@D@@YAHQEAPEADQEAPEAPEAD@Z 000000018001e7a4 f   libucrt:argv_wildcards.obj
 0001:0001d9e0       ??$copy_and_add_argument_to_buffer@D@@YAHQEBD0_KAEAV?$argument_list@D@?A0x5f5c8891@@@Z 000000018001e9e0 f   libucrt:argv_wildcards.obj
 0001:0001db64       ??$expand_argument_wildcards@D@@YAHQEAD0AEAV?$argument_list@D@?A0x5f5c8891@@@Z 000000018001eb64 f   libucrt:argv_wildcards.obj
 0001:0001e10c       ??$?RV<lambda_efdfa57d1f175319df784efa44bb7b81>@@AEAV<lambda_5f0a4c1567f8adc6734073e5d1e1b35c>@@V<lambda_2e8a7d3640ea6ccb4c2413664c2db6fd>@@@?$__crt_seh_guarded_call@X@@QEAAX$$QEAV<lambda_efdfa57d1f175319df784efa44bb7b81>@@AEAV<lambda_5f0a4c1567f8adc6734073e5d1e1b35c>@@$$QEAV<lambda_2e8a7d3640ea6ccb4c2413664c2db6fd>@@@Z 000000018001f10c f   libucrt:mbctype.obj
 0001:0001e2dc       ?getSystemCP@@YAHH@Z       000000018001f2dc f   libucrt:mbctype.obj
 0001:0001e35c       ?setSBCS@@YAXPEAU__crt_multibyte_data@@@Z 000000018001f35c f   libucrt:mbctype.obj
 0001:0001e3f4       ?setSBUpLow@@YAXPEAU__crt_multibyte_data@@@Z 000000018001f3f4 f   libucrt:mbctype.obj
 0001:0001e5ec       ?setmbcp_internal@@YAHH_NQEAU__acrt_ptd@@QEAPEAU__crt_multibyte_data@@@Z 000000018001f5ec f   libucrt:mbctype.obj
 0001:0001e85c       ?update_thread_multibyte_data_internal@@YAPEAU__crt_multibyte_data@@QEAU__acrt_ptd@@QEAPEAU1@@Z 000000018001f85c f   libucrt:mbctype.obj
 0001:0001ec58       ?x_ismbbtype_l@@YAHPEAU__crt_locale_pointers@@IHH@Z 000000018001fc58 f   libucrt:ismbbyte.obj
 0001:0001ef88       ??$common_set_variable_in_environment_nolock@D@@YAHQEADH@Z 000000018001ff88 f   libucrt:setenv.obj
 0001:0001f2e0       ??$copy_environment@D@@YAPEAPEADQEAPEAD@Z 00000001800202e0 f   libucrt:setenv.obj
 0001:0001f5a4       ??$?RV<lambda_450d765d439847d4c735a33c368b5fc0>@@AEAV<lambda_44731a7d0e6d81c3e6aa82d741081786>@@V<lambda_601a2a7da3b7a96e9554ac7215c4b07c>@@@?$__crt_seh_guarded_call@P6AXH@Z@@QEAAP6AXH@Z$$QEAV<lambda_450d765d439847d4c735a33c368b5fc0>@@AEAV<lambda_44731a7d0e6d81c3e6aa82d741081786>@@$$QEAV<lambda_601a2a7da3b7a96e9554ac7215c4b07c>@@@Z 00000001800205a4 f   libucrt:signal.obj
 0001:0001fdf0       ??$?RV<lambda_a37b2b86f63e897a80ea819b0eb08c01>@@AEAV<lambda_38ce7e780aa69e748d6df282ebc68efe>@@V<lambda_99fb1378e971ab6e7edea83e3a7a83a2>@@@?$__crt_seh_guarded_call@H@@QEAAH$$QEAV<lambda_a37b2b86f63e897a80ea819b0eb08c01>@@AEAV<lambda_38ce7e780aa69e748d6df282ebc68efe>@@$$QEAV<lambda_99fb1378e971ab6e7edea83e3a7a83a2>@@@Z 0000000180020df0 f   libucrt:commit.obj
 0001:0001ff10       ?write_double_translated_ansi_nolock@@YA?AUwrite_result@?A0x17268360@@HQEBDIAEAV__crt_cached_ptd_host@@@Z 0000000180020f10 f   libucrt:write.obj
 0001:000203a4       ?write_text_ansi_nolock@@YA?AUwrite_result@?A0x17268360@@HQEBDI@Z 00000001800213a4 f   libucrt:write.obj
 0001:000204ac       ?write_text_utf16le_nolock@@YA?AUwrite_result@?A0x17268360@@HQEBDI@Z 00000001800214ac f   libucrt:write.obj
 0001:000205c8       ?write_text_utf8_nolock@@YA?AUwrite_result@?A0x17268360@@HQEBDI@Z 00000001800215c8 f   libucrt:write.obj
 0001:00021148       ?should_round_up@@YA_NQEBD0HW4__acrt_has_trailing_digits@@W4__acrt_rounding_mode@@@Z 0000000180022148 f   libucrt:_fptostr.obj
 0001:00022a3c       memcpy_s                   0000000180023a3c f   libucrt:cfout.obj
 0001:00022ba4       ??$write_buffer_nolock@D@@YA_NDV__crt_stdio_stream@@AEAV__crt_cached_ptd_host@@@Z 0000000180023ba4 f   libucrt:_flsbuf.obj
 0001:00022c9c       ??$write_buffer_nolock@_W@@YA_N_WV__crt_stdio_stream@@AEAV__crt_cached_ptd_host@@@Z 0000000180023c9c f   libucrt:_flsbuf.obj
 0001:00022d98       ?stream_is_at_end_of_file_nolock@@YA_NV__crt_stdio_stream@@@Z 0000000180023d98 f   libucrt:_flsbuf.obj
 0001:00023190       ?free_crt_array_internal@@YAXQEAPEBX_K@Z 0000000180024190 f   libucrt:inittime.obj
 0001:000235f4       ??$common_sopen_dispatch@D@@YAHQEBDHHHQEAHH@Z 00000001800245f4 f   libucrt:open.obj
 0001:000236b8       ?configure_text_mode@@YAHHUfile_options@?A0xa9d50aae@@HAEAW4__crt_lowio_text_mode@@@Z 00000001800246b8 f   libucrt:open.obj
 0001:00023938       ?decode_options@@YA?AUfile_options@?A0xa9d50aae@@HHH@Z 0000000180024938 f   libucrt:open.obj
 0001:00023b4c       ?truncate_ctrl_z_if_present@@YAHH@Z 0000000180024b4c f   libucrt:open.obj
 0001:00024174       ?InternalCompareStringA@@YAHPEAU__crt_locale_pointers@@PEB_WKPEBDH2HH@Z 0000000180025174 f   libucrt:comparestringa.obj
 0001:00024a18       fallbackMethod             0000000180025a18 f   libucrt:strpbrk.obj
 0001:00024d8c       $LN79                      0000000180025d8c     libucrt:strpbrk.obj
 0001:00024dc8       $LN78                      0000000180025dc8     libucrt:strpbrk.obj
 0001:00024e08       $LN77                      0000000180025e08     libucrt:strpbrk.obj
 0001:00024ee4       ?__acrt_LCMapStringA_stat@@YAHPEAU__crt_locale_pointers@@PEB_WKPEBDHPEADHHH@Z 0000000180025ee4 f   libucrt:lcmapstringa.obj
 0001:000252b0       ?initialize_multibyte@@YAHXZ 00000001800262b0 f   libucrt:multibyte_initializer.obj
 0001:0002553c       ??$common_lseek@_J@@YA_JH_JHAEAV__crt_cached_ptd_host@@@Z 000000018002653c f   libucrt:lseek.obj
 0001:0002565c       ??$common_lseek_nolock@_J@@YA_JH_JHAEAV__crt_cached_ptd_host@@@Z 000000018002665c f   libucrt:lseek.obj
 0001:0002588c       ??$translate_text_mode_nolock@_W@@YAHHQEA_W_K@Z 000000018002688c f   libucrt:read.obj
 0001:00025a88       ?translate_ansi_or_utf8_nolock@@YAHHQEAD_KQEA_W1@Z 0000000180026a88 f   libucrt:read.obj
 0001:000263a0       ceil_soft                  00000001800273a0 f   libucrt:ceil.obj
 0001:00026450       $$000000                   0000000180027450     libucrt:log10.obj
 0001:00026467       Llog10_sse2                0000000180027467     libucrt:log10.obj
 0001:000264cf       Llog10_sse2_continue_common 00000001800274cf     libucrt:log10.obj
 0001:000265e0       Llog10_sse2_near_one       00000001800275e0     libucrt:log10.obj
 0001:000266a7       Llog10_sse2_denormal_adjust 00000001800276a7     libucrt:log10.obj
 0001:000266e0       Llog10_sse2_x_is_zero_or_neg 00000001800276e0     libucrt:log10.obj
 0001:00026700       Llog10_sse2_x_is_neg       0000000180027700     libucrt:log10.obj
 0001:00026720       Llog10_sse2_x_is_inf_or_nan 0000000180027720     libucrt:log10.obj
 0001:00026740       Llog10_sse2_finish         0000000180027740     libucrt:log10.obj
 0001:00026750       Llog10_fma3                0000000180027750     libucrt:log10.obj
 0001:000267ab       Llog10_fma3_continue_common 00000001800277ab     libucrt:log10.obj
 0001:00026890       Llog10_fma3_near_one       0000000180027890     libucrt:log10.obj
 0001:00026939       Llog10_fma3_denormal_adjust 0000000180027939     libucrt:log10.obj
 0001:00026970       Llog10_fma3_x_is_zero_or_neg 0000000180027970     libucrt:log10.obj
 0001:000269a0       Llog10_fma3_x_is_neg       00000001800279a0     libucrt:log10.obj
 0001:000269c0       Llog10_fma3_x_is_inf_or_nan 00000001800279c0     libucrt:log10.obj
 0001:000269f0       Llog10_fma3_finish         00000001800279f0     libucrt:log10.obj
 0001:00027260       common_control87           0000000180028260 f   libucrt:ieee.obj
 0001:00027500       _exception_enabled         0000000180028500 f   libucrt:libm_error.obj
 0001:00027770       $$000000                   0000000180028770     libucrt:floorceil_sse41.obj
 0001:00027854       _log_special_common        0000000180028854 f   libucrt:log_special.obj
 0001:00027eb0       $$000000                   0000000180028eb0     LIBCMT:chkstk.obj
 0001:00028120       $$000000                   0000000180029120     LIBCMT:guard_dispatch.obj
 0001:00028140       $$000000                   0000000180029140     LIBCMT:guard_xfg_dispatch.obj
 0001:00028170       $$000000                   0000000180029170     libucrt:dispatchcfg.obj
 0001:000281a0       $$000000                   00000001800291a0     libvcruntime:memcpy.obj
 0001:000281b0       $$000000                   00000001800291b0     libvcruntime:memcpy.obj
 0001:000281de       MoveSmall0                 00000001800291de     libvcruntime:memcpy.obj
 0001:000281e0       MoveSmall15                00000001800291e0     libvcruntime:memcpy.obj
 0001:00028200       MoveSmall11                0000000180029200     libvcruntime:memcpy.obj
 0001:00028218       MoveSmall2                 0000000180029218     libvcruntime:memcpy.obj
 0001:00028220       MoveSmall7                 0000000180029220     libvcruntime:memcpy.obj
 0001:00028238       MoveSmall14                0000000180029238     libvcruntime:memcpy.obj
 0001:0002824f       MoveSmall3                 000000018002924f     libvcruntime:memcpy.obj
 0001:00028260       MoveSmall13                0000000180029260     libvcruntime:memcpy.obj
 0001:00028276       MoveSmall10                0000000180029276     libvcruntime:memcpy.obj
 0001:00028285       MoveSmall9                 0000000180029285     libvcruntime:memcpy.obj
 0001:00028293       MoveSmall12                0000000180029293     libvcruntime:memcpy.obj
 0001:000282a0       MoveSmall6                 00000001800292a0     libvcruntime:memcpy.obj
 0001:000282af       MoveSmall5                 00000001800292af     libvcruntime:memcpy.obj
 0001:000282bd       MoveSmall8                 00000001800292bd     libvcruntime:memcpy.obj
 0001:000282c4       MoveSmall1                 00000001800292c4     libvcruntime:memcpy.obj
 0001:000282ca       MoveSmall4                 00000001800292ca     libvcruntime:memcpy.obj
 0001:000282d0       MoveAbove15                00000001800292d0     libvcruntime:memcpy.obj
 0001:000282ed       MoveAbove32                00000001800292ed     libvcruntime:memcpy.obj
 0001:0002832d       MoveWithYMM                000000018002932d     libvcruntime:memcpy.obj
 0001:00028380       YmmLoop                    0000000180029380     libvcruntime:memcpy.obj
 0001:00028408       MovUpTo256WithYMM          0000000180029408     libvcruntime:memcpy.obj
 0001:00028425       Mov8YmmBlocks              0000000180029425     libvcruntime:memcpy.obj
 0001:00028439       Mov7YmmBlocks              0000000180029439     libvcruntime:memcpy.obj
 0001:0002844d       Mov6YmmBlocks              000000018002944d     libvcruntime:memcpy.obj
 0001:00028461       Mov5YmmBlocks              0000000180029461     libvcruntime:memcpy.obj
 0001:00028475       Mov4YmmBlocks              0000000180029475     libvcruntime:memcpy.obj
 0001:00028483       Mov3YmmBlocks              0000000180029483     libvcruntime:memcpy.obj
 0001:00028491       Mov2YmmBlocks              0000000180029491     libvcruntime:memcpy.obj
 0001:0002849f       Mov1YmmBlocks              000000018002949f     libvcruntime:memcpy.obj
 0001:000284a6       Mov0YmmBlocks              00000001800294a6     libvcruntime:memcpy.obj
 0001:000284b0       YmmLoopNT                  00000001800294b0     libvcruntime:memcpy.obj
 0001:00028555       Mov8YmmBlocksNT            0000000180029555     libvcruntime:memcpy.obj
 0001:00028569       Mov7YmmBlocksNT            0000000180029569     libvcruntime:memcpy.obj
 0001:0002857d       Mov6YmmBlocksNT            000000018002957d     libvcruntime:memcpy.obj
 0001:00028591       Mov5YmmBlocksNT            0000000180029591     libvcruntime:memcpy.obj
 0001:000285a5       Mov4YmmBlocksNT            00000001800295a5     libvcruntime:memcpy.obj
 0001:000285b3       Mov3YmmBlocksNT            00000001800295b3     libvcruntime:memcpy.obj
 0001:000285c1       Mov2YmmBlocksNT            00000001800295c1     libvcruntime:memcpy.obj
 0001:000285cf       Mov1YmmBlocksNT            00000001800295cf     libvcruntime:memcpy.obj
 0001:000285d6       Mov0YmmBlocksNT            00000001800295d6     libvcruntime:memcpy.obj
 0001:000285f0       NoAVX                      00000001800295f0     libvcruntime:memcpy.obj
 0001:00028606       MoveWithXMM                0000000180029606     libvcruntime:memcpy.obj
 0001:00028640       XmmLoop                    0000000180029640     libvcruntime:memcpy.obj
 0001:000286ac       MovUpTo128WithXMM          00000001800296ac     libvcruntime:memcpy.obj
 0001:000286c9       Mov8XmmBlocks              00000001800296c9     libvcruntime:memcpy.obj
 0001:000286d7       Mov7XmmBlocks              00000001800296d7     libvcruntime:memcpy.obj
 0001:000286e5       Mov6XmmBlocks              00000001800296e5     libvcruntime:memcpy.obj
 0001:000286f3       Mov5XmmBlocks              00000001800296f3     libvcruntime:memcpy.obj
 0001:00028701       Mov4XmmBlocks              0000000180029701     libvcruntime:memcpy.obj
 0001:0002870f       Mov3XmmBlocks              000000018002970f     libvcruntime:memcpy.obj
 0001:0002871d       Mov2XmmBlocks              000000018002971d     libvcruntime:memcpy.obj
 0001:0002872b       Mov1XmmBlocks              000000018002972b     libvcruntime:memcpy.obj
 0001:00028732       Mov0XmmBlocks              0000000180029732     libvcruntime:memcpy.obj
 0001:00028740       CopyDown                   0000000180029740     libvcruntime:memcpy.obj
 0001:0002875b       XmmMovAlign                000000018002975b     libvcruntime:memcpy.obj
 0001:00028773       XmmMovLargeTest            0000000180029773     libvcruntime:memcpy.obj
 0001:00028790       XmmMovLargeOuter           0000000180029790     libvcruntime:memcpy.obj
 0001:00028797       XmmMovLargeInner           0000000180029797     libvcruntime:memcpy.obj
 0001:000287ed       XmmMovSmallTest            00000001800297ed     libvcruntime:memcpy.obj
 0001:00028800       XmmMovSmallLoop            0000000180029800     libvcruntime:memcpy.obj
 0001:00028810       XmmMovTrailing             0000000180029810     libvcruntime:memcpy.obj
 0001:00028819       XmmMovReturn               0000000180029819     libvcruntime:memcpy.obj
 0001:00028840       $$000000                   0000000180029840     libvcruntime:memset.obj
 0001:00028850       $$000000                   0000000180029850     libvcruntime:memset.obj
 0001:00028891       SetSmall15                 0000000180029891     libvcruntime:memset.obj
 0001:00028895       SetSmall7                  0000000180029895     libvcruntime:memset.obj
 0001:00028899       SetSmall3                  0000000180029899     libvcruntime:memset.obj
 0001:0002889e       SetSmall1                  000000018002989e     libvcruntime:memset.obj
 0001:000288a2       SetSmall0                  00000001800298a2     libvcruntime:memset.obj
 0001:000288a3       SetSmall14                 00000001800298a3     libvcruntime:memset.obj
 0001:000288a7       SetSmall6                  00000001800298a7     libvcruntime:memset.obj
 0001:000288ab       SetSmall2                  00000001800298ab     libvcruntime:memset.obj
 0001:000288b0       MoveSmall0                 00000001800298b0     libvcruntime:memset.obj
 0001:000288c0       SetSmall13                 00000001800298c0     libvcruntime:memset.obj
 0001:000288c4       SetSmall5                  00000001800298c4     libvcruntime:memset.obj
 0001:000288d0       SetSmall12                 00000001800298d0     libvcruntime:memset.obj
 0001:000288d4       SetSmall4                  00000001800298d4     libvcruntime:memset.obj
 0001:000288d9       SetSmall11                 00000001800298d9     libvcruntime:memset.obj
 0001:000288e7       SetSmall9                  00000001800298e7     libvcruntime:memset.obj
 0001:000288f0       SetSmall10                 00000001800298f0     libvcruntime:memset.obj
 0001:000288fa       SetSmall8                  00000001800298fa     libvcruntime:memset.obj
 0001:00028900       SetAbove15                 0000000180029900     libvcruntime:memset.obj
 0001:00028916       SetAbove32                 0000000180029916     libvcruntime:memset.obj
 0001:00028942       SetWithYMM                 0000000180029942     libvcruntime:memset.obj
 0001:00028980       YmmLoop                    0000000180029980     libvcruntime:memset.obj
 0001:000289ca       SetUpTo256WithYMM          00000001800299ca     libvcruntime:memset.obj
 0001:000289e7       Set8YmmBlocks              00000001800299e7     libvcruntime:memset.obj
 0001:000289f1       Set7YmmBlocks              00000001800299f1     libvcruntime:memset.obj
 0001:000289fb       Set6YmmBlocks              00000001800299fb     libvcruntime:memset.obj
 0001:00028a05       Set5YmmBlocks              0000000180029a05     libvcruntime:memset.obj
 0001:00028a0f       Set4YmmBlocks              0000000180029a0f     libvcruntime:memset.obj
 0001:00028a16       Set3YmmBlocks              0000000180029a16     libvcruntime:memset.obj
 0001:00028a1d       Set2YmmBlocks              0000000180029a1d     libvcruntime:memset.obj
 0001:00028a24       Set1YmmBlocks              0000000180029a24     libvcruntime:memset.obj
 0001:00028a2b       Set0YmmBlocks              0000000180029a2b     libvcruntime:memset.obj
 0001:00028a33       SetWithYMMNT               0000000180029a33     libvcruntime:memset.obj
 0001:00028a40       YmmLoopNT                  0000000180029a40     libvcruntime:memset.obj
 0001:00028aa7       Set8YmmBlocksNT            0000000180029aa7     libvcruntime:memset.obj
 0001:00028ab1       Set7YmmBlocksNT            0000000180029ab1     libvcruntime:memset.obj
 0001:00028abb       Set6YmmBlocksNT            0000000180029abb     libvcruntime:memset.obj
 0001:00028ac5       Set5YmmBlocksNT            0000000180029ac5     libvcruntime:memset.obj
 0001:00028acf       Set4YmmBlocksNT            0000000180029acf     libvcruntime:memset.obj
 0001:00028ad6       Set3YmmBlocksNT            0000000180029ad6     libvcruntime:memset.obj
 0001:00028add       Set2YmmBlocksNT            0000000180029add     libvcruntime:memset.obj
 0001:00028ae4       Set1YmmBlocksNT            0000000180029ae4     libvcruntime:memset.obj
 0001:00028aeb       Set0YmmBlocksNT            0000000180029aeb     libvcruntime:memset.obj
 0001:00028b00       NoAVX                      0000000180029b00     libvcruntime:memset.obj
 0001:00028b16       SetWithXMM                 0000000180029b16     libvcruntime:memset.obj
 0001:00028b40       XmmLoop                    0000000180029b40     libvcruntime:memset.obj
 0001:00028b7e       SetUpTo128WithXMM          0000000180029b7e     libvcruntime:memset.obj
 0001:00028b9b       Set8XmmBlocks              0000000180029b9b     libvcruntime:memset.obj
 0001:00028ba2       Set7XmmBlocks              0000000180029ba2     libvcruntime:memset.obj
 0001:00028ba9       Set6XmmBlocks              0000000180029ba9     libvcruntime:memset.obj
 0001:00028bb0       Set5XmmBlocks              0000000180029bb0     libvcruntime:memset.obj
 0001:00028bb7       Set4XmmBlocks              0000000180029bb7     libvcruntime:memset.obj
 0001:00028bbe       Set3XmmBlocks              0000000180029bbe     libvcruntime:memset.obj
 0001:00028bc5       Set2XmmBlocks              0000000180029bc5     libvcruntime:memset.obj
 0001:00028bcc       Set1XmmBlocks              0000000180029bcc     libvcruntime:memset.obj
 0001:00028bd3       Set0XmmBlocks              0000000180029bd3     libvcruntime:memset.obj
 0001:00028be0       $$000000                   0000000180029be0     libucrt:strcmp.obj
 0001:00028c60       $$000000                   0000000180029c60     libucrt:strcat.obj
 0001:00028dd0       $$000000                   0000000180029dd0     libucrt:strncpy.obj
 0001:00028f50       $$000000                   0000000180029f50     libucrt:strlen.obj
 0001:00029010       $$000000                   000000018002a010     libucrt:strncat.obj
 0001:000291c0       $$000000                   000000018002a1c0     libucrt:strncmp.obj
 0001:00029260       ?fin$0@?0??dllmain_crt_process_attach@@YAHQEAUHINSTANCE__@@QEAX@Z@4HA 000000018002a260 f   LIBCMT:dll_dllmain.obj
 0001:00029277       ?fin$0@?0??dllmain_crt_process_detach@@YAH_N@Z@4HA 000000018002a277 f   LIBCMT:dll_dllmain.obj
 0001:00029290       ?fin$1@?0??dllmain_crt_process_detach@@YAH_N@Z@4HA 000000018002a290 f   LIBCMT:dll_dllmain.obj
 0001:000292a4       ?filt$0@?0??dllmain_dispatch@@YAHQEAUHINSTANCE__@@KQEAX@Z@4HA 000000018002a2a4 f   LIBCMT:dll_dllmain.obj
 0001:000292da       __scrt_is_nonwritable_in_current_image$filt$0 000000018002a2da f   LIBCMT:utility.obj
 0001:000292f2       __DestructExceptionObject$filt$0 000000018002a2f2 f   libvcruntime:ehhelpers.obj
 0001:00029388       ?filt$0@?0???$_CallSETranslator@V__FrameHandler3@@@@YAHPEAUEHExceptionRecord@@PEA_KPEAU_CONTEXT@@PEAU_xDISPATCHER_CONTEXT@@PEBU_s_FuncInfo@@K1H@Z@4HA 000000018002a388 f   libvcruntime:risctrnsctrl.obj
 0001:00029430       ?filt$0@?0??CxxCallCatchBlock@__FrameHandler3@@SAPEAXPEAU_EXCEPTION_RECORD@@@Z@4HA 000000018002a430 f   libvcruntime:frame.obj
 0001:00029455       ?fin$1@?0??CxxCallCatchBlock@__FrameHandler3@@SAPEAXPEAU_EXCEPTION_RECORD@@@Z@4HA 000000018002a455 f   libvcruntime:frame.obj
 0001:000294db       ?filt$0@?0??FrameUnwindToState@__FrameHandler3@@SAXPEA_KPEAU_xDISPATCHER_CONTEXT@@PEBU_s_FuncInfo@@H@Z@4HA 000000018002a4db f   libvcruntime:frame.obj
 0001:000294f1       ?fin$1@?0??FrameUnwindToState@__FrameHandler3@@SAXPEA_KPEAU_xDISPATCHER_CONTEXT@@PEBU_s_FuncInfo@@H@Z@4HA 000000018002a4f1 f   libvcruntime:frame.obj
 0001:00029514       ?filt$0@?0???$thread_start@P6AIPEAX@Z$00@@YAKQEAX@Z@4HA 000000018002a514 f   libucrt:thread.obj
 0001:00029532       ?fin$0@?0???$?RV<lambda_842d9ff0dc9ef11c61343bbaebe7f885>@@AEAV<lambda_c5860995281e5c4ce005b3de8f5874ee>@@V<lambda_d90129c13df834fdcbf8d2b88dafcf2d>@@@?$__crt_seh_guarded_call@X@@QEAAX$$QEAV<lambda_842d9ff0dc9ef11c61343bbaebe7f885>@@AEAV<lambda_c5860995281e5c4ce005b3de8f5874ee>@@$$QEAV<lambda_d90129c13df834fdcbf8d2b88dafcf2d>@@@Z@4HA 000000018002a532 f   libucrt:fflush.obj
 0001:00029532       ?fin$0@?0???$?RV<lambda_613eff765f5c257adf68e381dfe80f05>@@AEAV<lambda_ebf663be9fcd9e0b17ed57bdb95b0759>@@V<lambda_872abebd861b7db59b42e49ea65623b0>@@@?$__crt_seh_guarded_call@H@@QEAAH$$QEAV<lambda_613eff765f5c257adf68e381dfe80f05>@@AEAV<lambda_ebf663be9fcd9e0b17ed57bdb95b0759>@@$$QEAV<lambda_872abebd861b7db59b42e49ea65623b0>@@@Z@4HA 000000018002a532 f   libucrt:output.obj
 0001:00029532       ?fin$0@?0???$?RV<lambda_d854c62834386a3b23916ad6dae2782d>@@AEAV<lambda_303760bc4008a2b3ec4768a30b06a80c>@@V<lambda_4780a7ea4f8cbd2590aec34bd14e2bbf>@@@?$__crt_seh_guarded_call@H@@QEAAH$$QEAV<lambda_d854c62834386a3b23916ad6dae2782d>@@AEAV<lambda_303760bc4008a2b3ec4768a30b06a80c>@@$$QEAV<lambda_4780a7ea4f8cbd2590aec34bd14e2bbf>@@@Z@4HA 000000018002a532 f   libucrt:output.obj
 0001:0002954d       ?fin$0@?0??_fclose_internal@@YAHQEAU_iobuf@@AEAV__crt_cached_ptd_host@@@Z@4HA 000000018002a54d f   libucrt:fclose.obj
 0001:00029565       ?fin$0@?0???$common_fsopen@D@@YAPEAU_iobuf@@QEBD0H@Z@4HA 000000018002a565 f   libucrt:fopen.obj
 0001:00029590       ?fin$0@?0???$common_getenv@D@@YAPEADQEBD@Z@4HA 000000018002a590 f   libucrt:getenv.obj
 0001:000295b0       _query_new_handler$fin$0   000000018002a5b0 f   libucrt:new_handler.obj
 0001:000295c6       _set_new_handler$fin$0     000000018002a5c6 f   libucrt:new_handler.obj
 0001:000295dc       ?fin$0@?0???$?RV<lambda_0ae27a3a962d80f24befdcbee591983d>@@AEAV<lambda_8d0ee55de4b1038c4002e0adecdf1839>@@V<lambda_dc504788e8f1664fe9b84e20bfb512f2>@@@?$__crt_seh_guarded_call@X@@QEAAX$$QEAV<lambda_0ae27a3a962d80f24befdcbee591983d>@@AEAV<lambda_8d0ee55de4b1038c4002e0adecdf1839>@@$$QEAV<lambda_dc504788e8f1664fe9b84e20bfb512f2>@@@Z@4HA 000000018002a5dc f   libucrt:per_thread_data.obj
 0001:000295dc       ?fin$0@?0???$?RV<lambda_2d41944a1d46af3157314b8a01080d33>@@AEAV<lambda_8f455de75cd7d7f24b4096f044d8b9e6>@@V<lambda_aa500f224e6afead328df44964fe2772>@@@?$__crt_seh_guarded_call@X@@QEAAX$$QEAV<lambda_2d41944a1d46af3157314b8a01080d33>@@AEAV<lambda_8f455de75cd7d7f24b4096f044d8b9e6>@@$$QEAV<lambda_aa500f224e6afead328df44964fe2772>@@@Z@4HA 000000018002a5dc f   libucrt:per_thread_data.obj
 0001:000295dc       ?fin$0@?0???$?RV<lambda_aa87e3671a710a21b5dc78c0bdf72e11>@@AEAV<lambda_92619d2358a28f41a33ba319515a20b9>@@V<lambda_6992ecaafeb10aed2b74cb1fae11a551>@@@?$__crt_seh_guarded_call@X@@QEAAX$$QEAV<lambda_aa87e3671a710a21b5dc78c0bdf72e11>@@AEAV<lambda_92619d2358a28f41a33ba319515a20b9>@@$$QEAV<lambda_6992ecaafeb10aed2b74cb1fae11a551>@@@Z@4HA 000000018002a5dc f   libucrt:per_thread_data.obj
 0001:000295dc       ?fin$0@?0???$?RV<lambda_f2e299630e499de9f9a165e60fcd3db5>@@AEAV<lambda_2ae9d31cdba2644fcbeaf08da7c24588>@@V<lambda_40d01ff24d0e7b3814fdbdcee8eab3c7>@@@?$__crt_seh_guarded_call@X@@QEAAX$$QEAV<lambda_f2e299630e499de9f9a165e60fcd3db5>@@AEAV<lambda_2ae9d31cdba2644fcbeaf08da7c24588>@@$$QEAV<lambda_40d01ff24d0e7b3814fdbdcee8eab3c7>@@@Z@4HA 000000018002a5dc f   libucrt:per_thread_data.obj
 0001:000295dc       ?fin$0@?0???$?RV<lambda_450d765d439847d4c735a33c368b5fc0>@@AEAV<lambda_44731a7d0e6d81c3e6aa82d741081786>@@V<lambda_601a2a7da3b7a96e9554ac7215c4b07c>@@@?$__crt_seh_guarded_call@P6AXH@Z@@QEAAP6AXH@Z$$QEAV<lambda_450d765d439847d4c735a33c368b5fc0>@@AEAV<lambda_44731a7d0e6d81c3e6aa82d741081786>@@$$QEAV<lambda_601a2a7da3b7a96e9554ac7215c4b07c>@@@Z@4HA 000000018002a5dc f   libucrt:signal.obj
 0001:000295dc       ?fin$0@?0???$?RV<lambda_d80eeec6fff315bfe5c115232f3240e3>@@AEAV<lambda_6e4b09c48022b2350581041d5f6b0c4c>@@V<lambda_2358e3775559c9db80273638284d5e45>@@@?$__crt_seh_guarded_call@X@@QEAAX$$QEAV<lambda_d80eeec6fff315bfe5c115232f3240e3>@@AEAV<lambda_6e4b09c48022b2350581041d5f6b0c4c>@@$$QEAV<lambda_2358e3775559c9db80273638284d5e45>@@@Z@4HA 000000018002a5dc f   libucrt:exit.obj
 0001:000295dc       ?fin$0@?0???$?RV<lambda_7777bce6b2f8c936911f934f8298dc43>@@AEAV<lambda_f03950bc5685219e0bcd2087efbe011e>@@V<lambda_3883c3dff614d5e0c5f61bb1ac94921c>@@@?$__crt_seh_guarded_call@H@@QEAAH$$QEAV<lambda_7777bce6b2f8c936911f934f8298dc43>@@AEAV<lambda_f03950bc5685219e0bcd2087efbe011e>@@$$QEAV<lambda_3883c3dff614d5e0c5f61bb1ac94921c>@@@Z@4HA 000000018002a5dc f   libucrt:onexit.obj
 0001:000295f6       ?filt$0@?0???R<lambda_6e4b09c48022b2350581041d5f6b0c4c>@@QEBA@XZ@4HA 000000018002a5f6 f   libucrt:exit.obj
 0001:00029623       _fcloseall$fin$0           000000018002a623 f   libucrt:closeall.obj
 0001:00029623       ?fin$0@?0??__acrt_stdio_allocate_stream@@YA?AV__crt_stdio_stream@@XZ@4HA 000000018002a623 f   libucrt:stream.obj
 0001:0002963c       ?fin$0@?0???$?RV<lambda_886d6c58226a84441f68b9f2b8217b83>@@AEAV<lambda_ab61a845afdef5b7c387490eaf3616ee>@@V<lambda_f7f22ab5edc0698d5f6905b0d3f44752>@@@?$__crt_seh_guarded_call@X@@QEAAX$$QEAV<lambda_886d6c58226a84441f68b9f2b8217b83>@@AEAV<lambda_ab61a845afdef5b7c387490eaf3616ee>@@$$QEAV<lambda_f7f22ab5edc0698d5f6905b0d3f44752>@@@Z@4HA 000000018002a63c f   libucrt:fflush.obj
 0001:00029659       __acrt_initialize_lowio$fin$0 000000018002a659 f   libucrt:ioinit.obj
 0001:00029659       __acrt_lowio_ensure_fh_exists$fin$0 000000018002a659 f   libucrt:osfinfo.obj
 0001:00029659       _alloc_osfhnd$fin$0        000000018002a659 f   libucrt:osfinfo.obj
 0001:00029672       ?fin$0@?0???$?RV<lambda_410d79af7f07d98d83a3f525b3859a53>@@AEAV<lambda_3e16ef9562a7dcce91392c22ab16ea36>@@V<lambda_38119f0e861e05405d8a144b9b982f0a>@@@?$__crt_seh_guarded_call@X@@QEAAX$$QEAV<lambda_410d79af7f07d98d83a3f525b3859a53>@@AEAV<lambda_3e16ef9562a7dcce91392c22ab16ea36>@@$$QEAV<lambda_38119f0e861e05405d8a144b9b982f0a>@@@Z@4HA 000000018002a672 f   libucrt:wsetlocale.obj
 0001:0002968c       ?fin$0@?0???$?RV<lambda_ad8af0d99a0adf03d037d7dffe354bb5>@@AEAV<lambda_c9ba49e555ba839a7b07aa3fbecb7617>@@V<lambda_2f1ebd5d68526518146ae959c9e734c8>@@@?$__crt_seh_guarded_call@H@@QEAAH$$QEAV<lambda_ad8af0d99a0adf03d037d7dffe354bb5>@@AEAV<lambda_c9ba49e555ba839a7b07aa3fbecb7617>@@$$QEAV<lambda_2f1ebd5d68526518146ae959c9e734c8>@@@Z@4HA 000000018002a68c f   libucrt:close.obj
 0001:0002968c       ?fin$0@?0???$?RV<lambda_a37b2b86f63e897a80ea819b0eb08c01>@@AEAV<lambda_38ce7e780aa69e748d6df282ebc68efe>@@V<lambda_99fb1378e971ab6e7edea83e3a7a83a2>@@@?$__crt_seh_guarded_call@H@@QEAAH$$QEAV<lambda_a37b2b86f63e897a80ea819b0eb08c01>@@AEAV<lambda_38ce7e780aa69e748d6df282ebc68efe>@@$$QEAV<lambda_99fb1378e971ab6e7edea83e3a7a83a2>@@@Z@4HA 000000018002a68c f   libucrt:commit.obj
 0001:000296a6       ?fin$0@?0???$?RV<lambda_efdfa57d1f175319df784efa44bb7b81>@@AEAV<lambda_5f0a4c1567f8adc6734073e5d1e1b35c>@@V<lambda_2e8a7d3640ea6ccb4c2413664c2db6fd>@@@?$__crt_seh_guarded_call@X@@QEAAX$$QEAV<lambda_efdfa57d1f175319df784efa44bb7b81>@@AEAV<lambda_5f0a4c1567f8adc6734073e5d1e1b35c>@@$$QEAV<lambda_2e8a7d3640ea6ccb4c2413664c2db6fd>@@@Z@4HA 000000018002a6a6 f   libucrt:mbctype.obj
 0001:000296c0       ?fin$0@?0??update_thread_multibyte_data_internal@@YAPEAU__crt_multibyte_data@@QEAU__acrt_ptd@@QEAPEAU1@@Z@4HA 000000018002a6c0 f   libucrt:mbctype.obj
 0001:000296d9       raise$fin$0                000000018002a6d9 f   libucrt:signal.obj
 0001:000296fa       __acrt_update_thread_locale_data$fin$0 000000018002a6fa f   libucrt:locale_refcounting.obj
 0001:00029713       ?fin$0@?0???$common_lseek@_J@@YA_JH_JHAEAV__crt_cached_ptd_host@@@Z@4HA 000000018002a713 f   libucrt:lseek.obj
 0001:00029713       _write_internal$fin$0      000000018002a713 f   libucrt:write.obj
 0001:0002972a       ?fin$0@?0???$common_sopen_dispatch@D@@YAHQEBDHHHQEAHH@Z@4HA 000000018002a72a f   libucrt:open.obj
 0001:000297a2       common_control87$filt$0    000000018002a7a2 f   libucrt:ieee.obj
 0001:000297ce       _ctrlfp$filt$0             000000018002a7ce f   libucrt:fpctrl.obj
 0001:00029800       _IsNonwritableInCurrentImage$filt$0 000000018002a800 f   LIBCMT:pesect.obj
 0002:0000fb08       GS_ExceptionPointers       000000018003ab08     LIBCMT:gs_report.obj
 0002:0000fb50       ?tokenTable@@3QBUStringLiteral@@B 000000018003ab50     libvcruntime:undname.obj
 0002:0000fc60       ?nameTable@@3QBUStringLiteral@@B 000000018003ac60     libvcruntime:undname.obj
 0002:00010190       ?rttiTable@@3QBUStringLiteral@@B 000000018003b190     libvcruntime:undname.obj
 0002:000101e0       ?IndirectionName@@3QBUStringLiteral@@B 000000018003b1e0     libvcruntime:undname.obj
 0002:00010240       ?PrefixName@@3QBUStringLiteral@@B 000000018003b240     libvcruntime:undname.obj
 0002:00010930       ?ExceptionTemplate@?1??UnwindNestedFrames@__FrameHandler3@@SAXPEA_KPEAUEHExceptionRecord@@PEAU_CONTEXT@@0PEAXPEBU_s_FuncInfo@@HHPEBU_s_HandlerType@@PEAU_xDISPATCHER_CONTEXT@@E@Z@4U_EXCEPTION_RECORD@@B 000000018003b930     libvcruntime:risctrnsctrl.obj
 0002:000109c8       ?module_names@?A0x14174aea@@3QBQEB_WB 000000018003b9c8     libvcruntime:winapi_downlevel.obj
 0002:00010a88       ?candidate_modules@?1??try_get_FlsAlloc@@YAP6AKP6AXPEAX@Z@ZXZ@4QBW4module_id@?A0x14174aea@@B 000000018003ba88     libvcruntime:winapi_downlevel.obj
 0002:00010aa0       ?candidate_modules@?1??try_get_FlsFree@@YAP6AHK@ZXZ@4QBW4module_id@?A0x14174aea@@B 000000018003baa0     libvcruntime:winapi_downlevel.obj
 0002:00010ab0       ?candidate_modules@?1??try_get_FlsGetValue@@YAP6APEAXK@ZXZ@4QBW4module_id@?A0x14174aea@@B 000000018003bab0     libvcruntime:winapi_downlevel.obj
 0002:00010ac8       ?candidate_modules@?1??try_get_FlsSetValue@@YAP6AHKPEAX@ZXZ@4QBW4module_id@?A0x14174aea@@B 000000018003bac8     libvcruntime:winapi_downlevel.obj
 0002:00010ae0       ?candidate_modules@?1??try_get_InitializeCriticalSectionEx@@YAP6AHPEAU_RTL_CRITICAL_SECTION@@KK@ZXZ@4QBW4module_id@?A0x14174aea@@B 000000018003bae0     libvcruntime:winapi_downlevel.obj
 0002:00010c30       $cppxdata$?state_case_type@?$output_processor@DV?$stream_output_adapter@D@__crt_stdio_output@@V?$standard_base@DV?$stream_output_adapter@D@__crt_stdio_output@@@2@@__crt_stdio_output@@AEAA_NXZ 000000018003bc30     libucrt:output.obj
 0002:00010c58       $cppxdata$?state_case_type@?$output_processor@_WV?$stream_output_adapter@_W@__crt_stdio_output@@V?$standard_base@_WV?$stream_output_adapter@_W@__crt_stdio_output@@@2@@__crt_stdio_output@@AEAA_NXZ 000000018003bc58     libucrt:output.obj
 0002:00010c80       $cppxdata$?type_case_s_compute_narrow_string_length@?$output_processor@_WV?$stream_output_adapter@_W@__crt_stdio_output@@V?$standard_base@_WV?$stream_output_adapter@_W@__crt_stdio_output@@@2@@__crt_stdio_output@@AEAAHH_W@Z 000000018003bc80     libucrt:output.obj
 0002:00010d88       $cppxdata$?try_cor_exit_process@@YAXI@Z 000000018003bd88     libucrt:exit.obj
 0002:00010db0       $cppxdata$?common_exit@@YAXHW4_crt_exit_cleanup_mode@@W4_crt_exit_return_mode@@@Z 000000018003bdb0     libucrt:exit.obj
 0002:00010e00       $cppxdata$__dcrt_uninitialize_environments_nolock 000000018003be00     libucrt:environment_initialization.obj
 0002:00010e00       $cppxdata$__acrt_freeptd   000000018003be00     libucrt:per_thread_data.obj
 0002:00010e00       $cppxdata$__acrt_getptd_head 000000018003be00     libucrt:per_thread_data.obj
 0002:00010e00       $cppxdata$__acrt_getptd_noexit 000000018003be00     libucrt:per_thread_data.obj
 0002:00010e00       $cppxdata$__acrt_getptd_noexit_explicit 000000018003be00     libucrt:per_thread_data.obj
 0002:00010e28       $cppxdata$_execute_onexit_table 000000018003be28     libucrt:onexit.obj
 0002:00010e50       __acrt_initializers        000000018003be50     libucrt:initialization.obj
 0002:00010f50       ?errtable@@3QBUerrentry@?A0x31fdb9ec@@B 000000018003bf50     libucrt:errno.obj
 0002:000110c0       ?module_names@?A0x391cf84c@@3QBQEB_WB 000000018003c0c0     libucrt:winapi_thunks.obj
 0002:000116a8       ?candidate_modules@?1??try_get_AreFileApisANSI@@YAP6AHXZXZ@4QBW4module_id@?A0x391cf84c@@B 000000018003c6a8     libucrt:winapi_thunks.obj
 0002:000116c0       ?candidate_modules@?1??try_get_CompareStringEx@@YAP6AHPEB_WK0H0HPEAU_nlsversioninfo@@PEAX_J@ZXZ@4QBW4module_id@?A0x391cf84c@@B 000000018003c6c0     libucrt:winapi_thunks.obj
 0002:000116d8       ?candidate_modules@?1??try_get_FlsGetValue2@@YAP6APEAXK@ZXZ@4QBW4module_id@?A0x391cf84c@@B 000000018003c6d8     libucrt:winapi_thunks.obj
 0002:000116f0       ?candidate_modules@?1??try_get_LCMapStringEx@@YAP6AHPEB_WK0HPEA_WHPEAU_nlsversioninfo@@PEAX_J@ZXZ@4QBW4module_id@?A0x391cf84c@@B 000000018003c6f0     libucrt:winapi_thunks.obj
 0002:00011708       ?candidate_modules@?1??try_get_LocaleNameToLCID@@YAP6AKPEB_WK@ZXZ@4QBW4module_id@?A0x391cf84c@@B 000000018003c708     libucrt:winapi_thunks.obj
 0002:00011724       ?candidate_modules@?1??try_get_RoInitialize@@YAP6AJW4RO_INIT_TYPE@@@ZXZ@4QBW4module_id@?A0x391cf84c@@B 000000018003c724     libucrt:winapi_thunks.obj
 0002:00011738       ?candidate_modules@?1??try_get_RoUninitialize@@YAP6AXXZXZ@4QBW4module_id@?A0x391cf84c@@B 000000018003c738     libucrt:winapi_thunks.obj
 0002:00011750       ?candidate_modules@?1??try_get_AppPolicyGetProcessTerminationMethod@@YAP6AJPEAXPEAW4AppPolicyProcessTerminationMethod@@@ZXZ@4QBW4module_id@?A0x391cf84c@@B 000000018003c750     libucrt:winapi_thunks.obj
 0002:00011780       ?candidate_modules@?1??try_get_AppPolicyGetThreadInitializationType@@YAP6AJPEAXPEAW4AppPolicyThreadInitializationType@@@ZXZ@4QBW4module_id@?A0x391cf84c@@B 000000018003c780     libucrt:winapi_thunks.obj
 0002:000117b0       ?strings@?1??fp_format_nan_or_infinity@@YAHW4__acrt_fp_class@@_NPEAD_K1@Z@4QAY03QEBDA 000000018003c7b0     libucrt:cvt.obj
 0002:00011f28       ?_mb_locale_names@@3QBQEB_WB 000000018003cf28     libucrt:mbctype.obj
 0002:00012590       ?LcidToLocaleNameTable@?A0x881e4c05@@3QBULcidToLocaleName@1@B 000000018003d590     libucrt:lcidtoname_downlevel.obj
 0002:00013ff0       ?LocaleNameToIndexTable@?A0x881e4c05@@3QBULocaleNameIndex@1@B 000000018003eff0     libucrt:lcidtoname_downlevel.obj
 0002:00015888       $cppxdata$?write_double_translated_ansi_nolock@@YA?AUwrite_result@?A0x17268360@@HQEBDIAEAV__crt_cached_ptd_host@@@Z 0000000180040888     libucrt:write.obj
 0002:000162b0       __real_ninf                00000001800412b0     libucrt:log10.obj
 0002:000162c0       __real_inf                 00000001800412c0     libucrt:log10.obj
 0002:000162d0       __real_neg_qnan            00000001800412d0     libucrt:log10.obj
 0002:000162e0       __real_qnanbit             00000001800412e0     libucrt:log10.obj
 0002:000162f0       __int_1023                 00000001800412f0     libucrt:log10.obj
 0002:00016300       __mask_001                 0000000180041300     libucrt:log10.obj
 0002:00016310       __mask_mant                0000000180041310     libucrt:log10.obj
 0002:00016320       __mask_mant_top8           0000000180041320     libucrt:log10.obj
 0002:00016330       __mask_mant9               0000000180041330     libucrt:log10.obj
 0002:00016340       __real_log10_e             0000000180041340     libucrt:log10.obj
 0002:00016350       __real_log10_e_lead        0000000180041350     libucrt:log10.obj
 0002:00016360       __real_log10_e_tail        0000000180041360     libucrt:log10.obj
 0002:00016370       __real_log10_2_lead        0000000180041370     libucrt:log10.obj
 0002:00016380       __real_log10_2_tail        0000000180041380     libucrt:log10.obj
 0002:00016390       __real_two                 0000000180041390     libucrt:log10.obj
 0002:000163a0       __real_one                 00000001800413a0     libucrt:log10.obj
 0002:000163b0       __real_half                00000001800413b0     libucrt:log10.obj
 0002:000163c0       __mask_100                 00000001800413c0     libucrt:log10.obj
 0002:000163d0       __real_1_over_512          00000001800413d0     libucrt:log10.obj
 0002:000163e0       __real_1_over_2            00000001800413e0     libucrt:log10.obj
 0002:000163f0       __real_1_over_3            00000001800413f0     libucrt:log10.obj
 0002:00016400       __real_1_over_4            0000000180041400     libucrt:log10.obj
 0002:00016410       __real_1_over_5            0000000180041410     libucrt:log10.obj
 0002:00016420       __real_1_over_6            0000000180041420     libucrt:log10.obj
 0002:00016430       __real_neg_1023            0000000180041430     libucrt:log10.obj
 0002:00016440       __mask_2045                0000000180041440     libucrt:log10.obj
 0002:00016450       __real_threshold           0000000180041450     libucrt:log10.obj
 0002:00016460       __real_near_one_lt         0000000180041460     libucrt:log10.obj
 0002:00016470       __real_near_one_gt         0000000180041470     libucrt:log10.obj
 0002:00016480       __real_min_norm            0000000180041480     libucrt:log10.obj
 0002:00016490       __real_notsign             0000000180041490     libucrt:log10.obj
 0002:000164a0       __real_ca1                 00000001800414a0     libucrt:log10.obj
 0002:000164b0       __real_ca2                 00000001800414b0     libucrt:log10.obj
 0002:000164c0       __real_ca3                 00000001800414c0     libucrt:log10.obj
 0002:000164d0       __real_ca4                 00000001800414d0     libucrt:log10.obj
 0002:000164e0       __mask_lower               00000001800414e0     libucrt:log10.obj
 0002:000164f0       __flag_x_zero              00000001800414f0     libucrt:log10.obj
 0002:000164f4       __flag_x_neg               00000001800414f4     libucrt:log10.obj
 0002:000164f8       __flag_x_nan               00000001800414f8     libucrt:log10.obj
 0002:00016510       DoubleNegZero              0000000180041510     libucrt:floorceil_sse41.obj
 0002:00016520       DoubleLargestNumBelowHalf  0000000180041520     libucrt:floorceil_sse41.obj
 0002:00016530       FloatNegZero               0000000180041530     libucrt:floorceil_sse41.obj
 0002:00016540       FloatLargestNumBelowHalf   0000000180041540     libucrt:floorceil_sse41.obj
 0002:00017f40       MoveSmall                  0000000180042f40     libvcruntime:memcpy.obj
 0002:00017f80       MoveSmallYmm               0000000180042f80     libvcruntime:memcpy.obj
 0002:00017fa4       MoveSmallYmmNT             0000000180042fa4     libvcruntime:memcpy.obj
 0002:00017fc8       MoveSmallXmm               0000000180042fc8     libvcruntime:memcpy.obj
 0002:00017ff0       SetSmall                   0000000180042ff0     libvcruntime:memset.obj
 0002:00018030       SetSmallYmm                0000000180043030     libvcruntime:memset.obj
 0002:00018054       SetSmallYmmNT              0000000180043054     libvcruntime:memset.obj
 0002:00018078       SetSmallXmm                0000000180043078     libvcruntime:memset.obj
 0002:00018838       $unwind$??0AccessBridgeATInstance@@QEAA@PEAUHWND__@@0PEADPEAV0@@Z 0000000180043838     AccessBridgeATInstance.obj
 0002:00018838       $unwind$??1AccessBridgeATInstance@@QEAA@XZ 0000000180043838     AccessBridgeATInstance.obj
 0002:00018838       $unwind$??0AccessBridgeJavaEntryPoints@@QEAA@PEAUJNIEnv_@@PEAV_jobject@@@Z 0000000180043838     AccessBridgeJavaEntryPoints.obj
 0002:00018838       $unwind$??0JavaAccessBridge@@QEAA@PEAUHINSTANCE__@@@Z 0000000180043838     JavaAccessBridge.obj
 0002:00018838       $unwind$DllMain            0000000180043838     JavaAccessBridge.obj
 0002:00018838       $unwind$__raise_securityfailure 0000000180043838     LIBCMT:gs_report.obj
 0002:00018838       $unwind$??2@YAPEAX_K@Z     0000000180043838     LIBCMT:new_scalar.obj
 0002:00018838       $unwind$??_Gtype_info@@UEAAPEAXI@Z 0000000180043838     LIBCMT:std_type_info_static.obj
 0002:00018838       $unwind$??0bad_alloc@std@@QEAA@AEBV01@@Z 0000000180043838     LIBCMT:throw_bad_alloc.obj
 0002:00018838       $unwind$??0bad_array_new_length@std@@QEAA@AEBV01@@Z 0000000180043838     LIBCMT:throw_bad_alloc.obj
 0002:00018838       $unwind$??0exception@std@@QEAA@AEBV01@@Z 0000000180043838     LIBCMT:throw_bad_alloc.obj
 0002:00018838       $unwind$__scrt_initialize_onexit_tables 0000000180043838     LIBCMT:utility.obj
 0002:00018838       $unwind$__scrt_release_startup_lock 0000000180043838     LIBCMT:utility.obj
 0002:00018838       $unwind$__scrt_uninitialize_crt 0000000180043838     LIBCMT:utility.obj
 0002:00018838       $unwind$_IsExceptionObjectToBeDestroyed 0000000180043838     libvcruntime:ehhelpers.obj
 0002:00018838       $unwind$?GetUnwindTryBlock@__FrameHandler3@@SAHPEA_KPEAU_xDISPATCHER_CONTEXT@@PEBU_s_FuncInfo@@@Z 0000000180043838     libvcruntime:ehstate.obj
 0002:00018838       $unwind$?StateFromIp@__FrameHandler3@@SAHPEBU_s_FuncInfo@@PEAU_xDISPATCHER_CONTEXT@@_K@Z 0000000180043838     libvcruntime:ehstate.obj
 0002:00018838       $unwind$??0bad_exception@std@@QEAA@AEBV01@@Z 0000000180043838     libvcruntime:frame.obj
 0002:00018838       $unwind$?ExFilterRethrow@@YAHPEAU_EXCEPTION_POINTERS@@PEAUEHExceptionRecord@@PEAH@Z 0000000180043838     libvcruntime:frame.obj
 0002:00018838       $unwind$__vcrt_initialize_locks 0000000180043838     libvcruntime:locks.obj
 0002:00018838       $unwind$__vcrt_uninitialize_locks 0000000180043838     libvcruntime:locks.obj
 0002:00018838       $unwind$__vcrt_freeptd_for_this_thread 0000000180043838     libvcruntime:per_thread_data.obj
 0002:00018838       $unwind$?ExecutionInCatch@__FrameHandler3@@SA_NPEAU_xDISPATCHER_CONTEXT@@PEBU_s_FuncInfo@@@Z 0000000180043838     libvcruntime:risctrnsctrl.obj
 0002:00018838       $unwind$_CreateFrameInfo   0000000180043838     libvcruntime:risctrnsctrl.obj
 0002:00018838       $unwind$_SetImageBase      0000000180043838     libvcruntime:risctrnsctrl.obj
 0002:00018838       $unwind$_SetThrowImageBase 0000000180043838     libvcruntime:risctrnsctrl.obj
 0002:00018838       $unwind$__std_exception_destroy 0000000180043838     libvcruntime:std_exception.obj
 0002:00018838       $unwind$__std_type_info_destroy_list 0000000180043838     libvcruntime:std_type_info.obj
 0002:00018838       $unwind$__vcrt_FlsAlloc    0000000180043838     libvcruntime:winapi_downlevel.obj
 0002:00018838       $unwind$__vcrt_FlsFree     0000000180043838     libvcruntime:winapi_downlevel.obj
 0002:00018838       $unwind$__vcrt_FlsGetValue 0000000180043838     libvcruntime:winapi_downlevel.obj
 0002:00018838       $unwind$?__c16rtomb_utf8@__crt_mbstring@@YA_KPEAD_SPEAU_Mbstatet@@AEAV__crt_cached_ptd_host@@@Z 0000000180043838     libucrt:c16rtomb.obj
 0002:00018838       $unwind$initialize_pointers 0000000180043838     libucrt:initialization.obj
 0002:00018838       $unwind$uninitialize_allocated_memory 0000000180043838     libucrt:initialization.obj
 0002:00018838       $unwind$__acrt_initialize_locks 0000000180043838     libucrt:locks.obj
 0002:00018838       $unwind$__acrt_uninitialize_locks 0000000180043838     libucrt:locks.obj
 0002:00018838       $unwind$__acrt_get_process_end_policy 0000000180043838     libucrt:win_policies.obj
 0002:00018838       $unwind$__acrt_AppPolicyGetProcessTerminationMethodInternal 0000000180043838     libucrt:winapi_thunks.obj
 0002:00018838       $unwind$__acrt_AppPolicyGetThreadInitializationTypeInternal 0000000180043838     libucrt:winapi_thunks.obj
 0002:00018838       $unwind$__acrt_RoInitialize 0000000180043838     libucrt:winapi_thunks.obj
 0002:00018838       $unwind$__acrt_uninitialize_winapi_thunks 0000000180043838     libucrt:winapi_thunks.obj
 0002:00018838       $unwind$__acrt_update_locale_info 0000000180043838     libucrt:locale_update.obj
 0002:00018838       $unwind$__acrt_update_locale_info_explicit 0000000180043838     libucrt:locale_update.obj
 0002:00018838       $unwind$__acrt_update_multibyte_info 0000000180043838     libucrt:locale_update.obj
 0002:00018838       $unwind$__acrt_update_multibyte_info_explicit 0000000180043838     libucrt:locale_update.obj
 0002:00018838       $unwind$__acrt_errno_map_os_error 0000000180043838     libucrt:errno.obj
 0002:00018838       $unwind$__acrt_errno_map_os_error_ptd 0000000180043838     libucrt:errno.obj
 0002:00018838       $unwind$__acrt_allocate_buffer_for_argv 0000000180043838     libucrt:argv_parsing.obj
 0002:00018838       $unwind$?exit_or_terminate_process@@YAXI_N@Z 0000000180043838     libucrt:exit.obj
 0002:00018838       $unwind$__acrt_uninitialize_stdio 0000000180043838     libucrt:_file.obj
 0002:00018838       $unwind$?stream_is_at_end_of_file_nolock@@YA_NV__crt_stdio_stream@@@Z 0000000180043838     libucrt:_flsbuf.obj
 0002:00018838       $unwind$__acrt_stdio_free_buffer_nolock 0000000180043838     libucrt:_freebuf.obj
 0002:00018838       $unwind$__acrt_should_use_temporary_buffer 0000000180043838     libucrt:_sftbuf.obj
 0002:00018838       $unwind$?type_case_s@?$output_processor@DV?$stream_output_adapter@D@__crt_stdio_output@@V?$standard_base@DV?$stream_output_adapter@D@__crt_stdio_output@@@2@@__crt_stdio_output@@AEAA_NXZ 0000000180043838     libucrt:output.obj
 0002:00018838       $unwind$strcpy_s           0000000180043838     libucrt:strcpy_s.obj
 0002:00018838       $unwind$_controlfp_s       0000000180043838     libucrt:contrlfp.obj
 0002:00018838       $unwind$fegetenv           0000000180043838     libucrt:fegetenv.obj
 0002:00018838       $unwind$feholdexcept       0000000180043838     libucrt:feholdexcept.obj
 0002:00018840       $unwind$?initiateIPC@AccessBridgeATInstance@@QEAA_JXZ 0000000180043840     AccessBridgeATInstance.obj
 0002:00018840       $unwind$?postHelloToWindowsDLLMsg@JavaAccessBridge@@QEAAXPEAUHWND__@@@Z 0000000180043840     JavaAccessBridge.obj
 0002:00018840       $unwind$?type_case_c_tchar@?$output_processor@DV?$stream_output_adapter@D@__crt_stdio_output@@V?$standard_base@DV?$stream_output_adapter@D@__crt_stdio_output@@@2@@__crt_stdio_output@@AEAA_ND@Z 0000000180043840     libucrt:output.obj
 0002:00018840       $unwind$?type_case_n@?$output_processor@DV?$stream_output_adapter@D@__crt_stdio_output@@V?$standard_base@DV?$stream_output_adapter@D@__crt_stdio_output@@@2@@__crt_stdio_output@@AEAA_NXZ 0000000180043840     libucrt:output.obj
 0002:00018840       $unwind$?type_case_n@?$output_processor@_WV?$stream_output_adapter@_W@__crt_stdio_output@@V?$standard_base@_WV?$stream_output_adapter@_W@__crt_stdio_output@@@2@@__crt_stdio_output@@AEAA_NXZ 0000000180043840     libucrt:output.obj
 0002:0001884c       $unwind$?sendAccessibilityEventPackage@AccessBridgeATInstance@@QEAA_JPEADHJ@Z 000000018004384c     AccessBridgeATInstance.obj
 0002:0001884c       $unwind$?sendJavaEventPackage@AccessBridgeATInstance@@QEAA_JPEADHJ@Z 000000018004384c     AccessBridgeATInstance.obj
 0002:0001884c       $unwind$?getAccessibleTableInfo@AccessBridgeJavaEntryPoints@@QEAAHPEAV_jobject@@PEAUAccessibleTableInfoTag@@@Z 000000018004384c     AccessBridgeJavaEntryPoints.obj
 0002:0001884c       $unwind$__scrt_dllmain_exception_filter 000000018004384c     LIBCMT:utility.obj
 0002:0001884c       $unwind$?GetHandlerSearchState@__FrameHandler3@@SAHPEA_KPEAU_xDISPATCHER_CONTEXT@@PEBU_s_FuncInfo@@@Z 000000018004384c     libvcruntime:frame.obj
 0002:0001884c       $unwind$?Is_bad_exception_allowed@@YAEPEBU_s_ESTypeList@@@Z 000000018004384c     libvcruntime:frame.obj
 0002:0001884c       $unwind$?CatchTryBlock@__FrameHandler3@@SAPEBU_s_TryBlockMapEntry@@PEBU_s_FuncInfo@@H@Z 000000018004384c     libvcruntime:risctrnsctrl.obj
 0002:0001884c       $unwind$?should_round_up@@YA_NQEBD0HW4__acrt_has_trailing_digits@@W4__acrt_rounding_mode@@@Z 000000018004384c     libucrt:_fptostr.obj
 0002:0001884c       $unwind$__acrt_free_locale 000000018004384c     libucrt:locale_refcounting.obj
 0002:0001884c       $unwind$__acrt_lowio_create_handle_array 000000018004384c     libucrt:osfinfo.obj
 0002:0001884c       $unwind$_seh_filter_exe    000000018004384c     libucrt:exception_filter.obj
 0002:0001884c       $unwind$__acrt_stdio_flush_nolock 000000018004384c     libucrt:fflush.obj
 0002:0001884c       $unwind$??$ensure_buffer_is_big_enough@D@formatting_buffer@__crt_stdio_output@@QEAA_N_KAEAV__crt_cached_ptd_host@@@Z 000000018004384c     libucrt:output.obj
 0002:0001884c       $unwind$??$ensure_buffer_is_big_enough@_W@formatting_buffer@__crt_stdio_output@@QEAA_N_KAEAV__crt_cached_ptd_host@@@Z 000000018004384c     libucrt:output.obj
 0002:00018860       $unwind$?JavaBridgeThread@@YAIPEAX@Z 0000000180043860     AccessBridgeATInstance.obj
 0002:00018868       $unwind$?do_event@@YAXPEADHPEAUHWND__@@1@Z 0000000180043868     AccessBridgeATInstance.obj
 0002:00018868       $unwind$?getAccessibleKeyBindings@AccessBridgeJavaEntryPoints@@QEAAHPEAV_jobject@@PEAUAccessibleKeyBindingsTag@@@Z 0000000180043868     AccessBridgeJavaEntryPoints.obj
 0002:00018868       $unwind$?getAccessibleTableCellInfo@AccessBridgeJavaEntryPoints@@QEAAHPEAV_jobject@@HHPEAUAccessibleTableCellInfoTag@@@Z 0000000180043868     AccessBridgeJavaEntryPoints.obj
 0002:00018868       $unwind$?getAccessibleTableColumnSelections@AccessBridgeJavaEntryPoints@@QEAAHPEAV_jobject@@HPEAH@Z 0000000180043868     AccessBridgeJavaEntryPoints.obj
 0002:00018868       $unwind$?getAccessibleTableRowSelections@AccessBridgeJavaEntryPoints@@QEAAHPEAV_jobject@@HPEAH@Z 0000000180043868     AccessBridgeJavaEntryPoints.obj
 0002:00018868       $unwind$?getAccessibleTextInfo@AccessBridgeJavaEntryPoints@@QEAAHPEAV_jobject@@PEAUAccessibleTextInfoTag@@HH@Z 0000000180043868     AccessBridgeJavaEntryPoints.obj
 0002:00018868       $unwind$?processPackage@JavaAccessBridge@@QEAA_JPEADH@Z 0000000180043868     JavaAccessBridge.obj
 0002:00018868       $unwind$??$create_environment@D@@YAQEAPEADQEAD@Z 0000000180043868     libucrt:environment_initialization.obj
 0002:00018868       $unwind$_mbtowc_internal   0000000180043868     libucrt:mbtowc.obj
 0002:00018868       $unwind$??$__acrt_convert_wcs_mbs_cp@D_WV<lambda_7c9dea7b4ca7285d2cdb541a38da6275>@@U__crt_win32_buffer_internal_dynamic_resizing@@@@YAHQEBDAEAV?$__crt_win32_buffer@_WU__crt_win32_buffer_internal_dynamic_resizing@@@@AEBV<lambda_7c9dea7b4ca7285d2cdb541a38da6275>@@I@Z 0000000180043868     libucrt:argv_wildcards.obj
 0002:00018868       $unwind$??$type_case_integer@$07@?$output_processor@DV?$stream_output_adapter@D@__crt_stdio_output@@V?$standard_base@DV?$stream_output_adapter@D@__crt_stdio_output@@@2@@__crt_stdio_output@@AEAA_N_N@Z 0000000180043868     libucrt:output.obj
 0002:00018868       $unwind$??$type_case_integer@$07@?$output_processor@_WV?$stream_output_adapter@_W@__crt_stdio_output@@V?$standard_base@_WV?$stream_output_adapter@_W@__crt_stdio_output@@@2@@__crt_stdio_output@@AEAA_N_N@Z 0000000180043868     libucrt:output.obj
 0002:00018868       $unwind$??$type_case_integer@$09@?$output_processor@DV?$stream_output_adapter@D@__crt_stdio_output@@V?$standard_base@DV?$stream_output_adapter@D@__crt_stdio_output@@@2@@__crt_stdio_output@@AEAA_N_N@Z 0000000180043868     libucrt:output.obj
 0002:00018868       $unwind$??$type_case_integer@$09@?$output_processor@_WV?$stream_output_adapter@_W@__crt_stdio_output@@V?$standard_base@_WV?$stream_output_adapter@_W@__crt_stdio_output@@@2@@__crt_stdio_output@@AEAA_N_N@Z 0000000180043868     libucrt:output.obj
 0002:00018868       $unwind$??$type_case_integer@$0BA@@?$output_processor@DV?$stream_output_adapter@D@__crt_stdio_output@@V?$standard_base@DV?$stream_output_adapter@D@__crt_stdio_output@@@2@@__crt_stdio_output@@AEAA_N_N@Z 0000000180043868     libucrt:output.obj
 0002:00018868       $unwind$??$type_case_integer@$0BA@@?$output_processor@_WV?$stream_output_adapter@_W@__crt_stdio_output@@V?$standard_base@_WV?$stream_output_adapter@_W@__crt_stdio_output@@@2@@__crt_stdio_output@@AEAA_N_N@Z 0000000180043868     libucrt:output.obj
 0002:00018868       $unwind$?process@?$output_processor@DV?$stream_output_adapter@D@__crt_stdio_output@@V?$standard_base@DV?$stream_output_adapter@D@__crt_stdio_output@@@2@@__crt_stdio_output@@QEAAHXZ 0000000180043868     libucrt:output.obj
 0002:00018868       $unwind$?process@?$output_processor@_WV?$stream_output_adapter@_W@__crt_stdio_output@@V?$standard_base@_WV?$stream_output_adapter@_W@__crt_stdio_output@@@2@@__crt_stdio_output@@QEAAHXZ 0000000180043868     libucrt:output.obj
 0002:00018880       $unwind$PrintDebugString   0000000180043880     AccessBridgeDebug.obj
 0002:00018880       $unwind$wPrintDebugString  0000000180043880     AccessBridgeDebug.obj
 0002:00018880       $unwind$wPrintJavaDebugString 0000000180043880     AccessBridgeDebug.obj
 0002:00018888       $unwind$initializeFileLogger 0000000180043888     AccessBridgeDebug.obj
 0002:00018888       $unwind$?getCurrentAccessibleValueFromContext@AccessBridgeJavaEntryPoints@@QEAAHPEAV_jobject@@PEAGF@Z 0000000180043888     AccessBridgeJavaEntryPoints.obj
 0002:00018888       $unwind$?getMaximumAccessibleValueFromContext@AccessBridgeJavaEntryPoints@@QEAAHPEAV_jobject@@PEAGF@Z 0000000180043888     AccessBridgeJavaEntryPoints.obj
 0002:00018888       $unwind$?getMinimumAccessibleValueFromContext@AccessBridgeJavaEntryPoints@@QEAAHPEAV_jobject@@PEAGF@Z 0000000180043888     AccessBridgeJavaEntryPoints.obj
 0002:00018888       $unwind$?getVirtualAccessibleName@AccessBridgeJavaEntryPoints@@QEAAHQEAV_jobject@@PEAGH@Z 0000000180043888     AccessBridgeJavaEntryPoints.obj
 0002:00018888       $unwind$?fp_format_f_internal@@YAHQEAD_KHQEAU_strflt@@_NAEAV__crt_cached_ptd_host@@@Z 0000000180043888     libucrt:cvt.obj
 0002:00018888       $unwind$__acrt_DownlevelLocaleNameToLCID 0000000180043888     libucrt:lcidtoname_downlevel.obj
 0002:00018888       $unwind$??R<lambda_f03950bc5685219e0bcd2087efbe011e>@@QEBA@XZ 0000000180043888     libucrt:onexit.obj
 0002:00018888       $unwind$?write_string_impl@?$output_adapter_common@DV?$stream_output_adapter@D@__crt_stdio_output@@@__crt_stdio_output@@IEBAXQEBDHQEAHAEAV__crt_cached_ptd_host@@@Z 0000000180043888     libucrt:output.obj
 0002:00018888       $unwind$?write_string_impl@?$output_adapter_common@_WV?$stream_output_adapter@_W@__crt_stdio_output@@@__crt_stdio_output@@IEBAXQEB_WHQEAHAEAV__crt_cached_ptd_host@@@Z 0000000180043888     libucrt:output.obj
 0002:000188a0       $unwind$finalizeFileLogger 00000001800438a0     AccessBridgeDebug.obj
 0002:000188a0       $unwind$getTimeStamp       00000001800438a0     AccessBridgeDebug.obj
 0002:000188a0       $unwind$?initBroadcastMessageIDs@@YAHXZ 00000001800438a0     AccessBridgeMessages.obj
 0002:000188a0       $unwind$__scrt_initialize_default_local_stdio_options 00000001800438a0     LIBCMT:default_local_stdio_options.obj
 0002:000188a0       $unwind$?dllmain_crt_dispatch@@YAHQEAUHINSTANCE__@@KQEAX@Z 00000001800438a0     LIBCMT:dll_dllmain.obj
 0002:000188a0       $unwind$__GSHandlerCheck   00000001800438a0     LIBCMT:gshandler.obj
 0002:000188a0       $unwind$__scrt_acquire_startup_lock 00000001800438a0     LIBCMT:utility.obj
 0002:000188a0       $unwind$__scrt_dllmain_after_initialize_c 00000001800438a0     LIBCMT:utility.obj
 0002:000188a0       $unwind$__scrt_dllmain_before_initialize_c 00000001800438a0     LIBCMT:utility.obj
 0002:000188a0       $unwind$__scrt_dllmain_crt_thread_attach 00000001800438a0     LIBCMT:utility.obj
 0002:000188a0       $unwind$__scrt_dllmain_crt_thread_detach 00000001800438a0     LIBCMT:utility.obj
 0002:000188a0       $unwind$__scrt_dllmain_uninitialize_c 00000001800438a0     LIBCMT:utility.obj
 0002:000188a0       $unwind$__scrt_dllmain_uninitialize_critical 00000001800438a0     LIBCMT:utility.obj
 0002:000188a0       $unwind$__scrt_initialize_crt 00000001800438a0     LIBCMT:utility.obj
 0002:000188a0       $unwind$__std_terminate    00000001800438a0     libvcruntime:ehhelpers.obj
 0002:000188a0       $unwind$?GetCurrentState@__FrameHandler3@@SAHPEA_KPEAU_xDISPATCHER_CONTEXT@@PEBU_s_FuncInfo@@@Z 00000001800438a0     libvcruntime:ehstate.obj
 0002:000188a0       $xdatasym$_CallSettingFrame 00000001800438a0     libvcruntime:handlers.obj
 0002:000188a0       $unwind$__vcrt_initialize  00000001800438a0     libvcruntime:initialization.obj
 0002:000188a0       $unwind$__vcrt_thread_attach 00000001800438a0     libvcruntime:initialization.obj
 0002:000188a0       $unwind$__vcrt_thread_detach 00000001800438a0     libvcruntime:initialization.obj
 0002:000188a0       $unwind$__vcrt_uninitialize 00000001800438a0     libvcruntime:initialization.obj
 0002:000188a0       $unwind$__vcrt_uninitialize_critical 00000001800438a0     libvcruntime:initialization.obj
 0002:000188a0       $unwind$__vcrt_freefls     00000001800438a0     libvcruntime:per_thread_data.obj
 0002:000188a0       $unwind$__vcrt_getptd      00000001800438a0     libvcruntime:per_thread_data.obj
 0002:000188a0       $unwind$__vcrt_initialize_ptd 00000001800438a0     libvcruntime:per_thread_data.obj
 0002:000188a0       $unwind$__vcrt_uninitialize_ptd 00000001800438a0     libvcruntime:per_thread_data.obj
 0002:000188a0       $unwind$_GetImageBase      00000001800438a0     libvcruntime:risctrnsctrl.obj
 0002:000188a0       $unwind$_GetThrowImageBase 00000001800438a0     libvcruntime:risctrnsctrl.obj
 0002:000188a0       $unwind$__dcrt_terminate_console_output 00000001800438a0     libucrt:initcon.obj
 0002:000188a0       $unwind$??$uninitialize_environment_internal@D@@YAXAEAPEAPEAD@Z 00000001800438a0     libucrt:environment_initialization.obj
 0002:000188a0       $unwind$??$uninitialize_environment_internal@_W@@YAXAEAPEAPEA_W@Z 00000001800438a0     libucrt:environment_initialization.obj
 0002:000188a0       $unwind$__dcrt_get_or_create_narrow_environment_nolock 00000001800438a0     libucrt:environment_initialization.obj
 0002:000188a0       $unwind$?initialize_multibyte@@YAHXZ 00000001800438a0     libucrt:multibyte_initializer.obj
 0002:000188a0       $unwind$__acrt_thread_attach 00000001800438a0     libucrt:initialization.obj
 0002:000188a0       $unwind$__acrt_thread_detach 00000001800438a0     libucrt:initialization.obj
 0002:000188a0       $unwind$__acrt_uninitialize 00000001800438a0     libucrt:initialization.obj
 0002:000188a0       $unwind$__acrt_uninitialize_critical 00000001800438a0     libucrt:initialization.obj
 0002:000188a0       $unwind$initialize_c       00000001800438a0     libucrt:initialization.obj
 0002:000188a0       $unwind$uninitialize_allocated_io_buffers 00000001800438a0     libucrt:initialization.obj
 0002:000188a0       $unwind$uninitialize_environment 00000001800438a0     libucrt:initialization.obj
 0002:000188a0       $unwind$__acrt_getptd      00000001800438a0     libucrt:per_thread_data.obj
 0002:000188a0       $unwind$__acrt_initialize_ptd 00000001800438a0     libucrt:per_thread_data.obj
 0002:000188a0       $unwind$__acrt_uninitialize_ptd 00000001800438a0     libucrt:per_thread_data.obj
 0002:000188a0       $unwind$__acrt_get_begin_thread_init_policy 00000001800438a0     libucrt:win_policies.obj
 0002:000188a0       $unwind$__acrt_AreFileApisANSI 00000001800438a0     libucrt:winapi_thunks.obj
 0002:000188a0       $unwind$__acrt_RoUninitialize 00000001800438a0     libucrt:winapi_thunks.obj
 0002:000188a0       $unwind$__acrt_initialize_winapi_thunks 00000001800438a0     libucrt:winapi_thunks.obj
 0002:000188a0       $unwind$__acrt_tls2_supported 00000001800438a0     libucrt:winapi_thunks.obj
 0002:000188a0       $unwind$__acrt_release_locale_ref 00000001800438a0     libucrt:locale_refcounting.obj
 0002:000188a0       $unwind$_isatty            00000001800438a0     libucrt:isatty.obj
 0002:000188a0       $unwind$_get_osfhandle     00000001800438a0     libucrt:osfinfo.obj
 0002:000188a0       $unwind$_get_fmode         00000001800438a0     libucrt:setmode.obj
 0002:000188a0       $unwind$__acrt_initialize_multibyte 00000001800438a0     libucrt:mbctype.obj
 0002:000188a0       $unwind$__acrt_update_thread_multibyte_data 00000001800438a0     libucrt:mbctype.obj
 0002:000188a0       $unwind$__doserrno         00000001800438a0     libucrt:errno.obj
 0002:000188a0       $unwind$_errno             00000001800438a0     libucrt:errno.obj
 0002:000188a0       $unwind$_invoke_watson     00000001800438a0     libucrt:invalid_parameter.obj
 0002:000188a0       $unwind$abort              00000001800438a0     libucrt:abort.obj
 0002:000188a0       $unwind$__acrt_initialize_command_line 00000001800438a0     libucrt:argv_data.obj
 0002:000188a0       $unwind$_endthreadex       00000001800438a0     libucrt:thread.obj
 0002:000188a0       $unwind$_fileno            00000001800438a0     libucrt:fileno.obj
 0002:000188a0       $unwind$?validate_stream_is_ansi_if_required@?$__acrt_stdio_char_traits@D@@SA_NQEAU_iobuf@@@Z 00000001800438a0     libucrt:output.obj
 0002:000188a0       $unwind$_strnicmp          00000001800438a0     libucrt:strnicmp.obj
 0002:000188a0       $unwind$_clearfp           00000001800438a0     libucrt:ieee.obj
 0002:000188a0       $unwind$fegetround         00000001800438a0     libucrt:fegetround.obj
 0002:000188a0       $unwind$_set_errno_from_matherr 00000001800438a0     libucrt:fpexcept.obj
 0002:000188a8       $unwind$fprintf            00000001800438a8     AccessBridgeDebug.obj
 0002:000188b4       $unwind$printf             00000001800438b4     AccessBridgeDebug.obj
 0002:000188c0       $unwind$?CallBooleanMethod@JNIEnv_@@QEAAEPEAV_jobject@@PEAU_jmethodID@@ZZ 00000001800438c0     AccessBridgeJavaEntryPoints.obj
 0002:000188c0       $unwind$?CallCharMethod@JNIEnv_@@QEAAGPEAV_jobject@@PEAU_jmethodID@@ZZ 00000001800438c0     AccessBridgeJavaEntryPoints.obj
 0002:000188c0       $unwind$?CallFloatMethod@JNIEnv_@@QEAAMPEAV_jobject@@PEAU_jmethodID@@ZZ 00000001800438c0     AccessBridgeJavaEntryPoints.obj
 0002:000188c0       $unwind$?CallIntMethod@JNIEnv_@@QEAAHPEAV_jobject@@PEAU_jmethodID@@ZZ 00000001800438c0     AccessBridgeJavaEntryPoints.obj
 0002:000188c0       $unwind$?CallObjectMethod@JNIEnv_@@QEAAPEAV_jobject@@PEAV2@PEAU_jmethodID@@ZZ 00000001800438c0     AccessBridgeJavaEntryPoints.obj
 0002:000188c0       $unwind$?CallVoidMethod@JNIEnv_@@QEAAXPEAV_jobject@@PEAU_jmethodID@@ZZ 00000001800438c0     AccessBridgeJavaEntryPoints.obj
 0002:000188c8       $unwind$?BuildJavaEntryPoints@AccessBridgeJavaEntryPoints@@QEAAHXZ 00000001800438c8     AccessBridgeJavaEntryPoints.obj
 0002:000188e0       $unwind$?addAccessibilityEventNotification@AccessBridgeJavaEntryPoints@@QEAAH_J@Z 00000001800438e0     AccessBridgeJavaEntryPoints.obj
 0002:000188e0       $unwind$?addJavaEventNotification@AccessBridgeJavaEntryPoints@@QEAAH_J@Z 00000001800438e0     AccessBridgeJavaEntryPoints.obj
 0002:000188e0       $unwind$?clearAccessibleSelectionFromContext@AccessBridgeJavaEntryPoints@@QEAAXPEAV_jobject@@@Z 00000001800438e0     AccessBridgeJavaEntryPoints.obj
 0002:000188e0       $unwind$?getAccessibleContextFromHWND@AccessBridgeJavaEntryPoints@@QEAAPEAV_jobject@@H@Z 00000001800438e0     AccessBridgeJavaEntryPoints.obj
 0002:000188e0       $unwind$?getAccessibleHyperlinkCount@AccessBridgeJavaEntryPoints@@QEAAHQEAV_jobject@@@Z 00000001800438e0     AccessBridgeJavaEntryPoints.obj
 0002:000188e0       $unwind$?getAccessibleSelectionCountFromContext@AccessBridgeJavaEntryPoints@@QEAAHPEAV_jobject@@@Z 00000001800438e0     AccessBridgeJavaEntryPoints.obj
 0002:000188e0       $unwind$?getAccessibleTableColumnSelectionCount@AccessBridgeJavaEntryPoints@@QEAAHPEAV_jobject@@@Z 00000001800438e0     AccessBridgeJavaEntryPoints.obj
 0002:000188e0       $unwind$?getAccessibleTableRowSelectionCount@AccessBridgeJavaEntryPoints@@QEAAHPEAV_jobject@@@Z 00000001800438e0     AccessBridgeJavaEntryPoints.obj
 0002:000188e0       $unwind$?getHWNDFromAccessibleContext@AccessBridgeJavaEntryPoints@@QEAAPEAUHWND__@@PEAV_jobject@@@Z 00000001800438e0     AccessBridgeJavaEntryPoints.obj
 0002:000188e0       $unwind$?getObjectDepth@AccessBridgeJavaEntryPoints@@QEAAHQEAV_jobject@@@Z 00000001800438e0     AccessBridgeJavaEntryPoints.obj
 0002:000188e0       $unwind$?getVisibleChildrenCount@AccessBridgeJavaEntryPoints@@QEAAHQEAV_jobject@@@Z 00000001800438e0     AccessBridgeJavaEntryPoints.obj
 0002:000188e0       $unwind$?isJavaWindow@AccessBridgeJavaEntryPoints@@QEAAHH@Z 00000001800438e0     AccessBridgeJavaEntryPoints.obj
 0002:000188e0       $unwind$?removeAccessibilityEventNotification@AccessBridgeJavaEntryPoints@@QEAAH_J@Z 00000001800438e0     AccessBridgeJavaEntryPoints.obj
 0002:000188e0       $unwind$?removeJavaEventNotification@AccessBridgeJavaEntryPoints@@QEAAH_J@Z 00000001800438e0     AccessBridgeJavaEntryPoints.obj
 0002:000188e0       $unwind$?requestFocus@AccessBridgeJavaEntryPoints@@QEAAHQEAV_jobject@@@Z 00000001800438e0     AccessBridgeJavaEntryPoints.obj
 0002:000188e0       $unwind$?selectAllAccessibleSelectionFromContext@AccessBridgeJavaEntryPoints@@QEAAXPEAV_jobject@@@Z 00000001800438e0     AccessBridgeJavaEntryPoints.obj
 0002:000188e0       $unwind$??1JavaAccessBridge@@QEAA@XZ 00000001800438e0     JavaAccessBridge.obj
 0002:000188e0       $unwind$?releaseJavaObject@JavaAccessBridge@@QEAAXPEAV_jobject@@@Z 00000001800438e0     JavaAccessBridge.obj
 0002:000188e0       $unwind$AccessBridgeDialogProc 00000001800438e0     JavaAccessBridge.obj
 0002:000188e0       $unwind$Java_com_sun_java_accessibility_internal_AccessBridge_runDLL 00000001800438e0     JavaAccessBridge.obj
 0002:000188e0       $unwind$_RTC_Initialize    00000001800438e0     LIBCMT:initsect.obj
 0002:000188e0       $unwind$_RTC_Terminate     00000001800438e0     LIBCMT:initsect.obj
 0002:000188e0       $unwind$??_Gbad_alloc@std@@UEAAPEAXI@Z 00000001800438e0     LIBCMT:throw_bad_alloc.obj
 0002:000188e0       $unwind$??_Gbad_array_new_length@std@@UEAAPEAXI@Z 00000001800438e0     LIBCMT:throw_bad_alloc.obj
 0002:000188e0       $unwind$??_Gexception@std@@UEAAPEAXI@Z 00000001800438e0     LIBCMT:throw_bad_alloc.obj
 0002:000188e0       $unwind$__C_specific_handler_noexcept 00000001800438e0     libvcruntime:chandler_noexcept.obj
 0002:000188e0       $unwind$__FrameUnwindFilter 00000001800438e0     libvcruntime:ehhelpers.obj
 0002:000188e0       $unwind$?SetUnwindTryBlock@__FrameHandler3@@SAXPEA_KPEAU_xDISPATCHER_CONTEXT@@PEBU_s_FuncInfo@@H@Z 00000001800438e0     libvcruntime:ehstate.obj
 0002:000188e0       $unwind$??_Gbad_exception@std@@UEAAPEAXI@Z 00000001800438e0     libvcruntime:frame.obj
 0002:000188e0       $unwind$_FindAndUnlinkFrame 00000001800438e0     libvcruntime:risctrnsctrl.obj
 0002:000188e0       $unwind$__vcrt_FlsSetValue 00000001800438e0     libvcruntime:winapi_downlevel.obj
 0002:000188e0       $unwind$??$common_initialize_environment_nolock@D@@YAHXZ 00000001800438e0     libucrt:environment_initialization.obj
 0002:000188e0       $unwind$?replace_current_thread_locale_nolock@@YAXQEAU__acrt_ptd@@QEAU__crt_locale_data@@@Z 00000001800438e0     libucrt:per_thread_data.obj
 0002:000188e0       $unwind$__acrt_execute_uninitializers 00000001800438e0     libucrt:shared_initialization.obj
 0002:000188e0       $unwind$__acrt_LocaleNameToLCID 00000001800438e0     libucrt:winapi_thunks.obj
 0002:000188e0       $unwind$?free_crt_array_internal@@YAXQEAPEBX_K@Z 00000001800438e0     libucrt:inittime.obj
 0002:000188e0       $unwind$_updatetlocinfoEx_nolock 00000001800438e0     libucrt:locale_refcounting.obj
 0002:000188e0       $unwind$__acrt_uninitialize_lowio 00000001800438e0     libucrt:ioinit.obj
 0002:000188e0       $unwind$?setSBCS@@YAXPEAU__crt_multibyte_data@@@Z 00000001800438e0     libucrt:mbctype.obj
 0002:000188e0       $unwind$_initterm_e        00000001800438e0     libucrt:initterm.obj
 0002:000188e0       $unwind$?common_end_thread@@YAXI@Z 00000001800438e0     libucrt:thread.obj
 0002:000188e0       $unwind$__acrt_stdio_allocate_buffer_nolock 00000001800438e0     libucrt:_getbuf.obj
 0002:000188e0       $unwind$__acrt_stdio_begin_temporary_buffering_nolock 00000001800438e0     libucrt:_sftbuf.obj
 0002:000188e0       $unwind$?type_case_Z@?$output_processor@_WV?$stream_output_adapter@_W@__crt_stdio_output@@V?$standard_base@_WV?$stream_output_adapter@_W@__crt_stdio_output@@@2@@__crt_stdio_output@@AEAA_NXZ 00000001800438e0     libucrt:output.obj
 0002:000188ec       $unwind$?getVersionInfo@AccessBridgeJavaEntryPoints@@QEAAHPEAUAccessBridgeVersionInfoTag@@@Z 00000001800438ec     AccessBridgeJavaEntryPoints.obj
 0002:000188ec       $unwind$?should_round_up@@YA_NQEBN_KFW4__acrt_rounding_mode@@@Z 00000001800438ec     libucrt:cvt.obj
 0002:000188ec       $unwind$_chsize_nolock_internal 00000001800438ec     libucrt:chsize.obj
 0002:000188ec       $unwind$??$parse_command_line@D@@YAXPEADPEAPEAD0PEA_K2@Z 00000001800438ec     libucrt:argv_parsing.obj
 0002:00018908       $unwind$?verifyAccessibleText@AccessBridgeJavaEntryPoints@@QEAAHPEAV_jobject@@@Z 0000000180043908     AccessBridgeJavaEntryPoints.obj
 0002:00018908       $unwind$?get_raw_ptd_noexit@__crt_cached_ptd_host@@QEAAPEAU__acrt_ptd@@XZ 0000000180043908     libucrt:invalid_parameter.obj
 0002:00018908       $unwind$?type_case_c_tchar@?$output_processor@_WV?$stream_output_adapter@_W@__crt_stdio_output@@V?$standard_base@_WV?$stream_output_adapter@_W@__crt_stdio_output@@@2@@__crt_stdio_output@@AEAA_N_W@Z 0000000180043908     libucrt:output.obj
 0002:00018918       $unwind$?getAccessibleContextWithFocus@AccessBridgeJavaEntryPoints@@QEAAPEAV_jobject@@XZ 0000000180043918     AccessBridgeJavaEntryPoints.obj
 0002:00018918       $unwind$?getAccessibleParentFromContext@AccessBridgeJavaEntryPoints@@QEAAPEAV_jobject@@PEAV2@@Z 0000000180043918     AccessBridgeJavaEntryPoints.obj
 0002:00018918       $unwind$?getAccessibleTableColumnHeader@AccessBridgeJavaEntryPoints@@QEAAHPEAV_jobject@@PEAUAccessibleTableInfoTag@@@Z 0000000180043918     AccessBridgeJavaEntryPoints.obj
 0002:00018918       $unwind$?getAccessibleTableRowHeader@AccessBridgeJavaEntryPoints@@QEAAHPEAV_jobject@@PEAUAccessibleTableInfoTag@@@Z 0000000180043918     AccessBridgeJavaEntryPoints.obj
 0002:00018918       $unwind$?getActiveDescendent@AccessBridgeJavaEntryPoints@@QEAAPEAV_jobject@@QEAV2@@Z 0000000180043918     AccessBridgeJavaEntryPoints.obj
 0002:00018918       $unwind$?getTopLevelObject@AccessBridgeJavaEntryPoints@@QEAAPEAV_jobject@@QEAV2@@Z 0000000180043918     AccessBridgeJavaEntryPoints.obj
 0002:00018918       $unwind$?isSameObject@AccessBridgeJavaEntryPoints@@QEAAHPEAV_jobject@@0@Z 0000000180043918     AccessBridgeJavaEntryPoints.obj
 0002:00018918       $unwind$?WindowsATDestroyed@JavaAccessBridge@@QEAAXPEAUHWND__@@@Z 0000000180043918     JavaAccessBridge.obj
 0002:00018918       $unwind$?receiveMemoryPackage@JavaAccessBridge@@QEAAHPEAUHWND__@@J@Z 0000000180043918     JavaAccessBridge.obj
 0002:00018918       $unwind$Java_com_sun_java_accessibility_internal_AccessBridge_sendDebugString 0000000180043918     JavaAccessBridge.obj
 0002:00018918       $unwind$_DllMainCRTStartup 0000000180043918     LIBCMT:dll_dllmain.obj
 0002:00018918       $unwind$__vcrt_getptd_noexit 0000000180043918     libvcruntime:per_thread_data.obj
 0002:00018918       $unwind$?FrameUnwindToEmptyState@__FrameHandler3@@SAXPEA_KPEAU_xDISPATCHER_CONTEXT@@PEBU_s_FuncInfo@@@Z 0000000180043918     libvcruntime:risctrnsctrl.obj
 0002:00018918       $unwind$__vcrt_InitializeCriticalSectionEx 0000000180043918     libvcruntime:winapi_downlevel.obj
 0002:00018918       $unwind$??$common_getenv_nolock@D@@YAPEADQEBD@Z 0000000180043918     libucrt:getenv.obj
 0002:00018918       $unwind$memcpy_s           0000000180043918     libucrt:cfout.obj
 0002:00018918       $unwind$?internal_get_ptd_head_slow@@YAPEAU__acrt_ptd@@XZ 0000000180043918     libucrt:per_thread_data.obj
 0002:00018918       $unwind$__acrt_execute_initializers 0000000180043918     libucrt:shared_initialization.obj
 0002:00018918       $unwind$_close_nolock_internal 0000000180043918     libucrt:close.obj
 0002:00018918       $unwind$?value@?$dual_state_global@P6AXPEB_W00I_K@Z@__crt_state_management@@QEAAAEAP6AXPEB_W00I_K@ZAEAV__crt_cached_ptd_host@@@Z 0000000180043918     libucrt:invalid_parameter.obj
 0002:00018918       $unwind$?create_thread_parameter@@YAPEAU__acrt_thread_parameter@@QEAX0@Z 0000000180043918     libucrt:thread.obj
 0002:00018918       $unwind$__acrt_stdio_flush_and_write_narrow_nolock 0000000180043918     libucrt:_flsbuf.obj
 0002:00018918       $unwind$__acrt_stdio_flush_and_write_wide_nolock 0000000180043918     libucrt:_flsbuf.obj
 0002:00018918       $unwind$??$__acrt_stdio_parse_mode@D@@YA?AU__acrt_stdio_stream_mode@@QEBD@Z 0000000180043918     libucrt:openfile.obj
 0002:00018918       $unwind$?type_case_s@?$output_processor@_WV?$stream_output_adapter@_W@__crt_stdio_output@@V?$standard_base@_WV?$stream_output_adapter@_W@__crt_stdio_output@@@2@@__crt_stdio_output@@AEAA_NXZ 0000000180043918     libucrt:output.obj
 0002:00018918       $unwind$?update_locale_slow@__crt_cached_ptd_host@@AEAAXXZ 0000000180043918     libucrt:output.obj
 0002:00018918       $unwind$strncpy_s          0000000180043918     libucrt:strncpy_s.obj
 0002:00018918       $unwind$??0_LocaleUpdate@@QEAA@QEAU__crt_locale_pointers@@@Z 0000000180043918     libucrt:wcsnicol.obj
 0002:00018928       $unwind$?activateAccessibleHyperlink@AccessBridgeJavaEntryPoints@@QEAAHPEAV_jobject@@0@Z 0000000180043928     AccessBridgeJavaEntryPoints.obj
 0002:00018928       $unwind$?addAccessibleSelectionFromContext@AccessBridgeJavaEntryPoints@@QEAAXPEAV_jobject@@H@Z 0000000180043928     AccessBridgeJavaEntryPoints.obj
 0002:00018928       $unwind$?getAccessibleChildFromContext@AccessBridgeJavaEntryPoints@@QEAAPEAV_jobject@@PEAV2@H@Z 0000000180043928     AccessBridgeJavaEntryPoints.obj
 0002:00018928       $unwind$?getAccessibleHypertextLinkIndex@AccessBridgeJavaEntryPoints@@QEAAHQEAV_jobject@@H@Z 0000000180043928     AccessBridgeJavaEntryPoints.obj
 0002:00018928       $unwind$?getAccessibleSelectionFromContext@AccessBridgeJavaEntryPoints@@QEAAPEAV_jobject@@PEAV2@H@Z 0000000180043928     AccessBridgeJavaEntryPoints.obj
 0002:00018928       $unwind$?getAccessibleTableColumn@AccessBridgeJavaEntryPoints@@QEAAHPEAV_jobject@@H@Z 0000000180043928     AccessBridgeJavaEntryPoints.obj
 0002:00018928       $unwind$?getAccessibleTableColumnDescription@AccessBridgeJavaEntryPoints@@QEAAPEAV_jobject@@PEAV2@H@Z 0000000180043928     AccessBridgeJavaEntryPoints.obj
 0002:00018928       $unwind$?getAccessibleTableRow@AccessBridgeJavaEntryPoints@@QEAAHPEAV_jobject@@H@Z 0000000180043928     AccessBridgeJavaEntryPoints.obj
 0002:00018928       $unwind$?getAccessibleTableRowDescription@AccessBridgeJavaEntryPoints@@QEAAPEAV_jobject@@PEAV2@H@Z 0000000180043928     AccessBridgeJavaEntryPoints.obj
 0002:00018928       $unwind$?getParentWithRole@AccessBridgeJavaEntryPoints@@QEAAPEAV_jobject@@QEAV2@PEBG@Z 0000000180043928     AccessBridgeJavaEntryPoints.obj
 0002:00018928       $unwind$?getParentWithRoleElseRoot@AccessBridgeJavaEntryPoints@@QEAAPEAV_jobject@@QEAV2@PEBG@Z 0000000180043928     AccessBridgeJavaEntryPoints.obj
 0002:00018928       $unwind$?isAccessibleChildSelectedFromContext@AccessBridgeJavaEntryPoints@@QEAAHPEAV_jobject@@H@Z 0000000180043928     AccessBridgeJavaEntryPoints.obj
 0002:00018928       $unwind$?isAccessibleTableColumnSelected@AccessBridgeJavaEntryPoints@@QEAAHPEAV_jobject@@H@Z 0000000180043928     AccessBridgeJavaEntryPoints.obj
 0002:00018928       $unwind$?isAccessibleTableRowSelected@AccessBridgeJavaEntryPoints@@QEAAHPEAV_jobject@@H@Z 0000000180043928     AccessBridgeJavaEntryPoints.obj
 0002:00018928       $unwind$?removeAccessibleSelectionFromContext@AccessBridgeJavaEntryPoints@@QEAAXPEAV_jobject@@H@Z 0000000180043928     AccessBridgeJavaEntryPoints.obj
 0002:00018928       $unwind$?setCaretPosition@AccessBridgeJavaEntryPoints@@QEAAHQEAV_jobject@@H@Z 0000000180043928     AccessBridgeJavaEntryPoints.obj
 0002:00018928       $unwind$?setTextContents@AccessBridgeJavaEntryPoints@@QEAAHQEAV_jobject@@PEBG@Z 0000000180043928     AccessBridgeJavaEntryPoints.obj
 0002:00018928       $unwind$?MemoryMappedFileCreated@JavaAccessBridge@@QEAA_JPEAUHWND__@@PEAD@Z 0000000180043928     JavaAccessBridge.obj
 0002:00018938       $unwind$?getAccessibleContextAt@AccessBridgeJavaEntryPoints@@QEAAPEAV_jobject@@HHPEAV2@@Z 0000000180043938     AccessBridgeJavaEntryPoints.obj
 0002:00018938       $unwind$?getAccessibleTableIndex@AccessBridgeJavaEntryPoints@@QEAAHPEAV_jobject@@HH@Z 0000000180043938     AccessBridgeJavaEntryPoints.obj
 0002:00018938       $unwind$?getAccessibleTextLineBounds@AccessBridgeJavaEntryPoints@@QEAAHPEAV_jobject@@HPEAH1@Z 0000000180043938     AccessBridgeJavaEntryPoints.obj
 0002:00018938       $unwind$?getAccessibleTextRect@AccessBridgeJavaEntryPoints@@QEAAHPEAV_jobject@@PEAUAccessibleTextRectInfoTag@@H@Z 0000000180043938     AccessBridgeJavaEntryPoints.obj
 0002:00018938       $unwind$?getCaretLocation@AccessBridgeJavaEntryPoints@@QEAAHPEAV_jobject@@PEAUAccessibleTextRectInfoTag@@H@Z 0000000180043938     AccessBridgeJavaEntryPoints.obj
 0002:00018938       $unwind$?selectTextRange@AccessBridgeJavaEntryPoints@@QEAAHQEAV_jobject@@HH@Z 0000000180043938     AccessBridgeJavaEntryPoints.obj
 0002:00018938       $unwind$__acrt_fp_strflt_to_string 0000000180043938     libucrt:_fptostr.obj
 0002:00018938       $unwind$??$common_lseek_nolock@_J@@YA_JH_JHAEAV__crt_cached_ptd_host@@@Z 0000000180043938     libucrt:lseek.obj
 0002:00018938       $unwind$_invalid_parameter_internal 0000000180043938     libucrt:invalid_parameter.obj
 0002:0001894c       $unwind$?getAccessibleContextInfo@AccessBridgeJavaEntryPoints@@QEAAHPEAV_jobject@@PEAUAccessibleContextInfoTag@@@Z 000000018004394c     AccessBridgeJavaEntryPoints.obj
 0002:0001894c       $unwind$?try_get_function@@YAPEAXW4function_id@?A0x14174aea@@QEBDQEBW4module_id@2@2@Z 000000018004394c     libvcruntime:winapi_downlevel.obj
 0002:00018968       $unwind$?getAccessibleRelationSet@AccessBridgeJavaEntryPoints@@QEAAHPEAV_jobject@@PEAUAccessibleRelationSetInfoTag@@@Z 0000000180043968     AccessBridgeJavaEntryPoints.obj
 0002:00018980       $unwind$?getAccessibleActions@AccessBridgeJavaEntryPoints@@QEAAHPEAV_jobject@@PEAUAccessibleActionsTag@@@Z 0000000180043980     AccessBridgeJavaEntryPoints.obj
 0002:00018980       $unwind$?getAccessibleHypertext@AccessBridgeJavaEntryPoints@@QEAAHPEAV_jobject@@PEAUAccessibleHypertextInfoTag@@@Z 0000000180043980     AccessBridgeJavaEntryPoints.obj
 0002:00018980       $unwind$?getAccessibleHypertextExt@AccessBridgeJavaEntryPoints@@QEAAHQEAV_jobject@@HPEAUAccessibleHypertextInfoTag@@@Z 0000000180043980     AccessBridgeJavaEntryPoints.obj
 0002:00018980       $unwind$?getAccessibleIcons@AccessBridgeJavaEntryPoints@@QEAAHPEAV_jobject@@PEAUAccessibleIconsTag@@@Z 0000000180043980     AccessBridgeJavaEntryPoints.obj
 0002:00018980       $unwind$?__mbsrtowcs_utf8@__crt_mbstring@@YA_KPEA_WPEAPEBD_KPEAU_Mbstatet@@AEAV__crt_cached_ptd_host@@@Z 0000000180043980     libucrt:mbrtowc.obj
 0002:0001899c       $unwind$?getAccessibleHyperlink@AccessBridgeJavaEntryPoints@@QEAAHQEAV_jobject@@HPEAUAccessibleHyperlinkInfoTag@@@Z 000000018004399c     AccessBridgeJavaEntryPoints.obj
 0002:000189b4       $unwind$?doAccessibleActions@AccessBridgeJavaEntryPoints@@QEAAHPEAV_jobject@@PEAUAccessibleActionsToDoTag@@PEAH@Z 00000001800439b4     AccessBridgeJavaEntryPoints.obj
 0002:000189b4       $unwind$?getAccessibleTextRange@AccessBridgeJavaEntryPoints@@QEAAHPEAV_jobject@@HHPEAGF@Z 00000001800439b4     AccessBridgeJavaEntryPoints.obj
 0002:000189d0       $unwind$?getAccessibleTextItems@AccessBridgeJavaEntryPoints@@QEAAHPEAV_jobject@@PEAUAccessibleTextItemsInfoTag@@H@Z 00000001800439d0     AccessBridgeJavaEntryPoints.obj
 0002:000189d0       $unwind$??$copy_and_add_argument_to_buffer@D@@YAHQEBD0_KAEAV?$argument_list@D@?A0x5f5c8891@@@Z 00000001800439d0     libucrt:argv_wildcards.obj
 0002:000189d0       $unwind$??$parse_integer@KV?$c_string_character_source@D@__crt_strtox@@$0A@@__crt_strtox@@YAKAEAV__crt_cached_ptd_host@@V?$c_string_character_source@D@0@H_N@Z 00000001800439d0     libucrt:output.obj
 0002:000189ec       $unwind$?getAccessibleTextSelectionInfo@AccessBridgeJavaEntryPoints@@QEAAHPEAV_jobject@@PEAUAccessibleTextSelectionInfoTag@@@Z 00000001800439ec     AccessBridgeJavaEntryPoints.obj
 0002:00018a04       $unwind$?getAccessibleTextAttributes@AccessBridgeJavaEntryPoints@@QEAAHPEAV_jobject@@HPEAUAccessibleTextAttributesInfoTag@@@Z 0000000180043a04     AccessBridgeJavaEntryPoints.obj
 0002:00018a20       $unwind$?getTextAttributesInRange@AccessBridgeJavaEntryPoints@@QEAAHQEAV_jobject@@HHPEAUAccessibleTextAttributesInfoTag@@PEAF@Z 0000000180043a20     AccessBridgeJavaEntryPoints.obj
 0002:00018a40       $unwind$?getVisibleChildren@AccessBridgeJavaEntryPoints@@QEAAHQEAV_jobject@@HPEAUVisibleChildenInfoTag@@@Z 0000000180043a40     AccessBridgeJavaEntryPoints.obj
 0002:00018a5c       $unwind$?javaRun@JavaAccessBridge@@QEAAXPEAUJNIEnv_@@PEAV_jobject@@@Z 0000000180043a5c     JavaAccessBridge.obj
 0002:00018a5c       $unwind$?fp_format_e@@YAHQEBNQEAD_K12H_NIW4__acrt_rounding_mode@@AEAV__crt_cached_ptd_host@@@Z 0000000180043a5c     libucrt:cvt.obj
 0002:00018a74       $unwind$?initWindow@JavaAccessBridge@@QEAAHXZ 0000000180043a74     JavaAccessBridge.obj
 0002:00018a7c       $unwind$?addAccessibilityEventNotification@JavaAccessBridge@@QEAAX_JPEAUHWND__@@@Z 0000000180043a7c     JavaAccessBridge.obj
 0002:00018a7c       $unwind$?addJavaEventNotification@JavaAccessBridge@@QEAAX_JPEAUHWND__@@@Z 0000000180043a7c     JavaAccessBridge.obj
 0002:00018a7c       $unwind$?removeAccessibilityEventNotification@JavaAccessBridge@@QEAAX_JPEAUHWND__@@@Z 0000000180043a7c     JavaAccessBridge.obj
 0002:00018a7c       $unwind$?removeJavaEventNotification@JavaAccessBridge@@QEAAX_JPEAUHWND__@@@Z 0000000180043a7c     JavaAccessBridge.obj
 0002:00018a7c       $unwind$__GSHandlerCheck_EH 0000000180043a7c     LIBCMT:gshandlereh.obj
 0002:00018a7c       $unwind$??$TypeMatchHelper@V__FrameHandler3@@@@YAHPEBU_s_HandlerType@@PEBU_s_CatchableType@@PEBU_s_ThrowInfo@@@Z 0000000180043a7c     libvcruntime:frame.obj
 0002:00018a7c       $unwind$?initialize_stdio_handles_nolock@@YAXXZ 0000000180043a7c     libucrt:ioinit.obj
 0002:00018a7c       $unwind$__acrt_lowio_set_os_handle 0000000180043a7c     libucrt:osfinfo.obj
 0002:00018a7c       $unwind$__acrt_initialize_stdio 0000000180043a7c     libucrt:_file.obj
 0002:00018a94       $unwind$?javaShutdown@JavaAccessBridge@@QEAAXPEAUJNIEnv_@@PEAV_jobject@@@Z 0000000180043a94     JavaAccessBridge.obj
 0002:00018aa8       $unwind$?fireCaretUpdate@JavaAccessBridge@@QEAAXPEAUJNIEnv_@@PEAV_jobject@@11@Z 0000000180043aa8     JavaAccessBridge.obj
 0002:00018aa8       $unwind$?fireFocusGained@JavaAccessBridge@@QEAAXPEAUJNIEnv_@@PEAV_jobject@@11@Z 0000000180043aa8     JavaAccessBridge.obj
 0002:00018aa8       $unwind$?fireFocusLost@JavaAccessBridge@@QEAAXPEAUJNIEnv_@@PEAV_jobject@@11@Z 0000000180043aa8     JavaAccessBridge.obj
 0002:00018aa8       $unwind$?fireMouseClicked@JavaAccessBridge@@QEAAXPEAUJNIEnv_@@PEAV_jobject@@11@Z 0000000180043aa8     JavaAccessBridge.obj
 0002:00018aa8       $unwind$?fireMouseEntered@JavaAccessBridge@@QEAAXPEAUJNIEnv_@@PEAV_jobject@@11@Z 0000000180043aa8     JavaAccessBridge.obj
 0002:00018aa8       $unwind$?fireMouseExited@JavaAccessBridge@@QEAAXPEAUJNIEnv_@@PEAV_jobject@@11@Z 0000000180043aa8     JavaAccessBridge.obj
 0002:00018aa8       $unwind$?fireMousePressed@JavaAccessBridge@@QEAAXPEAUJNIEnv_@@PEAV_jobject@@11@Z 0000000180043aa8     JavaAccessBridge.obj
 0002:00018ac0       $unwind$?fireMenuCanceled@JavaAccessBridge@@QEAAXPEAUJNIEnv_@@PEAV_jobject@@11@Z 0000000180043ac0     JavaAccessBridge.obj
 0002:00018ac0       $unwind$?fireMenuDeselected@JavaAccessBridge@@QEAAXPEAUJNIEnv_@@PEAV_jobject@@11@Z 0000000180043ac0     JavaAccessBridge.obj
 0002:00018ac0       $unwind$?fireMenuSelected@JavaAccessBridge@@QEAAXPEAUJNIEnv_@@PEAV_jobject@@11@Z 0000000180043ac0     JavaAccessBridge.obj
 0002:00018ac0       $unwind$?fireMouseReleased@JavaAccessBridge@@QEAAXPEAUJNIEnv_@@PEAV_jobject@@11@Z 0000000180043ac0     JavaAccessBridge.obj
 0002:00018ac0       $unwind$?firePopupMenuCanceled@JavaAccessBridge@@QEAAXPEAUJNIEnv_@@PEAV_jobject@@11@Z 0000000180043ac0     JavaAccessBridge.obj
 0002:00018ac0       $unwind$?firePopupMenuWillBecomeInvisible@JavaAccessBridge@@QEAAXPEAUJNIEnv_@@PEAV_jobject@@11@Z 0000000180043ac0     JavaAccessBridge.obj
 0002:00018ac0       $unwind$?firePopupMenuWillBecomeVisible@JavaAccessBridge@@QEAAXPEAUJNIEnv_@@PEAV_jobject@@11@Z 0000000180043ac0     JavaAccessBridge.obj
 0002:00018adc       $unwind$?firePropertyCaretChange@JavaAccessBridge@@QEAAXPEAUJNIEnv_@@PEAV_jobject@@11HH@Z 0000000180043adc     JavaAccessBridge.obj
 0002:00018af8       $unwind$?firePropertyDescriptionChange@JavaAccessBridge@@QEAAXPEAUJNIEnv_@@PEAV_jobject@@11PEAV_jstring@@2@Z 0000000180043af8     JavaAccessBridge.obj
 0002:00018af8       $unwind$?firePropertyNameChange@JavaAccessBridge@@QEAAXPEAUJNIEnv_@@PEAV_jobject@@11PEAV_jstring@@2@Z 0000000180043af8     JavaAccessBridge.obj
 0002:00018af8       $unwind$?firePropertyStateChange@JavaAccessBridge@@QEAAXPEAUJNIEnv_@@PEAV_jobject@@11PEAV_jstring@@2@Z 0000000180043af8     JavaAccessBridge.obj
 0002:00018af8       $unwind$?firePropertyTableModelChange@JavaAccessBridge@@QEAAXPEAUJNIEnv_@@PEAV_jobject@@11PEAV_jstring@@2@Z 0000000180043af8     JavaAccessBridge.obj
 0002:00018af8       $unwind$?firePropertyValueChange@JavaAccessBridge@@QEAAXPEAUJNIEnv_@@PEAV_jobject@@11PEAV_jstring@@2@Z 0000000180043af8     JavaAccessBridge.obj
 0002:00018b18       $unwind$?firePropertySelectionChange@JavaAccessBridge@@QEAAXPEAUJNIEnv_@@PEAV_jobject@@11@Z 0000000180043b18     JavaAccessBridge.obj
 0002:00018b18       $unwind$?firePropertyTextChange@JavaAccessBridge@@QEAAXPEAUJNIEnv_@@PEAV_jobject@@11@Z 0000000180043b18     JavaAccessBridge.obj
 0002:00018b18       $unwind$?firePropertyVisibleDataChange@JavaAccessBridge@@QEAAXPEAUJNIEnv_@@PEAV_jobject@@11@Z 0000000180043b18     JavaAccessBridge.obj
 0002:00018b30       $unwind$?firePropertyActiveDescendentChange@JavaAccessBridge@@QEAAXPEAUJNIEnv_@@PEAV_jobject@@1111@Z 0000000180043b30     JavaAccessBridge.obj
 0002:00018b30       $unwind$?firePropertyChildChange@JavaAccessBridge@@QEAAXPEAUJNIEnv_@@PEAV_jobject@@1111@Z 0000000180043b30     JavaAccessBridge.obj
 0002:00018b4c       $unwind$Java_com_sun_java_accessibility_internal_AccessBridge_jawtGetComponentFromNativeWindowHandle 0000000180043b4c     JavaAccessBridge.obj
 0002:00018b4c       $unwind$Java_com_sun_java_accessibility_internal_AccessBridge_jawtGetNativeWindowHandleFromComponent 0000000180043b4c     JavaAccessBridge.obj
 0002:00018b58       $unwind$Java_com_sun_java_accessibility_internal_AccessBridge_propertyActiveDescendentChange 0000000180043b58     JavaAccessBridge.obj
 0002:00018b58       $unwind$Java_com_sun_java_accessibility_internal_AccessBridge_propertyCaretChange 0000000180043b58     JavaAccessBridge.obj
 0002:00018b58       $unwind$Java_com_sun_java_accessibility_internal_AccessBridge_propertyChildChange 0000000180043b58     JavaAccessBridge.obj
 0002:00018b58       $unwind$Java_com_sun_java_accessibility_internal_AccessBridge_propertyDescriptionChange 0000000180043b58     JavaAccessBridge.obj
 0002:00018b58       $unwind$Java_com_sun_java_accessibility_internal_AccessBridge_propertyNameChange 0000000180043b58     JavaAccessBridge.obj
 0002:00018b58       $unwind$Java_com_sun_java_accessibility_internal_AccessBridge_propertyStateChange 0000000180043b58     JavaAccessBridge.obj
 0002:00018b58       $unwind$Java_com_sun_java_accessibility_internal_AccessBridge_propertyTableModelChange 0000000180043b58     JavaAccessBridge.obj
 0002:00018b58       $unwind$Java_com_sun_java_accessibility_internal_AccessBridge_propertyValueChange 0000000180043b58     JavaAccessBridge.obj
 0002:00018b58       $unwind$?__scrt_throw_std_bad_alloc@@YAXXZ 0000000180043b58     LIBCMT:throw_bad_alloc.obj
 0002:00018b58       $unwind$?__scrt_throw_std_bad_array_new_length@@YAXXZ 0000000180043b58     LIBCMT:throw_bad_alloc.obj
 0002:00018b58       $unwind$_raise_exc         0000000180043b58     libucrt:fpexcept.obj
 0002:00018b60       $unwind$Java_com_sun_java_accessibility_internal_AccessBridge_caretUpdate 0000000180043b60     JavaAccessBridge.obj
 0002:00018b60       $unwind$Java_com_sun_java_accessibility_internal_AccessBridge_focusGained 0000000180043b60     JavaAccessBridge.obj
 0002:00018b60       $unwind$Java_com_sun_java_accessibility_internal_AccessBridge_focusLost 0000000180043b60     JavaAccessBridge.obj
 0002:00018b60       $unwind$Java_com_sun_java_accessibility_internal_AccessBridge_menuCanceled 0000000180043b60     JavaAccessBridge.obj
 0002:00018b60       $unwind$Java_com_sun_java_accessibility_internal_AccessBridge_menuDeselected 0000000180043b60     JavaAccessBridge.obj
 0002:00018b60       $unwind$Java_com_sun_java_accessibility_internal_AccessBridge_menuSelected 0000000180043b60     JavaAccessBridge.obj
 0002:00018b60       $unwind$Java_com_sun_java_accessibility_internal_AccessBridge_mouseClicked 0000000180043b60     JavaAccessBridge.obj
 0002:00018b60       $unwind$Java_com_sun_java_accessibility_internal_AccessBridge_mouseEntered 0000000180043b60     JavaAccessBridge.obj
 0002:00018b60       $unwind$Java_com_sun_java_accessibility_internal_AccessBridge_mouseExited 0000000180043b60     JavaAccessBridge.obj
 0002:00018b60       $unwind$Java_com_sun_java_accessibility_internal_AccessBridge_mousePressed 0000000180043b60     JavaAccessBridge.obj
 0002:00018b60       $unwind$Java_com_sun_java_accessibility_internal_AccessBridge_mouseReleased 0000000180043b60     JavaAccessBridge.obj
 0002:00018b60       $unwind$Java_com_sun_java_accessibility_internal_AccessBridge_popupMenuCanceled 0000000180043b60     JavaAccessBridge.obj
 0002:00018b60       $unwind$Java_com_sun_java_accessibility_internal_AccessBridge_popupMenuWillBecomeInvisible 0000000180043b60     JavaAccessBridge.obj
 0002:00018b60       $unwind$Java_com_sun_java_accessibility_internal_AccessBridge_popupMenuWillBecomeVisible 0000000180043b60     JavaAccessBridge.obj
 0002:00018b60       $unwind$Java_com_sun_java_accessibility_internal_AccessBridge_propertySelectionChange 0000000180043b60     JavaAccessBridge.obj
 0002:00018b60       $unwind$Java_com_sun_java_accessibility_internal_AccessBridge_propertyTextChange 0000000180043b60     JavaAccessBridge.obj
 0002:00018b60       $unwind$Java_com_sun_java_accessibility_internal_AccessBridge_propertyVisibleDataChange 0000000180043b60     JavaAccessBridge.obj
 0002:00018b60       $unwind$_sopen_s           0000000180043b60     libucrt:open.obj
 0002:00018b60       $unwind$_invalid_parameter_noinfo 0000000180043b60     libucrt:invalid_parameter.obj
 0002:00018b60       $unwind$?state_case_size@?$output_processor@DV?$stream_output_adapter@D@__crt_stdio_output@@V?$standard_base@DV?$stream_output_adapter@D@__crt_stdio_output@@@2@@__crt_stdio_output@@AEAA_NXZ 0000000180043b60     libucrt:output.obj
 0002:00018b60       $unwind$?state_case_size@?$output_processor@_WV?$stream_output_adapter@_W@__crt_stdio_output@@V?$standard_base@_WV?$stream_output_adapter@_W@__crt_stdio_output@@@2@@__crt_stdio_output@@AEAA_NXZ 0000000180043b60     libucrt:output.obj
 0002:00018b60       $unwind$_log10_special     0000000180043b60     libucrt:log_special.obj
 0002:00018b68       $unwind$__GSHandlerCheckCommon 0000000180043b68     LIBCMT:gshandler.obj
 0002:00018b70       $xdatasym                  0000000180043b70     LIBCMT:amdsecgs.obj
 0002:00018b74       $unwind$?dllmain_crt_process_attach@@YAHQEAUHINSTANCE__@@QEAX@Z 0000000180043b74     LIBCMT:dll_dllmain.obj
 0002:00018bb0       $unwind$?fin$0@?0??dllmain_crt_process_attach@@YAHQEAUHINSTANCE__@@QEAX@Z@4HA 0000000180043bb0     LIBCMT:dll_dllmain.obj
 0002:00018bb0       $unwind$?fin$0@?0??dllmain_crt_process_detach@@YAH_N@Z@4HA 0000000180043bb0     LIBCMT:dll_dllmain.obj
 0002:00018bb0       $unwind$?fin$1@?0??dllmain_crt_process_detach@@YAH_N@Z@4HA 0000000180043bb0     LIBCMT:dll_dllmain.obj
 0002:00018bb0       $unwind$_IsNonwritableInCurrentImage$filt$0 0000000180043bb0     LIBCMT:pesect.obj
 0002:00018bb0       $unwind$?filt$0@?0??CxxCallCatchBlock@__FrameHandler3@@SAPEAXPEAU_EXCEPTION_RECORD@@@Z@4HA 0000000180043bb0     libvcruntime:frame.obj
 0002:00018bb0       $unwind$?filt$0@?0??FrameUnwindToState@__FrameHandler3@@SAXPEA_KPEAU_xDISPATCHER_CONTEXT@@PEBU_s_FuncInfo@@H@Z@4HA 0000000180043bb0     libvcruntime:frame.obj
 0002:00018bb0       $unwind$?fin$1@?0??FrameUnwindToState@__FrameHandler3@@SAXPEA_KPEAU_xDISPATCHER_CONTEXT@@PEBU_s_FuncInfo@@H@Z@4HA 0000000180043bb0     libvcruntime:frame.obj
 0002:00018bb0       $unwind$?fin$0@?0???$common_getenv@D@@YAPEADQEBD@Z@4HA 0000000180043bb0     libucrt:getenv.obj
 0002:00018bb0       $unwind$?fin$0@?0???$?RV<lambda_0ae27a3a962d80f24befdcbee591983d>@@AEAV<lambda_8d0ee55de4b1038c4002e0adecdf1839>@@V<lambda_dc504788e8f1664fe9b84e20bfb512f2>@@@?$__crt_seh_guarded_call@X@@QEAAX$$QEAV<lambda_0ae27a3a962d80f24befdcbee591983d>@@AEAV<lambda_8d0ee55de4b1038c4002e0adecdf1839>@@$$QEAV<lambda_dc504788e8f1664fe9b84e20bfb512f2>@@@Z@4HA 0000000180043bb0     libucrt:per_thread_data.obj
 0002:00018bb0       $unwind$?fin$0@?0???$?RV<lambda_2d41944a1d46af3157314b8a01080d33>@@AEAV<lambda_8f455de75cd7d7f24b4096f044d8b9e6>@@V<lambda_aa500f224e6afead328df44964fe2772>@@@?$__crt_seh_guarded_call@X@@QEAAX$$QEAV<lambda_2d41944a1d46af3157314b8a01080d33>@@AEAV<lambda_8f455de75cd7d7f24b4096f044d8b9e6>@@$$QEAV<lambda_aa500f224e6afead328df44964fe2772>@@@Z@4HA 0000000180043bb0     libucrt:per_thread_data.obj
 0002:00018bb0       $unwind$?fin$0@?0???$?RV<lambda_aa87e3671a710a21b5dc78c0bdf72e11>@@AEAV<lambda_92619d2358a28f41a33ba319515a20b9>@@V<lambda_6992ecaafeb10aed2b74cb1fae11a551>@@@?$__crt_seh_guarded_call@X@@QEAAX$$QEAV<lambda_aa87e3671a710a21b5dc78c0bdf72e11>@@AEAV<lambda_92619d2358a28f41a33ba319515a20b9>@@$$QEAV<lambda_6992ecaafeb10aed2b74cb1fae11a551>@@@Z@4HA 0000000180043bb0     libucrt:per_thread_data.obj
 0002:00018bb0       $unwind$?fin$0@?0???$?RV<lambda_f2e299630e499de9f9a165e60fcd3db5>@@AEAV<lambda_2ae9d31cdba2644fcbeaf08da7c24588>@@V<lambda_40d01ff24d0e7b3814fdbdcee8eab3c7>@@@?$__crt_seh_guarded_call@X@@QEAAX$$QEAV<lambda_f2e299630e499de9f9a165e60fcd3db5>@@AEAV<lambda_2ae9d31cdba2644fcbeaf08da7c24588>@@$$QEAV<lambda_40d01ff24d0e7b3814fdbdcee8eab3c7>@@@Z@4HA 0000000180043bb0     libucrt:per_thread_data.obj
 0002:00018bb0       $unwind$__acrt_update_thread_locale_data$fin$0 0000000180043bb0     libucrt:locale_refcounting.obj
 0002:00018bb0       $unwind$?fin$0@?0???$?RV<lambda_410d79af7f07d98d83a3f525b3859a53>@@AEAV<lambda_3e16ef9562a7dcce91392c22ab16ea36>@@V<lambda_38119f0e861e05405d8a144b9b982f0a>@@@?$__crt_seh_guarded_call@X@@QEAAX$$QEAV<lambda_410d79af7f07d98d83a3f525b3859a53>@@AEAV<lambda_3e16ef9562a7dcce91392c22ab16ea36>@@$$QEAV<lambda_38119f0e861e05405d8a144b9b982f0a>@@@Z@4HA 0000000180043bb0     libucrt:wsetlocale.obj
 0002:00018bb0       $unwind$?fin$0@?0???$?RV<lambda_ad8af0d99a0adf03d037d7dffe354bb5>@@AEAV<lambda_c9ba49e555ba839a7b07aa3fbecb7617>@@V<lambda_2f1ebd5d68526518146ae959c9e734c8>@@@?$__crt_seh_guarded_call@H@@QEAAH$$QEAV<lambda_ad8af0d99a0adf03d037d7dffe354bb5>@@AEAV<lambda_c9ba49e555ba839a7b07aa3fbecb7617>@@$$QEAV<lambda_2f1ebd5d68526518146ae959c9e734c8>@@@Z@4HA 0000000180043bb0     libucrt:close.obj
 0002:00018bb0       $unwind$?fin$0@?0???$?RV<lambda_a37b2b86f63e897a80ea819b0eb08c01>@@AEAV<lambda_38ce7e780aa69e748d6df282ebc68efe>@@V<lambda_99fb1378e971ab6e7edea83e3a7a83a2>@@@?$__crt_seh_guarded_call@H@@QEAAH$$QEAV<lambda_a37b2b86f63e897a80ea819b0eb08c01>@@AEAV<lambda_38ce7e780aa69e748d6df282ebc68efe>@@$$QEAV<lambda_99fb1378e971ab6e7edea83e3a7a83a2>@@@Z@4HA 0000000180043bb0     libucrt:commit.obj
 0002:00018bb0       $unwind$__acrt_initialize_lowio$fin$0 0000000180043bb0     libucrt:ioinit.obj
 0002:00018bb0       $unwind$__acrt_lowio_ensure_fh_exists$fin$0 0000000180043bb0     libucrt:osfinfo.obj
 0002:00018bb0       $unwind$_alloc_osfhnd$fin$0 0000000180043bb0     libucrt:osfinfo.obj
 0002:00018bb0       $unwind$?fin$0@?0???$?RV<lambda_efdfa57d1f175319df784efa44bb7b81>@@AEAV<lambda_5f0a4c1567f8adc6734073e5d1e1b35c>@@V<lambda_2e8a7d3640ea6ccb4c2413664c2db6fd>@@@?$__crt_seh_guarded_call@X@@QEAAX$$QEAV<lambda_efdfa57d1f175319df784efa44bb7b81>@@AEAV<lambda_5f0a4c1567f8adc6734073e5d1e1b35c>@@$$QEAV<lambda_2e8a7d3640ea6ccb4c2413664c2db6fd>@@@Z@4HA 0000000180043bb0     libucrt:mbctype.obj
 0002:00018bb0       $unwind$?fin$0@?0??update_thread_multibyte_data_internal@@YAPEAU__crt_multibyte_data@@QEAU__acrt_ptd@@QEAPEAU1@@Z@4HA 0000000180043bb0     libucrt:mbctype.obj
 0002:00018bb0       $unwind$?fin$0@?0???$?RV<lambda_450d765d439847d4c735a33c368b5fc0>@@AEAV<lambda_44731a7d0e6d81c3e6aa82d741081786>@@V<lambda_601a2a7da3b7a96e9554ac7215c4b07c>@@@?$__crt_seh_guarded_call@P6AXH@Z@@QEAAP6AXH@Z$$QEAV<lambda_450d765d439847d4c735a33c368b5fc0>@@AEAV<lambda_44731a7d0e6d81c3e6aa82d741081786>@@$$QEAV<lambda_601a2a7da3b7a96e9554ac7215c4b07c>@@@Z@4HA 0000000180043bb0     libucrt:signal.obj
 0002:00018bb0       $unwind$raise$fin$0        0000000180043bb0     libucrt:signal.obj
 0002:00018bb0       $unwind$?filt$0@?0???R<lambda_6e4b09c48022b2350581041d5f6b0c4c>@@QEBA@XZ@4HA 0000000180043bb0     libucrt:exit.obj
 0002:00018bb0       $unwind$?fin$0@?0???$?RV<lambda_d80eeec6fff315bfe5c115232f3240e3>@@AEAV<lambda_6e4b09c48022b2350581041d5f6b0c4c>@@V<lambda_2358e3775559c9db80273638284d5e45>@@@?$__crt_seh_guarded_call@X@@QEAAX$$QEAV<lambda_d80eeec6fff315bfe5c115232f3240e3>@@AEAV<lambda_6e4b09c48022b2350581041d5f6b0c4c>@@$$QEAV<lambda_2358e3775559c9db80273638284d5e45>@@@Z@4HA 0000000180043bb0     libucrt:exit.obj
 0002:00018bb0       $unwind$?fin$0@?0???$?RV<lambda_7777bce6b2f8c936911f934f8298dc43>@@AEAV<lambda_f03950bc5685219e0bcd2087efbe011e>@@V<lambda_3883c3dff614d5e0c5f61bb1ac94921c>@@@?$__crt_seh_guarded_call@H@@QEAAH$$QEAV<lambda_7777bce6b2f8c936911f934f8298dc43>@@AEAV<lambda_f03950bc5685219e0bcd2087efbe011e>@@$$QEAV<lambda_3883c3dff614d5e0c5f61bb1ac94921c>@@@Z@4HA 0000000180043bb0     libucrt:onexit.obj
 0002:00018bb0       $unwind$?filt$0@?0???$thread_start@P6AIPEAX@Z$00@@YAKQEAX@Z@4HA 0000000180043bb0     libucrt:thread.obj
 0002:00018bb0       $unwind$_fcloseall$fin$0   0000000180043bb0     libucrt:closeall.obj
 0002:00018bb0       $unwind$?fin$0@?0???$?RV<lambda_842d9ff0dc9ef11c61343bbaebe7f885>@@AEAV<lambda_c5860995281e5c4ce005b3de8f5874ee>@@V<lambda_d90129c13df834fdcbf8d2b88dafcf2d>@@@?$__crt_seh_guarded_call@X@@QEAAX$$QEAV<lambda_842d9ff0dc9ef11c61343bbaebe7f885>@@AEAV<lambda_c5860995281e5c4ce005b3de8f5874ee>@@$$QEAV<lambda_d90129c13df834fdcbf8d2b88dafcf2d>@@@Z@4HA 0000000180043bb0     libucrt:fflush.obj
 0002:00018bb0       $unwind$?fin$0@?0???$?RV<lambda_886d6c58226a84441f68b9f2b8217b83>@@AEAV<lambda_ab61a845afdef5b7c387490eaf3616ee>@@V<lambda_f7f22ab5edc0698d5f6905b0d3f44752>@@@?$__crt_seh_guarded_call@X@@QEAAX$$QEAV<lambda_886d6c58226a84441f68b9f2b8217b83>@@AEAV<lambda_ab61a845afdef5b7c387490eaf3616ee>@@$$QEAV<lambda_f7f22ab5edc0698d5f6905b0d3f44752>@@@Z@4HA 0000000180043bb0     libucrt:fflush.obj
 0002:00018bb0       $unwind$?fin$0@?0???$common_fsopen@D@@YAPEAU_iobuf@@QEBD0H@Z@4HA 0000000180043bb0     libucrt:fopen.obj
 0002:00018bb0       $unwind$?fin$0@?0???$?RV<lambda_613eff765f5c257adf68e381dfe80f05>@@AEAV<lambda_ebf663be9fcd9e0b17ed57bdb95b0759>@@V<lambda_872abebd861b7db59b42e49ea65623b0>@@@?$__crt_seh_guarded_call@H@@QEAAH$$QEAV<lambda_613eff765f5c257adf68e381dfe80f05>@@AEAV<lambda_ebf663be9fcd9e0b17ed57bdb95b0759>@@$$QEAV<lambda_872abebd861b7db59b42e49ea65623b0>@@@Z@4HA 0000000180043bb0     libucrt:output.obj
 0002:00018bb0       $unwind$?fin$0@?0???$?RV<lambda_d854c62834386a3b23916ad6dae2782d>@@AEAV<lambda_303760bc4008a2b3ec4768a30b06a80c>@@V<lambda_4780a7ea4f8cbd2590aec34bd14e2bbf>@@@?$__crt_seh_guarded_call@H@@QEAAH$$QEAV<lambda_d854c62834386a3b23916ad6dae2782d>@@AEAV<lambda_303760bc4008a2b3ec4768a30b06a80c>@@$$QEAV<lambda_4780a7ea4f8cbd2590aec34bd14e2bbf>@@@Z@4HA 0000000180043bb0     libucrt:output.obj
 0002:00018bb0       $unwind$?fin$0@?0??__acrt_stdio_allocate_stream@@YA?AV__crt_stdio_stream@@XZ@4HA 0000000180043bb0     libucrt:stream.obj
 0002:00018bb0       $unwind$common_control87$filt$0 0000000180043bb0     libucrt:ieee.obj
 0002:00018bb8       $unwind$?dllmain_crt_process_detach@@YAH_N@Z 0000000180043bb8     LIBCMT:dll_dllmain.obj
 0002:00018c0c       $unwind$?dllmain_dispatch@@YAHQEAUHINSTANCE__@@KQEAX@Z 0000000180043c0c     LIBCMT:dll_dllmain.obj
 0002:00018c34       $unwind$?filt$0@?0??dllmain_dispatch@@YAHQEAUHINSTANCE__@@KQEAX@Z@4HA 0000000180043c34     LIBCMT:dll_dllmain.obj
 0002:00018c34       $unwind$?fin$0@?0???$common_lseek@_J@@YA_JH_JHAEAV__crt_cached_ptd_host@@@Z@4HA 0000000180043c34     libucrt:lseek.obj
 0002:00018c34       $unwind$_write_internal$fin$0 0000000180043c34     libucrt:write.obj
 0002:00018c34       $unwind$?fin$0@?0??_fclose_internal@@YAHQEAU_iobuf@@AEAV__crt_cached_ptd_host@@@Z@4HA 0000000180043c34     libucrt:fclose.obj
 0002:00018c3c       $unwind$__report_gsfailure 0000000180043c3c     LIBCMT:gs_report.obj
 0002:00018c44       $unwind$capture_previous_context 0000000180043c44     LIBCMT:gs_report.obj
 0002:00018c50       $unwind$__security_init_cookie 0000000180043c50     LIBCMT:gs_support.obj
 0002:00018c5c       $unwind$__scrt_is_nonwritable_in_current_image 0000000180043c5c     LIBCMT:utility.obj
 0002:00018c7c       $unwind$__scrt_is_nonwritable_in_current_image$filt$0 0000000180043c7c     LIBCMT:utility.obj
 0002:00018c7c       $unwind$_ctrlfp$filt$0     0000000180043c7c     libucrt:fpctrl.obj
 0002:00018c84       $unwind$__scrt_fastfail    0000000180043c84     LIBCMT:utility_desktop.obj
 0002:00018c94       $unwind$__isa_available_init 0000000180043c94     LIBCMT:cpu_disp.obj
 0002:00018ca8       $xdatasym                  0000000180043ca8     LIBCMT:guard_dispatch.obj
 0002:00018cb0       $xdatasym                  0000000180043cb0     LIBCMT:guard_xfg_dispatch.obj
 0002:00018cb8       $xdatasym$memcpy_repmovs   0000000180043cb8     libvcruntime:memcpy.obj
 0002:00018cc8       $xdatasym$memcpy           0000000180043cc8     libvcruntime:memcpy.obj
 0002:00018cc8       $xdatasym$memset           0000000180043cc8     libvcruntime:memset.obj
 0002:00018cc8       $xdatasym$_NLG_Notify      0000000180043cc8     libvcruntime:notify.obj
 0002:00018cc8       $xdatasym$__NLG_Dispatch2  0000000180043cc8     libvcruntime:notify.obj
 0002:00018cc8       $xdatasym$__NLG_Return2    0000000180043cc8     libvcruntime:notify.obj
 0002:00018cc8       $xdatasym$_guard_dispatch_icall 0000000180043cc8     libucrt:dispatchcfg.obj
 0002:00018cd0       $xdatasym$memset_repstos   0000000180043cd0     libvcruntime:memset.obj
 0002:00018cdc       $unwind$__C_specific_handler 0000000180043cdc     libvcruntime:riscchandler.obj
 0002:00018cdc       $unwind$?GetRangeOfTrysToCheck@__FrameHandler3@@SA?AU?$pair@Viterator@TryBlockMap@__FrameHandler3@@V123@@std@@AEAVTryBlockMap@1@HPEAU_xDISPATCHER_CONTEXT@@PEBU_s_FuncInfo@@H@Z 0000000180043cdc     libvcruntime:risctrnsctrl.obj
 0002:00018cf8       $unwind$__std_exception_copy 0000000180043cf8     libvcruntime:std_exception.obj
 0002:00018cf8       $unwind$_free_osfhnd       0000000180043cf8     libucrt:osfinfo.obj
 0002:00018d0c       $unwind$_CxxThrowException 0000000180043d0c     libvcruntime:throw.obj
 0002:00018d1c       $unwind$__DestructExceptionObject 0000000180043d1c     libvcruntime:ehhelpers.obj
 0002:00018d3c       $unwind$__DestructExceptionObject$filt$0 0000000180043d3c     libvcruntime:ehhelpers.obj
 0002:00018d3c       $unwind$?fin$1@?0??CxxCallCatchBlock@__FrameHandler3@@SAPEAXPEAU_EXCEPTION_RECORD@@@Z@4HA 0000000180043d3c     libvcruntime:frame.obj
 0002:00018d48       $unwind$?GetEstablisherFrame@__FrameHandler3@@SAPEA_KPEA_KPEAU_xDISPATCHER_CONTEXT@@PEBU_s_FuncInfo@@0@Z 0000000180043d48     libvcruntime:risctrnsctrl.obj
 0002:00018d60       $unwind$?UnwindNestedFrames@__FrameHandler3@@SAXPEA_KPEAUEHExceptionRecord@@PEAU_CONTEXT@@0PEAXPEBU_s_FuncInfo@@HHPEBU_s_HandlerType@@PEAU_xDISPATCHER_CONTEXT@@E@Z 0000000180043d60     libvcruntime:risctrnsctrl.obj
 0002:00018d74       $unwind$__CxxFrameHandler3 0000000180043d74     libvcruntime:risctrnsctrl.obj
 0002:00018d88       $unwind$??$_CallSETranslator@V__FrameHandler3@@@@YAHPEAUEHExceptionRecord@@PEA_KPEAU_CONTEXT@@PEAU_xDISPATCHER_CONTEXT@@PEBU_s_FuncInfo@@K1H@Z 0000000180043d88     libvcruntime:risctrnsctrl.obj
 0002:00018da8       $unwind$?filt$0@?0???$_CallSETranslator@V__FrameHandler3@@@@YAHPEAUEHExceptionRecord@@PEA_KPEAU_CONTEXT@@PEAU_xDISPATCHER_CONTEXT@@PEBU_s_FuncInfo@@K1H@Z@4HA 0000000180043da8     libvcruntime:risctrnsctrl.obj
 0002:00018db4       $unwind$?FrameUnwindToState@__FrameHandler3@@SAXPEA_KPEAU_xDISPATCHER_CONTEXT@@PEBU_s_FuncInfo@@H@Z 0000000180043db4     libvcruntime:frame.obj
 0002:00018e00       $unwind$?CxxCallCatchBlock@__FrameHandler3@@SAPEAXPEAU_EXCEPTION_RECORD@@@Z 0000000180043e00     libvcruntime:frame.obj
 0002:00018e3c       $unwind$?IsInExceptionSpec@@YAEPEAUEHExceptionRecord@@PEBU_s_ESTypeList@@@Z 0000000180043e3c     libvcruntime:frame.obj
 0002:00018e58       $unwind$??$BuildCatchObjectHelperInternal@V__FrameHandler3@@@@YAHPEAUEHExceptionRecord@@PEAXPEBU_s_HandlerType@@PEBU_s_CatchableType@@@Z 0000000180043e58     libvcruntime:frame.obj
 0002:00018e98       $unwind$??$BuildCatchObjectInternal@V__FrameHandler3@@@@YAXPEAUEHExceptionRecord@@PEAXPEBU_s_HandlerType@@PEBU_s_CatchableType@@@Z 0000000180043e98     libvcruntime:frame.obj
 0002:00018ec4       $unwind$??$__InternalCxxFrameHandler@V__FrameHandler3@@@@YA?AW4_EXCEPTION_DISPOSITION@@PEAUEHExceptionRecord@@PEA_KPEAU_CONTEXT@@PEAU_xDISPATCHER_CONTEXT@@PEBU_s_FuncInfo@@H1E@Z 0000000180043ec4     libvcruntime:frame.obj
 0002:00018edc       $unwind$??$FindHandler@V__FrameHandler3@@@@YAXPEAUEHExceptionRecord@@PEA_KPEAU_CONTEXT@@PEAU_xDISPATCHER_CONTEXT@@PEBU_s_FuncInfo@@EH1@Z 0000000180043edc     libvcruntime:frame.obj
 0002:00018efc       $unwind$??$CatchIt@V__FrameHandler3@@@@YAXPEAUEHExceptionRecord@@PEA_KPEAU_CONTEXT@@PEAU_xDISPATCHER_CONTEXT@@PEBU_s_FuncInfo@@PEBU_s_HandlerType@@PEBU_s_CatchableType@@PEBU_s_TryBlockMapEntry@@H1EE@Z 0000000180043efc     libvcruntime:frame.obj
 0002:00018f14       $unwind$??$FindHandlerForForeignException@V__FrameHandler3@@@@YAXPEAUEHExceptionRecord@@PEA_KPEAU_CONTEXT@@PEAU_xDISPATCHER_CONTEXT@@PEBU_s_FuncInfo@@HH1@Z 0000000180043f14     libvcruntime:frame.obj
 0002:00018f30       $xdatasym                  0000000180043f30     libucrt:strcmp.obj
 0002:00018f38       $xdatasym                  0000000180043f38     libucrt:strcat.obj
 0002:00018f40       $xdatasym                  0000000180043f40     libucrt:strncpy.obj
 0002:00018f44       $unwind$_beginthreadex     0000000180043f44     libucrt:thread.obj
 0002:00018f58       $unwind$??$thread_start@P6AIPEAX@Z$00@@YAKQEAX@Z 0000000180043f58     libucrt:thread.obj
 0002:00018f78       $xdatasym                  0000000180043f78     libucrt:strlen.obj
 0002:00018f80       $xdatasym                  0000000180043f80     libucrt:strncat.obj
 0002:00018f84       $unwind$__stdio_common_vfprintf 0000000180043f84     libucrt:output.obj
 0002:00018f84       $unwind$__stdio_common_vfwprintf 0000000180043f84     libucrt:output.obj
 0002:00018f94       $unwind$?get_raw_ptd@__crt_cached_ptd_host@@QEAAPEAU__acrt_ptd@@XZ 0000000180043f94     libucrt:output.obj
 0002:00018f9c       $chain$0$?get_raw_ptd@__crt_cached_ptd_host@@QEAAPEAU__acrt_ptd@@XZ 0000000180043f9c     libucrt:output.obj
 0002:00018fb0       $chain$1$?get_raw_ptd@__crt_cached_ptd_host@@QEAAPEAU__acrt_ptd@@XZ 0000000180043fb0     libucrt:output.obj
 0002:00018fc0       $unwind$?parse_int_from_format_string@?$output_processor@DV?$stream_output_adapter@D@__crt_stdio_output@@V?$standard_base@DV?$stream_output_adapter@D@__crt_stdio_output@@@2@@__crt_stdio_output@@AEAA_NQEAH@Z 0000000180043fc0     libucrt:output.obj
 0002:00018fc0       $unwind$?parse_int_from_format_string@?$output_processor@_WV?$stream_output_adapter@_W@__crt_stdio_output@@V?$standard_base@_WV?$stream_output_adapter@_W@__crt_stdio_output@@@2@@__crt_stdio_output@@AEAA_NQEAH@Z 0000000180043fc0     libucrt:output.obj
 0002:00018fd4       $unwind$?state_case_type@?$output_processor@DV?$stream_output_adapter@D@__crt_stdio_output@@V?$standard_base@DV?$stream_output_adapter@D@__crt_stdio_output@@@2@@__crt_stdio_output@@AEAA_NXZ 0000000180043fd4     libucrt:output.obj
 0002:00018ffc       $stateUnwindMap$__dcrt_uninitialize_environments_nolock 0000000180043ffc     libucrt:environment_initialization.obj
 0002:00018ffc       $stateUnwindMap$__acrt_freeptd 0000000180043ffc     libucrt:per_thread_data.obj
 0002:00018ffc       $stateUnwindMap$__acrt_getptd_head 0000000180043ffc     libucrt:per_thread_data.obj
 0002:00018ffc       $stateUnwindMap$__acrt_getptd_noexit 0000000180043ffc     libucrt:per_thread_data.obj
 0002:00018ffc       $stateUnwindMap$__acrt_getptd_noexit_explicit 0000000180043ffc     libucrt:per_thread_data.obj
 0002:00018ffc       $stateUnwindMap$?common_exit@@YAXHW4_crt_exit_cleanup_mode@@W4_crt_exit_return_mode@@@Z 0000000180043ffc     libucrt:exit.obj
 0002:00018ffc       $stateUnwindMap$_execute_onexit_table 0000000180043ffc     libucrt:onexit.obj
 0002:00018ffc       $stateUnwindMap$?state_case_type@?$output_processor@DV?$stream_output_adapter@D@__crt_stdio_output@@V?$standard_base@DV?$stream_output_adapter@D@__crt_stdio_output@@@2@@__crt_stdio_output@@AEAA_NXZ 0000000180043ffc     libucrt:output.obj
 0002:00018ffc       $stateUnwindMap$?state_case_type@?$output_processor@_WV?$stream_output_adapter@_W@__crt_stdio_output@@V?$standard_base@_WV?$stream_output_adapter@_W@__crt_stdio_output@@@2@@__crt_stdio_output@@AEAA_NXZ 0000000180043ffc     libucrt:output.obj
 0002:00019008       $ip2state$?state_case_type@?$output_processor@DV?$stream_output_adapter@D@__crt_stdio_output@@V?$standard_base@DV?$stream_output_adapter@D@__crt_stdio_output@@@2@@__crt_stdio_output@@AEAA_NXZ 0000000180044008     libucrt:output.obj
 0002:00019018       $unwind$?type_case_a@?$output_processor@DV?$stream_output_adapter@D@__crt_stdio_output@@V?$standard_base@DV?$stream_output_adapter@D@__crt_stdio_output@@@2@@__crt_stdio_output@@AEAA_NXZ 0000000180044018     libucrt:output.obj
 0002:00019028       $unwind$??R<lambda_303760bc4008a2b3ec4768a30b06a80c>@@QEBAHXZ 0000000180044028     libucrt:output.obj
 0002:0001904c       $unwind$?state_case_type@?$output_processor@_WV?$stream_output_adapter@_W@__crt_stdio_output@@V?$standard_base@_WV?$stream_output_adapter@_W@__crt_stdio_output@@@2@@__crt_stdio_output@@AEAA_NXZ 000000018004404c     libucrt:output.obj
 0002:00019078       $ip2state$?state_case_type@?$output_processor@_WV?$stream_output_adapter@_W@__crt_stdio_output@@V?$standard_base@_WV?$stream_output_adapter@_W@__crt_stdio_output@@@2@@__crt_stdio_output@@AEAA_NXZ 0000000180044078     libucrt:output.obj
 0002:00019088       $unwind$?type_case_s_compute_narrow_string_length@?$output_processor@_WV?$stream_output_adapter@_W@__crt_stdio_output@@V?$standard_base@_WV?$stream_output_adapter@_W@__crt_stdio_output@@@2@@__crt_stdio_output@@AEAAHH_W@Z 0000000180044088     libucrt:output.obj
 0002:000190a0       $ip2state$?type_case_s_compute_narrow_string_length@?$output_processor@_WV?$stream_output_adapter@_W@__crt_stdio_output@@V?$standard_base@_WV?$stream_output_adapter@_W@__crt_stdio_output@@@2@@__crt_stdio_output@@AEAAHH_W@Z 00000001800440a0     libucrt:output.obj
 0002:000190a8       $unwind$?type_case_a@?$output_processor@_WV?$stream_output_adapter@_W@__crt_stdio_output@@V?$standard_base@_WV?$stream_output_adapter@_W@__crt_stdio_output@@@2@@__crt_stdio_output@@AEAA_NXZ 00000001800440a8     libucrt:output.obj
 0002:000190bc       $unwind$??R<lambda_ebf663be9fcd9e0b17ed57bdb95b0759>@@QEBAHXZ 00000001800440bc     libucrt:output.obj
 0002:000190e0       $unwind$??$?RV<lambda_d854c62834386a3b23916ad6dae2782d>@@AEAV<lambda_303760bc4008a2b3ec4768a30b06a80c>@@V<lambda_4780a7ea4f8cbd2590aec34bd14e2bbf>@@@?$__crt_seh_guarded_call@H@@QEAAH$$QEAV<lambda_d854c62834386a3b23916ad6dae2782d>@@AEAV<lambda_303760bc4008a2b3ec4768a30b06a80c>@@$$QEAV<lambda_4780a7ea4f8cbd2590aec34bd14e2bbf>@@@Z 00000001800440e0     libucrt:output.obj
 0002:00019104       $unwind$??$?RV<lambda_613eff765f5c257adf68e381dfe80f05>@@AEAV<lambda_ebf663be9fcd9e0b17ed57bdb95b0759>@@V<lambda_872abebd861b7db59b42e49ea65623b0>@@@?$__crt_seh_guarded_call@H@@QEAAH$$QEAV<lambda_613eff765f5c257adf68e381dfe80f05>@@AEAV<lambda_ebf663be9fcd9e0b17ed57bdb95b0759>@@$$QEAV<lambda_872abebd861b7db59b42e49ea65623b0>@@@Z 0000000180044104     libucrt:output.obj
 0002:00019128       $unwind$??$parse_integer@KV?$c_string_character_source@_W@__crt_strtox@@$0A@@__crt_strtox@@YAKAEAV__crt_cached_ptd_host@@V?$c_string_character_source@_W@0@H_N@Z 0000000180044128     libucrt:output.obj
 0002:00019144       $unwind$strrchr            0000000180044144     libvcruntime:strrchr.obj
 0002:00019144       $unwind$??$type_case_integer_parse_into_buffer@I$09@?$output_processor@DV?$stream_output_adapter@D@__crt_stdio_output@@V?$standard_base@DV?$stream_output_adapter@D@__crt_stdio_output@@@2@@__crt_stdio_output@@AEAAXI_N@Z 0000000180044144     libucrt:output.obj
 0002:00019144       $unwind$??$type_case_integer_parse_into_buffer@I$09@?$output_processor@_WV?$stream_output_adapter@_W@__crt_stdio_output@@V?$standard_base@_WV?$stream_output_adapter@_W@__crt_stdio_output@@@2@@__crt_stdio_output@@AEAAXI_N@Z 0000000180044144     libucrt:output.obj
 0002:00019144       $unwind$??$type_case_integer_parse_into_buffer@_K$09@?$output_processor@DV?$stream_output_adapter@D@__crt_stdio_output@@V?$standard_base@DV?$stream_output_adapter@D@__crt_stdio_output@@@2@@__crt_stdio_output@@AEAAX_K_N@Z 0000000180044144     libucrt:output.obj
 0002:00019144       $unwind$??$type_case_integer_parse_into_buffer@_K$09@?$output_processor@_WV?$stream_output_adapter@_W@__crt_stdio_output@@V?$standard_base@_WV?$stream_output_adapter@_W@__crt_stdio_output@@@2@@__crt_stdio_output@@AEAAX_K_N@Z 0000000180044144     libucrt:output.obj
 0002:00019144       $unwind$wcsnlen            0000000180044144     libucrt:strnlen.obj
 0002:0001914c       $unwind$_chsize_nolock     000000018004414c     libucrt:chsize.obj
 0002:0001914c       $unwind$_close_nolock      000000018004414c     libucrt:close.obj
 0002:0001914c       $unwind$_lseeki64          000000018004414c     libucrt:lseek.obj
 0002:0001914c       $unwind$_lseeki64_nolock   000000018004414c     libucrt:lseek.obj
 0002:0001914c       $unwind$_write             000000018004414c     libucrt:write.obj
 0002:0001914c       $unwind$fclose             000000018004414c     libucrt:fclose.obj
 0002:0001914c       $unwind$_fflush_nolock     000000018004414c     libucrt:fflush.obj
 0002:0001915c       $unwind$?_fclose_nolock_internal@@YAHQEAU_iobuf@@AEAV__crt_cached_ptd_host@@@Z 000000018004415c     libucrt:fclose.obj
 0002:0001916c       $unwind$?_fclose_internal@@YAHQEAU_iobuf@@AEAV__crt_cached_ptd_host@@@Z 000000018004416c     libucrt:fclose.obj
 0002:00019190       $unwind$??$common_fsopen@D@@YAPEAU_iobuf@@QEBD0H@Z 0000000180044190     libucrt:fopen.obj
 0002:000191b8       $unwind$??$common_getenv@D@@YAPEADQEBD@Z 00000001800441b8     libucrt:getenv.obj
 0002:000191d8       $unwind$wcsncpy            00000001800441d8     libucrt:wcsncpy.obj
 0002:000191f0       $unwind$_callnewh          00000001800441f0     libucrt:new_handler.obj
 0002:000191fc       $unwind$_query_new_handler 00000001800441fc     libucrt:new_handler.obj
 0002:0001921c       $unwind$_query_new_handler$fin$0 000000018004421c     libucrt:new_handler.obj
 0002:00019224       $unwind$_set_new_handler   0000000180044224     libucrt:new_handler.obj
 0002:00019248       $unwind$_set_new_handler$fin$0 0000000180044248     libucrt:new_handler.obj
 0002:00019250       $unwind$??$free_environment@D@@YAXQEAPEAD@Z 0000000180044250     libucrt:environment_initialization.obj
 0002:00019250       $unwind$??$free_environment@_W@@YAXQEAPEA_W@Z 0000000180044250     libucrt:environment_initialization.obj
 0002:00019250       $unwind$_initterm          0000000180044250     libucrt:initterm.obj
 0002:0001925c       $unwind$?try_cor_exit_process@@YAXI@Z 000000018004425c     libucrt:exit.obj
 0002:00019270       $ip2state$?try_cor_exit_process@@YAXI@Z 0000000180044270     libucrt:exit.obj
 0002:00019278       $unwind$?common_exit@@YAXHW4_crt_exit_cleanup_mode@@W4_crt_exit_return_mode@@@Z 0000000180044278     libucrt:exit.obj
 0002:00019290       $ip2state$?common_exit@@YAXHW4_crt_exit_cleanup_mode@@W4_crt_exit_return_mode@@@Z 0000000180044290     libucrt:exit.obj
 0002:00019298       $unwind$??R<lambda_6e4b09c48022b2350581041d5f6b0c4c>@@QEBA@XZ 0000000180044298     libucrt:exit.obj
 0002:000192b8       $unwind$??$?RV<lambda_d80eeec6fff315bfe5c115232f3240e3>@@AEAV<lambda_6e4b09c48022b2350581041d5f6b0c4c>@@V<lambda_2358e3775559c9db80273638284d5e45>@@@?$__crt_seh_guarded_call@X@@QEAAX$$QEAV<lambda_d80eeec6fff315bfe5c115232f3240e3>@@AEAV<lambda_6e4b09c48022b2350581041d5f6b0c4c>@@$$QEAV<lambda_2358e3775559c9db80273638284d5e45>@@@Z 00000001800442b8     libucrt:exit.obj
 0002:000192dc       $unwind$_configure_narrow_argv 00000001800442dc     libucrt:argv_parsing.obj
 0002:000192f0       $unwind$__dcrt_uninitialize_environments_nolock 00000001800442f0     libucrt:environment_initialization.obj
 0002:000192f0       $unwind$__acrt_getptd_head 00000001800442f0     libucrt:per_thread_data.obj
 0002:00019300       $unwind$??$initialize_environment_by_cloning_nolock@D@@YAHXZ 0000000180044300     libucrt:environment_initialization.obj
 0002:00019314       $unwind$_execute_onexit_table 0000000180044314     libucrt:onexit.obj
 0002:00019328       $ip2state$_execute_onexit_table 0000000180044328     libucrt:onexit.obj
 0002:00019330       $unwind$??$?RV<lambda_7777bce6b2f8c936911f934f8298dc43>@@AEAV<lambda_f03950bc5685219e0bcd2087efbe011e>@@V<lambda_3883c3dff614d5e0c5f61bb1ac94921c>@@@?$__crt_seh_guarded_call@H@@QEAAH$$QEAV<lambda_7777bce6b2f8c936911f934f8298dc43>@@AEAV<lambda_f03950bc5685219e0bcd2087efbe011e>@@$$QEAV<lambda_3883c3dff614d5e0c5f61bb1ac94921c>@@@Z 0000000180044330     libucrt:onexit.obj
 0002:00019354       $unwind$terminate          0000000180044354     libucrt:terminate.obj
 0002:00019378       $xdatasym                  0000000180044378     libucrt:strncmp.obj
 0002:0001937c       $unwind$__acrt_call_reportfault 000000018004437c     libucrt:invalid_parameter.obj
 0002:0001939c       $unwind$_invalid_parameter 000000018004439c     libucrt:invalid_parameter.obj
 0002:000193a8       $unwind$__acrt_errno_from_os_error 00000001800443a8     libucrt:errno.obj
 0002:000193b8       $unwind$_calloc_base       00000001800443b8     libucrt:calloc_base.obj
 0002:000193c0       $unwind$_free_base         00000001800443c0     libucrt:free_base.obj
 0002:000193c8       $unwind$__acrt_getptd_noexit 00000001800443c8     libucrt:per_thread_data.obj
 0002:000193c8       $unwind$__acrt_getptd_noexit_explicit 00000001800443c8     libucrt:per_thread_data.obj
 0002:000193dc       $unwind$__acrt_freeptd     00000001800443dc     libucrt:per_thread_data.obj
 0002:000193ec       $unwind$?destroy_fls@@YAXPEAX@Z 00000001800443ec     libucrt:per_thread_data.obj
 0002:000193ec       $unwind$__acrt_locale_free_numeric 00000001800443ec     libucrt:initnum.obj
 0002:000193ec       $unwind$__acrt_locale_free_lc_time_if_unreferenced 00000001800443ec     libucrt:locale_refcounting.obj
 0002:000193f4       $unwind$?construct_ptd_array@@YAXQEAU__acrt_ptd@@@Z 00000001800443f4     libucrt:per_thread_data.obj
 0002:000193fc       $unwind$?destroy_ptd_array@@YAXQEAU__acrt_ptd@@@Z 00000001800443fc     libucrt:per_thread_data.obj
 0002:00019404       $unwind$??$?RV<lambda_0ae27a3a962d80f24befdcbee591983d>@@AEAV<lambda_8d0ee55de4b1038c4002e0adecdf1839>@@V<lambda_dc504788e8f1664fe9b84e20bfb512f2>@@@?$__crt_seh_guarded_call@X@@QEAAX$$QEAV<lambda_0ae27a3a962d80f24befdcbee591983d>@@AEAV<lambda_8d0ee55de4b1038c4002e0adecdf1839>@@$$QEAV<lambda_dc504788e8f1664fe9b84e20bfb512f2>@@@Z 0000000180044404     libucrt:per_thread_data.obj
 0002:00019428       $unwind$??$?RV<lambda_aa87e3671a710a21b5dc78c0bdf72e11>@@AEAV<lambda_92619d2358a28f41a33ba319515a20b9>@@V<lambda_6992ecaafeb10aed2b74cb1fae11a551>@@@?$__crt_seh_guarded_call@X@@QEAAX$$QEAV<lambda_aa87e3671a710a21b5dc78c0bdf72e11>@@AEAV<lambda_92619d2358a28f41a33ba319515a20b9>@@$$QEAV<lambda_6992ecaafeb10aed2b74cb1fae11a551>@@@Z 0000000180044428     libucrt:per_thread_data.obj
 0002:0001944c       $unwind$??$?RV<lambda_f2e299630e499de9f9a165e60fcd3db5>@@AEAV<lambda_2ae9d31cdba2644fcbeaf08da7c24588>@@V<lambda_40d01ff24d0e7b3814fdbdcee8eab3c7>@@@?$__crt_seh_guarded_call@X@@QEAAX$$QEAV<lambda_f2e299630e499de9f9a165e60fcd3db5>@@AEAV<lambda_2ae9d31cdba2644fcbeaf08da7c24588>@@$$QEAV<lambda_40d01ff24d0e7b3814fdbdcee8eab3c7>@@@Z 000000018004444c     libucrt:per_thread_data.obj
 0002:00019470       $unwind$??$?RV<lambda_2d41944a1d46af3157314b8a01080d33>@@AEAV<lambda_8f455de75cd7d7f24b4096f044d8b9e6>@@V<lambda_aa500f224e6afead328df44964fe2772>@@@?$__crt_seh_guarded_call@X@@QEAAX$$QEAV<lambda_2d41944a1d46af3157314b8a01080d33>@@AEAV<lambda_8f455de75cd7d7f24b4096f044d8b9e6>@@$$QEAV<lambda_aa500f224e6afead328df44964fe2772>@@@Z 0000000180044470     libucrt:per_thread_data.obj
 0002:00019494       $unwind$?fp_format_f@@YAHQEBNQEAD_K12HW4__acrt_rounding_mode@@AEAV__crt_cached_ptd_host@@@Z 0000000180044494     libucrt:cvt.obj
 0002:00019494       $unwind$__acrt_CompareStringEx 0000000180044494     libucrt:winapi_thunks.obj
 0002:00019494       $unwind$__acrt_LCMapStringEx 0000000180044494     libucrt:winapi_thunks.obj
 0002:000194a8       $unwind$?try_get_function_slow@@YAPEAXW4function_id@?A0x391cf84c@@QEBDQEBW4module_id@2@2@Z 00000001800444a8     libucrt:winapi_thunks.obj
 0002:000194c8       $unwind$_fcloseall         00000001800444c8     libucrt:closeall.obj
 0002:000194ec       $unwind$?common_flush_all@@YAH_N@Z 00000001800444ec     libucrt:fflush.obj
 0002:000194f4       $unwind$??$?RV<lambda_842d9ff0dc9ef11c61343bbaebe7f885>@@AEAV<lambda_c5860995281e5c4ce005b3de8f5874ee>@@V<lambda_d90129c13df834fdcbf8d2b88dafcf2d>@@@?$__crt_seh_guarded_call@X@@QEAAX$$QEAV<lambda_842d9ff0dc9ef11c61343bbaebe7f885>@@AEAV<lambda_c5860995281e5c4ce005b3de8f5874ee>@@$$QEAV<lambda_d90129c13df834fdcbf8d2b88dafcf2d>@@@Z 00000001800444f4     libucrt:fflush.obj
 0002:00019518       $unwind$??$?RV<lambda_886d6c58226a84441f68b9f2b8217b83>@@AEAV<lambda_ab61a845afdef5b7c387490eaf3616ee>@@V<lambda_f7f22ab5edc0698d5f6905b0d3f44752>@@@?$__crt_seh_guarded_call@X@@QEAAX$$QEAV<lambda_886d6c58226a84441f68b9f2b8217b83>@@AEAV<lambda_ab61a845afdef5b7c387490eaf3616ee>@@$$QEAV<lambda_f7f22ab5edc0698d5f6905b0d3f44752>@@@Z 0000000180044518     libucrt:fflush.obj
 0002:00019540       $unwind$__acrt_initialize_lowio 0000000180044540     libucrt:ioinit.obj
 0002:00019560       $unwind$?initialize_inherited_file_handles_nolock@@YAXXZ 0000000180044560     libucrt:ioinit.obj
 0002:0001957c       $unwind$_malloc_base       000000018004457c     libucrt:malloc_base.obj
 0002:00019584       $unwind$__acrt_fp_format   0000000180044584     libucrt:cvt.obj
 0002:00019594       $unwind$?fp_format_e_internal@@YAHQEAD_KH_NIQEAU_strflt@@2AEAV__crt_cached_ptd_host@@@Z 0000000180044594     libucrt:cvt.obj
 0002:000195b0       $unwind$?fp_format_a@@YAHQEBNPEAD_KQEAD2H_NIW4__acrt_rounding_mode@@AEAV__crt_cached_ptd_host@@@Z 00000001800445b0     libucrt:cvt.obj
 0002:000195cc       $unwind$?fp_format_g@@YAHQEBNQEAD_K12H_NIW4__acrt_rounding_mode@@AEAV__crt_cached_ptd_host@@@Z 00000001800445cc     libucrt:cvt.obj
 0002:000195e4       $unwind$_wctomb_internal   00000001800445e4     libucrt:wctomb.obj
 0002:000195f8       $unwind$?__mbrtoc32_utf8@__crt_mbstring@@YA_KPEA_UPEBD_KPEAU_Mbstatet@@AEAV__crt_cached_ptd_host@@@Z 00000001800445f8     libucrt:mbrtoc32.obj
 0002:00019614       $unwind$__dcrt_lowio_ensure_console_output_initialized 0000000180044614     libucrt:initcon.obj
 0002:00019614       $unwind$?__mbrtowc_utf8@__crt_mbstring@@YA_KPEA_WPEBD_KPEAU_Mbstatet@@AEAV__crt_cached_ptd_host@@@Z 0000000180044614     libucrt:mbrtowc.obj
 0002:00019614       $unwind$?getSystemCP@@YAHH@Z 0000000180044614     libucrt:mbctype.obj
 0002:0001961c       $unwind$_fputwc_nolock_internal 000000018004461c     libucrt:fputwc.obj
 0002:00019638       $unwind$__acrt_stdio_end_temporary_buffering_nolock 0000000180044638     libucrt:_sftbuf.obj
 0002:00019640       $unwind$__acrt_uninitialize_locale 0000000180044640     libucrt:wsetlocale.obj
 0002:00019640       $unwind$__acrt_get_sigabrt_handler 0000000180044640     libucrt:signal.obj
 0002:00019648       $unwind$??$?RV<lambda_410d79af7f07d98d83a3f525b3859a53>@@AEAV<lambda_3e16ef9562a7dcce91392c22ab16ea36>@@V<lambda_38119f0e861e05405d8a144b9b982f0a>@@@?$__crt_seh_guarded_call@X@@QEAAX$$QEAV<lambda_410d79af7f07d98d83a3f525b3859a53>@@AEAV<lambda_3e16ef9562a7dcce91392c22ab16ea36>@@$$QEAV<lambda_38119f0e861e05405d8a144b9b982f0a>@@@Z 0000000180044648     libucrt:wsetlocale.obj
 0002:00019670       $unwind$_close_internal    0000000180044670     libucrt:close.obj
 0002:00019678       $unwind$??$?RV<lambda_ad8af0d99a0adf03d037d7dffe354bb5>@@AEAV<lambda_c9ba49e555ba839a7b07aa3fbecb7617>@@V<lambda_2f1ebd5d68526518146ae959c9e734c8>@@@?$__crt_seh_guarded_call@H@@QEAAH$$QEAV<lambda_ad8af0d99a0adf03d037d7dffe354bb5>@@AEAV<lambda_c9ba49e555ba839a7b07aa3fbecb7617>@@$$QEAV<lambda_2f1ebd5d68526518146ae959c9e734c8>@@@Z 0000000180044678     libucrt:close.obj
 0002:0001969c       $unwind$?__acrt_stdio_allocate_stream@@YA?AV__crt_stdio_stream@@XZ 000000018004469c     libucrt:stream.obj
 0002:000196bc       $unwind$?find_or_allocate_unused_stream_nolock@@YA?AV__crt_stdio_stream@@XZ 00000001800446bc     libucrt:stream.obj
 0002:000196d0       $unwind$_openfile          00000001800446d0     libucrt:openfile.obj
 0002:000196e4       $unwind$_strnicoll_l       00000001800446e4     libucrt:strnicol.obj
 0002:000196f8       $unwind$??$common_expand_argv_wildcards@D@@YAHQEAPEADQEAPEAPEAD@Z 00000001800446f8     libucrt:argv_wildcards.obj
 0002:00019710       $unwind$__dcrt_get_narrow_environment_from_os 0000000180044710     libucrt:get_environment_from_os.obj
 0002:00019710       $unwind$??$__acrt_convert_wcs_mbs_cp@_WDV<lambda_d8593a27d1aa8c02be35c86a17d324c4>@@U__crt_win32_buffer_internal_dynamic_resizing@@@@YAHQEB_WAEAV?$__crt_win32_buffer@DU__crt_win32_buffer_internal_dynamic_resizing@@@@AEBV<lambda_d8593a27d1aa8c02be35c86a17d324c4>@@I@Z 0000000180044710     libucrt:argv_wildcards.obj
 0002:00019728       $unwind$??$expand_argument_wildcards@D@@YAHQEAD0AEAV?$argument_list@D@?A0x5f5c8891@@@Z 0000000180044728     libucrt:argv_wildcards.obj
 0002:00019748       $unwind$__acrt_GetModuleFileNameA 0000000180044748     libucrt:getmodulefilenamea.obj
 0002:00019764       $unwind$__dcrt_write_console 0000000180044764     libucrt:initcon.obj
 0002:00019764       $unwind$??$__acrt_convert_wcs_mbs_cp@_WDV<lambda_f788ae46380686e8b737efdd8c720d07>@@U__crt_win32_buffer_no_resizing@@@@YAHQEB_WAEAV?$__crt_win32_buffer@DU__crt_win32_buffer_no_resizing@@@@AEBV<lambda_f788ae46380686e8b737efdd8c720d07>@@I@Z 0000000180044764     libucrt:getmodulefilenamea.obj
 0002:00019778       $unwind$_setmbcp_nolock    0000000180044778     libucrt:mbctype.obj
 0002:00019798       $unwind$?update_thread_multibyte_data_internal@@YAPEAU__crt_multibyte_data@@QEAU__acrt_ptd@@QEAPEAU1@@Z 0000000180044798     libucrt:mbctype.obj
 0002:000197c0       $unwind$?setmbcp_internal@@YAHH_NQEAU__acrt_ptd@@QEAPEAU__crt_multibyte_data@@@Z 00000001800447c0     libucrt:mbctype.obj
 0002:000197d8       $unwind$?setSBUpLow@@YAXPEAU__crt_multibyte_data@@@Z 00000001800447d8     libucrt:mbctype.obj
 0002:000197f4       $unwind$??$?RV<lambda_efdfa57d1f175319df784efa44bb7b81>@@AEAV<lambda_5f0a4c1567f8adc6734073e5d1e1b35c>@@V<lambda_2e8a7d3640ea6ccb4c2413664c2db6fd>@@@?$__crt_seh_guarded_call@X@@QEAAX$$QEAV<lambda_efdfa57d1f175319df784efa44bb7b81>@@AEAV<lambda_5f0a4c1567f8adc6734073e5d1e1b35c>@@$$QEAV<lambda_2e8a7d3640ea6ccb4c2413664c2db6fd>@@@Z 00000001800447f4     libucrt:mbctype.obj
 0002:00019818       $unwind$?x_ismbbtype_l@@YAHPEAU__crt_locale_pointers@@IHH@Z 0000000180044818     libucrt:ismbbyte.obj
 0002:00019818       $unwind$_strnicmp_l        0000000180044818     libucrt:strnicmp.obj
 0002:00019828       $unwind$__acrt_WideCharToMultiByte 0000000180044828     libucrt:widechartomultibyte.obj
 0002:00019834       $unwind$??$common_set_variable_in_environment_nolock@D@@YAHQEADH@Z 0000000180044834     libucrt:setenv.obj
 0002:0001984c       $unwind$??$copy_environment@D@@YAPEAPEADQEAPEAD@Z 000000018004484c     libucrt:setenv.obj
 0002:00019860       $unwind$_recalloc_base     0000000180044860     libucrt:recalloc.obj
 0002:00019874       $unwind$__acrt_initialize_heap 0000000180044874     libucrt:heap_handle.obj
 0002:0001987c       $unwind$raise              000000018004487c     libucrt:signal.obj
 0002:000198bc       $unwind$??$?RV<lambda_450d765d439847d4c735a33c368b5fc0>@@AEAV<lambda_44731a7d0e6d81c3e6aa82d741081786>@@V<lambda_601a2a7da3b7a96e9554ac7215c4b07c>@@@?$__crt_seh_guarded_call@P6AXH@Z@@QEAAP6AXH@Z$$QEAV<lambda_450d765d439847d4c735a33c368b5fc0>@@AEAV<lambda_44731a7d0e6d81c3e6aa82d741081786>@@$$QEAV<lambda_601a2a7da3b7a96e9554ac7215c4b07c>@@@Z 00000001800448bc     libucrt:signal.obj
 0002:000198e0       $unwind$_set_new_mode      00000001800448e0     libucrt:new_mode.obj
 0002:000198e8       $unwind$__acrt_update_thread_locale_data 00000001800448e8     libucrt:locale_refcounting.obj
 0002:0001990c       $unwind$_commit            000000018004490c     libucrt:commit.obj
 0002:00019914       $unwind$??$?RV<lambda_a37b2b86f63e897a80ea819b0eb08c01>@@AEAV<lambda_38ce7e780aa69e748d6df282ebc68efe>@@V<lambda_99fb1378e971ab6e7edea83e3a7a83a2>@@@?$__crt_seh_guarded_call@H@@QEAAH$$QEAV<lambda_a37b2b86f63e897a80ea819b0eb08c01>@@AEAV<lambda_38ce7e780aa69e748d6df282ebc68efe>@@$$QEAV<lambda_99fb1378e971ab6e7edea83e3a7a83a2>@@@Z 0000000180044914     libucrt:commit.obj
 0002:00019938       $unwind$_write_nolock      0000000180044938     libucrt:write.obj
 0002:00019950       $unwind$_write_internal    0000000180044950     libucrt:write.obj
 0002:0001997c       $unwind$?write_double_translated_ansi_nolock@@YA?AUwrite_result@?A0x17268360@@HQEBDIAEAV__crt_cached_ptd_host@@@Z 000000018004497c     libucrt:write.obj
 0002:000199a8       $ip2state$?write_double_translated_ansi_nolock@@YA?AUwrite_result@?A0x17268360@@HQEBDIAEAV__crt_cached_ptd_host@@@Z 00000001800449a8     libucrt:write.obj
 0002:000199b0       $unwind$?write_text_ansi_nolock@@YA?AUwrite_result@?A0x17268360@@HQEBDI@Z 00000001800449b0     libucrt:write.obj
 0002:000199b0       $unwind$?write_text_utf16le_nolock@@YA?AUwrite_result@?A0x17268360@@HQEBDI@Z 00000001800449b0     libucrt:write.obj
 0002:000199d0       $unwind$?write_text_utf8_nolock@@YA?AUwrite_result@?A0x17268360@@HQEBDI@Z 00000001800449d0     libucrt:write.obj
 0002:000199f4       $unwind$_alloc_osfhnd      00000001800449f4     libucrt:osfinfo.obj
 0002:00019a24       $unwind$__acrt_lowio_destroy_handle_array 0000000180044a24     libucrt:osfinfo.obj
 0002:00019a34       $unwind$__acrt_lowio_ensure_fh_exists 0000000180044a34     libucrt:osfinfo.obj
 0002:00019a60       $unwind$__acrt_fltout      0000000180044a60     libucrt:cfout.obj
 0002:00019a84       $unwind$?divide@__crt_strtox@@YA_KAEAUbig_integer@1@AEBU21@@Z 0000000180044a84     libucrt:cfout.obj
 0002:00019a9c       $chain$0$?divide@__crt_strtox@@YA_KAEAUbig_integer@1@AEBU21@@Z 0000000180044a9c     libucrt:cfout.obj
 0002:00019ab0       $chain$1$?divide@__crt_strtox@@YA_KAEAUbig_integer@1@AEBU21@@Z 0000000180044ab0     libucrt:cfout.obj
 0002:00019ac0       $unwind$??$write_buffer_nolock@D@@YA_NDV__crt_stdio_stream@@AEAV__crt_cached_ptd_host@@@Z 0000000180044ac0     libucrt:_flsbuf.obj
 0002:00019ad4       $unwind$??$write_buffer_nolock@_W@@YA_N_WV__crt_stdio_stream@@AEAV__crt_cached_ptd_host@@@Z 0000000180044ad4     libucrt:_flsbuf.obj
 0002:00019ae8       $unwind$__acrt_locale_free_monetary 0000000180044ae8     libucrt:initmon.obj
 0002:00019af0       $unwind$__acrt_locale_free_time 0000000180044af0     libucrt:inittime.obj
 0002:00019b00       $unwind$__acrt_GetStringTypeA 0000000180044b00     libucrt:getstringtypea.obj
 0002:00019b28       $unwind$_sopen_nolock      0000000180044b28     libucrt:open.obj
 0002:00019b44       $unwind$_wsopen_nolock     0000000180044b44     libucrt:open.obj
 0002:00019b64       $unwind$??$common_sopen_dispatch@D@@YAHQEBDHHHQEAHH@Z 0000000180044b64     libucrt:open.obj
 0002:00019b88       $unwind$?fin$0@?0???$common_sopen_dispatch@D@@YAHQEBDHHHQEAHH@Z@4HA 0000000180044b88     libucrt:open.obj
 0002:00019b90       $unwind$?decode_options@@YA?AUfile_options@?A0xa9d50aae@@HHH@Z 0000000180044b90     libucrt:open.obj
 0002:00019ba4       $unwind$?truncate_ctrl_z_if_present@@YAHH@Z 0000000180044ba4     libucrt:open.obj
 0002:00019bb4       $unwind$?configure_text_mode@@YAHHUfile_options@?A0xa9d50aae@@HAEAW4__crt_lowio_text_mode@@@Z 0000000180044bb4     libucrt:open.obj
 0002:00019bcc       $unwind$__acrt_CompareStringA 0000000180044bcc     libucrt:comparestringa.obj
 0002:00019bdc       $unwind$?InternalCompareStringA@@YAHPEAU__crt_locale_pointers@@PEB_WKPEBDH2HH@Z 0000000180044bdc     libucrt:comparestringa.obj
 0002:00019c00       $unwind$qsort              0000000180044c00     libucrt:qsort.obj
 0002:00019c18       $chain$3$qsort             0000000180044c18     libucrt:qsort.obj
 0002:00019c38       $chain$4$qsort             0000000180044c38     libucrt:qsort.obj
 0002:00019c48       $unwind$strpbrk            0000000180044c48     libucrt:strpbrk.obj
 0002:00019c58       $unwind$fallbackMethod     0000000180044c58     libucrt:strpbrk.obj
 0002:00019c68       $unwind$_mbsdec_l          0000000180044c68     libucrt:mbsdec.obj
 0002:00019c74       $unwind$__acrt_LCMapStringA 0000000180044c74     libucrt:lcmapstringa.obj
 0002:00019c84       $unwind$?__acrt_LCMapStringA_stat@@YAHPEAU__crt_locale_pointers@@PEB_WKPEBDHPEADHHH@Z 0000000180044c84     libucrt:lcmapstringa.obj
 0002:00019cac       $unwind$__acrt_SetEnvironmentVariableA 0000000180044cac     libucrt:setenvironmentvariablea.obj
 0002:00019cc8       $unwind$_msize_base        0000000180044cc8     libucrt:msize.obj
 0002:00019cd0       $unwind$_realloc_base      0000000180044cd0     libucrt:realloc_base.obj
 0002:00019cdc       $unwind$??$common_lseek@_J@@YA_JH_JHAEAV__crt_cached_ptd_host@@@Z 0000000180044cdc     libucrt:lseek.obj
 0002:00019d08       $unwind$_putwch_nolock     0000000180044d08     libucrt:putwch.obj
 0002:00019d10       $unwind$_read_nolock       0000000180044d10     libucrt:read.obj
 0002:00019d28       $unwind$?translate_ansi_or_utf8_nolock@@YAHHQEAD_KQEA_W1@Z 0000000180044d28     libucrt:read.obj
 0002:00019d40       $unwind$??$translate_text_mode_nolock@_W@@YAHHQEA_W_K@Z 0000000180044d40     libucrt:read.obj
 0002:00019d58       $unwind$fesetenv           0000000180044d58     libucrt:fesetenv.obj
 0002:00019d68       $xdatasym$log10            0000000180044d68     libucrt:log10.obj
 0002:00019d74       $unwind$__acrt_fenv_set_control 0000000180044d74     libucrt:_fenvutils.obj
 0002:00019d80       $chain$0$__acrt_fenv_set_control 0000000180044d80     libucrt:_fenvutils.obj
 0002:00019d94       $chain$1$__acrt_fenv_set_control 0000000180044d94     libucrt:_fenvutils.obj
 0002:00019da4       $unwind$_setmode_nolock    0000000180044da4     libucrt:setmode.obj
 0002:00019db4       $unwind$_guard_check_icall 0000000180044db4     libucrt:checkcfg.obj
 0002:00019dc0       $unwind$common_control87   0000000180044dc0     libucrt:ieee.obj
 0002:00019dec       $unwind$_exception_enabled 0000000180044dec     libucrt:libm_error.obj
 0002:00019e00       $chain$0$_exception_enabled 0000000180044e00     libucrt:libm_error.obj
 0002:00019e14       $chain$1$_exception_enabled 0000000180044e14     libucrt:libm_error.obj
 0002:00019e24       $unwind$_handle_error      0000000180044e24     libucrt:libm_error.obj
 0002:00019e40       $unwind$__acrt_initialize_fma3 0000000180044e40     libucrt:fma3_available.obj
 0002:00019e48       $unwind$_log_special_common 0000000180044e48     libucrt:log_special.obj
 0002:00019e54       $unwind$_ctrlfp            0000000180044e54     libucrt:fpctrl.obj
 0002:00019e74       $unwind$_raise_exc_ex      0000000180044e74     libucrt:fpexcept.obj
 0002:00019e88       $unwind$_IsNonwritableInCurrentImage 0000000180044e88     LIBCMT:pesect.obj
 0002:00019eb0       $xdatasym                  0000000180044eb0     LIBCMT:chkstk.obj
 0002:0001a010       .edata                     0000000180045010     javaaccessbridge.exp
 0002:0001a038       rgpv                       0000000180045038     javaaccessbridge.exp
 0002:0001a0b0       rgszName                   00000001800450b0     javaaccessbridge.exp
 0002:0001a128       rgwOrd                     0000000180045128     javaaccessbridge.exp
 0002:0001a164       szName                     0000000180045164     javaaccessbridge.exp
 0002:0001a179       $N00001                    0000000180045179     javaaccessbridge.exp
 0002:0001a1bb       $N00002                    00000001800451bb     javaaccessbridge.exp
 0002:0001a1fd       $N00003                    00000001800451fd     javaaccessbridge.exp
 0002:0001a23d       $N00004                    000000018004523d     javaaccessbridge.exp
 0002:0001a280       $N00005                    0000000180045280     javaaccessbridge.exp
 0002:0001a2dd       $N00006                    00000001800452dd     javaaccessbridge.exp
 0002:0001a33a       $N00007                    000000018004533a     javaaccessbridge.exp
 0002:0001a37d       $N00008                    000000018004537d     javaaccessbridge.exp
 0002:0001a3c2       $N00009                    00000001800453c2     javaaccessbridge.exp
 0002:0001a405       $N00010                    0000000180045405     javaaccessbridge.exp
 0002:0001a448       $N00011                    0000000180045448     javaaccessbridge.exp
 0002:0001a48b       $N00012                    000000018004548b     javaaccessbridge.exp
 0002:0001a4cd       $N00013                    00000001800454cd     javaaccessbridge.exp
 0002:0001a510       $N00014                    0000000180045510     javaaccessbridge.exp
 0002:0001a554       $N00015                    0000000180045554     javaaccessbridge.exp
 0002:0001a59c       $N00016                    000000018004559c     javaaccessbridge.exp
 0002:0001a5ef       $N00017                    00000001800455ef     javaaccessbridge.exp
 0002:0001a640       $N00018                    0000000180045640     javaaccessbridge.exp
 0002:0001a695       $N00019                    0000000180045695     javaaccessbridge.exp
 0002:0001a6df       $N00020                    00000001800456df     javaaccessbridge.exp
 0002:0001a729       $N00021                    0000000180045729     javaaccessbridge.exp
 0002:0001a779       $N00022                    0000000180045779     javaaccessbridge.exp
 0002:0001a7c2       $N00023                    00000001800457c2     javaaccessbridge.exp
 0002:0001a810       $N00024                    0000000180045810     javaaccessbridge.exp
 0002:0001a85a       $N00025                    000000018004585a     javaaccessbridge.exp
 0002:0001a8a9       $N00026                    00000001800458a9     javaaccessbridge.exp
 0002:0001a8f2       $N00027                    00000001800458f2     javaaccessbridge.exp
 0002:0001a93c       $N00028                    000000018004593c     javaaccessbridge.exp
 0002:0001a98c       $N00029                    000000018004598c     javaaccessbridge.exp
 0002:0001a9c9       $N00030                    00000001800459c9     javaaccessbridge.exp
 0002:0001ad96       .idata$6                   0000000180045d96     jawt:jawt.dll
 0002:0001ae7a       .idata$6                   0000000180045e7a     kernel32:KERNEL32.dll
 0002:0001af36       .idata$6                   0000000180045f36     user32:USER32.dll
 0003:00000070       ?__vcrt_flsindex@@3KA      0000000180047070     libvcruntime:per_thread_data.obj
 0003:00000190       ?errno_no_memory@@3HA      0000000180047190     libucrt:errno.obj
 0003:00000194       ?doserrno_no_memory@@3KA   0000000180047194     libucrt:errno.obj
 0003:00000198       ?__acrt_flsindex@@3KA      0000000180047198     libucrt:per_thread_data.obj
 0003:00000590       _mbctypes                  0000000180047590     libucrt:mbctype.obj
 0003:000006a0       _mbcasemaps                00000001800476a0     libucrt:mbctype.obj
 0003:000007a0       ?__rgctypeflag@@3PADA      00000001800477a0     libucrt:mbctype.obj
 0003:000007b0       ?__rgcode_page_info@@3PAUcode_page_info@@A 00000001800477b0     libucrt:mbctype.obj
 0003:00000a50       ?__dcrt_lowio_console_output_handle@@3PEAXEA 0000000180047a50     libucrt:initcon.obj
 0003:00000a58       ?dazSupported@?1??common_control87@@9@9 0000000180047a58     libucrt:ieee.obj
 0003:00000a60       ?dazSupported@?1??_ctrlfp@@9@9 0000000180047a60     libucrt:fpctrl.obj
 0003:00000b50       logFP                      0000000180047b50     AccessBridgeDebug.obj
 0003:00000b98       ?__proc_attached@@3HA      0000000180047b98     LIBCMT:dll_dllmain.obj
 0003:00000ba0       GS_ExceptionRecord         0000000180047ba0     LIBCMT:gs_report.obj
 0003:00000c40       GS_ContextRecord           0000000180047c40     LIBCMT:gs_report.obj
 0003:00001138       ?is_initialized_as_dll@@3_NA 0000000180048138     LIBCMT:utility.obj
 0003:00001139       ?module_local_atexit_table_initialized@@3_NA 0000000180048139     LIBCMT:utility.obj
 0003:00001140       ?module_local_atexit_table@@3U_onexit_table_t@@A 0000000180048140     LIBCMT:utility.obj
 0003:00001158       ?module_local_at_quick_exit_table@@3U_onexit_table_t@@A 0000000180048158     LIBCMT:utility.obj
 0003:000011c8       ?heap@@3V_HeapManager@@A   00000001800481c8     libvcruntime:undname.obj
 0003:000011f0       ?__vcrt_startup_thread_ptd@@3U__vcrt_ptd@@A 00000001800481f0     libvcruntime:per_thread_data.obj
 0003:00001270       __vcrt_lock_table          0000000180048270     libvcruntime:locks.obj
 0003:00001298       __vcrt_locks_initialized   0000000180048298     libvcruntime:locks.obj
 0003:000012a0       ?module_handles@@3PAPEAUHINSTANCE__@@A 00000001800482a0     libvcruntime:winapi_downlevel.obj
 0003:000012b8       ?function_pointers@@3PAPEAXA 00000001800482b8     libvcruntime:winapi_downlevel.obj
 0003:00001300       ?__acrt_new_handler@@3V?$dual_state_global@P6AH_K@Z@__crt_state_management@@A 0000000180048300     libucrt:new_handler.obj
 0003:00001308       ?c_termination_complete@@3JA 0000000180048308     libucrt:exit.obj
 0003:00001310       ?thread_local_exit_callback_func@@3P6AXPEAXK0@ZEA 0000000180048310     libucrt:exit.obj
 0003:00001318       ?c_exit_complete@?1???R<lambda_6e4b09c48022b2350581041d5f6b0c4c>@@QEBA@XZ@4_NA 0000000180048318     libucrt:exit.obj
 0003:00001320       ?program_name@?1???$common_configure_argv@D@@YAHW4_crt_argv_mode@@@Z@4PADA 0000000180048320     libucrt:argv_parsing.obj
 0003:00001478       ?__acrt_invalid_parameter_handler@@3V?$dual_state_global@P6AXPEB_W00I_K@Z@__crt_state_management@@A 0000000180048478     libucrt:invalid_parameter.obj
 0003:00001490       ?module_handles@@3PAPEAUHINSTANCE__@@A 0000000180048490     libucrt:winapi_thunks.obj
 0003:00001548       ?state_cache@?1???$get_cached_win_policy@Ubegin_thread_init_policy_properties@?1??__acrt_get_begin_thread_init_policy@@YA?AW4begin_thread_init_policy@@XZ@@@YA?AW4begin_thread_init_policy@@W4AppPolicyThreadInitializationType@@@Z@4JA 0000000180048548     libucrt:win_policies.obj
 0003:00001958       ?internal_state@?1??_mbtowc_internal@@9@4U_Mbstatet@@A 0000000180048958     libucrt:mbtowc.obj
 0003:00001960       ?internal_pst@?1??__mbrtoc32_utf8@__crt_mbstring@@YA_KPEA_UPEBD_KPEAU_Mbstatet@@AEAV__crt_cached_ptd_host@@@Z@4U3@A 0000000180048960     libucrt:mbrtoc32.obj
 0003:00001968       ?internal_pst@?1??__c16rtomb_utf8@__crt_mbstring@@YA_KPEAD_SPEAU_Mbstatet@@AEAV__crt_cached_ptd_host@@@Z@4U3@A 0000000180048968     libucrt:c16rtomb.obj
 0003:00001970       ?enable_percent_n@@3_KA    0000000180048970     libucrt:printf_count_output.obj
 0003:000019a0       ?__acrt_lock_table@@3PAU_RTL_CRITICAL_SECTION@@A 00000001800489a0     libucrt:locks.obj
 0003:00001bf8       ?__acrt_locks_initialized@@3IA 0000000180048bf8     libucrt:locks.obj
 0003:00001c18       ?fSystemSet@@3HA           0000000180048c18     libucrt:mbctype.obj
 0003:00001c1c       ?initialized@?1??__acrt_initialize_multibyte@@9@4_NA 0000000180048c1c     libucrt:mbctype.obj
 0003:00001c58       ?ctrlc_action@@3V?$dual_state_global@P6AXH@Z@__crt_state_management@@A 0000000180048c58     libucrt:signal.obj
 0003:00001c60       ?ctrlbreak_action@@3V?$dual_state_global@P6AXH@Z@__crt_state_management@@A 0000000180048c60     libucrt:signal.obj
 0003:00001c68       ?abort_action@@3V?$dual_state_global@P6AXH@Z@__crt_state_management@@A 0000000180048c68     libucrt:signal.obj
 0003:00001c70       ?term_action@@3V?$dual_state_global@P6AXH@Z@__crt_state_management@@A 0000000180048c70     libucrt:signal.obj
 0003:00001c78       ?user_matherr@@3V?$dual_state_global@P6AHPEAU_exception@@@Z@__crt_state_management@@A 0000000180048c78     libucrt:matherr.obj
 0003:00001c80       ?__acrt_global_new_mode@@3V?$dual_state_global@J@__crt_state_management@@A 0000000180048c80     libucrt:new_mode.obj
 0003:00001c90       ?__acrt_app_type@@3W4_crt_app_type@@A 0000000180048c90     libucrt:report_runtime_error.obj
 0005:00000000       ?function_pointers@@3PAPEAXA 000000018004b000     libucrt:winapi_thunks.obj
 0006:00000120       $R000000                   000000018004c120     javaaccessbridge.dll.res
 0006:000004a0       $R000380                   000000018004c4a0     javaaccessbridge.dll.res
 0006:000006b8       $R000598                   000000018004c6b8     javaaccessbridge.dll.res
